 qagamex86

 Timestamp is 4839b7bd (Sun May 25 23:02:21 2008)

 Preferred load address is 20000000

 Start         Length     Name                   Class
 0001:00000000 0006572aH .text                   CODE
 0002:00000000 00000150H .idata$5                DATA
 0002:00000150 000098caH .rdata                  DATA
 0002:00009a1c 00000056H .rdata$debug            DATA
 0002:00009a74 00000004H .rtc$IAA                DATA
 0002:00009a78 00000004H .rtc$IZZ                DATA
 0002:00009a7c 00000004H .rtc$TAA                DATA
 0002:00009a80 00000004H .rtc$TZZ                DATA
 0002:00009a84 00000014H .idata$2                DATA
 0002:00009a98 00000014H .idata$3                DATA
 0002:00009aac 00000150H .idata$4                DATA
 0002:00009bfc 000005feH .idata$6                DATA
 0002:0000a200 0000005aH .edata                  DATA
 0003:00000000 00000004H .CRT$XCA                DATA
 0003:00000004 00000004H .CRT$XCAA               DATA
 0003:00000008 00000004H .CRT$XCZ                DATA
 0003:0000000c 00000004H .CRT$XIA                DATA
 0003:00000010 00000010H .CRT$XIC                DATA
 0003:00000020 00000004H .CRT$XIZ                DATA
 0003:00000024 00000004H .CRT$XPA                DATA
 0003:00000028 00000004H .CRT$XPX                DATA
 0003:0000002c 00000004H .CRT$XPZ                DATA
 0003:00000030 00000004H .CRT$XTA                DATA
 0003:00000034 00000004H .CRT$XTZ                DATA
 0003:00000040 00002cecH .data                   DATA
 0003:00002d40 0014c954H .bss                    DATA

  Address         Publics by Value              Rva+Base     Lib:Object

 0000:00000000       __except_list              00000000     <absolute>
 0000:00000000       ___safe_se_handler_table   00000000     <absolute>
 0000:00000000       ___safe_se_handler_count   00000000     <absolute>
 0001:00000000       _BotNumActivePlayers       20001000 f   ai_chat.obj
 0001:000000f0       _BotIsFirstInRankings      200010f0 f   ai_chat.obj
 0001:00000200       _BotIsLastInRankings       20001200 f   ai_chat.obj
 0001:00000310       _BotFirstClientInRankings  20001310 f   ai_chat.obj
 0001:00000440       _BotLastClientInRankings   20001440 f   ai_chat.obj
 0001:00000570       _BotRandomOpponentName     20001570 f   ai_chat.obj
 0001:00000740       _BotMapTitle               20001740 f   ai_chat.obj
 0001:000007a0       _BotWeaponNameForMeansOfDeath 200017a0 f   ai_chat.obj
 0001:00000870       _BotRandomWeaponName       20001870 f   ai_chat.obj
 0001:00000920       _BotVisibleEnemies         20001920 f   ai_chat.obj
 0001:00000a30       _BotValidChatPosition      20001a30 f   ai_chat.obj
 0001:00000bf0       _BotChat_EnterGame         20001bf0 f   ai_chat.obj
 0001:00000d30       _BotChat_ExitGame          20001d30 f   ai_chat.obj
 0001:00000e60       _BotChat_StartLevel        20001e60 f   ai_chat.obj
 0001:00000fa0       _BotChat_EndLevel          20001fa0 f   ai_chat.obj
 0001:000011c0       _BotChat_Death             200021c0 f   ai_chat.obj
 0001:00001650       _BotChat_Kill              20002650 f   ai_chat.obj
 0001:000018e0       _BotChat_EnemySuicide      200028e0 f   ai_chat.obj
 0001:00001a40       _BotChat_HitTalking        20002a40 f   ai_chat.obj
 0001:00001c00       _BotChat_HitNoDeath        20002c00 f   ai_chat.obj
 0001:00001df0       _BotChat_HitNoKill         20002df0 f   ai_chat.obj
 0001:00001fa0       _BotChat_Random            20002fa0 f   ai_chat.obj
 0001:00002260       _BotChatTime               20003260 f   ai_chat.obj
 0001:000022a0       _BotChatTest               200032a0 f   ai_chat.obj
 0001:00003000       _BotPrintTeamGoal          20004000 f   ai_cmd.obj
 0001:00003230       _BotGetItemTeamGoal        20004230 f   ai_cmd.obj
 0001:000032a0       _BotGetMessageTeamGoal     200042a0 f   ai_cmd.obj
 0001:00003310       _BotGetTime                20004310 f   ai_cmd.obj
 0001:00003440       _FindClientByName          20004440 f   ai_cmd.obj
 0001:00003530       _FindEnemyByName           20004530 f   ai_cmd.obj
 0001:00003640       _NumPlayersOnSameTeam      20004640 f   ai_cmd.obj
 0001:000036f0       _BotGetPatrolWaypoints     200046f0 f   ai_cmd.obj
 0001:000039a0       _BotAddressedToBot         200049a0 f   ai_cmd.obj
 0001:00003c30       _BotGPSToPosition          20004c30 f   ai_cmd.obj
 0001:00003d40       _BotMatch_HelpAccompany    20004d40 f   ai_cmd.obj
 0001:000041e0       _BotMatch_DefendKeyArea    200051e0 f   ai_cmd.obj
 0001:00004360       _BotMatch_GetItem          20005360 f   ai_cmd.obj
 0001:000044a0       _BotMatch_Camp             200054a0 f   ai_cmd.obj
 0001:00004870       _BotMatch_Patrol           20005870 f   ai_cmd.obj
 0001:000049c0       _BotMatch_GetFlag          200059c0 f   ai_cmd.obj
 0001:00004b10       _BotMatch_AttackEnemyBase  20005b10 f   ai_cmd.obj
 0001:00004c40       _BotMatch_RushBase         20005c40 f   ai_cmd.obj
 0001:00004d70       _BotMatch_TaskPreference   20005d70 f   ai_cmd.obj
 0001:00004f20       _BotMatch_ReturnFlag       20005f20 f   ai_cmd.obj
 0001:00005030       _BotMatch_JoinSubteam      20006030 f   ai_cmd.obj
 0001:00005110       _BotMatch_LeaveSubteam     20006110 f   ai_cmd.obj
 0001:000051e0       _BotMatch_WhichTeam        200061e0 f   ai_cmd.obj
 0001:00005280       _BotMatch_CheckPoint       20006280 f   ai_cmd.obj
 0001:00005540       _BotMatch_FormationSpace   20006540 f   ai_cmd.obj
 0001:00005620       _BotMatch_Dismiss          20006620 f   ai_cmd.obj
 0001:000056f0       _BotMatch_Suicide          200066f0 f   ai_cmd.obj
 0001:000057a0       _BotMatch_StartTeamLeaderShip 200067a0 f   ai_cmd.obj
 0001:00005860       _BotMatch_StopTeamLeaderShip 20006860 f   ai_cmd.obj
 0001:00005940       _BotMatch_WhoIsTeamLeader  20006940 f   ai_cmd.obj
 0001:000059b0       _BotMatch_WhatAreYouDoing  200069b0 f   ai_cmd.obj
 0001:00005c40       _BotMatch_WhatIsMyCommand  20006c40 f   ai_cmd.obj
 0001:00005c90       _BotNearestVisibleItem     20006c90 f   ai_cmd.obj
 0001:00005e10       _BotMatch_WhereAreYou      20006e10 f   ai_cmd.obj
 0001:000060f0       _BotMatch_LeadTheWay       200070f0 f   ai_cmd.obj
 0001:000063d0       _BotMatch_Kill             200073d0 f   ai_cmd.obj
 0001:00006530       _BotMatch_CTF              20007530 f   ai_cmd.obj
 0001:000066f0       _BotMatch_EnterGame        200076f0 f   ai_cmd.obj
 0001:00006740       _BotMatch_NewLeader        20007740 f   ai_cmd.obj
 0001:000067b0       _BotMatchMessage           200077b0 f   ai_cmd.obj
 0001:00006b90       _BotResetNodeSwitches      20007b90 f   ai_dmnet.obj
 0001:00006bb0       _BotDumpNodeSwitches       20007bb0 f   ai_dmnet.obj
 0001:00006c40       _BotRecordNodeSwitch       20007c40 f   ai_dmnet.obj
 0001:00006ce0       _BotGetAirGoal             20007ce0 f   ai_dmnet.obj
 0001:00006e90       _BotGoForAir               20007e90 f   ai_dmnet.obj
 0001:00006f80       _BotNearbyGoal             20007f80 f   ai_dmnet.obj
 0001:00007040       _BotReachedGoal            20008040 f   ai_dmnet.obj
 0001:00007200       _BotGetItemLongTermGoal    20008200 f   ai_dmnet.obj
 0001:00007350       _BotGetLongTermGoal        20008350 f   ai_dmnet.obj
 0001:00009190       _BotLongTermGoal           2000a190 f   ai_dmnet.obj
 0001:000096a0       _AIEnter_Intermission      2000a6a0 f   ai_dmnet.obj
 0001:00009720       _AINode_Intermission       2000a720 f   ai_dmnet.obj
 0001:000097a0       _AIEnter_Observer          2000a7a0 f   ai_dmnet.obj
 0001:000097f0       _AINode_Observer           2000a7f0 f   ai_dmnet.obj
 0001:00009830       _AIEnter_Stand             2000a830 f   ai_dmnet.obj
 0001:00009880       _AINode_Stand              2000a880 f   ai_dmnet.obj
 0001:000099b0       _AIEnter_Respawn           2000a9b0 f   ai_dmnet.obj
 0001:00009ac0       _AINode_Respawn            2000aac0 f   ai_dmnet.obj
 0001:00009bd0       _BotSelectActivateWeapon   2000abd0 f   ai_dmnet.obj
 0001:00009cd0       _BotClearPath              2000acd0 f   ai_dmnet.obj
 0001:0000a140       _AIEnter_Seek_ActivateEntity 2000b140 f   ai_dmnet.obj
 0001:0000a180       _AINode_Seek_ActivateEntity 2000b180 f   ai_dmnet.obj
 0001:0000a990       _AIEnter_Seek_NBG          2000b990 f   ai_dmnet.obj
 0001:0000aa20       _AINode_Seek_NBG           2000ba20 f   ai_dmnet.obj
 0001:0000aed0       _AIEnter_Seek_LTG          2000bed0 f   ai_dmnet.obj
 0001:0000af60       _AINode_Seek_LTG           2000bf60 f   ai_dmnet.obj
 0001:0000b5d0       _AIEnter_Battle_Fight      2000c5d0 f   ai_dmnet.obj
 0001:0000b620       _AIEnter_Battle_SuicidalFight 2000c620 f   ai_dmnet.obj
 0001:0000b680       _AINode_Battle_Fight       2000c680 f   ai_dmnet.obj
 0001:0000bbe0       _AIEnter_Battle_Chase      2000cbe0 f   ai_dmnet.obj
 0001:0000bc30       _AINode_Battle_Chase       2000cc30 f   ai_dmnet.obj
 0001:0000c190       _AIEnter_Battle_Retreat    2000d190 f   ai_dmnet.obj
 0001:0000c1d0       _AINode_Battle_Retreat     2000d1d0 f   ai_dmnet.obj
 0001:0000c820       _AIEnter_Battle_NBG        2000d820 f   ai_dmnet.obj
 0001:0000c860       _AINode_Battle_NBG         2000d860 f   ai_dmnet.obj
 0001:0000cd90       _BotSetUserInfo            2000dd90 f   ai_dmq3.obj
 0001:0000ce00       _BotCTFCarryingFlag        2000de00 f   ai_dmq3.obj
 0001:0000ce50       _BotTeam                   2000de50 f   ai_dmq3.obj
 0001:0000cef0       _BotOppositeTeam           2000def0 f   ai_dmq3.obj
 0001:0000cf30       _BotEnemyFlag              2000df30 f   ai_dmq3.obj
 0001:0000cf60       _BotTeamFlag               2000df60 f   ai_dmq3.obj
 0001:0000cf90       _EntityIsDead              2000df90 f   ai_dmq3.obj
 0001:0000cfe0       _EntityCarriesFlag         2000dfe0 f   ai_dmq3.obj
 0001:0000d020       _EntityIsInvisible         2000e020 f   ai_dmq3.obj
 0001:0000d060       _EntityIsShooting          2000e060 f   ai_dmq3.obj
 0001:0000d090       _EntityIsChatting          2000e090 f   ai_dmq3.obj
 0001:0000d0c0       _EntityHasQuad             2000e0c0 f   ai_dmq3.obj
 0001:0000d0f0       _BotRememberLastOrderedTask 2000e0f0 f   ai_dmq3.obj
 0001:0000d170       _BotSetTeamStatus          2000e170 f   ai_dmq3.obj
 0001:0000d180       _BotSetLastOrderedTask     2000e180 f   ai_dmq3.obj
 0001:0000d340       _BotRefuseOrder            2000e340 f   ai_dmq3.obj
 0001:0000d3d0       _BotCTFSeekGoals           2000e3d0 f   ai_dmq3.obj
 0001:0000df10       _BotCTFRetreatGoals        2000ef10 f   ai_dmq3.obj
 0001:0000dfa0       _BotTeamGoals              2000efa0 f   ai_dmq3.obj
 0001:0000dff0       _BotPointAreaNum           2000eff0 f   ai_dmq3.obj
 0001:0000e070       _ClientName                2000f070 f   ai_dmq3.obj
 0001:0000e110       _ClientSkin                2000f110 f   ai_dmq3.obj
 0001:0000e1a0       _ClientFromName            2000f1a0 f   ai_dmq3.obj
 0001:0000e250       _ClientOnSameTeamFromName  2000f250 f   ai_dmq3.obj
 0001:0000e320       _stristr                   2000f320 f   ai_dmq3.obj
 0001:0000e3c0       _EasyClientName            2000f3c0 f   ai_dmq3.obj
 0001:0000e660       _BotSynonymContext         2000f660 f   ai_dmq3.obj
 0001:0000e6b0       _BotChooseWeapon           2000f6b0 f   ai_dmq3.obj
 0001:0000e760       _BotSetupForMovement       2000f760 f   ai_dmq3.obj
 0001:0000e8d0       _BotCheckItemPickup        2000f8d0 f   ai_dmq3.obj
 0001:0000e8e0       _BotUpdateInventory        2000f8e0 f   ai_dmq3.obj
 0001:0000ebf0       _BotUpdateBattleInventory  2000fbf0 f   ai_dmq3.obj
 0001:0000ec80       _BotBattleUseItems         2000fc80 f   ai_dmq3.obj
 0001:0000ecf0       _BotSetTeleportTime        2000fcf0 f   ai_dmq3.obj
 0001:0000ed40       _BotIsDead                 2000fd40 f   ai_dmq3.obj
 0001:0000ed60       _BotIsObserver             2000fd60 f   ai_dmq3.obj
 0001:0000edd0       _BotIntermission           2000fdd0 f   ai_dmq3.obj
 0001:0000ee20       _BotInLavaOrSlime          2000fe20 f   ai_dmq3.obj
 0001:0000ee70       _BotCreateWayPoint         2000fe70 f   ai_dmq3.obj
 0001:0000ef70       _BotFindWayPoint           2000ff70 f   ai_dmq3.obj
 0001:0000efc0       _BotFreeWaypoints          2000ffc0 f   ai_dmq3.obj
 0001:0000f000       _BotInitWaypoints          20010000 f   ai_dmq3.obj
 0001:0000f060       _TeamPlayIsOn              20010060 f   ai_dmq3.obj
 0001:0000f080       _BotAggression             20010080 f   ai_dmq3.obj
 0001:0000f210       _BotFeelingBad             20010210 f   ai_dmq3.obj
 0001:0000f280       _BotWantsToRetreat         20010280 f   ai_dmq3.obj
 0001:0000f330       _BotWantsToChase           20010330 f   ai_dmq3.obj
 0001:0000f3d0       _BotWantsToHelp            200103d0 f   ai_dmq3.obj
 0001:0000f3f0       _BotCanAndWantsToRocketJump 200103f0 f   ai_dmq3.obj
 0001:0000f4b0       _BotHasPersistantPowerupAndWeapon 200104b0 f   ai_dmq3.obj
 0001:0000f600       _BotGoCamp                 20010600 f   ai_dmq3.obj
 0001:0000f710       _BotWantsToCamp            20010710 f   ai_dmq3.obj
 0001:0000f950       _BotDontAvoid              20010950 f   ai_dmq3.obj
 0001:0000f9b0       _BotGoForPowerups          200109b0 f   ai_dmq3.obj
 0001:0000fa30       _BotRoamGoal               20010a30 f   ai_dmq3.obj
 0001:0000fd90       _BotAttackMove             20010d90 f   ai_dmq3.obj
 0001:00010480       _BotSameTeam               20011480 f   ai_dmq3.obj
 0001:00010560       _InFieldOfVision           20011560 f   ai_dmq3.obj
 0001:00010670       _BotEntityVisible          20011670 f   ai_dmq3.obj
 0001:00010be0       _BotFindEnemy              20011be0 f   ai_dmq3.obj
 0001:000110f0       _BotTeamFlagCarrierVisible 200120f0 f   ai_dmq3.obj
 0001:000111d0       _BotTeamFlagCarrier        200121d0 f   ai_dmq3.obj
 0001:00011270       _BotEnemyFlagCarrierVisible 20012270 f   ai_dmq3.obj
 0001:00011350       _BotVisibleTeamMatesAndEnemies 20012350 f   ai_dmq3.obj
 0001:000114d0       _BotAimAtEnemy             200124d0 f   ai_dmq3.obj
 0001:00012650       _BotCheckAttack            20013650 f   ai_dmq3.obj
 0001:00012bb0       _BotMapScripts             20013bb0 f   ai_dmq3.obj
 0001:00013000       _BotSetMovedir             20014000 f   ai_dmq3.obj
 0001:00013100       _BotModelMinsMaxs          20014100 f   ai_dmq3.obj
 0001:00013280       _BotFuncButtonActivateGoal 20014280 f   ai_dmq3.obj
 0001:00013df0       _BotFuncDoorActivateGoal   20014df0 f   ai_dmq3.obj
 0001:00013fd0       _BotTriggerMultipleActivateGoal 20014fd0 f   ai_dmq3.obj
 0001:000142c0       _BotPopFromActivateGoalStack 200152c0 f   ai_dmq3.obj
 0001:00014340       _BotPushOntoActivateGoalStack 20015340 f   ai_dmq3.obj
 0001:00014460       _BotClearActivateGoalStack 20015460 f   ai_dmq3.obj
 0001:00014490       _BotEnableActivateGoalAreas 20015490 f   ai_dmq3.obj
 0001:00014510       _BotIsGoingToActivateEntity 20015510 f   ai_dmq3.obj
 0001:000145f0       _BotGetActivateGoal        200155f0 f   ai_dmq3.obj
 0001:00014e80       _BotGoForActivateGoal      20015e80 f   ai_dmq3.obj
 0001:00014f40       _BotPrintActivateGoalInfo  20015f40 f   ai_dmq3.obj
 0001:00015050       _BotRandomMove             20016050 f   ai_dmq3.obj
 0001:000150f0       _BotAIBlocked              200160f0 f   ai_dmq3.obj
 0001:00015490       _BotAIPredictObstacles     20016490 f   ai_dmq3.obj
 0001:00015640       _BotCheckConsoleMessages   20016640 f   ai_dmq3.obj
 0001:00015a80       _BotCheckForGrenades       20016a80 f   ai_dmq3.obj
 0001:00015ad0       _BotCheckEvents            20016ad0 f   ai_dmq3.obj
 0001:00015f60       _BotCheckSnapshot          20016f60 f   ai_dmq3.obj
 0001:00016040       _BotCheckAir               20017040 f   ai_dmq3.obj
 0001:00016090       _BotAlternateRoute         20017090 f   ai_dmq3.obj
 0001:00016140       _BotGetAlternateRouteGoal  20017140 f   ai_dmq3.obj
 0001:00016280       _BotSetupAlternativeRouteGoals 20017280 f   ai_dmq3.obj
 0001:000162b0       _BotDeathmatchAI           200172b0 f   ai_dmq3.obj
 0001:00016680       _BotSetEntityNumForGoalWithModel 20017680 f   ai_dmq3.obj
 0001:00016760       _BotSetEntityNumForGoal    20017760 f   ai_dmq3.obj
 0001:00016820       _BotGoalForBSPEntity       20017820 f   ai_dmq3.obj
 0001:000169c0       _BotSetupDeathmatchAI      200179c0 f   ai_dmq3.obj
 0001:00016ba0       _BotShutdownDeathmatchAI   20017ba0 f   ai_dmq3.obj
 0001:00016bc0       _BotAI_Print               20017bc0 f   ai_main.obj
 0001:00016cc0       _BotAI_Trace               20017cc0 f   ai_main.obj
 0001:00016d90       _BotAI_GetClientState      20017d90 f   ai_main.obj
 0001:00016e00       _BotAI_GetEntityState      20017e00 f   ai_main.obj
 0001:00016e80       _BotAI_GetSnapshotEntity   20017e80 f   ai_main.obj
 0001:00016ee0       _BotAI_BotInitialChat      20017ee0 f   ai_main.obj
 0001:00016fb0       _BotTestAAS                20017fb0 f   ai_main.obj
 0001:00017090       _BotReportStatus           20018090 f   ai_main.obj
 0001:00017490       _BotTeamplayReport         20018490 f   ai_main.obj
 0001:00017680       _BotSetInfoConfigString    20018680 f   ai_main.obj
 0001:00017a40       _BotUpdateInfoConfigStrings 20018a40 f   ai_main.obj
 0001:00017b10       _BotInterbreedBots         20018b10 f   ai_main.obj
 0001:00017cd0       _BotWriteInterbreeded      20018cd0 f   ai_main.obj
 0001:00017da0       _BotInterbreedEndMatch     20018da0 f   ai_main.obj
 0001:00017e30       _BotInterbreeding          20018e30 f   ai_main.obj
 0001:00017f60       _BotEntityInfo             20018f60 f   ai_main.obj
 0001:00017f80       _NumBots                   20018f80 f   ai_main.obj
 0001:00017fa0       _BotTeamLeader             20018fa0 f   ai_main.obj
 0001:00018000       _AngleDifference           20019000 f   ai_main.obj
 0001:00018070       _BotChangeViewAngle        20019070 f   ai_main.obj
 0001:00018160       _BotChangeViewAngles       20019160 f   ai_main.obj
 0001:000184c0       _BotInputToUserCommand     200194c0 f   ai_main.obj
 0001:000188d0       _BotUpdateInput            200198d0 f   ai_main.obj
 0001:00018a10       _BotAIRegularUpdate        20019a10 f   ai_main.obj
 0001:00018a50       _RemoveColorEscapeSequences 20019a50 f   ai_main.obj
 0001:00018b00       _BotAI                     20019b00 f   ai_main.obj
 0001:00018f70       _BotScheduleBotThink       20019f70 f   ai_main.obj
 0001:00018ff0       _BotWriteSessionData       20019ff0 f   ai_main.obj
 0001:00019110       _BotReadSessionData        2001a110 f   ai_main.obj
 0001:00019210       _BotAISetupClient          2001a210 f   ai_main.obj
 0001:000196a0       _BotAIShutdownClient       2001a6a0 f   ai_main.obj
 0001:000197d0       _BotResetState             2001a7d0 f   ai_main.obj
 0001:00019a00       _BotAILoadMap              2001aa00 f   ai_main.obj
 0001:00019ab0       _BotAIStartFrame           2001aab0 f   ai_main.obj
 0001:0001a140       _BotInitLibrary            2001b140 f   ai_main.obj
 0001:0001a5f0       _BotAISetup                2001b5f0 f   ai_main.obj
 0001:0001a780       _BotAIShutdown             2001b780 f   ai_main.obj
 0001:0001a800       _BotValidTeamLeader        2001b800 f   ai_team.obj
 0001:0001a850       _BotNumTeamMates           2001b850 f   ai_team.obj
 0001:0001a950       _BotClientTravelTimeToGoal 2001b950 f   ai_team.obj
 0001:0001a9c0       _BotSortTeamMatesByBaseTravelTime 2001b9c0 f   ai_team.obj
 0001:0001abb0       _BotSetTeamMateTaskPreference 2001bbb0 f   ai_team.obj
 0001:0001ac00       _BotGetTeamMateTaskPreference 2001bc00 f   ai_team.obj
 0001:0001ac70       _BotSortTeamMatesByTaskPreference 2001bc70 f   ai_team.obj
 0001:0001ae20       _BotSayTeamOrderAlways     2001be20 f   ai_team.obj
 0001:0001aed0       _BotSayTeamOrder           2001bed0 f   ai_team.obj
 0001:0001aef0       _BotVoiceChat              2001bef0 f   ai_team.obj
 0001:0001af00       _BotVoiceChatOnly          2001bf00 f   ai_team.obj
 0001:0001af10       _BotSayVoiceTeamOrder      2001bf10 f   ai_team.obj
 0001:0001af20       _BotCTFOrders_BothFlagsNotAtBase 2001bf20 f   ai_team.obj
 0001:0001b4a0       _BotCTFOrders_FlagNotAtBase 2001c4a0 f   ai_team.obj
 0001:0001bc20       _BotCTFOrders_EnemyFlagNotAtBase 2001cc20 f   ai_team.obj
 0001:0001c100       _BotCTFOrders_BothFlagsAtBase 2001d100 f   ai_team.obj
 0001:0001c880       _BotCTFOrders              2001d880 f   ai_team.obj
 0001:0001c930       _BotCreateGroup            2001d930 f   ai_team.obj
 0001:0001c9f0       _BotTeamOrders             2001d9f0 f   ai_team.obj
 0001:0001cc40       _FindHumanTeamLeader       2001dc40 f   ai_team.obj
 0001:0001cd00       _BotTeamAI                 2001dd00 f   ai_team.obj
 0001:0001d1a0       _BotVoiceChat_GetFlag      2001e1a0 f   ai_vcmd.obj
 0001:0001d290       _BotVoiceChat_Offense      2001e290 f   ai_vcmd.obj
 0001:0001d370       _BotVoiceChat_Defend       2001e370 f   ai_vcmd.obj
 0001:0001d490       _BotVoiceChat_DefendFlag   2001e490 f   ai_vcmd.obj
 0001:0001d4c0       _BotVoiceChat_Patrol       2001e4c0 f   ai_vcmd.obj
 0001:0001d560       _BotVoiceChat_Camp         2001e560 f   ai_vcmd.obj
 0001:0001d750       _BotVoiceChat_FollowMe     2001e750 f   ai_vcmd.obj
 0001:0001d960       _BotVoiceChat_FollowFlagCarrier 2001e960 f   ai_vcmd.obj
 0001:0001d9b0       _BotVoiceChat_ReturnFlag   2001e9b0 f   ai_vcmd.obj
 0001:0001da70       _BotVoiceChat_StartLeader  2001ea70 f   ai_vcmd.obj
 0001:0001daa0       _BotVoiceChat_StopLeader   2001eaa0 f   ai_vcmd.obj
 0001:0001db00       _BotVoiceChat_WhoIsLeader  2001eb00 f   ai_vcmd.obj
 0001:0001dba0       _BotVoiceChat_WantOnDefense 2001eba0 f   ai_vcmd.obj
 0001:0001dc60       _BotVoiceChat_WantOnOffense 2001ec60 f   ai_vcmd.obj
 0001:0001dd20       _BotVoiceChat_Dummy        2001ed20 f   ai_vcmd.obj
 0001:0001dd30       _BotVoiceChatCommand       2001ed30 f   ai_vcmd.obj
 0001:0001df70       _BG_FindItemForPowerup     2001ef70 f   bg_misc.obj
 0001:0001dff0       _BG_FindItemForHoldable    2001eff0 f   bg_misc.obj
 0001:0001e060       _BG_FindItemForWeapon      2001f060 f   bg_misc.obj
 0001:0001e0c0       _BG_FindItem               2001f0c0 f   bg_misc.obj
 0001:0001e110       _BG_PlayerTouchesItem      2001f110 f   bg_misc.obj
 0001:0001e1d0       _BG_CanItemBeGrabbed       2001f1d0 f   bg_misc.obj
 0001:0001e400       _BG_EvaluateTrajectory     2001f400 f   bg_misc.obj
 0001:0001e660       _BG_EvaluateTrajectoryDelta 2001f660 f   bg_misc.obj
 0001:0001e820       _BG_AddPredictableEventToPlayerstate 2001f820 f   bg_misc.obj
 0001:0001e8d0       _BG_TouchJumpPad           2001f8d0 f   bg_misc.obj
 0001:0001e9c0       _BG_PlayerStateToEntityState 2001f9c0 f   bg_misc.obj
 0001:0001ed20       _BG_PlayerStateToEntityStateExtraPolate 2001fd20 f   bg_misc.obj
 0001:0001f090       _PM_AddEvent               20020090 f   bg_pmove.obj
 0001:0001f0c0       _PM_AddTouchEnt            200200c0 f   bg_pmove.obj
 0001:0001f150       _PM_ClipVelocity           20020150 f   bg_pmove.obj
 0001:0001f1f0       _PM_UpdateViewAngles       200201f0 f   bg_pmove.obj
 0001:0001f2f0       _PmoveSingle               200202f0 f   bg_pmove.obj
 0001:000226b0       _Pmove                     200236b0 f   bg_pmove.obj
 0001:000227a0       _PM_SlideMove              200237a0 f   bg_slidemove.obj
 0001:00023040       _PM_StepSlideMove          20024040 f   bg_slidemove.obj
 0001:00023460       _P_DamageFeedback          20024460 f   g_active.obj
 0001:000235f0       _P_WorldEffects            200245f0 f   g_active.obj
 0001:00023890       _G_SetClientSound          20024890 f   g_active.obj
 0001:000238f0       _ClientImpacts             200248f0 f   g_active.obj
 0001:000239f0       _G_TouchTriggers           200249f0 f   g_active.obj
 0001:00023d50       _SpectatorThink            20024d50 f   g_active.obj
 0001:00023ec0       _ClientInactivityTimer     20024ec0 f   g_active.obj
 0001:00024000       _ClientTimerActions        20025000 f   g_active.obj
 0001:000241b0       _ClientIntermissionThink   200251b0 f   g_active.obj
 0001:00024240       _ClientEvents              20025240 f   g_active.obj
 0001:000244e0       _SendPendingPredictableEvents 200254e0 f   g_active.obj
 0001:000245f0       _ClientThink_real          200255f0 f   g_active.obj
 0001:00024cf0       _ClientThink               20025cf0 f   g_active.obj
 0001:00024d70       _G_RunClient               20025d70 f   g_active.obj
 0001:00024dc0       _SpectatorClientEndFrame   20025dc0 f   g_active.obj
 0001:00024f50       _ClientEndFrame            20025f50 f   g_active.obj
 0001:000250d0       _UpdateTournamentInfo      200260d0 f   g_arenas.obj
 0001:00025370       _SpawnModelsOnVictoryPads  20026370 f   g_arenas.obj
 0001:00025f60       _Svcmd_AbortPodium_f       20026f60 f   g_arenas.obj
 0001:00025fb0       _trap_Cvar_VariableValue   20026fb0 f   g_bot.obj
 0001:00025ff0       _G_ParseInfos              20026ff0 f   g_bot.obj
 0001:000261c0       _G_GetArenaInfoByMap       200271c0 f   g_bot.obj
 0001:00026230       _G_AddRandomBot            20027230 f   g_bot.obj
 0001:000264d0       _G_RemoveRandomBot         200274d0 f   g_bot.obj
 0001:000265a0       _G_CountHumanPlayers       200275a0 f   g_bot.obj
 0001:00026640       _G_CountBotPlayers         20027640 f   g_bot.obj
 0001:00026720       _G_CheckMinimumPlayers     20027720 f   g_bot.obj
 0001:00026930       _G_CheckBotSpawn           20027930 f   g_bot.obj
 0001:00026a90       _G_RemoveQueuedBotBegin    20027a90 f   g_bot.obj
 0001:00026ae0       _G_BotConnect              20027ae0 f   g_bot.obj
 0001:00026bc0       _Svcmd_AddBot_f            20027bc0 f   g_bot.obj
 0001:00027260       _Svcmd_BotList_f           20028260 f   g_bot.obj
 0001:00027400       _G_GetBotInfoByNumber      20028400 f   g_bot.obj
 0001:00027450       _G_GetBotInfoByName        20028450 f   g_bot.obj
 0001:000274c0       _G_InitBots                200284c0 f   g_bot.obj
 0001:00027cd0       _SP_info_player_deathmatch 20028cd0 f   g_client.obj
 0001:00027d50       _SP_info_player_start      20028d50 f   g_client.obj
 0001:00027d80       _SP_info_player_intermission 20028d80 f   g_client.obj
 0001:00027d90       _SpotWouldTelefrag         20028d90 f   g_client.obj
 0001:00027e90       _SelectNearestDeathmatchSpawnPoint 20028e90 f   g_client.obj
 0001:00027f80       _SelectRandomDeathmatchSpawnPoint 20028f80 f   g_client.obj
 0001:00028020       _SelectRandomFurthestSpawnPoint 20029020 f   g_client.obj
 0001:00028380       _SelectSpawnPoint          20029380 f   g_client.obj
 0001:000283b0       _SelectInitialSpawnPoint   200293b0 f   g_client.obj
 0001:00028480       _SelectSpectatorSpawnPoint 20029480 f   g_client.obj
 0001:000284e0       _InitBodyQue               200294e0 f   g_client.obj
 0001:00028550       _BodySink                  20029550 f   g_client.obj
 0001:000285c0       _CopyToBodyQue             200295c0 f   g_client.obj
 0001:00028940       _SetClientViewAngle        20029940 f   g_client.obj
 0001:00028a20       _respawn                   20029a20 f   g_client.obj
 0001:00028a80       _TeamCount                 20029a80 f   g_client.obj
 0001:00028b10       _TeamLeader                20029b10 f   g_client.obj
 0001:00028ba0       _PickTeam                  20029ba0 f   g_client.obj
 0001:00028c10       _ClientUserinfoChanged     20029c10 f   g_client.obj
 0001:000293a0       _ClientConnect             2002a3a0 f   g_client.obj
 0001:000295d0       _ClientBegin               2002a5d0 f   g_client.obj
 0001:00029720       _ClientSpawn               2002a720 f   g_client.obj
 0001:00029ea0       _ClientDisconnect          2002aea0 f   g_client.obj
 0001:0002a0e0       _DeathmatchScoreboardMessage 2002b0e0 f   g_cmds.obj
 0001:0002a3b0       _Cmd_Score_f               2002b3b0 f   g_cmds.obj
 0001:0002a3d0       _CheatsOk                  2002b3d0 f   g_cmds.obj
 0001:0002a450       _ConcatArgs                2002b450 f   g_cmds.obj
 0001:0002a520       _SanitizeString            2002b520 f   g_cmds.obj
 0001:0002a5a0       _ClientNumberFromString    2002b5a0 f   g_cmds.obj
 0001:0002a740       _Cmd_Give_f                2002b740 f   g_cmds.obj
 0001:0002aa90       _Cmd_God_f                 2002ba90 f   g_cmds.obj
 0001:0002ab10       _Cmd_Notarget_f            2002bb10 f   g_cmds.obj
 0001:0002ab90       _Cmd_Noclip_f              2002bb90 f   g_cmds.obj
 0001:0002ac30       _Cmd_LevelShot_f           2002bc30 f   g_cmds.obj
 0001:0002aca0       _Cmd_TeamTask_f            2002bca0 f   g_cmds.obj
 0001:0002ad80       _Cmd_Kill_f                2002bd80 f   g_cmds.obj
 0001:0002ae10       _BroadcastTeamChange       2002be10 f   g_cmds.obj
 0001:0002aef0       _SetTeam                   2002bef0 f   g_cmds.obj
 0001:0002b300       _StopFollowing             2002c300 f   g_cmds.obj
 0001:0002b3a0       _Cmd_Team_f                2002c3a0 f   g_cmds.obj
 0001:0002b540       _Cmd_Follow_f              2002c540 f   g_cmds.obj
 0001:0002b680       _Cmd_FollowCycle_f         2002c680 f   g_cmds.obj
 0001:0002b7c0       _G_Say                     2002c7c0 f   g_cmds.obj
 0001:0002bb50       _G_Voice                   2002cb50 f   g_cmds.obj
 0001:0002bcf0       _Cmd_GameCommand_f         2002ccf0 f   g_cmds.obj
 0001:0002bdc0       _Cmd_Where_f               2002cdc0 f   g_cmds.obj
 0001:0002be10       _Cmd_CallVote_f            2002ce10 f   g_cmds.obj
 0001:0002c430       _Cmd_Vote_f                2002d430 f   g_cmds.obj
 0001:0002c5a0       _Cmd_CallTeamVote_f        2002d5a0 f   g_cmds.obj
 0001:0002cc30       _Cmd_TeamVote_f            2002dc30 f   g_cmds.obj
 0001:0002ce00       _Cmd_SetViewpos_f          2002de00 f   g_cmds.obj
 0001:0002cf30       _Cmd_Stats_f               2002df30 f   g_cmds.obj
 0001:0002cf40       _ClientCommand             2002df40 f   g_cmds.obj
 0001:0002daa0       _ScorePlum                 2002eaa0 f   g_combat.obj
 0001:0002db00       _AddScore                  2002eb00 f   g_combat.obj
 0001:0002dba0       _TossClientItems           2002eba0 f   g_combat.obj
 0001:0002dd20       _LookAtKiller              2002ed20 f   g_combat.obj
 0001:0002de10       _GibEntity                 2002ee10 f   g_combat.obj
 0001:0002dee0       _body_die                  2002eee0 f   g_combat.obj
 0001:0002df30       _CheckAlmostCapture        2002ef30 f   g_combat.obj
 0001:0002e120       _CheckAlmostScored         2002f120 f   g_combat.obj
 0001:0002e230       _player_die                2002f230 f   g_combat.obj
 0001:0002e990       _CheckArmor                2002f990 f   g_combat.obj
 0001:0002ea30       _RaySphereIntersections    2002fa30 f   g_combat.obj
 0001:0002ec40       _G_Damage                  2002fc40 f   g_combat.obj
 0001:0002f280       _CanDamage                 20030280 f   g_combat.obj
 0001:0002f500       _G_RadiusDamage            20030500 f   g_combat.obj
 0001:0002f7f0       _Pickup_Powerup            200307f0 f   g_items.obj
 0001:0002fa30       _Pickup_Holdable           20030a30 f   g_items.obj
 0001:0002faa0       _Add_Ammo                  20030aa0 f   g_items.obj
 0001:0002fb10       _Pickup_Ammo               20030b10 f   g_items.obj
 0001:0002fb70       _Pickup_Weapon             20030b70 f   g_items.obj
 0001:0002fcc0       _Pickup_Health             20030cc0 f   g_items.obj
 0001:0002fdb0       _Pickup_Armor              20030db0 f   g_items.obj
 0001:0002fe40       _RespawnItem               20030e40 f   g_items.obj
 0001:00030050       _Touch_Item                20031050 f   g_items.obj
 0001:00030460       _LaunchItem                20031460 f   g_items.obj
 0001:00030600       _Drop_Item                 20031600 f   g_items.obj
 0001:000306c0       _Use_Item                  200316c0 f   g_items.obj
 0001:000306e0       _FinishSpawningItem        200316e0 f   g_items.obj
 0001:00030960       _G_CheckTeamItems          20031960 f   g_items.obj
 0001:00030a00       _ClearRegisteredItems      20031a00 f   g_items.obj
 0001:00030a50       _RegisterItem              20031a50 f   g_items.obj
 0001:00030a90       _SaveRegisteredItems       20031a90 f   g_items.obj
 0001:00030b50       _G_ItemDisabled            20031b50 f   g_items.obj
 0001:00030b90       _G_SpawnItem               20031b90 f   g_items.obj
 0001:00030c60       _G_BounceItem              20031c60 f   g_items.obj
 0001:00030e80       _G_RunItem                 20031e80 f   g_items.obj
 0001:00031010       _vmMain                    20032010 f   g_main.obj
 0001:00031130       _G_Printf                  20032130 f   g_main.obj
 0001:00031180       _G_Error                   20032180 f   g_main.obj
 0001:000311d0       _G_FindTeams               200321d0 f   g_main.obj
 0001:000313a0       _G_RemapTeamShaders        200323a0 f   g_main.obj
 0001:000313b0       _G_RegisterCvars           200323b0 f   g_main.obj
 0001:00031490       _G_UpdateCvars             20032490 f   g_main.obj
 0001:00031560       _G_InitGame                20032560 f   g_main.obj
 0001:00031810       _G_ShutdownGame            20032810 f   g_main.obj
 0001:00031880       _Com_Error                 20032880 f   g_main.obj
 0001:000318d0       _Com_Printf                200328d0 f   g_main.obj
 0001:00031920       _AddTournamentPlayer       20032920 f   g_main.obj
 0001:00031a20       _RemoveTournamentLoser     20032a20 f   g_main.obj
 0001:00031a80       _RemoveTournamentWinner    20032a80 f   g_main.obj
 0001:00031ae0       _AdjustTournamentScores    20032ae0 f   g_main.obj
 0001:00031bb0       _SortRanks                 20032bb0 f   g_main.obj
 0001:00031d00       _CalculateRanks            20032d00 f   g_main.obj
 0001:000321e0       _SendScoreboardMessageToAllClients 200331e0 f   g_main.obj
 0001:00032240       _MoveClientToIntermission  20033240 f   g_main.obj
 0001:00032390       _FindIntermissionPoint     20033390 f   g_main.obj
 0001:00032490       _BeginIntermission         20033490 f   g_main.obj
 0001:00032550       _ExitLevel                 20033550 f   g_main.obj
 0001:00032690       _G_LogPrintf               20033690 f   g_main.obj
 0001:000327b0       _LogExit                   200337b0 f   g_main.obj
 0001:000328e0       _CheckIntermissionExit     200338e0 f   g_main.obj
 0001:00032a60       _ScoreIsTied               20033a60 f   g_main.obj
 0001:00032ae0       _CheckExitRules            20033ae0 f   g_main.obj
 0001:00032d10       _CheckTournament           20033d10 f   g_main.obj
 0001:00032fe0       _CheckVote                 20033fe0 f   g_main.obj
 0001:000330d0       _PrintTeam                 200340d0 f   g_main.obj
 0001:00033130       _SetLeader                 20034130 f   g_main.obj
 0001:000332c0       _CheckTeamLeader           200342c0 f   g_main.obj
 0001:00033400       _CheckTeamVote             20034400 f   g_main.obj
 0001:00033560       _CheckCvars                20034560 f   g_main.obj
 0001:000335d0       _G_RunThink                200345d0 f   g_main.obj
 0001:00033650       _G_RunFrame                20034650 f   g_main.obj
 0001:00033920       _G_Alloc                   20034920 f   g_mem.obj
 0001:000339b0       _G_InitMemory              200349b0 f   g_mem.obj
 0001:000339d0       _Svcmd_GameMem_f           200349d0 f   g_mem.obj
 0001:00033a00       _SP_info_camp              20034a00 f   g_misc.obj
 0001:00033a30       _SP_info_null              20034a30 f   g_misc.obj
 0001:00033a50       _SP_info_notnull           20034a50 f   g_misc.obj
 0001:00033a80       _SP_light                  20034a80 f   g_misc.obj
 0001:00033aa0       _TeleportPlayer            20034aa0 f   g_misc.obj
 0001:00033cd0       _SP_misc_teleporter_dest   20034cd0 f   g_misc.obj
 0001:00033ce0       _SP_misc_model             20034ce0 f   g_misc.obj
 0001:00033d00       _locateCamera              20034d00 f   g_misc.obj
 0001:00033e70       _SP_misc_portal_surface    20034e70 f   g_misc.obj
 0001:00033f50       _SP_misc_portal_camera     20034f50 f   g_misc.obj
 0001:00033ff0       _Use_Shooter               20034ff0 f   g_misc.obj
 0001:00034240       _InitShooter               20035240 f   g_misc.obj
 0001:00034370       _SP_shooter_rocket         20035370 f   g_misc.obj
 0001:00034390       _SP_shooter_plasma         20035390 f   g_misc.obj
 0001:000343b0       _SP_shooter_grenade        200353b0 f   g_misc.obj
 0001:000343d0       _G_BounceMissile           200353d0 f   g_missile.obj
 0001:000345f0       _G_ExplodeMissile          200355f0 f   g_missile.obj
 0001:00034740       _G_MissileImpact           20035740 f   g_missile.obj
 0001:00034c80       _G_RunMissile              20035c80 f   g_missile.obj
 0001:00034e30       _fire_plasma               20035e30 f   g_missile.obj
 0001:00035000       _fire_grenade              20036000 f   g_missile.obj
 0001:000351e0       _fire_bfg                  200361e0 f   g_missile.obj
 0001:000353b0       _fire_rocket               200363b0 f   g_missile.obj
 0001:00035580       _fire_grapple              20036580 f   g_missile.obj
 0001:00035740       _G_TestEntityPosition      20036740 f   g_mover.obj
 0001:00035820       _G_CreateRotationMatrix    20036820 f   g_mover.obj
 0001:00035860       _G_TransposeMatrix         20036860 f   g_mover.obj
 0001:000358d0       _G_RotatePoint             200368d0 f   g_mover.obj
 0001:00035970       _G_TryPushingEntity        20036970 f   g_mover.obj
 0001:00035eb0       _G_CheckProxMinePosition   20036eb0 f   g_mover.obj
 0001:00035f90       _G_TryPushingProxMine      20036f90 f   g_mover.obj
 0001:00036140       _G_MoverPush               20037140 f   g_mover.obj
 0001:000366e0       _G_MoverTeam               200376e0 f   g_mover.obj
 0001:000368f0       _G_RunMover                200378f0 f   g_mover.obj
 0001:00036940       _SetMoverState             20037940 f   g_mover.obj
 0001:00036b90       _MatchTeam                 20037b90 f   g_mover.obj
 0001:00036bd0       _ReturnToPos1              20037bd0 f   g_mover.obj
 0001:00036c30       _Reached_BinaryMover       20037c30 f   g_mover.obj
 0001:00036d70       _Use_BinaryMover           20037d70 f   g_mover.obj
 0001:00036f60       _InitMover                 20037f60 f   g_mover.obj
 0001:00037290       _Blocked_Door              20038290 f   g_mover.obj
 0001:00037350       _Touch_DoorTrigger         20038350 f   g_mover.obj
 0001:00037540       _Think_SpawnNewDoorTrigger 20038540 f   g_mover.obj
 0001:00037750       _Think_MatchTeam           20038750 f   g_mover.obj
 0001:00037780       _SP_func_door              20038780 f   g_mover.obj
 0001:00037af0       _Touch_Plat                20038af0 f   g_mover.obj
 0001:00037b40       _Touch_PlatCenterTrigger   20038b40 f   g_mover.obj
 0001:00037b90       _SpawnPlatTrigger          20038b90 f   g_mover.obj
 0001:00037d50       _SP_func_plat              20038d50 f   g_mover.obj
 0001:00037f50       _Touch_Button              20038f50 f   g_mover.obj
 0001:00037f90       _SP_func_button            20038f90 f   g_mover.obj
 0001:000381c0       _Think_BeginMoving         200391c0 f   g_mover.obj
 0001:000381f0       _Reached_Train             200391f0 f   g_mover.obj
 0001:000383e0       _Think_SetupTrainTargets   200393e0 f   g_mover.obj
 0001:00038530       _SP_path_corner            20039530 f   g_mover.obj
 0001:00038580       _SP_func_train             20039580 f   g_mover.obj
 0001:00038690       _SP_func_static            20039690 f   g_mover.obj
 0001:00038720       _SP_func_rotating          20039720 f   g_mover.obj
 0001:00038880       _SP_func_bobbing           20039880 f   g_mover.obj
 0001:000389e0       _SP_func_pendulum          200399e0 f   g_mover.obj
 0001:00038b80       _G_WriteClientSessionData  20039b80 f   g_session.obj
 0001:00038c20       _G_ReadSessionData         20039c20 f   g_session.obj
 0001:00038cf0       _G_InitSessionData         20039cf0 f   g_session.obj
 0001:00038df0       _G_InitWorldSession        20039df0 f   g_session.obj
 0001:00038e60       _G_WriteSessionData        20039e60 f   g_session.obj
 0001:00038ef0       _G_SpawnString             20039ef0 f   g_spawn.obj
 0001:00038f70       _G_SpawnFloat              20039f70 f   g_spawn.obj
 0001:00038fb0       _G_SpawnInt                20039fb0 f   g_spawn.obj
 0001:00038ff0       _G_SpawnVector             20039ff0 f   g_spawn.obj
 0001:00039040       _SP_item_botroam           2003a040 f   g_spawn.obj
 0001:00039050       _G_CallSpawn               2003a050 f   g_spawn.obj
 0001:00039140       _G_NewString               2003a140 f   g_spawn.obj
 0001:00039200       _G_ParseField              2003a200 f   g_spawn.obj
 0001:00039370       _G_SpawnGEntityFromSpawnVars 2003a370 f   g_spawn.obj
 0001:00039560       _G_AddSpawnVarToken        2003a560 f   g_spawn.obj
 0001:000395e0       _G_ParseSpawnVars          2003a5e0 f   g_spawn.obj
 0001:00039730       _SP_worldspawn             2003a730 f   g_spawn.obj
 0001:00039900       _G_SpawnEntitiesFromString 2003a900 f   g_spawn.obj
 0001:00039960       _G_FilterPacket            2003a960 f   g_svcmds.obj
 0001:00039a60       _G_ProcessIPBans           2003aa60 f   g_svcmds.obj
 0001:00039eb0       _Svcmd_AddIP_f             2003aeb0 f   g_svcmds.obj
 0001:00039f10       _Svcmd_RemoveIP_f          2003af10 f   g_svcmds.obj
 0001:00039ff0       _Svcmd_EntityList_f        2003aff0 f   g_svcmds.obj
 0001:0003a1b0       _ClientForString           2003b1b0 f   g_svcmds.obj
 0001:0003a2c0       _Svcmd_ForceTeam_f         2003b2c0 f   g_svcmds.obj
 0001:0003a350       _ConsoleCommand            2003b350 f   g_svcmds.obj
 0001:0003a560       _dllEntry                  2003b560 f   g_syscalls.obj
 0001:0003a580       _PASSFLOAT                 2003b580 f   g_syscalls.obj
 0001:0003a5a0       _trap_Printf               2003b5a0 f   g_syscalls.obj
 0001:0003a5c0       _trap_Error                2003b5c0 f   g_syscalls.obj
 0001:0003a5e0       _trap_Milliseconds         2003b5e0 f   g_syscalls.obj
 0001:0003a600       _trap_Argc                 2003b600 f   g_syscalls.obj
 0001:0003a620       _trap_Argv                 2003b620 f   g_syscalls.obj
 0001:0003a650       _trap_FS_FOpenFile         2003b650 f   g_syscalls.obj
 0001:0003a680       _trap_FS_Read              2003b680 f   g_syscalls.obj
 0001:0003a6b0       _trap_FS_Write             2003b6b0 f   g_syscalls.obj
 0001:0003a6e0       _trap_FS_FCloseFile        2003b6e0 f   g_syscalls.obj
 0001:0003a700       _trap_FS_GetFileList       2003b700 f   g_syscalls.obj
 0001:0003a730       _trap_FS_Seek              2003b730 f   g_syscalls.obj
 0001:0003a760       _trap_SendConsoleCommand   2003b760 f   g_syscalls.obj
 0001:0003a790       _trap_Cvar_Register        2003b790 f   g_syscalls.obj
 0001:0003a7c0       _trap_Cvar_Update          2003b7c0 f   g_syscalls.obj
 0001:0003a7e0       _trap_Cvar_Set             2003b7e0 f   g_syscalls.obj
 0001:0003a810       _trap_Cvar_VariableIntegerValue 2003b810 f   g_syscalls.obj
 0001:0003a830       _trap_Cvar_VariableStringBuffer 2003b830 f   g_syscalls.obj
 0001:0003a860       _trap_LocateGameData       2003b860 f   g_syscalls.obj
 0001:0003a890       _trap_DropClient           2003b890 f   g_syscalls.obj
 0001:0003a8c0       _trap_SendServerCommand    2003b8c0 f   g_syscalls.obj
 0001:0003a8f0       _trap_SetConfigstring      2003b8f0 f   g_syscalls.obj
 0001:0003a920       _trap_GetConfigstring      2003b920 f   g_syscalls.obj
 0001:0003a950       _trap_GetUserinfo          2003b950 f   g_syscalls.obj
 0001:0003a980       _trap_SetUserinfo          2003b980 f   g_syscalls.obj
 0001:0003a9b0       _trap_GetServerinfo        2003b9b0 f   g_syscalls.obj
 0001:0003a9e0       _trap_SetBrushModel        2003b9e0 f   g_syscalls.obj
 0001:0003aa10       _trap_Trace                2003ba10 f   g_syscalls.obj
 0001:0003aa50       _trap_TraceCapsule         2003ba50 f   g_syscalls.obj
 0001:0003aa90       _trap_PointContents        2003ba90 f   g_syscalls.obj
 0001:0003aac0       _trap_InPVS                2003bac0 f   g_syscalls.obj
 0001:0003aaf0       _trap_InPVSIgnorePortals   2003baf0 f   g_syscalls.obj
 0001:0003ab20       _trap_AdjustAreaPortalState 2003bb20 f   g_syscalls.obj
 0001:0003ab50       _trap_AreasConnected       2003bb50 f   g_syscalls.obj
 0001:0003ab80       _trap_LinkEntity           2003bb80 f   g_syscalls.obj
 0001:0003aba0       _trap_UnlinkEntity         2003bba0 f   g_syscalls.obj
 0001:0003abc0       _trap_EntitiesInBox        2003bbc0 f   g_syscalls.obj
 0001:0003abf0       _trap_EntityContact        2003bbf0 f   g_syscalls.obj
 0001:0003ac20       _trap_EntityContactCapsule 2003bc20 f   g_syscalls.obj
 0001:0003ac50       _trap_BotAllocateClient    2003bc50 f   g_syscalls.obj
 0001:0003ac70       _trap_BotFreeClient        2003bc70 f   g_syscalls.obj
 0001:0003ac90       _trap_GetUsercmd           2003bc90 f   g_syscalls.obj
 0001:0003acc0       _trap_GetEntityToken       2003bcc0 f   g_syscalls.obj
 0001:0003acf0       _trap_DebugPolygonCreate   2003bcf0 f   g_syscalls.obj
 0001:0003ad20       _trap_DebugPolygonDelete   2003bd20 f   g_syscalls.obj
 0001:0003ad40       _trap_RealTime             2003bd40 f   g_syscalls.obj
 0001:0003ad60       _trap_SnapVector           2003bd60 f   g_syscalls.obj
 0001:0003ad80       _trap_BotLibSetup          2003bd80 f   g_syscalls.obj
 0001:0003ada0       _trap_BotLibShutdown       2003bda0 f   g_syscalls.obj
 0001:0003adc0       _trap_BotLibVarSet         2003bdc0 f   g_syscalls.obj
 0001:0003adf0       _trap_BotLibVarGet         2003bdf0 f   g_syscalls.obj
 0001:0003ae20       _trap_BotLibDefine         2003be20 f   g_syscalls.obj
 0001:0003ae50       _trap_BotLibStartFrame     2003be50 f   g_syscalls.obj
 0001:0003ae80       _trap_BotLibLoadMap        2003be80 f   g_syscalls.obj
 0001:0003aeb0       _trap_BotLibUpdateEntity   2003beb0 f   g_syscalls.obj
 0001:0003aee0       _trap_BotLibTest           2003bee0 f   g_syscalls.obj
 0001:0003af10       _trap_BotGetSnapshotEntity 2003bf10 f   g_syscalls.obj
 0001:0003af40       _trap_BotGetServerCommand  2003bf40 f   g_syscalls.obj
 0001:0003af70       _trap_BotUserCommand       2003bf70 f   g_syscalls.obj
 0001:0003afa0       _trap_AAS_EntityInfo       2003bfa0 f   g_syscalls.obj
 0001:0003afd0       _trap_AAS_Initialized      2003bfd0 f   g_syscalls.obj
 0001:0003aff0       _trap_AAS_PresenceTypeBoundingBox 2003bff0 f   g_syscalls.obj
 0001:0003b020       _trap_AAS_Time             2003c020 f   g_syscalls.obj
 0001:0003b050       _trap_AAS_PointAreaNum     2003c050 f   g_syscalls.obj
 0001:0003b080       _trap_AAS_PointReachabilityAreaIndex 2003c080 f   g_syscalls.obj
 0001:0003b0b0       _trap_AAS_TraceAreas       2003c0b0 f   g_syscalls.obj
 0001:0003b0f0       _trap_AAS_BBoxAreas        2003c0f0 f   g_syscalls.obj
 0001:0003b120       _trap_AAS_AreaInfo         2003c120 f   g_syscalls.obj
 0001:0003b150       _trap_AAS_PointContents    2003c150 f   g_syscalls.obj
 0001:0003b180       _trap_AAS_NextBSPEntity    2003c180 f   g_syscalls.obj
 0001:0003b1b0       _trap_AAS_ValueForBSPEpairKey 2003c1b0 f   g_syscalls.obj
 0001:0003b1e0       _trap_AAS_VectorForBSPEpairKey 2003c1e0 f   g_syscalls.obj
 0001:0003b210       _trap_AAS_FloatForBSPEpairKey 2003c210 f   g_syscalls.obj
 0001:0003b240       _trap_AAS_IntForBSPEpairKey 2003c240 f   g_syscalls.obj
 0001:0003b270       _trap_AAS_AreaReachability 2003c270 f   g_syscalls.obj
 0001:0003b2a0       _trap_AAS_AreaTravelTimeToGoalArea 2003c2a0 f   g_syscalls.obj
 0001:0003b2d0       _trap_AAS_EnableRoutingArea 2003c2d0 f   g_syscalls.obj
 0001:0003b300       _trap_AAS_PredictRoute     2003c300 f   g_syscalls.obj
 0001:0003b350       _trap_AAS_AlternativeRouteGoals 2003c350 f   g_syscalls.obj
 0001:0003b390       _trap_AAS_Swimming         2003c390 f   g_syscalls.obj
 0001:0003b3c0       _trap_AAS_PredictClientMovement 2003c3c0 f   g_syscalls.obj
 0001:0003b420       _trap_EA_Say               2003c420 f   g_syscalls.obj
 0001:0003b450       _trap_EA_SayTeam           2003c450 f   g_syscalls.obj
 0001:0003b480       _trap_EA_Command           2003c480 f   g_syscalls.obj
 0001:0003b4b0       _trap_EA_Action            2003c4b0 f   g_syscalls.obj
 0001:0003b4e0       _trap_EA_Gesture           2003c4e0 f   g_syscalls.obj
 0001:0003b510       _trap_EA_Talk              2003c510 f   g_syscalls.obj
 0001:0003b540       _trap_EA_Attack            2003c540 f   g_syscalls.obj
 0001:0003b570       _trap_EA_Use               2003c570 f   g_syscalls.obj
 0001:0003b5a0       _trap_EA_Respawn           2003c5a0 f   g_syscalls.obj
 0001:0003b5d0       _trap_EA_Crouch            2003c5d0 f   g_syscalls.obj
 0001:0003b600       _trap_EA_MoveUp            2003c600 f   g_syscalls.obj
 0001:0003b630       _trap_EA_MoveDown          2003c630 f   g_syscalls.obj
 0001:0003b660       _trap_EA_MoveForward       2003c660 f   g_syscalls.obj
 0001:0003b690       _trap_EA_MoveBack          2003c690 f   g_syscalls.obj
 0001:0003b6c0       _trap_EA_MoveLeft          2003c6c0 f   g_syscalls.obj
 0001:0003b6f0       _trap_EA_MoveRight         2003c6f0 f   g_syscalls.obj
 0001:0003b720       _trap_EA_SelectWeapon      2003c720 f   g_syscalls.obj
 0001:0003b750       _trap_EA_Jump              2003c750 f   g_syscalls.obj
 0001:0003b780       _trap_EA_DelayedJump       2003c780 f   g_syscalls.obj
 0001:0003b7b0       _trap_EA_Move              2003c7b0 f   g_syscalls.obj
 0001:0003b7f0       _trap_EA_View              2003c7f0 f   g_syscalls.obj
 0001:0003b820       _trap_EA_EndRegular        2003c820 f   g_syscalls.obj
 0001:0003b850       _trap_EA_GetInput          2003c850 f   g_syscalls.obj
 0001:0003b890       _trap_EA_ResetInput        2003c890 f   g_syscalls.obj
 0001:0003b8c0       _trap_BotLoadCharacter     2003c8c0 f   g_syscalls.obj
 0001:0003b8f0       _trap_BotFreeCharacter     2003c8f0 f   g_syscalls.obj
 0001:0003b920       _trap_Characteristic_Float 2003c920 f   g_syscalls.obj
 0001:0003b950       _trap_Characteristic_BFloat 2003c950 f   g_syscalls.obj
 0001:0003b9a0       _trap_Characteristic_Integer 2003c9a0 f   g_syscalls.obj
 0001:0003b9d0       _trap_Characteristic_BInteger 2003c9d0 f   g_syscalls.obj
 0001:0003ba00       _trap_Characteristic_String 2003ca00 f   g_syscalls.obj
 0001:0003ba30       _trap_BotAllocChatState    2003ca30 f   g_syscalls.obj
 0001:0003ba50       _trap_BotFreeChatState     2003ca50 f   g_syscalls.obj
 0001:0003ba80       _trap_BotQueueConsoleMessage 2003ca80 f   g_syscalls.obj
 0001:0003bab0       _trap_BotRemoveConsoleMessage 2003cab0 f   g_syscalls.obj
 0001:0003bae0       _trap_BotNextConsoleMessage 2003cae0 f   g_syscalls.obj
 0001:0003bb10       _trap_BotNumConsoleMessages 2003cb10 f   g_syscalls.obj
 0001:0003bb40       _trap_BotInitialChat       2003cb40 f   g_syscalls.obj
 0001:0003bb90       _trap_BotNumInitialChats   2003cb90 f   g_syscalls.obj
 0001:0003bbc0       _trap_BotReplyChat         2003cbc0 f   g_syscalls.obj
 0001:0003bc10       _trap_BotChatLength        2003cc10 f   g_syscalls.obj
 0001:0003bc40       _trap_BotEnterChat         2003cc40 f   g_syscalls.obj
 0001:0003bc70       _trap_BotGetChatMessage    2003cc70 f   g_syscalls.obj
 0001:0003bca0       _trap_StringContains       2003cca0 f   g_syscalls.obj
 0001:0003bcd0       _trap_BotFindMatch         2003ccd0 f   g_syscalls.obj
 0001:0003bd00       _trap_BotMatchVariable     2003cd00 f   g_syscalls.obj
 0001:0003bd30       _trap_UnifyWhiteSpaces     2003cd30 f   g_syscalls.obj
 0001:0003bd60       _trap_BotReplaceSynonyms   2003cd60 f   g_syscalls.obj
 0001:0003bd90       _trap_BotLoadChatFile      2003cd90 f   g_syscalls.obj
 0001:0003bdc0       _trap_BotSetChatGender     2003cdc0 f   g_syscalls.obj
 0001:0003bdf0       _trap_BotSetChatName       2003cdf0 f   g_syscalls.obj
 0001:0003be20       _trap_BotResetGoalState    2003ce20 f   g_syscalls.obj
 0001:0003be50       _trap_BotResetAvoidGoals   2003ce50 f   g_syscalls.obj
 0001:0003be80       _trap_BotRemoveFromAvoidGoals 2003ce80 f   g_syscalls.obj
 0001:0003beb0       _trap_BotPushGoal          2003ceb0 f   g_syscalls.obj
 0001:0003bee0       _trap_BotPopGoal           2003cee0 f   g_syscalls.obj
 0001:0003bf10       _trap_BotEmptyGoalStack    2003cf10 f   g_syscalls.obj
 0001:0003bf40       _trap_BotDumpAvoidGoals    2003cf40 f   g_syscalls.obj
 0001:0003bf70       _trap_BotDumpGoalStack     2003cf70 f   g_syscalls.obj
 0001:0003bfa0       _trap_BotGoalName          2003cfa0 f   g_syscalls.obj
 0001:0003bfd0       _trap_BotGetTopGoal        2003cfd0 f   g_syscalls.obj
 0001:0003c000       _trap_BotGetSecondGoal     2003d000 f   g_syscalls.obj
 0001:0003c030       _trap_BotChooseLTGItem     2003d030 f   g_syscalls.obj
 0001:0003c060       _trap_BotChooseNBGItem     2003d060 f   g_syscalls.obj
 0001:0003c0a0       _trap_BotTouchingGoal      2003d0a0 f   g_syscalls.obj
 0001:0003c0d0       _trap_BotItemGoalInVisButNotVisible 2003d0d0 f   g_syscalls.obj
 0001:0003c100       _trap_BotGetLevelItemGoal  2003d100 f   g_syscalls.obj
 0001:0003c130       _trap_BotGetNextCampSpotGoal 2003d130 f   g_syscalls.obj
 0001:0003c160       _trap_BotGetMapLocationGoal 2003d160 f   g_syscalls.obj
 0001:0003c190       _trap_BotAvoidGoalTime     2003d190 f   g_syscalls.obj
 0001:0003c1c0       _trap_BotSetAvoidGoalTime  2003d1c0 f   g_syscalls.obj
 0001:0003c200       _trap_BotInitLevelItems    2003d200 f   g_syscalls.obj
 0001:0003c220       _trap_BotUpdateEntityItems 2003d220 f   g_syscalls.obj
 0001:0003c240       _trap_BotLoadItemWeights   2003d240 f   g_syscalls.obj
 0001:0003c270       _trap_BotFreeItemWeights   2003d270 f   g_syscalls.obj
 0001:0003c2a0       _trap_BotInterbreedGoalFuzzyLogic 2003d2a0 f   g_syscalls.obj
 0001:0003c2d0       _trap_BotSaveGoalFuzzyLogic 2003d2d0 f   g_syscalls.obj
 0001:0003c300       _trap_BotMutateGoalFuzzyLogic 2003d300 f   g_syscalls.obj
 0001:0003c330       _trap_BotAllocGoalState    2003d330 f   g_syscalls.obj
 0001:0003c360       _trap_BotFreeGoalState     2003d360 f   g_syscalls.obj
 0001:0003c390       _trap_BotResetMoveState    2003d390 f   g_syscalls.obj
 0001:0003c3c0       _trap_BotAddAvoidSpot      2003d3c0 f   g_syscalls.obj
 0001:0003c400       _trap_BotMoveToGoal        2003d400 f   g_syscalls.obj
 0001:0003c430       _trap_BotMoveInDirection   2003d430 f   g_syscalls.obj
 0001:0003c470       _trap_BotResetAvoidReach   2003d470 f   g_syscalls.obj
 0001:0003c4a0       _trap_BotResetLastAvoidReach 2003d4a0 f   g_syscalls.obj
 0001:0003c4d0       _trap_BotReachabilityArea  2003d4d0 f   g_syscalls.obj
 0001:0003c500       _trap_BotMovementViewTarget 2003d500 f   g_syscalls.obj
 0001:0003c540       _trap_BotPredictVisiblePosition 2003d540 f   g_syscalls.obj
 0001:0003c580       _trap_BotAllocMoveState    2003d580 f   g_syscalls.obj
 0001:0003c5a0       _trap_BotFreeMoveState     2003d5a0 f   g_syscalls.obj
 0001:0003c5d0       _trap_BotInitMoveState     2003d5d0 f   g_syscalls.obj
 0001:0003c600       _trap_BotChooseBestFightWeapon 2003d600 f   g_syscalls.obj
 0001:0003c630       _trap_BotGetWeaponInfo     2003d630 f   g_syscalls.obj
 0001:0003c660       _trap_BotLoadWeaponWeights 2003d660 f   g_syscalls.obj
 0001:0003c690       _trap_BotAllocWeaponState  2003d690 f   g_syscalls.obj
 0001:0003c6b0       _trap_BotFreeWeaponState   2003d6b0 f   g_syscalls.obj
 0001:0003c6e0       _trap_BotResetWeaponState  2003d6e0 f   g_syscalls.obj
 0001:0003c710       _trap_GeneticParentsAndChildSelection 2003d710 f   g_syscalls.obj
 0001:0003c750       _trap_PC_LoadSource        2003d750 f   g_syscalls.obj
 0001:0003c780       _trap_PC_FreeSource        2003d780 f   g_syscalls.obj
 0001:0003c7b0       _trap_PC_ReadToken         2003d7b0 f   g_syscalls.obj
 0001:0003c7e0       _trap_PC_SourceFileAndLine 2003d7e0 f   g_syscalls.obj
 0001:0003c810       _Use_Target_Give           2003d810 f   g_target.obj
 0001:0003c8c0       _SP_target_give            2003d8c0 f   g_target.obj
 0001:0003c8e0       _Use_target_remove_powerups 2003d8e0 f   g_target.obj
 0001:0003c980       _SP_target_remove_powerups 2003d980 f   g_target.obj
 0001:0003c9a0       _Think_Target_Delay        2003d9a0 f   g_target.obj
 0001:0003c9d0       _Use_Target_Delay          2003d9d0 f   g_target.obj
 0001:0003ca60       _SP_target_delay           2003da60 f   g_target.obj
 0001:0003cae0       _Use_Target_Score          2003dae0 f   g_target.obj
 0001:0003cb10       _SP_target_score           2003db10 f   g_target.obj
 0001:0003cb50       _Use_Target_Print          2003db50 f   g_target.obj
 0001:0003cc50       _SP_target_print           2003dc50 f   g_target.obj
 0001:0003cc70       _Use_Target_Speaker        2003dc70 f   g_target.obj
 0001:0003cd30       _SP_target_speaker         2003dd30 f   g_target.obj
 0001:0003cf00       _target_laser_think        2003df00 f   g_target.obj
 0001:0003d130       _target_laser_on           2003e130 f   g_target.obj
 0001:0003d170       _target_laser_off          2003e170 f   g_target.obj
 0001:0003d1a0       _target_laser_use          2003e1a0 f   g_target.obj
 0001:0003d1f0       _target_laser_start        2003e1f0 f   g_target.obj
 0001:0003d2f0       _SP_target_laser           2003e2f0 f   g_target.obj
 0001:0003d320       _target_teleporter_use     2003e320 f   g_target.obj
 0001:0003d390       _SP_target_teleporter      2003e390 f   g_target.obj
 0001:0003d3e0       _target_relay_use          2003e3e0 f   g_target.obj
 0001:0003d4b0       _SP_target_relay           2003e4b0 f   g_target.obj
 0001:0003d4d0       _target_kill_use           2003e4d0 f   g_target.obj
 0001:0003d500       _SP_target_kill            2003e500 f   g_target.obj
 0001:0003d520       _SP_target_position        2003e520 f   g_target.obj
 0001:0003d550       _SP_target_location        2003e550 f   g_target.obj
 0001:0003d690       _Team_InitGame             2003e690 f   g_team.obj
 0001:0003d6f0       _OtherTeam                 2003e6f0 f   g_team.obj
 0001:0003d720       _TeamName                  2003e720 f   g_team.obj
 0001:0003d760       _OtherTeamName             2003e760 f   g_team.obj
 0001:0003d7a0       _TeamColorString           2003e7a0 f   g_team.obj
 0001:0003d7e0       _PrintMsg                  2003e7e0 f   g_team.obj
 0001:0003d8b0       _AddTeamScore              2003e8b0 f   g_team.obj
 0001:0003d9c0       _OnSameTeam                2003e9c0 f   g_team.obj
 0001:0003da30       _Team_SetFlagStatus        2003ea30 f   g_team.obj
 0001:0003db10       _Team_CheckDroppedItem     2003eb10 f   g_team.obj
 0001:0003db80       _Team_ForceGesture         2003eb80 f   g_team.obj
 0001:0003dc10       _Team_FragBonuses          2003ec10 f   g_team.obj
 0001:0003e600       _Team_CheckHurtCarrier     2003f600 f   g_team.obj
 0001:0003e6f0       _Team_ResetFlag            2003f6f0 f   g_team.obj
 0001:0003e7b0       _Team_ResetFlags           2003f7b0 f   g_team.obj
 0001:0003e7e0       _Team_ReturnFlagSound      2003f7e0 f   g_team.obj
 0001:0003e850       _Team_TakeFlagSound        2003f850 f   g_team.obj
 0001:0003e930       _Team_CaptureFlagSound     2003f930 f   g_team.obj
 0001:0003e9a0       _Team_ReturnFlag           2003f9a0 f   g_team.obj
 0001:0003ea00       _Team_FreeEntity           2003fa00 f   g_team.obj
 0001:0003ea60       _Team_DroppedFlagThink     2003fa60 f   g_team.obj
 0001:0003eae0       _Team_TouchOurFlag         2003fae0 f   g_team.obj
 0001:0003efa0       _Team_TouchEnemyFlag       2003ffa0 f   g_team.obj
 0001:0003f060       _Pickup_Team               20040060 f   g_team.obj
 0001:0003f120       _Team_GetLocation          20040120 f   g_team.obj
 0001:0003f220       _Team_GetLocationMsg       20040220 f   g_team.obj
 0001:0003f2e0       _SelectRandomTeamSpawnPoint 200402e0 f   g_team.obj
 0001:0003f3f0       _SelectCTFSpawnPoint       200403f0 f   g_team.obj
 0001:0003f490       _TeamplayInfoMessage       20040490 f   g_team.obj
 0001:0003f7c0       _CheckTeamStatus           200407c0 f   g_team.obj
 0001:0003f930       _SP_team_CTF_redplayer     20040930 f   g_team.obj
 0001:0003f940       _SP_team_CTF_blueplayer    20040940 f   g_team.obj
 0001:0003f950       _SP_team_CTF_redspawn      20040950 f   g_team.obj
 0001:0003f960       _SP_team_CTF_bluespawn     20040960 f   g_team.obj
 0001:0003f970       _InitTrigger               20040970 f   g_trigger.obj
 0001:0003f9e0       _multi_wait                200409e0 f   g_trigger.obj
 0001:0003fa00       _multi_trigger             20040a00 f   g_trigger.obj
 0001:0003fbb0       _Use_Multi                 20040bb0 f   g_trigger.obj
 0001:0003fbd0       _Touch_Multi               20040bd0 f   g_trigger.obj
 0001:0003fc00       _SP_trigger_multiple       20040c00 f   g_trigger.obj
 0001:0003fcd0       _trigger_always_think      20040cd0 f   g_trigger.obj
 0001:0003fd00       _SP_trigger_always         20040d00 f   g_trigger.obj
 0001:0003fd30       _trigger_push_touch        20040d30 f   g_trigger.obj
 0001:0003fd70       _AimAtTarget               20040d70 f   g_trigger.obj
 0001:0003fef0       _SP_trigger_push           20040ef0 f   g_trigger.obj
 0001:0003ff70       _Use_target_push           20040f70 f   g_trigger.obj
 0001:00040030       _SP_target_push            20041030 f   g_trigger.obj
 0001:00040190       _trigger_teleporter_touch  20041190 f   g_trigger.obj
 0001:00040230       _SP_trigger_teleport       20041230 f   g_trigger.obj
 0001:000402c0       _hurt_use                  200412c0 f   g_trigger.obj
 0001:00040300       _hurt_touch                20041300 f   g_trigger.obj
 0001:000403e0       _SP_trigger_hurt           200413e0 f   g_trigger.obj
 0001:00040480       _func_timer_think          20041480 f   g_trigger.obj
 0001:00040500       _func_timer_use            20041500 f   g_trigger.obj
 0001:00040550       _SP_func_timer             20041550 f   g_trigger.obj
 0001:00040640       _AddRemap                  20041640 f   g_utils.obj
 0001:00040730       _BuildShaderStateConfig    20041730 f   g_utils.obj
 0001:00040800       _G_FindConfigstringIndex   20041800 f   g_utils.obj
 0001:000408c0       _G_ModelIndex              200418c0 f   g_utils.obj
 0001:000408f0       _G_SoundIndex              200418f0 f   g_utils.obj
 0001:00040920       _G_TeamCommand             20041920 f   g_utils.obj
 0001:000409b0       _G_Find                    200419b0 f   g_utils.obj
 0001:00040a40       _G_PickTarget              20041a40 f   g_utils.obj
 0001:00040af0       _G_UseTargets              20041af0 f   g_utils.obj
 0001:00040c00       _tv                        20041c00 f   g_utils.obj
 0001:00040c50       _vtos                      20041c50 f   g_utils.obj
 0001:00040cc0       _G_SetMovedir              20041cc0 f   g_utils.obj
 0001:00040de0       _vectoyaw                  20041de0 f   g_utils.obj
 0001:00040eb0       _G_InitGentity             20041eb0 f   g_utils.obj
 0001:00040f00       _G_Spawn                   20041f00 f   g_utils.obj
 0001:00041070       _G_EntitiesFree            20042070 f   g_utils.obj
 0001:000410d0       _G_FreeEntity              200420d0 f   g_utils.obj
 0001:00041140       _G_TempEntity              20042140 f   g_utils.obj
 0001:00041200       _G_KillBox                 20042200 f   g_utils.obj
 0001:00041350       _G_AddPredictableEvent     20042350 f   g_utils.obj
 0001:00041390       _G_AddEvent                20042390 f   g_utils.obj
 0001:00041480       _G_Sound                   20042480 f   g_utils.obj
 0001:000414c0       _G_SetOrigin               200424c0 f   g_utils.obj
 0001:00041560       _DebugLine                 20042560 f   g_utils.obj
 0001:000417c0       _G_BounceProjectile        200427c0 f   g_weapon.obj
 0001:000418b0       _Weapon_Gauntlet           200428b0 f   g_weapon.obj
 0001:000418c0       _CheckGauntletAttack       200428c0 f   g_weapon.obj
 0001:00041a90       _SnapVectorTowards         20042a90 f   g_weapon.obj
 0001:00041b20       _Bullet_Fire               20042b20 f   g_weapon.obj
 0001:00041de0       _BFG_Fire                  20042de0 f   g_weapon.obj
 0001:00041e50       _ShotgunPellet             20042e50 f   g_weapon.obj
 0001:00041f60       _ShotgunPattern            20042f60 f   g_weapon.obj
 0001:00042150       _weapon_supershotgun_fire  20043150 f   g_weapon.obj
 0001:00042240       _weapon_grenadelauncher_fire 20043240 f   g_weapon.obj
 0001:000422d0       _Weapon_RocketLauncher_Fire 200432d0 f   g_weapon.obj
 0001:00042340       _Weapon_Plasmagun_Fire     20043340 f   g_weapon.obj
 0001:000423b0       _weapon_railgun_fire       200433b0 f   g_weapon.obj
 0001:00042750       _Weapon_GrapplingHook_Fire 20043750 f   g_weapon.obj
 0001:000427b0       _Weapon_HookFree           200437b0 f   g_weapon.obj
 0001:00042810       _Weapon_HookThink          20043810 f   g_weapon.obj
 0001:00042970       _Weapon_LightningFire      20043970 f   g_weapon.obj
 0001:00042b30       _LogAccuracyHit            20043b30 f   g_weapon.obj
 0001:00042bb0       _CalcMuzzlePoint           20043bb0 f   g_weapon.obj
 0001:00042c90       _CalcMuzzlePointOrigin     20043c90 f   g_weapon.obj
 0001:00042d70       _FireWeapon                20043d70 f   g_weapon.obj
 0001:00042f50       _Q_rand                    20043f50 f   q_math.obj
 0001:00042f80       _Q_random                  20043f80 f   q_math.obj
 0001:00042fb0       _Q_crandom                 20043fb0 f   q_math.obj
 0001:00042fe0       _ClampChar                 20043fe0 f   q_math.obj
 0001:00043010       _ClampShort                20044010 f   q_math.obj
 0001:00043050       _DirToByte                 20044050 f   q_math.obj
 0001:000430f0       _ByteToDir                 200440f0 f   q_math.obj
 0001:00043170       _ColorBytes3               20044170 f   q_math.obj
 0001:000431c0       _ColorBytes4               200441c0 f   q_math.obj
 0001:00043220       _NormalizeColor            20044220 f   q_math.obj
 0001:000432d0       _PlaneFromPoints           200442d0 f   q_math.obj
 0001:00043410       _RotatePointAroundVector   20044410 f   q_math.obj
 0001:00043640       _RotateAroundDirection     20044640 f   q_math.obj
 0001:000436d0       _vectoangles               200446d0 f   q_math.obj
 0001:00043850       _AnglesToAxis              20044850 f   q_math.obj
 0001:000438b0       _AxisClear                 200448b0 f   q_math.obj
 0001:00043920       _AxisCopy                  20044920 f   q_math.obj
 0001:000439a0       _ProjectPointOnPlane       200449a0 f   q_math.obj
 0001:00043aa0       _MakeNormalVectors         20044aa0 f   q_math.obj
 0001:00043b70       _VectorRotate              20044b70 f   q_math.obj
 0001:00043c10       _Q_rsqrt                   20044c10 f   q_math.obj
 0001:00043c70       _Q_fabs                    20044c70 f   q_math.obj
 0001:00043ca0       _LerpAngle                 20044ca0 f   q_math.obj
 0001:00043d00       _AngleSubtract             20044d00 f   q_math.obj
 0001:00043d60       _AnglesSubtract            20044d60 f   q_math.obj
 0001:00043dd0       _AngleMod                  20044dd0 f   q_math.obj
 0001:00043e10       _AngleNormalize360         20044e10 f   q_math.obj
 0001:00043e50       _AngleNormalize180         20044e50 f   q_math.obj
 0001:00043e90       _AngleDelta                20044e90 f   q_math.obj
 0001:00043ec0       _SetPlaneSignbits          20044ec0 f   q_math.obj
 0001:00043f20       _BoxOnPlaneSide            20044f20 f   q_math.obj
 0001:00044160       _RadiusFromBounds          20045160 f   q_math.obj
 0001:00044240       _ClearBounds               20045240 f   q_math.obj
 0001:00044290       _AddPointToBounds          20045290 f   q_math.obj
 0001:00044360       _VectorNormalize           20045360 f   q_math.obj
 0001:00044400       _VectorNormalize2          20045400 f   q_math.obj
 0001:000444c0       __VectorMA                 200454c0 f   q_math.obj
 0001:00044510       __DotProduct               20045510 f   q_math.obj
 0001:00044550       __VectorSubtract           20045550 f   q_math.obj
 0001:000445a0       __VectorAdd                200455a0 f   q_math.obj
 0001:000445f0       __VectorCopy               200455f0 f   q_math.obj
 0001:00044630       __VectorScale              20045630 f   q_math.obj
 0001:00044670       _Vector4Scale              20045670 f   q_math.obj
 0001:000446c0       _Q_log2                    200456c0 f   q_math.obj
 0001:00044700       _MatrixMultiply            20045700 f   q_math.obj
 0001:000448b0       _AngleVectors              200458b0 f   q_math.obj
 0001:00044aa0       _PerpendicularVector       20045aa0 f   q_math.obj
 0001:00044b60       _Com_Clamp                 20045b60 f   q_shared.obj
 0001:00044ba0       _COM_SkipPath              20045ba0 f   q_shared.obj
 0001:00044bf0       _COM_StripExtension        20045bf0 f   q_shared.obj
 0001:00044c40       _COM_DefaultExtension      20045c40 f   q_shared.obj
 0001:00044cd0       _ShortSwap                 20045cd0 f   q_shared.obj
 0001:00044d10       _ShortNoSwap               20045d10 f   q_shared.obj
 0001:00044d30       _LongSwap                  20045d30 f   q_shared.obj
 0001:00044da0       _LongNoSwap                20045da0 f   q_shared.obj
 0001:00044dc0       _Long64Swap                20045dc0 f   q_shared.obj
 0001:00044e10       _Long64NoSwap              20045e10 f   q_shared.obj
 0001:00044e30       _FloatSwap                 20045e30 f   q_shared.obj
 0001:00044e60       _FloatNoSwap               20045e60 f   q_shared.obj
 0001:00044e80       _COM_BeginParseSession     20045e80 f   q_shared.obj
 0001:00044ec0       _COM_GetCurrentParseLine   20045ec0 f   q_shared.obj
 0001:00044ee0       _COM_Parse                 20045ee0 f   q_shared.obj
 0001:00044f00       _COM_ParseError            20045f00 f   q_shared.obj
 0001:00044f50       _COM_ParseWarning          20045f50 f   q_shared.obj
 0001:00044fa0       _COM_Compress              20045fa0 f   q_shared.obj
 0001:000451a0       _COM_ParseExt              200461a0 f   q_shared.obj
 0001:00045430       _COM_MatchToken            20046430 f   q_shared.obj
 0001:00045480       _SkipBracedSection         20046480 f   q_shared.obj
 0001:000454f0       _SkipRestOfLine            200464f0 f   q_shared.obj
 0001:00045540       _Parse1DMatrix             20046540 f   q_shared.obj
 0001:000455c0       _Parse2DMatrix             200465c0 f   q_shared.obj
 0001:00045630       _Parse3DMatrix             20046630 f   q_shared.obj
 0001:000456b0       _Q_isprint                 200466b0 f   q_shared.obj
 0001:000456e0       _Q_islower                 200466e0 f   q_shared.obj
 0001:00045710       _Q_isupper                 20046710 f   q_shared.obj
 0001:00045740       _Q_isalpha                 20046740 f   q_shared.obj
 0001:00045780       _Q_strrchr                 20046780 f   q_shared.obj
 0001:000457e0       _Q_strncpyz                200467e0 f   q_shared.obj
 0001:00045850       _Q_stricmpn                20046850 f   q_shared.obj
 0001:00045920       _Q_strncmp                 20046920 f   q_shared.obj
 0001:00045990       _Q_stricmp                 20046990 f   q_shared.obj
 0001:000459d0       _Q_strlwr                  200469d0 f   q_shared.obj
 0001:00045a20       _Q_strupr                  20046a20 f   q_shared.obj
 0001:00045a70       _Q_strcat                  20046a70 f   q_shared.obj
 0001:00045ac0       _Q_PrintStrlen             20046ac0 f   q_shared.obj
 0001:00045b40       _Q_CleanStr                20046b40 f   q_shared.obj
 0001:00045bd0       _Com_sprintf               20046bd0 f   q_shared.obj
 0001:00045c60       _va                        20046c60 f   q_shared.obj
 0001:00045cc0       _Info_ValueForKey          20046cc0 f   q_shared.obj
 0001:00045e40       _Info_NextPair             20046e40 f   q_shared.obj
 0001:00045f20       _Info_RemoveKey            20046f20 f   q_shared.obj
 0001:00046090       _Info_RemoveKey_Big        20047090 f   q_shared.obj
 0001:00046200       _Info_Validate             20047200 f   q_shared.obj
 0001:00046250       _Info_SetValueForKey       20047250 f   q_shared.obj
 0001:000463d0       _Info_SetValueForKey_Big   200473d0 f   q_shared.obj
 0001:00046540       _atol                      20047540 f   LIBCMTD:atox.obj
 0001:00046650       _atoi                      20047650 f   LIBCMTD:atox.obj
 0001:00046670       __atoi64                   20047670 f   LIBCMTD:atox.obj
 0001:000467b0       _strlen                    200477b0 f   LIBCMTD:strlen.obj
 0001:00046840       _srand                     20047840 f   LIBCMTD:rand.obj
 0001:00046850       _rand                      20047850 f   LIBCMTD:rand.obj
 0001:00046890       __fpmath                   20047890 f   LIBCMTD:fpinit.obj
 0001:000468c0       __fpclear                  200478c0 f   LIBCMTD:fpinit.obj
 0001:000468d0       __cfltcvt_init             200478d0 f   LIBCMTD:fpinit.obj
 0001:00046920       ___setfflag                20047920 f   LIBCMTD:fpinit.obj
 0001:0004693c       __ftol2                    2004793c f   LIBCMTD:ftol2.obj
 0001:000469c0       _strncpy                   200479c0 f   LIBCMTD:strncpy.obj
 0001:00046af0       _strcpy                    20047af0 f   LIBCMTD:strcat.obj
 0001:00046b00       _strcat                    20047b00 f   LIBCMTD:strcat.obj
 0001:00046bf0       _memcpy                    20047bf0 f   LIBCMTD:memcpy.obj
 0001:00046f30       _atof                      20047f30 f   LIBCMTD:atof.obj
 0001:00046f80       _sscanf                    20047f80 f   LIBCMTD:sscanf.obj
 0001:00047030       __CIsqrt                   20048030 f   LIBCMTD:sqrt.obj
 0001:00047044       _sqrt                      20048044     LIBCMTD:sqrt.obj
 0001:000470f0       _memset                    200480f0 f   LIBCMTD:memset.obj
 0001:00047150       __toupper                  20048150 f   LIBCMTD:toupper.obj
 0001:00047160       _toupper                   20048160 f   LIBCMTD:toupper.obj
 0001:000471a0       ___toupper_mt              200481a0 f   LIBCMTD:toupper.obj
 0001:000472e0       _memmove                   200482e0 f   LIBCMTD:memmove.obj
 0001:00047620       _strstr                    20048620 f   LIBCMTD:strstr.obj
 0001:000476b0       _fabs                      200486b0 f   LIBCMTD:fabs.obj
 0001:000477b0       _strcmp                    200487b0 f   LIBCMTD:strcmp.obj
 0001:00047840       _vsprintf                  20048840 f   LIBCMTD:vsprintf.obj
 0001:00047930       __vscprintf                20048930 f   LIBCMTD:vsprintf.obj
 0001:000479b0       _abs                       200489b0 f   LIBCMTD:abs.obj
 0001:000479e0       __abs64                    200489e0 f   LIBCMTD:abs.obj
 0001:00047a30       _strchr                    20048a30 f   LIBCMTD:strchr.obj
 0001:00047a36       ___from_strstr_to_strchr   20048a36     LIBCMTD:strchr.obj
 0001:00047af0       __CIsin                    20048af0 f   LIBCMTD:sin.obj
 0001:00047b04       _sin                       20048b04     LIBCMTD:sin.obj
 0001:00047ba0       __CIcos                    20048ba0 f   LIBCMTD:cos.obj
 0001:00047bb4       _cos                       20048bb4     LIBCMTD:cos.obj
 0001:00047c50       __alloca_probe             20048c50     LIBCMTD:chkstk.obj
 0001:00047c50       __chkstk                   20048c50 f   LIBCMTD:chkstk.obj
 0001:00047c90       __tolower                  20048c90 f   LIBCMTD:tolower.obj
 0001:00047ca0       _tolower                   20048ca0 f   LIBCMTD:tolower.obj
 0001:00047ce0       ___tolower_mt              20048ce0 f   LIBCMTD:tolower.obj
 0001:00047e20       _ceil                      20048e20 f   LIBCMTD:ceil_pentium4.obj
 0001:00047e60       __ceil_pentium4            20048e60 f   LIBCMTD:ceil_pentium4.obj
 0001:00047f40       _qsort                     20048f40 f   LIBCMTD:qsort.obj
 0001:000483a0       _atan2                     200493a0 f   LIBCMTD:87ctriga.obj
 0001:000483aa       __CIatan2                  200493aa f   LIBCMTD:87ctriga.obj
 0001:000483c0       __assert                   200493c0 f   LIBCMTD:assert.obj
 0001:000489c0       __CRT_INIT@12              200499c0 f   LIBCMTD:dllcrt0.obj
 0001:00048c10       __DllMainCRTStartup@12     20049c10 f   LIBCMTD:dllcrt0.obj
 0001:00048d90       __amsg_exit                20049d90 f   LIBCMTD:dllcrt0.obj
 0001:00048dd0       __chvalidator              20049dd0 f   LIBCMTD:isctype.obj
 0001:00048e10       __chvalidator_mt           20049e10 f   LIBCMTD:isctype.obj
 0001:00048e50       __isctype                  20049e50 f   LIBCMTD:isctype.obj
 0001:00048e90       ___isctype_mt              20049e90 f   LIBCMTD:isctype.obj
 0001:00048f50       ____setlc_active_func      20049f50 f   LIBCMTD:setlocal.obj
 0001:00048f60       ____unguarded_readlc_active_add_func 20049f60 f   LIBCMTD:setlocal.obj
 0001:00048f70       ___freetlocinfo            20049f70 f   LIBCMTD:setlocal.obj
 0001:000490f0       ___updatetlocinfo          2004a0f0 f   LIBCMTD:setlocal.obj
 0001:00049330       _setlocale                 2004a330 f   LIBCMTD:setlocal.obj
 0001:00049de0       __expandlocale             2004ade0 f   LIBCMTD:setlocal.obj
 0001:00049fc0       ___init_dummy              2004afc0 f   LIBCMTD:setlocal.obj
 0001:00049fd0       __strcats                  2004afd0 f   LIBCMTD:setlocal.obj
 0001:0004a020       ___lc_strtolc              2004b020 f   LIBCMTD:setlocal.obj
 0001:0004a190       ___lc_lctostr              2004b190 f   LIBCMTD:setlocal.obj
 0001:0004a200       ___crtTlsAlloc@4           2004b200 f   LIBCMTD:tidtable.obj
 0001:0004a210       __mtinit                   2004b210 f   LIBCMTD:tidtable.obj
 0001:0004a360       __mtterm                   2004b360 f   LIBCMTD:tidtable.obj
 0001:0004a390       __initptd                  2004b390 f   LIBCMTD:tidtable.obj
 0001:0004a3b0       __getptd                   2004b3b0 f   LIBCMTD:tidtable.obj
 0001:0004a450       __freefls@4                2004b450 f   LIBCMTD:tidtable.obj
 0001:0004a6d0       __freeptd                  2004b6d0 f   LIBCMTD:tidtable.obj
 0001:0004a710       ___threadid                2004b710 f   LIBCMTD:tidtable.obj
 0001:0004a720       ___threadhandle            2004b720 f   LIBCMTD:tidtable.obj
 0001:0004a730       __allmul                   2004b730 f   LIBCMTD:llmul.obj
 0001:0004a770       __setdefaultprecision      2004b770 f   LIBCMTD:fp8.obj
 0001:0004a790       __ms_p5_test_fdiv          2004b790 f   LIBCMTD:testfdiv.obj
 0001:0004a7e0       __ms_p5_mp_test_fdiv       2004b7e0 f   LIBCMTD:testfdiv.obj
 0001:0004a830       __forcdecpt                2004b830 f   LIBCMTD:cvt.obj
 0001:0004a8b0       __cropzeros                2004b8b0 f   LIBCMTD:cvt.obj
 0001:0004a990       __positive                 2004b990 f   LIBCMTD:cvt.obj
 0001:0004a9c0       __fassign                  2004b9c0 f   LIBCMTD:cvt.obj
 0001:0004aa10       __cftoe                    2004ba10 f   LIBCMTD:cvt.obj
 0001:0004ac10       __cftof                    2004bc10 f   LIBCMTD:cvt.obj
 0001:0004add0       __cftog                    2004bdd0 f   LIBCMTD:cvt.obj
 0001:0004aed0       __cfltcvt                  2004bed0 f   LIBCMTD:cvt.obj
 0001:0004af60       __fltin2                   2004bf60 f   LIBCMTD:cfin.obj
 0001:0004b040       _isalpha                   2004c040 f   LIBCMTD:_ctype.obj
 0001:0004b0b0       _isupper                   2004c0b0 f   LIBCMTD:_ctype.obj
 0001:0004b110       _islower                   2004c110 f   LIBCMTD:_ctype.obj
 0001:0004b170       _isdigit                   2004c170 f   LIBCMTD:_ctype.obj
 0001:0004b1d0       _isxdigit                  2004c1d0 f   LIBCMTD:_ctype.obj
 0001:0004b240       _isspace                   2004c240 f   LIBCMTD:_ctype.obj
 0001:0004b2a0       _ispunct                   2004c2a0 f   LIBCMTD:_ctype.obj
 0001:0004b300       _isalnum                   2004c300 f   LIBCMTD:_ctype.obj
 0001:0004b370       _isprint                   2004c370 f   LIBCMTD:_ctype.obj
 0001:0004b3e0       _isgraph                   2004c3e0 f   LIBCMTD:_ctype.obj
 0001:0004b450       _iscntrl                   2004c450 f   LIBCMTD:_ctype.obj
 0001:0004b4b0       ___isascii                 2004c4b0 f   LIBCMTD:_ctype.obj
 0001:0004b4c0       ___toascii                 2004c4c0 f   LIBCMTD:_ctype.obj
 0001:0004b4d0       ___iscsymf                 2004c4d0 f   LIBCMTD:_ctype.obj
 0001:0004b510       ___iscsym                  2004c510 f   LIBCMTD:_ctype.obj
 0001:0004b550       __input                    2004c550 f   LIBCMTD:input.obj
 0001:0004c9c0       __CrtDbgBreak              2004d9c0 f   LIBCMTD:dbgrpt.obj
 0001:0004c9d0       __CrtSetReportMode         2004d9d0 f   LIBCMTD:dbgrpt.obj
 0001:0004ca30       __CrtSetReportFile         2004da30 f   LIBCMTD:dbgrpt.obj
 0001:0004cab0       __CrtSetReportHook         2004dab0 f   LIBCMTD:dbgrpt.obj
 0001:0004cad0       __CrtSetReportHook2        2004dad0 f   LIBCMTD:dbgrpt.obj
 0001:0004cd20       __CrtDbgReport             2004dd20 f   LIBCMTD:dbgrpt.obj
 0001:0004d490       __trandisp1                2004e490 f   LIBCMTD:87disp.obj
 0001:0004d4f7       __trandisp2                2004e4f7 f   LIBCMTD:87disp.obj
 0001:0004d583       __rttospopde               2004e583     LIBCMTD:87disp.obj
 0001:0004d588       __rttospop                 2004e588     LIBCMTD:87disp.obj
 0001:0004d58a       __rtnospop                 2004e58a     LIBCMTD:87disp.obj
 0001:0004d58c       __rttosnpop                2004e58c     LIBCMTD:87disp.obj
 0001:0004d58d       __rtnospopde               2004e58d     LIBCMTD:87disp.obj
 0001:0004d594       __rtzeropop                2004e594     LIBCMTD:87disp.obj
 0001:0004d596       __rtzeronpop               2004e596     LIBCMTD:87disp.obj
 0001:0004d59b       __rtonepop                 2004e59b     LIBCMTD:87disp.obj
 0001:0004d59d       __rtonenpop                2004e59d     LIBCMTD:87disp.obj
 0001:0004d5a2       __tosnan1                  2004e5a2     LIBCMTD:87disp.obj
 0001:0004d5cd       __nosnan2                  2004e5cd     LIBCMTD:87disp.obj
 0001:0004d5cf       __tosnan2                  2004e5cf     LIBCMTD:87disp.obj
 0001:0004d5f7       __nan2                     2004e5f7     LIBCMTD:87disp.obj
 0001:0004d636       __rtindfpop                2004e636     LIBCMTD:87disp.obj
 0001:0004d638       __rtindfnpop               2004e638     LIBCMTD:87disp.obj
 0001:0004d649       __rttosnpopde              2004e649     LIBCMTD:87disp.obj
 0001:0004d653       __rtchsifneg               2004e653     LIBCMTD:87disp.obj
 0001:0004d660       __startTwoArgErrorHandling 2004e660 f   LIBCMTD:genexcep.obj
 0001:0004d677       __startOneArgErrorHandling 2004e677 f   LIBCMTD:genexcep.obj
 0001:0004d6c0       __twoToTOS                 2004e6c0 f   LIBCMTD:common.obj
 0001:0004d6d5       __load_CW                  2004e6d5 f   LIBCMTD:common.obj
 0001:0004d6ec       __convertTOStoQNaN         2004e6ec f   LIBCMTD:common.obj
 0001:0004d705       __fload_withFB             2004e705 f   LIBCMTD:common.obj
 0001:0004d748       __checkTOS_withFB          2004e748 f   LIBCMTD:common.obj
 0001:0004d75e       __fast_exit                2004e75e f   LIBCMTD:common.obj
 0001:0004d76b       __math_exit                2004e76b f   LIBCMTD:common.obj
 0001:0004d795       __check_overflow_exit      2004e795 f   LIBCMTD:common.obj
 0001:0004d7a9       __check_range_exit         2004e7a9 f   LIBCMTD:common.obj
 0001:0004d850       ___crtLCMapStringA         2004e850 f   LIBCMTD:a_map.obj
 0001:0004de10       __handle_qnan1             2004ee10 f   LIBCMTD:fpexcept.obj
 0001:0004de70       __handle_qnan2             2004ee70 f   LIBCMTD:fpexcept.obj
 0001:0004dee0       __except1                  2004eee0 f   LIBCMTD:fpexcept.obj
 0001:0004dfe0       __except2                  2004efe0 f   LIBCMTD:fpexcept.obj
 0001:0004e0f0       __raise_exc                2004f0f0 f   LIBCMTD:fpexcept.obj
 0001:0004e5a0       __handle_exc               2004f5a0 f   LIBCMTD:fpexcept.obj
 0001:0004e8c0       __umatherr                 2004f8c0 f   LIBCMTD:fpexcept.obj
 0001:0004e960       __set_errno                2004f960 f   LIBCMTD:fpexcept.obj
 0001:0004e9e0       __errcode                  2004f9e0 f   LIBCMTD:fpexcept.obj
 0001:0004ea50       __set_exp                  2004fa50 f   LIBCMTD:util.obj
 0001:0004ea90       __get_exp                  2004fa90 f   LIBCMTD:util.obj
 0001:0004eac0       __add_exp                  2004fac0 f   LIBCMTD:util.obj
 0001:0004eaf0       __set_bexp                 2004faf0 f   LIBCMTD:util.obj
 0001:0004eb20       __sptype                   2004fb20 f   LIBCMTD:util.obj
 0001:0004eba0       __decomp                   2004fba0 f   LIBCMTD:util.obj
 0001:0004ecd0       __statfp                   2004fcd0 f   LIBCMTD:fpctrl.obj
 0001:0004ece0       __clrfp                    2004fce0 f   LIBCMTD:fpctrl.obj
 0001:0004ed00       __ctrlfp                   2004fd00 f   LIBCMTD:fpctrl.obj
 0001:0004ed30       __set_statfp               2004fd30 f   LIBCMTD:fpctrl.obj
 0001:0004eda0       __flsbuf                   2004fda0 f   LIBCMTD:_flsbuf.obj
 0001:0004f000       __output                   20050000 f   LIBCMTD:output.obj
 0001:0004ff80       ___libm_error_support      20050f80 f   LIBCMTD:libm_error.obj
 0001:00050990       ___sse2_available_init     20051990 f   LIBCMTD:cpu_disp.obj
 0001:00050b20       __set_SSE2_enable          20051b20 f   LIBCMTD:cpu_disp.obj
 0001:00050b40       __ceil_default             20051b40 f   LIBCMTD:ceil.obj
 0001:00050c9c       __fFATN2                   20051c9c     LIBCMTD:87triga.obj
 0001:00050cec       __rtpiby2                  20051cec     LIBCMTD:87triga.obj
 0001:00050d30       __cintrindisp2             20051d30 f   LIBCMTD:87cdisp.obj
 0001:00050d6e       __cintrindisp1             20051d6e f   LIBCMTD:87cdisp.obj
 0001:00050dab       __ctrandisp2               20051dab f   LIBCMTD:87cdisp.obj
 0001:00050f41       __ctrandisp1               20051f41 f   LIBCMTD:87cdisp.obj
 0001:00050f74       __fload                    20051f74 f   LIBCMTD:87cdisp.obj
 0001:00050fb0       _abort                     20051fb0 f   LIBCMTD:abort.obj
 0001:00050fd0       __cinit                    20051fd0 f   LIBCMTD:crt0dat.obj
 0001:00051030       _exit                      20052030 f   LIBCMTD:crt0dat.obj
 0001:00051050       __exit                     20052050 f   LIBCMTD:crt0dat.obj
 0001:00051070       __cexit                    20052070 f   LIBCMTD:crt0dat.obj
 0001:00051090       __c_exit                   20052090 f   LIBCMTD:crt0dat.obj
 0001:000511e0       ___crtExitProcess          200521e0 f   LIBCMTD:crt0dat.obj
 0001:00051230       __lockexit                 20052230 f   LIBCMTD:crt0dat.obj
 0001:00051240       __unlockexit               20052240 f   LIBCMTD:crt0dat.obj
 0001:000512c0       _signal                    200522c0 f   LIBCMTD:winsig.obj
 0001:00051600       _raise                     20052600 f   LIBCMTD:winsig.obj
 0001:000518c0       ___fpecode                 200528c0 f   LIBCMTD:winsig.obj
 0001:000518d0       ___pxcptinfoptrs           200528d0 f   LIBCMTD:winsig.obj
 0001:000518e0       ___crtMessageBoxA          200528e0 f   LIBCMTD:crtmbox.obj
 0001:00051a50       __itoa                     20052a50 f   LIBCMTD:xtoa.obj
 0001:00051b70       __ltoa                     20052b70 f   LIBCMTD:xtoa.obj
 0001:00051bb0       __ultoa                    20052bb0 f   LIBCMTD:xtoa.obj
 0001:00051bd0       __i64toa                   20052bd0 f   LIBCMTD:xtoa.obj
 0001:00051d20       __ui64toa                  20052d20 f   LIBCMTD:xtoa.obj
 0001:00051d40       _strncat                   20052d40 f   LIBCMTD:strncat.obj
 0001:00051e80       _fflush                    20052e80 f   LIBCMTD:fflush.obj
 0001:00051f10       __fflush_lk                20052f10 f   LIBCMTD:fflush.obj
 0001:00051f50       __flush                    20052f50 f   LIBCMTD:fflush.obj
 0001:00052010       __flushall                 20053010 f   LIBCMTD:fflush.obj
 0001:000521b0       _fprintf                   200531b0 f   LIBCMTD:fprintf.obj
 0001:000522a0       _setvbuf                   200532a0 f   LIBCMTD:setvbuf.obj
 0001:00052440       ___iob_func                20053440 f   LIBCMTD:_file.obj
 0001:00052450       ___initstdio               20053450 f   LIBCMTD:_file.obj
 0001:00052580       ___endstdio                20053580 f   LIBCMTD:_file.obj
 0001:000525a0       __lock_file                200535a0 f   LIBCMTD:_file.obj
 0001:000525e0       __lock_file2               200535e0 f   LIBCMTD:_file.obj
 0001:00052610       __unlock_file              20053610 f   LIBCMTD:_file.obj
 0001:00052650       __unlock_file2             20053650 f   LIBCMTD:_file.obj
 0001:00052680       @__security_check_cookie@4 20053680 f   LIBCMTD:secchk.obj
 0001:00052700       _malloc                    20053700 f   LIBCMTD:dbgheap.obj
 0001:00052730       __malloc_dbg               20053730 f   LIBCMTD:dbgheap.obj
 0001:00052760       __nh_malloc                20053760 f   LIBCMTD:dbgheap.obj
 0001:00052780       __nh_malloc_dbg            20053780 f   LIBCMTD:dbgheap.obj
 0001:00052820       __heap_alloc               20053820 f   LIBCMTD:dbgheap.obj
 0001:00052840       __heap_alloc_dbg           20053840 f   LIBCMTD:dbgheap.obj
 0001:00052b60       _calloc                    20053b60 f   LIBCMTD:dbgheap.obj
 0001:00052b90       __calloc_dbg               20053b90 f   LIBCMTD:dbgheap.obj
 0001:00052bf0       _realloc                   20053bf0 f   LIBCMTD:dbgheap.obj
 0001:00052c20       __realloc_dbg              20053c20 f   LIBCMTD:dbgheap.obj
 0001:000531c0       __expand                   200541c0 f   LIBCMTD:dbgheap.obj
 0001:000531f0       __expand_dbg               200541f0 f   LIBCMTD:dbgheap.obj
 0001:00053280       _free                      20054280 f   LIBCMTD:dbgheap.obj
 0001:000532a0       __free_lk                  200542a0 f   LIBCMTD:dbgheap.obj
 0001:000532c0       __free_dbg                 200542c0 f   LIBCMTD:dbgheap.obj
 0001:00053330       __free_dbg_lk              20054330 f   LIBCMTD:dbgheap.obj
 0001:00053740       __msize                    20054740 f   LIBCMTD:dbgheap.obj
 0001:00053760       __msize_dbg                20054760 f   LIBCMTD:dbgheap.obj
 0001:000538d0       __CrtSetBreakAlloc         200548d0 f   LIBCMTD:dbgheap.obj
 0001:000538f0       __CrtSetDbgBlockType       200548f0 f   LIBCMTD:dbgheap.obj
 0001:000539d0       __CrtSetAllocHook          200549d0 f   LIBCMTD:dbgheap.obj
 0001:00053a40       __CrtCheckMemory           20054a40 f   LIBCMTD:dbgheap.obj
 0001:00053db0       __CrtSetDbgFlag            20054db0 f   LIBCMTD:dbgheap.obj
 0001:00053e60       __CrtDoForAllClientObjects 20054e60 f   LIBCMTD:dbgheap.obj
 0001:00053f10       __CrtIsValidPointer        20054f10 f   LIBCMTD:dbgheap.obj
 0001:00053f60       __CrtIsValidHeapPointer    20054f60 f   LIBCMTD:dbgheap.obj
 0001:00054010       __CrtIsMemoryBlock         20055010 f   LIBCMTD:dbgheap.obj
 0001:00054140       __CrtReportBlockType       20055140 f   LIBCMTD:dbgheap.obj
 0001:00054170       __CrtSetDumpClient         20055170 f   LIBCMTD:dbgheap.obj
 0001:00054190       __CrtMemCheckpoint         20055190 f   LIBCMTD:dbgheap.obj
 0001:00054330       __CrtMemDifference         20055330 f   LIBCMTD:dbgheap.obj
 0001:00054450       __CrtMemDumpAllObjectsSince 20055450 f   LIBCMTD:dbgheap.obj
 0001:00054850       __CrtDumpMemoryLeaks       20055850 f   LIBCMTD:dbgheap.obj
 0001:000548c0       __CrtMemDumpStatistics     200558c0 f   LIBCMTD:dbgheap.obj
 0001:00054970       __aligned_malloc           20055970 f   LIBCMTD:dbgheap.obj
 0001:00054990       __aligned_malloc_dbg       20055990 f   LIBCMTD:dbgheap.obj
 0001:000549b0       __aligned_realloc          200559b0 f   LIBCMTD:dbgheap.obj
 0001:000549d0       __aligned_realloc_dbg      200559d0 f   LIBCMTD:dbgheap.obj
 0001:00054a00       __aligned_offset_malloc    20055a00 f   LIBCMTD:dbgheap.obj
 0001:00054a20       __aligned_offset_malloc_dbg 20055a20 f   LIBCMTD:dbgheap.obj
 0001:00054b60       __aligned_offset_realloc   20055b60 f   LIBCMTD:dbgheap.obj
 0001:00054b90       __aligned_offset_realloc_dbg 20055b90 f   LIBCMTD:dbgheap.obj
 0001:00054df0       __aligned_free             20055df0 f   LIBCMTD:dbgheap.obj
 0001:00054e10       __aligned_free_dbg         20055e10 f   LIBCMTD:dbgheap.obj
 0001:00054ec0       __ioinit                   20055ec0 f   LIBCMTD:ioinit.obj
 0001:00055250       __ioterm                   20056250 f   LIBCMTD:ioinit.obj
 0001:000552f0       __setenvp                  200562f0 f   LIBCMTD:stdenvp.obj
 0001:00055470       __setargv                  20056470 f   LIBCMTD:stdargv.obj
 0001:000558d0       ___crtGetEnvironmentStringsA 200568d0 f   LIBCMTD:a_env.obj
 0001:00055af0       __RTC_Initialize           20056af0 f   LIBCMTD:initsect.obj
 0001:00055b70       __RTC_Terminate            20056b70 f   LIBCMTD:initsect.obj
 0001:00055bf0       ___heap_select             20056bf0 f   LIBCMTD:heapinit.obj
 0001:00055c20       __heap_init                20056c20 f   LIBCMTD:heapinit.obj
 0001:00055c90       __heap_term                20056c90 f   LIBCMTD:heapinit.obj
 0001:00055d40       __get_heap_handle          20056d40 f   LIBCMTD:heapinit.obj
 0001:00055d50       ___CppXcptFilter           20056d50 f   LIBCMTD:winxfltr.obj
 0001:00055d80       __XcptFilter               20056d80 f   LIBCMTD:winxfltr.obj
 0001:00055fa0       _DllMain@12                20056fa0 f   LIBCMTD:dllmain.obj
 0001:00055fac       __global_unwind2           20056fac f   LIBCMTD:exsup.obj
 0001:00055fee       __local_unwind2            20056fee f   LIBCMTD:exsup.obj
 0001:00056046       __NLG_Return2              20057046     LIBCMTD:exsup.obj
 0001:00056056       __abnormal_termination     20057056 f   LIBCMTD:exsup.obj
 0001:00056079       __NLG_Notify1              20057079 f   LIBCMTD:exsup.obj
 0001:00056082       __NLG_Notify               20057082 f   LIBCMTD:exsup.obj
 0001:00056095       __NLG_Dispatch             20057095     LIBCMTD:exsup.obj
 0001:000560a4       __except_handler3          200570a4 f   LIBCMTD:exsup3.obj
 0001:0005618a       __seh_longjmp_unwind@4     2005718a f   LIBCMTD:exsup3.obj
 0001:000561b0       __FF_MSGBANNER             200571b0 f   LIBCMTD:crt0msg.obj
 0001:00056200       __NMSG_WRITE               20057200 f   LIBCMTD:crt0msg.obj
 0001:00056410       __GET_RTERRMSG             20057410 f   LIBCMTD:crt0msg.obj
 0001:00056460       ___pwctype_func            20057460 f   LIBCMTD:ctype.obj
 0001:00056470       ___pctype_func             20057470 f   LIBCMTD:ctype.obj
 0001:00056480       ___crtGetStringTypeA       20057480 f   LIBCMTD:a_str.obj
 0001:00056720       __Getdays                  20057720 f   LIBCMTD:strftime.obj
 0001:00056850       __Getmonths                20057850 f   LIBCMTD:strftime.obj
 0001:00056980       __Gettnames                20057980 f   LIBCMTD:strftime.obj
 0001:00056d10       _strftime                  20057d10 f   LIBCMTD:strftime.obj
 0001:00056d30       __Strftime                 20057d30 f   LIBCMTD:strftime.obj
 0001:00056d80       __Strftime_mt              20057d80 f   LIBCMTD:strftime.obj
 0001:00057fa0       _localeconv                20058fa0 f   LIBCMTD:lconv.obj
 0001:00057fb0       ___init_time               20058fb0 f   LIBCMTD:inittime.obj
 0001:000585c0       ___free_lc_time            200595c0 f   LIBCMTD:inittime.obj
 0001:000588d0       ___init_numeric            200598d0 f   LIBCMTD:initnum.obj
 0001:00058c10       ___free_lconv_num          20059c10 f   LIBCMTD:initnum.obj
 0001:00058cb0       ___init_monetary           20059cb0 f   LIBCMTD:initmon.obj
 0001:000590b0       ___free_lconv_mon          2005a0b0 f   LIBCMTD:initmon.obj
 0001:00059210       ___init_ctype              2005a210 f   LIBCMTD:initctyp.obj
 0001:000594d0       ____mb_cur_max_func        2005a4d0 f   LIBCMTD:initctyp.obj
 0001:000594e0       ____lc_codepage_func       2005a4e0 f   LIBCMTD:initctyp.obj
 0001:00059510       ____lc_collate_cp_func     2005a510 f   LIBCMTD:initctyp.obj
 0001:00059540       ____lc_handle_func         2005a540 f   LIBCMTD:initctyp.obj
 0001:00059570       ___init_collate            2005a570 f   LIBCMTD:initcoll.obj
 0001:00059580       __mtinitlocks              2005a580 f   LIBCMTD:mlock.obj
 0001:00059610       __mtdeletelocks            2005a610 f   LIBCMTD:mlock.obj
 0001:000596d0       __mtinitlocknum            2005a6d0 f   LIBCMTD:mlock.obj
 0001:000597f0       __lock                     2005a7f0 f   LIBCMTD:mlock.obj
 0001:00059830       __unlock                   2005a830 f   LIBCMTD:mlock.obj
 0001:00059850       __lockerr_exit             2005a850 f   LIBCMTD:mlock.obj
 0001:00059870       _strcspn                   2005a870 f   LIBCMTD:strcspn.obj
 0001:000598c0       _strncmp                   2005a8c0 f   LIBCMTD:strncmp.obj
 0001:00059900       _strpbrk                   2005a900 f   LIBCMTD:strpbrk.obj
 0001:00059940       _memcmp                    2005a940 f   LIBCMTD:memcmp.obj
 0001:00059a00       ___get_qualified_locale    2005aa00 f   LIBCMTD:getqloc.obj
 0001:0005a830       ___updatetmbcinfo          2005b830 f   LIBCMTD:mbctype.obj
 0001:0005a900       __setmbcp                  2005b900 f   LIBCMTD:mbctype.obj
 0001:0005b240       __getmbcp                  2005c240 f   LIBCMTD:mbctype.obj
 0001:0005b260       ___initmbctable            2005c260 f   LIBCMTD:mbctype.obj
 0001:0005b290       __statusfp                 2005c290 f   LIBCMTD:ieee87.obj
 0001:0005b2b0       __clearfp                  2005c2b0 f   LIBCMTD:ieee87.obj
 0001:0005b2d0       __control87                2005c2d0 f   LIBCMTD:ieee87.obj
 0001:0005b320       __controlfp                2005c320 f   LIBCMTD:ieee87.obj
 0001:0005b340       __fpreset                  2005c340 f   LIBCMTD:ieee87.obj
 0001:0005b6d0       __ZeroTail                 2005c6d0 f   LIBCMTD:intrncvt.obj
 0001:0005b760       __IncMan                   2005c760 f   LIBCMTD:intrncvt.obj
 0001:0005b810       __RoundMan                 2005c810 f   LIBCMTD:intrncvt.obj
 0001:0005b8f0       __CopyMan                  2005c8f0 f   LIBCMTD:intrncvt.obj
 0001:0005b940       __FillZeroMan              2005c940 f   LIBCMTD:intrncvt.obj
 0001:0005b970       __IsZeroMan                2005c970 f   LIBCMTD:intrncvt.obj
 0001:0005b9b0       __ShrMan                   2005c9b0 f   LIBCMTD:intrncvt.obj
 0001:0005baa0       __ld12cvt                  2005caa0 f   LIBCMTD:intrncvt.obj
 0001:0005bce0       __ld12tod                  2005cce0 f   LIBCMTD:intrncvt.obj
 0001:0005bd00       __ld12tof                  2005cd00 f   LIBCMTD:intrncvt.obj
 0001:0005bd20       __ld12told                 2005cd20 f   LIBCMTD:intrncvt.obj
 0001:0005bdd0       __atodbl                   2005cdd0 f   LIBCMTD:intrncvt.obj
 0001:0005be20       __atoldbl                  2005ce20 f   LIBCMTD:intrncvt.obj
 0001:0005be70       __atoflt                   2005ce70 f   LIBCMTD:intrncvt.obj
 0001:0005bec0       __fptostr                  2005cec0 f   LIBCMTD:_fptostr.obj
 0001:0005bfc0       __fltout2                  2005cfc0 f   LIBCMTD:cfout.obj
 0001:0005c050       ___dtold                   2005d050 f   LIBCMTD:cfout.obj
 0001:0005c1a0       __fptrap                   2005d1a0 f   LIBCMTD:crt0fp.obj
 0001:0005c1b0       ___strgtold12              2005d1b0 f   LIBCMTD:strgtold.obj
 0001:0005cbb0       ___STRINGTOLD              2005dbb0 f   LIBCMTD:strgtold.obj
 0001:0005cc10       _mbtowc                    2005dc10 f   LIBCMTD:mbtowc.obj
 0001:0005cc50       ___mbtowc_mt               2005dc50 f   LIBCMTD:mbtowc.obj
 0001:0005cda0       __resetstkoflw             2005dda0 f   LIBCMTD:resetstk.obj
 0001:0005cef0       __allshl                   2005def0 f   LIBCMTD:llshl.obj
 0001:0005cf10       __filbuf                   2005df10 f   LIBCMTD:_filbuf.obj
 0001:0005d0e0       _ungetc                    2005e0e0 f   LIBCMTD:ungetc.obj
 0001:0005d180       __ungetc_lk                2005e180 f   LIBCMTD:ungetc.obj
 0001:0005d2b0       __dosmaperr                2005e2b0 f   LIBCMTD:dosmap.obj
 0001:0005d350       __errno                    2005e350 f   LIBCMTD:dosmap.obj
 0001:0005d360       ___doserrno                2005e360 f   LIBCMTD:dosmap.obj
 0001:0005d370       __snprintf                 2005e370 f   LIBCMTD:snprintf.obj
 0001:0005d460       __vsnprintf                2005e460 f   LIBCMTD:vsnprint.obj
 0001:0005d530       __87except                 2005e530 f   LIBCMTD:87except.obj
 0001:0005d6e0       ___ansicp                  2005e6e0 f   LIBCMTD:convrtcp.obj
 0001:0005d740       ___convertcp               2005e740 f   LIBCMTD:convrtcp.obj
 0001:0005d9e0       __matherr                  2005e9e0 f   LIBCMTD:matherr.obj
 0001:0005d9f0       __lseek                    2005e9f0 f   LIBCMTD:lseek.obj
 0001:0005db00       __lseek_lk                 2005eb00 f   LIBCMTD:lseek.obj
 0001:0005dbc0       __write                    2005ebc0 f   LIBCMTD:write.obj
 0001:0005dcd0       __write_lk                 2005ecd0 f   LIBCMTD:write.obj
 0001:0005dfc0       __getbuf                   2005efc0 f   LIBCMTD:_getbuf.obj
 0001:0005e080       __isatty                   2005f080 f   LIBCMTD:isatty.obj
 0001:0005e0c0       _wctomb                    2005f0c0 f   LIBCMTD:wctomb.obj
 0001:0005e100       ___wctomb_mt               2005f100 f   LIBCMTD:wctomb.obj
 0001:0005e1a0       __aulldiv                  2005f1a0 f   LIBCMTD:ulldiv.obj
 0001:0005e210       __aullrem                  2005f210 f   LIBCMTD:ullrem.obj
 0001:0005e290       __frnd                     2005f290 f   LIBCMTD:frnd.obj
 0001:0005e2b0       __onexit                   2005f2b0 f   LIBCMTD:onexit.obj
 0001:0005e410       _atexit                    2005f410 f   LIBCMTD:onexit.obj
 0001:0005e430       ___onexitinit              2005f430 f   LIBCMTD:onexit.obj
 0001:0005e480       __commit                   2005f480 f   LIBCMTD:commit.obj
 0001:0005e590       __stbuf                    2005f590 f   LIBCMTD:_sftbuf.obj
 0001:0005e6e0       __ftbuf                    2005f6e0 f   LIBCMTD:_sftbuf.obj
 0001:0005e770       __freebuf                  2005f770 f   LIBCMTD:_freebuf.obj
 0001:0005e800       __fcloseall                2005f800 f   LIBCMTD:closeall.obj
 0001:0005e920       ___security_init_cookie    2005f920 f   LIBCMTD:seccinit.obj
 0001:0005e9c0       ___security_error_handler  2005f9c0 f   LIBCMTD:secfail.obj
 0001:0005ebf0       __set_security_error_handler 2005fbf0 f   LIBCMTD:secfail.obj
 0001:0005ec10       ___buffer_overrun          2005fc10 f   LIBCMTD:secfail.obj
 0001:0005ec30       ___set_buffer_overrun_handler 2005fc30 f   LIBCMTD:secfail.obj
 0001:0005ec50       ?_set_new_handler@@YAP6AHI@ZP6AHI@Z@Z 2005fc50 f   LIBCMTD:handler.obj
 0001:0005ec80       ?_query_new_handler@@YAP6AHI@ZXZ 2005fc80 f   LIBCMTD:handler.obj
 0001:0005ec90       __callnewh                 2005fc90 f   LIBCMTD:handler.obj
 0001:0005ecc0       __malloc_base              2005fcc0 f   LIBCMTD:malloc.obj
 0001:0005ece0       __nh_malloc_base           2005fce0 f   LIBCMTD:malloc.obj
 0001:0005ed40       __heap_alloc_base          2005fd40 f   LIBCMTD:malloc.obj
 0001:0005ee10       __CrtDefaultAllocHook      2005fe10 f   LIBCMTD:dbghook.obj
 0001:0005ee20       __expand_base              2005fe20 f   LIBCMTD:expand.obj
 0001:0005ef40       __realloc_base             2005ff40 f   LIBCMTD:realloc.obj
 0001:0005f1f0       __free_base                200601f0 f   LIBCMTD:free.obj
 0001:0005f2c0       __heapchk                  200602c0 f   LIBCMTD:heapchk.obj
 0001:0005f380       __heapset                  20060380 f   LIBCMTD:heapchk.obj
 0001:0005f390       __get_sbh_threshold        20060390 f   LIBCMTD:sbheap.obj
 0001:0005f3b0       __set_sbh_threshold        200603b0 f   LIBCMTD:sbheap.obj
 0001:0005f420       ___sbh_heap_init           20060420 f   LIBCMTD:sbheap.obj
 0001:0005f490       ___sbh_find_block          20060490 f   LIBCMTD:sbheap.obj
 0001:0005f4f0       ___sbh_verify_block        200604f0 f   LIBCMTD:sbheap.obj
 0001:0005f550       ___sbh_free_block          20060550 f   LIBCMTD:sbheap.obj
 0001:0005fb10       ___sbh_alloc_block         20060b10 f   LIBCMTD:sbheap.obj
 0001:00060030       ___sbh_alloc_new_region    20061030 f   LIBCMTD:sbheap.obj
 0001:00060140       ___sbh_alloc_new_group     20061140 f   LIBCMTD:sbheap.obj
 0001:00060330       ___sbh_resize_block        20061330 f   LIBCMTD:sbheap.obj
 0001:00060900       ___sbh_heapmin             20061900 f   LIBCMTD:sbheap.obj
 0001:00060a30       ___sbh_heap_check          20061a30 f   LIBCMTD:sbheap.obj
 0001:00060f40       _sprintf                   20061f40 f   LIBCMTD:sprintf.obj
 0001:00061030       __scprintf                 20062030 f   LIBCMTD:sprintf.obj
 0001:000610b0       ___crtInitCritSecAndSpinCount 200620b0 f   LIBCMTD:initcrit.obj
 0001:000611d0       __ValidateEH3RN            200621d0 f   LIBCMTD:eh3valid.obj
 0001:000615c0       ___tzset                   200625c0 f   LIBCMTD:tzset.obj
 0001:00061650       __tzset                    20062650 f   LIBCMTD:tzset.obj
 0001:00061ae0       __isindst                  20062ae0 f   LIBCMTD:tzset.obj
 0001:000620c0       ___ascii_stricmp           200630c0 f   LIBCMTD:_stricmp.obj
 0001:00062110       ___getlocaleinfo           20063110 f   LIBCMTD:inithelp.obj
 0001:00062370       __stricmp                  20063370 f   LIBCMTD:stricmp.obj
 0001:00062420       __strnicmp                 20063420 f   LIBCMTD:strnicmp.obj
 0001:000624e0       ___addl                    200634e0 f   LIBCMTD:mantold.obj
 0001:00062520       ___add_12                  20063520 f   LIBCMTD:mantold.obj
 0001:000625d0       ___shl_12                  200635d0 f   LIBCMTD:mantold.obj
 0001:00062630       ___shr_12                  20063630 f   LIBCMTD:mantold.obj
 0001:000626a0       ___mtold12                 200636a0 f   LIBCMTD:mantold.obj
 0001:000627f0       _$I10_OUTPUT               200637f0 f   LIBCMTD:x10fout.obj
 0001:00062cd0       ___ld12mul                 20063cd0 f   LIBCMTD:tenpow.obj
 0001:000630c0       ___multtenpow12            200640c0 f   LIBCMTD:tenpow.obj
 0001:00063190       __read                     20064190 f   LIBCMTD:read.obj
 0001:000632a0       __read_lk                  200642a0 f   LIBCMTD:read.obj
 0001:000636e0       __alloc_osfhnd             200646e0 f   LIBCMTD:osfinfo.obj
 0001:00063960       __set_osfhnd               20064960 f   LIBCMTD:osfinfo.obj
 0001:00063a20       __free_osfhnd              20064a20 f   LIBCMTD:osfinfo.obj
 0001:00063b00       __get_osfhandle            20064b00 f   LIBCMTD:osfinfo.obj
 0001:00063b70       __open_osfhandle           20064b70 f   LIBCMTD:osfinfo.obj
 0001:00063cc0       __lock_fhandle             20064cc0 f   LIBCMTD:osfinfo.obj
 0001:00063db0       __unlock_fhandle           20064db0 f   LIBCMTD:osfinfo.obj
 0001:00063de0       __lseeki64                 20064de0 f   LIBCMTD:lseeki64.obj
 0001:00063f00       __lseeki64_lk              20064f00 f   LIBCMTD:lseeki64.obj
 0001:00063fd0       _fclose                    20064fd0 f   LIBCMTD:fclose.obj
 0001:00064090       __fclose_lk                20065090 f   LIBCMTD:fclose.obj
 0001:00064140       _getenv                    20065140 f   LIBCMTD:getenv.obj
 0001:000641b0       __getenv_lk                200651b0 f   LIBCMTD:getenv.obj
 0001:00064280       ___crtGetLocaleInfoW       20065280 f   LIBCMTD:w_loc.obj
 0001:00064460       ___crtGetLocaleInfoA       20065460 f   LIBCMTD:a_loc.obj
 0001:00064650       ___ascii_strnicmp          20065650 f   LIBCMTD:_strnicm.obj
 0001:000646c0       __close                    200656c0 f   LIBCMTD:close.obj
 0001:000647b0       __close_lk                 200657b0 f   LIBCMTD:close.obj
 0001:00064860       __mbsnbicoll               20065860 f   LIBCMTD:mbsnbico.obj
 0001:000648d0       ___wtomb_environ           200658d0 f   LIBCMTD:wtombenv.obj
 0001:000649c0       ___crtCompareStringA       200659c0 f   LIBCMTD:a_cmp.obj
 0001:00064f80       ___crtsetenv               20065f80 f   LIBCMTD:setenv.obj
 0001:00065470       __mbschr                   20066470 f   LIBCMTD:mbschr.obj
 0001:00065538       _GetModuleFileNameA@12     20066538 f   kernel32:KERNEL32.dll
 0001:0006553e       _GetCurrentThreadId@0      2006653e f   kernel32:KERNEL32.dll
 0001:00065544       _GetCommandLineA@0         20066544 f   kernel32:KERNEL32.dll
 0001:0006554a       _GetVersionExA@4           2006654a f   kernel32:KERNEL32.dll
 0001:00065550       _TlsAlloc@0                20066550 f   kernel32:KERNEL32.dll
 0001:00065556       _TlsFree@4                 20066556 f   kernel32:KERNEL32.dll
 0001:0006555c       _TlsSetValue@8             2006655c f   kernel32:KERNEL32.dll
 0001:00065562       _TlsGetValue@4             20066562 f   kernel32:KERNEL32.dll
 0001:00065568       _GetProcAddress@8          20066568 f   kernel32:KERNEL32.dll
 0001:0006556e       _GetModuleHandleA@4        2006656e f   kernel32:KERNEL32.dll
 0001:00065574       _SetLastError@4            20066574 f   kernel32:KERNEL32.dll
 0001:0006557a       _GetLastError@0            2006657a f   kernel32:KERNEL32.dll
 0001:00065580       _GetCurrentThread@0        20066580 f   kernel32:KERNEL32.dll
 0001:00065586       _DebugBreak@0              20066586 f   kernel32:KERNEL32.dll
 0001:0006558c       _GetStdHandle@4            2006658c f   kernel32:KERNEL32.dll
 0001:00065592       _WriteFile@20              20066592 f   kernel32:KERNEL32.dll
 0001:00065598       _InterlockedDecrement@4    20066598 f   kernel32:KERNEL32.dll
 0001:0006559e       _OutputDebugStringA@4      2006659e f   kernel32:KERNEL32.dll
 0001:000655a4       _LoadLibraryA@4            200665a4 f   kernel32:KERNEL32.dll
 0001:000655aa       _InterlockedIncrement@4    200665aa f   kernel32:KERNEL32.dll
 0001:000655b0       _WideCharToMultiByte@32    200665b0 f   kernel32:KERNEL32.dll
 0001:000655b6       _MultiByteToWideChar@24    200665b6 f   kernel32:KERNEL32.dll
 0001:000655bc       _LCMapStringA@24           200665bc f   kernel32:KERNEL32.dll
 0001:000655c2       _LCMapStringW@24           200665c2 f   kernel32:KERNEL32.dll
 0001:000655c8       _RaiseException@16         200665c8 f   kernel32:KERNEL32.dll
 0001:000655ce       _TerminateProcess@8        200665ce f   kernel32:KERNEL32.dll
 0001:000655d4       _GetCurrentProcess@0       200665d4 f   kernel32:KERNEL32.dll
 0001:000655da       _ExitProcess@4             200665da f   kernel32:KERNEL32.dll
 0001:000655e0       _SetConsoleCtrlHandler@8   200665e0 f   kernel32:KERNEL32.dll
 0001:000655e6       _EnterCriticalSection@4    200665e6 f   kernel32:KERNEL32.dll
 0001:000655ec       _LeaveCriticalSection@4    200665ec f   kernel32:KERNEL32.dll
 0001:000655f2       _IsBadWritePtr@8           200665f2 f   kernel32:KERNEL32.dll
 0001:000655f8       _IsBadReadPtr@8            200665f8 f   kernel32:KERNEL32.dll
 0001:000655fe       _HeapValidate@12           200665fe f   kernel32:KERNEL32.dll
 0001:00065604       _SetHandleCount@4          20066604 f   kernel32:KERNEL32.dll
 0001:0006560a       _GetFileType@4             2006660a f   kernel32:KERNEL32.dll
 0001:00065610       _GetStartupInfoA@4         20066610 f   kernel32:KERNEL32.dll
 0001:00065616       _DeleteCriticalSection@4   20066616 f   kernel32:KERNEL32.dll
 0001:0006561c       _FreeEnvironmentStringsA@4 2006661c f   kernel32:KERNEL32.dll
 0001:00065622       _GetEnvironmentStrings@0   20066622 f   kernel32:KERNEL32.dll
 0001:00065628       _FreeEnvironmentStringsW@4 20066628 f   kernel32:KERNEL32.dll
 0001:0006562e       _GetEnvironmentStringsW@0  2006662e f   kernel32:KERNEL32.dll
 0001:00065634       _HeapDestroy@4             20066634 f   kernel32:KERNEL32.dll
 0001:0006563a       _HeapCreate@12             2006663a f   kernel32:KERNEL32.dll
 0001:00065640       _HeapFree@12               20066640 f   kernel32:KERNEL32.dll
 0001:00065646       _VirtualFree@12            20066646 f   kernel32:KERNEL32.dll
 0001:0006564c       _UnhandledExceptionFilter@4 2006664c f   kernel32:KERNEL32.dll
 0001:00065652       _RtlUnwind@16              20066652 f   kernel32:KERNEL32.dll
 0001:00065658       _GetStringTypeA@20         20066658 f   kernel32:KERNEL32.dll
 0001:0006565e       _GetStringTypeW@16         2006665e f   kernel32:KERNEL32.dll
 0001:00065664       _GetTimeFormatA@24         20066664 f   kernel32:KERNEL32.dll
 0001:0006566a       _GetDateFormatA@24         2006666a f   kernel32:KERNEL32.dll
 0001:00065670       _GetCPInfo@8               20066670 f   kernel32:KERNEL32.dll
 0001:00065676       _FatalAppExitA@8           20066676 f   kernel32:KERNEL32.dll
 0001:0006567c       _IsValidLocale@8           2006667c f   kernel32:KERNEL32.dll
 0001:00065682       _IsValidCodePage@4         20066682 f   kernel32:KERNEL32.dll
 0001:00065688       _GetLocaleInfoA@16         20066688 f   kernel32:KERNEL32.dll
 0001:0006568e       _EnumSystemLocalesA@8      2006668e f   kernel32:KERNEL32.dll
 0001:00065694       _GetUserDefaultLCID@0      20066694 f   kernel32:KERNEL32.dll
 0001:0006569a       _GetACP@0                  2006669a f   kernel32:KERNEL32.dll
 0001:000656a0       _GetOEMCP@0                200666a0 f   kernel32:KERNEL32.dll
 0001:000656a6       _VirtualProtect@16         200666a6 f   kernel32:KERNEL32.dll
 0001:000656ac       _VirtualAlloc@16           200666ac f   kernel32:KERNEL32.dll
 0001:000656b2       _GetSystemInfo@4           200666b2 f   kernel32:KERNEL32.dll
 0001:000656b8       _VirtualQuery@12           200666b8 f   kernel32:KERNEL32.dll
 0001:000656be       _SetFilePointer@16         200666be f   kernel32:KERNEL32.dll
 0001:000656c4       _FlushFileBuffers@4        200666c4 f   kernel32:KERNEL32.dll
 0001:000656ca       _QueryPerformanceCounter@4 200666ca f   kernel32:KERNEL32.dll
 0001:000656d0       _GetTickCount@0            200666d0 f   kernel32:KERNEL32.dll
 0001:000656d6       _GetCurrentProcessId@0     200666d6 f   kernel32:KERNEL32.dll
 0001:000656dc       _GetSystemTimeAsFileTime@4 200666dc f   kernel32:KERNEL32.dll
 0001:000656e2       _HeapAlloc@12              200666e2 f   kernel32:KERNEL32.dll
 0001:000656e8       _HeapReAlloc@16            200666e8 f   kernel32:KERNEL32.dll
 0001:000656ee       _InitializeCriticalSection@4 200666ee f   kernel32:KERNEL32.dll
 0001:000656f4       _InterlockedExchange@8     200666f4 f   kernel32:KERNEL32.dll
 0001:000656fa       _GetTimeZoneInformation@4  200666fa f   kernel32:KERNEL32.dll
 0001:00065700       _ReadFile@20               20066700 f   kernel32:KERNEL32.dll
 0001:00065706       _SetStdHandle@8            20066706 f   kernel32:KERNEL32.dll
 0001:0006570c       _GetLocaleInfoW@16         2006670c f   kernel32:KERNEL32.dll
 0001:00065712       _CloseHandle@4             20066712 f   kernel32:KERNEL32.dll
 0001:00065718       _CompareStringA@24         20066718 f   kernel32:KERNEL32.dll
 0001:0006571e       _CompareStringW@24         2006671e f   kernel32:KERNEL32.dll
 0001:00065724       _SetEnvironmentVariableA@8 20066724 f   kernel32:KERNEL32.dll
 0002:00000000       __imp__GetModuleFileNameA@12 20067000     kernel32:KERNEL32.dll
 0002:00000004       __imp__GetCurrentThreadId@0 20067004     kernel32:KERNEL32.dll
 0002:00000008       __imp__GetCommandLineA@0   20067008     kernel32:KERNEL32.dll
 0002:0000000c       __imp__GetVersionExA@4     2006700c     kernel32:KERNEL32.dll
 0002:00000010       __imp__TlsAlloc@0          20067010     kernel32:KERNEL32.dll
 0002:00000014       __imp__TlsFree@4           20067014     kernel32:KERNEL32.dll
 0002:00000018       __imp__TlsSetValue@8       20067018     kernel32:KERNEL32.dll
 0002:0000001c       __imp__TlsGetValue@4       2006701c     kernel32:KERNEL32.dll
 0002:00000020       __imp__GetProcAddress@8    20067020     kernel32:KERNEL32.dll
 0002:00000024       __imp__GetModuleHandleA@4  20067024     kernel32:KERNEL32.dll
 0002:00000028       __imp__SetLastError@4      20067028     kernel32:KERNEL32.dll
 0002:0000002c       __imp__GetLastError@0      2006702c     kernel32:KERNEL32.dll
 0002:00000030       __imp__GetCurrentThread@0  20067030     kernel32:KERNEL32.dll
 0002:00000034       __imp__DebugBreak@0        20067034     kernel32:KERNEL32.dll
 0002:00000038       __imp__GetStdHandle@4      20067038     kernel32:KERNEL32.dll
 0002:0000003c       __imp__WriteFile@20        2006703c     kernel32:KERNEL32.dll
 0002:00000040       __imp__InterlockedDecrement@4 20067040     kernel32:KERNEL32.dll
 0002:00000044       __imp__OutputDebugStringA@4 20067044     kernel32:KERNEL32.dll
 0002:00000048       __imp__LoadLibraryA@4      20067048     kernel32:KERNEL32.dll
 0002:0000004c       __imp__InterlockedIncrement@4 2006704c     kernel32:KERNEL32.dll
 0002:00000050       __imp__WideCharToMultiByte@32 20067050     kernel32:KERNEL32.dll
 0002:00000054       __imp__MultiByteToWideChar@24 20067054     kernel32:KERNEL32.dll
 0002:00000058       __imp__LCMapStringA@24     20067058     kernel32:KERNEL32.dll
 0002:0000005c       __imp__LCMapStringW@24     2006705c     kernel32:KERNEL32.dll
 0002:00000060       __imp__RaiseException@16   20067060     kernel32:KERNEL32.dll
 0002:00000064       __imp__TerminateProcess@8  20067064     kernel32:KERNEL32.dll
 0002:00000068       __imp__GetCurrentProcess@0 20067068     kernel32:KERNEL32.dll
 0002:0000006c       __imp__ExitProcess@4       2006706c     kernel32:KERNEL32.dll
 0002:00000070       __imp__SetConsoleCtrlHandler@8 20067070     kernel32:KERNEL32.dll
 0002:00000074       __imp__EnterCriticalSection@4 20067074     kernel32:KERNEL32.dll
 0002:00000078       __imp__LeaveCriticalSection@4 20067078     kernel32:KERNEL32.dll
 0002:0000007c       __imp__IsBadWritePtr@8     2006707c     kernel32:KERNEL32.dll
 0002:00000080       __imp__IsBadReadPtr@8      20067080     kernel32:KERNEL32.dll
 0002:00000084       __imp__HeapValidate@12     20067084     kernel32:KERNEL32.dll
 0002:00000088       __imp__SetHandleCount@4    20067088     kernel32:KERNEL32.dll
 0002:0000008c       __imp__GetFileType@4       2006708c     kernel32:KERNEL32.dll
 0002:00000090       __imp__GetStartupInfoA@4   20067090     kernel32:KERNEL32.dll
 0002:00000094       __imp__DeleteCriticalSection@4 20067094     kernel32:KERNEL32.dll
 0002:00000098       __imp__FreeEnvironmentStringsA@4 20067098     kernel32:KERNEL32.dll
 0002:0000009c       __imp__GetEnvironmentStrings@0 2006709c     kernel32:KERNEL32.dll
 0002:000000a0       __imp__FreeEnvironmentStringsW@4 200670a0     kernel32:KERNEL32.dll
 0002:000000a4       __imp__GetEnvironmentStringsW@0 200670a4     kernel32:KERNEL32.dll
 0002:000000a8       __imp__HeapDestroy@4       200670a8     kernel32:KERNEL32.dll
 0002:000000ac       __imp__HeapCreate@12       200670ac     kernel32:KERNEL32.dll
 0002:000000b0       __imp__HeapFree@12         200670b0     kernel32:KERNEL32.dll
 0002:000000b4       __imp__VirtualFree@12      200670b4     kernel32:KERNEL32.dll
 0002:000000b8       __imp__UnhandledExceptionFilter@4 200670b8     kernel32:KERNEL32.dll
 0002:000000bc       __imp__RtlUnwind@16        200670bc     kernel32:KERNEL32.dll
 0002:000000c0       __imp__GetStringTypeA@20   200670c0     kernel32:KERNEL32.dll
 0002:000000c4       __imp__GetStringTypeW@16   200670c4     kernel32:KERNEL32.dll
 0002:000000c8       __imp__GetTimeFormatA@24   200670c8     kernel32:KERNEL32.dll
 0002:000000cc       __imp__GetDateFormatA@24   200670cc     kernel32:KERNEL32.dll
 0002:000000d0       __imp__GetCPInfo@8         200670d0     kernel32:KERNEL32.dll
 0002:000000d4       __imp__FatalAppExitA@8     200670d4     kernel32:KERNEL32.dll
 0002:000000d8       __imp__IsValidLocale@8     200670d8     kernel32:KERNEL32.dll
 0002:000000dc       __imp__IsValidCodePage@4   200670dc     kernel32:KERNEL32.dll
 0002:000000e0       __imp__GetLocaleInfoA@16   200670e0     kernel32:KERNEL32.dll
 0002:000000e4       __imp__EnumSystemLocalesA@8 200670e4     kernel32:KERNEL32.dll
 0002:000000e8       __imp__GetUserDefaultLCID@0 200670e8     kernel32:KERNEL32.dll
 0002:000000ec       __imp__GetACP@0            200670ec     kernel32:KERNEL32.dll
 0002:000000f0       __imp__GetOEMCP@0          200670f0     kernel32:KERNEL32.dll
 0002:000000f4       __imp__VirtualProtect@16   200670f4     kernel32:KERNEL32.dll
 0002:000000f8       __imp__VirtualAlloc@16     200670f8     kernel32:KERNEL32.dll
 0002:000000fc       __imp__GetSystemInfo@4     200670fc     kernel32:KERNEL32.dll
 0002:00000100       __imp__VirtualQuery@12     20067100     kernel32:KERNEL32.dll
 0002:00000104       __imp__SetFilePointer@16   20067104     kernel32:KERNEL32.dll
 0002:00000108       __imp__FlushFileBuffers@4  20067108     kernel32:KERNEL32.dll
 0002:0000010c       __imp__QueryPerformanceCounter@4 2006710c     kernel32:KERNEL32.dll
 0002:00000110       __imp__GetTickCount@0      20067110     kernel32:KERNEL32.dll
 0002:00000114       __imp__GetCurrentProcessId@0 20067114     kernel32:KERNEL32.dll
 0002:00000118       __imp__GetSystemTimeAsFileTime@4 20067118     kernel32:KERNEL32.dll
 0002:0000011c       __imp__HeapAlloc@12        2006711c     kernel32:KERNEL32.dll
 0002:00000120       __imp__HeapReAlloc@16      20067120     kernel32:KERNEL32.dll
 0002:00000124       __imp__InitializeCriticalSection@4 20067124     kernel32:KERNEL32.dll
 0002:00000128       __imp__InterlockedExchange@8 20067128     kernel32:KERNEL32.dll
 0002:0000012c       __imp__GetTimeZoneInformation@4 2006712c     kernel32:KERNEL32.dll
 0002:00000130       __imp__ReadFile@20         20067130     kernel32:KERNEL32.dll
 0002:00000134       __imp__SetStdHandle@8      20067134     kernel32:KERNEL32.dll
 0002:00000138       __imp__GetLocaleInfoW@16   20067138     kernel32:KERNEL32.dll
 0002:0000013c       __imp__CloseHandle@4       2006713c     kernel32:KERNEL32.dll
 0002:00000140       __imp__CompareStringA@24   20067140     kernel32:KERNEL32.dll
 0002:00000144       __imp__CompareStringW@24   20067144     kernel32:KERNEL32.dll
 0002:00000148       __imp__SetEnvironmentVariableA@8 20067148     kernel32:KERNEL32.dll
 0002:0000014c       \177KERNEL32_NULL_THUNK_DATA 2006714c     kernel32:KERNEL32.dll
 0002:0000016c       ??_C@_01PFHFFBPC@t?$AA@    2006716c     ai_chat.obj
 0002:00000170       ??_C@_01EFFIKLCJ@n?$AA@    20067170     ai_chat.obj
 0002:00000174       ??_C@_0O@OCOCOONB@sv_maxclients?$AA@ 20067174     ai_chat.obj
 0002:00000184       __real@46fffe00            20067184     ai_chat.obj
 0002:00000188       ??_C@_07KMNEBLH@mapname?$AA@ 20067188     ai_chat.obj
 0002:00000190       ??_C@_0BB@FPHHFAJG@?$FLunknown?5weapon?$FN?$AA@ 20067190     ai_chat.obj
 0002:000001a4       ??_C@_07MKHABLGK@Grapple?$AA@ 200671a4     ai_chat.obj
 0002:000001ac       ??_C@_06PNKEMFGD@BFG10K?$AA@ 200671ac     ai_chat.obj
 0002:000001b4       ??_C@_0O@HOCKKNKE@Lightning?5Gun?$AA@ 200671b4     ai_chat.obj
 0002:000001c4       ??_C@_07NMJDHEIK@Railgun?$AA@ 200671c4     ai_chat.obj
 0002:000001cc       ??_C@_09MBHKGILD@Plasmagun?$AA@ 200671cc     ai_chat.obj
 0002:000001d8       ??_C@_0BA@DJIGCIDL@Rocket?5Launcher?$AA@ 200671d8     ai_chat.obj
 0002:000001e8       ??_C@_0BB@GIEOMMBO@Grenade?5Launcher?$AA@ 200671e8     ai_chat.obj
 0002:000001fc       ??_C@_0L@KDNGMPND@Machinegun?$AA@ 200671fc     ai_chat.obj
 0002:00000208       ??_C@_08ELAHAPJB@Gauntlet?$AA@ 20067208     ai_chat.obj
 0002:00000214       ??_C@_07DGIAOJJ@Shotgun?$AA@ 20067214     ai_chat.obj
 0002:00000220       __real@4021cccccccccccd    20067220     ai_chat.obj
 0002:00000228       __real@00000000            20067228     ai_chat.obj
 0002:0000022c       __real@41200000            2006722c     ai_chat.obj
 0002:00000230       __real@3f800000            20067230     ai_chat.obj
 0002:00000234       __real@42000000            20067234     ai_chat.obj
 0002:00000238       __real@41c00000            20067238     ai_chat.obj
 0002:0000023c       ??_C@_0L@PKHLIBCF@game_enter?$AA@ 2006723c     ai_chat.obj
 0002:00000248       ??_C@_0O@IGAOFANI@?$FLinvalid?5var?$FN?$AA@ 20067248     ai_chat.obj
 0002:00000258       __real@41c80000            20067258     ai_chat.obj
 0002:0000025c       ??_C@_09PIOCENHO@game_exit?$AA@ 2006725c     ai_chat.obj
 0002:00000268       ??_C@_0M@CJNDJGDH@level_start?$AA@ 20067268     ai_chat.obj
 0002:00000274       ??_C@_06IMDBNOMM@vtaunt?$AA@ 20067274     ai_chat.obj
 0002:0000027c       ??_C@_09PILOJEEK@level_end?$AA@ 2006727c     ai_chat.obj
 0002:00000288       ??_C@_0P@LPKGAAGE@level_end_lose?$AA@ 20067288     ai_chat.obj
 0002:00000298       ??_C@_0BC@GKFLFIDK@level_end_victory?$AA@ 20067298     ai_chat.obj
 0002:000002ac       ??_C@_0N@INLGGPBP@death_praise?$AA@ 200672ac     ai_chat.obj
 0002:000002bc       ??_C@_0N@EPKIJPHK@death_insult?$AA@ 200672bc     ai_chat.obj
 0002:000002cc       ??_C@_09HPMGADCC@death_bfg?$AA@ 200672cc     ai_chat.obj
 0002:000002d8       ??_C@_0L@OLPOCBHN@death_rail?$AA@ 200672d8     ai_chat.obj
 0002:000002e4       ??_C@_0P@GODBEIFH@death_gauntlet?$AA@ 200672e4     ai_chat.obj
 0002:000002f8       __real@3fe0000000000000    200672f8     ai_chat.obj
 0002:00000300       ??_C@_0P@CLLHBMMH@death_telefrag?$AA@ 20067300     ai_chat.obj
 0002:00000310       ??_C@_0O@EGKCFKBF@death_suicide?$AA@ 20067310     ai_chat.obj
 0002:00000320       ??_C@_0P@FHLBDKHM@death_cratered?$AA@ 20067320     ai_chat.obj
 0002:00000330       ??_C@_0L@JGPKJCJO@death_lava?$AA@ 20067330     ai_chat.obj
 0002:0000033c       ??_C@_0M@ENLBBGB@death_slime?$AA@ 2006733c     ai_chat.obj
 0002:00000348       ??_C@_0M@BCPGKKBA@death_drown?$AA@ 20067348     ai_chat.obj
 0002:00000354       ??_C@_0P@LLJEDFBD@death_teammate?$AA@ 20067354     ai_chat.obj
 0002:00000364       ??_C@_07PANFCHNN@?$FLworld?$FN?$AA@ 20067364     ai_chat.obj
 0002:0000036c       ??_C@_0M@NDKPNHB@kill_praise?$AA@ 2006736c     ai_chat.obj
 0002:00000378       ??_C@_0M@MPCEANBE@kill_insult?$AA@ 20067378     ai_chat.obj
 0002:00000384       ??_C@_0O@MOMICIAK@kill_telefrag?$AA@ 20067384     ai_chat.obj
 0002:00000394       ??_C@_09HNPOIBHL@kill_rail?$AA@ 20067394     ai_chat.obj
 0002:000003a0       ??_C@_0O@ILEOHMJK@kill_gauntlet?$AA@ 200673a0     ai_chat.obj
 0002:000003b0       ??_C@_0O@FOOLABNO@kill_teammate?$AA@ 200673b0     ai_chat.obj
 0002:000003c0       ??_C@_0O@CCLFCPCH@enemy_suicide?$AA@ 200673c0     ai_chat.obj
 0002:000003ce       ??_C@_00CNPNBAHC@?$AA@     200673ce     ai_chat.obj
 0002:000003d0       ??_C@_0M@GJHANCBL@hit_talking?$AA@ 200673d0     ai_chat.obj
 0002:000003dc       ??_C@_0M@NEMKKKCP@hit_nodeath?$AA@ 200673dc     ai_chat.obj
 0002:000003e8       ??_C@_0L@HALGAHGK@hit_nokill?$AA@ 200673e8     ai_chat.obj
 0002:000003f4       ??_C@_0O@BCFFFDNI@random_insult?$AA@ 200673f4     ai_chat.obj
 0002:00000404       ??_C@_0M@DCDJELGA@random_misc?$AA@ 20067404     ai_chat.obj
 0002:00000410       __real@3fd0000000000000    20067410     ai_chat.obj
 0002:00000418       __real@3fb999999999999a    20067418     ai_chat.obj
 0002:00000420       __real@40000000            20067420     ai_chat.obj
 0002:00000424       ??_C@_0BN@OHELPGJE@?$CFs?3?5I?8ve?5got?5a?5regular?5goal?6?$AA@ 20067424     ai_cmd.obj
 0002:00000444       ??_C@_0CD@LMLPDLJC@?$CFs?3?5I?8m?5gonna?5roam?5for?5?$CF1?40f?5sec@ 20067444     ai_cmd.obj
 0002:00000468       ??_C@_0CF@DLPLJMNN@?$CFs?3?5I?8m?5gonna?5patrol?5for?5?$CF1?40f?5s@ 20067468     ai_cmd.obj
 0002:00000490       ??_C@_0CD@EMLIGCBD@?$CFs?3?5I?8m?5gonna?5camp?5for?5?$CF1?40f?5sec@ 20067490     ai_cmd.obj
 0002:000004b4       ??_C@_0CL@DDPGIFJG@?$CFs?3?5I?8m?5gonna?5kill?5someone?5for?5?$CF@ 200674b4     ai_cmd.obj
 0002:000004e0       ??_C@_0CK@DNEMKHBG@?$CFs?3?5I?8m?5gonna?5get?5an?5item?5for?5?$CF1@ 200674e0     ai_cmd.obj
 0002:0000050c       ??_C@_0DA@LGFLAKNG@?$CFs?3?5I?8m?5gonna?5defend?5a?5key?5area?5@ 2006750c     ai_cmd.obj
 0002:0000053c       ??_C@_0DF@COPPFAKG@?$CFs?3?5I?8m?5gonna?5try?5to?5return?5the?5@ 2006753c     ai_cmd.obj
 0002:00000574       ??_C@_0CP@EDGAPFMF@?$CFs?3?5I?8m?5gonna?5rush?5to?5the?5base?5f@ 20067574     ai_cmd.obj
 0002:000005a4       ??_C@_0CL@EMAFNDIM@?$CFs?3?5I?8m?5gonna?5get?5the?5flag?5for?5?$CF@ 200675a4     ai_cmd.obj
 0002:000005d0       ??_C@_0DE@GKHGGPOB@?$CFs?3?5I?8m?5gonna?5accompany?5a?5team?5m@ 200675d0     ai_cmd.obj
 0002:00000604       ??_C@_0CP@DNGNKLJC@?$CFs?3?5I?8m?5gonna?5help?5a?5team?5mate?5f@ 20067604     ai_cmd.obj
 0002:00000638       __real@404e000000000000    20067638     ai_cmd.obj
 0002:00000640       ??_C@_0CC@BCALNIDF@I?5need?5more?5key?5points?5to?5patrol@ 20067640     ai_cmd.obj
 0002:00000664       ??_C@_0BB@PGBIDPPC@what?5do?5you?5say?$DP?$AA@ 20067664     ai_cmd.obj
 0002:00000678       ??_C@_03PMGGPEJJ@?$CFd?6?$AA@ 20067678     ai_cmd.obj
 0002:0000067c       __real@44160000            2006767c     ai_cmd.obj
 0002:00000680       __real@42700000            20067680     ai_cmd.obj
 0002:00000684       ??_C@_0M@HCHCFBDA@whereareyou?$AA@ 20067684     ai_cmd.obj
 0002:00000690       ??_C@_07BANGEKHA@whereis?$AA@ 20067690     ai_cmd.obj
 0002:00000698       ??_C@_05NBAJGCGG@whois?$AA@ 20067698     ai_cmd.obj
 0002:000006a0       __real@42f00000            200676a0     ai_cmd.obj
 0002:000006a4       ??_C@_03ICICOMAL@yes?$AA@  200676a4     ai_cmd.obj
 0002:000006a8       ??_C@_0L@CCGDOBMA@keepinmind?$AA@ 200676a8     ai_cmd.obj
 0002:000006b4       __real@43340000            200676b4     ai_cmd.obj
 0002:000006b8       ??_C@_0L@OAEJIBOJ@joinedteam?$AA@ 200676b8     ai_cmd.obj
 0002:000006c4       ??_C@_08NKJDPEPF@leftteam?$AA@ 200676c4     ai_cmd.obj
 0002:000006d0       ??_C@_06NJFEFPHF@noteam?$AA@ 200676d0     ai_cmd.obj
 0002:000006d8       ??_C@_06NHKPLCFO@inteam?$AA@ 200676d8     ai_cmd.obj
 0002:000006e0       ??_C@_0BD@PGFNLHLB@checkpoint_confirm?$AA@ 200676e0     ai_cmd.obj
 0002:000006f4       ??_C@_0BC@PAJMIFOG@?$CF1?40f?5?$CF1?40f?5?$CF1?40f?$AA@ 200676f4     ai_cmd.obj
 0002:00000708       ??_C@_0BD@GKCAPLMB@checkpoint_invalid?$AA@ 20067708     ai_cmd.obj
 0002:0000071c       ??_C@_08OEKJENGB@?$CFf?5?$CFf?5?$CFf?$AA@ 2006771c     ai_cmd.obj
 0002:00000728       __real@43fa0000            20067728     ai_cmd.obj
 0002:0000072c       __real@42400000            2006772c     ai_cmd.obj
 0002:00000730       __real@4040000000000000    20067730     ai_cmd.obj
 0002:00000738       __real@402381d7dbf487fd    20067738     ai_cmd.obj
 0002:00000740       ??_C@_09FLIJNDLN@dismissed?$AA@ 20067740     ai_cmd.obj
 0002:0000074c       ??_C@_05CPCHEFAA@taunt?$AA@ 2006774c     ai_cmd.obj
 0002:00000754       ??_C@_04BJJEOANI@kill?$AA@ 20067754     ai_cmd.obj
 0002:0000075c       ??_C@_0BF@EGOEAANC@I?8m?5the?5team?5leader?6?$AA@ 2006775c     ai_cmd.obj
 0002:00000774       ??_C@_07IFIHEGLH@roaming?$AA@ 20067774     ai_cmd.obj
 0002:0000077c       ??_C@_0O@PNEKPGNP@returningflag?$AA@ 2006777c     ai_cmd.obj
 0002:0000078c       ??_C@_0M@BGGCILAH@rushingbase?$AA@ 2006778c     ai_cmd.obj
 0002:00000798       ??_C@_0O@KMOOAPPA@capturingflag?$AA@ 20067798     ai_cmd.obj
 0002:000007a8       ??_C@_0L@GHJELNDI@patrolling?$AA@ 200677a8     ai_cmd.obj
 0002:000007b4       ??_C@_07IKBLJPBH@camping?$AA@ 200677b4     ai_cmd.obj
 0002:000007bc       ??_C@_07EFNGDOD@killing?$AA@ 200677bc     ai_cmd.obj
 0002:000007c4       ??_C@_0M@EEGCLMEK@gettingitem?$AA@ 200677c4     ai_cmd.obj
 0002:000007d0       ??_C@_09GNBACBHC@defending?$AA@ 200677d0     ai_cmd.obj
 0002:000007dc       ??_C@_0N@FBKCFEPP@accompanying?$AA@ 200677dc     ai_cmd.obj
 0002:000007ec       ??_C@_07OIGCHEPH@helping?$AA@ 200677ec     ai_cmd.obj
 0002:000007f8       __real@3ff0000000000000    200677f8     ai_cmd.obj
 0002:00000800       ??_C@_08CBBFJFMD@location?$AA@ 20067800     ai_cmd.obj
 0002:0000080c       ??_C@_04OBGPFBCN@blue?$AA@ 2006780c     ai_cmd.obj
 0002:00000814       ??_C@_0N@LHJHAMNN@teamlocation?$AA@ 20067814     ai_cmd.obj
 0002:00000824       ??_C@_03FAAAOPJM@red?$AA@  20067824     ai_cmd.obj
 0002:00000828       __real@3fd999999999999a    20067828     ai_cmd.obj
 0002:00000830       ??_C@_09MDBFHCAB@Blue?5Flag?$AA@ 20067830     ai_cmd.obj
 0002:0000083c       ??_C@_08GAOGPIJL@Red?5Flag?$AA@ 2006783c     ai_cmd.obj
 0002:00000848       ??_C@_0M@ICCAHGAD@Heavy?5Armor?$AA@ 20067848     ai_cmd.obj
 0002:00000854       ??_C@_05JOOFIMIN@Armor?$AA@ 20067854     ai_cmd.obj
 0002:0000085c       ??_C@_06FDKFDAP@Flight?$AA@ 2006785c     ai_cmd.obj
 0002:00000864       ??_C@_0N@LCCEENAK@Invisibility?$AA@ 20067864     ai_cmd.obj
 0002:00000874       ??_C@_05HOIAGEJD@Speed?$AA@ 20067874     ai_cmd.obj
 0002:0000087c       ??_C@_0M@ONKEJEFE@Battle?5Suit?$AA@ 2006787c     ai_cmd.obj
 0002:00000888       ??_C@_0N@CBPBLBHG@Regeneration?$AA@ 20067888     ai_cmd.obj
 0002:00000898       ??_C@_0M@KOJLOALK@Quad?5Damage?$AA@ 20067898     ai_cmd.obj
 0002:000008a4       ??_C@_0BE@NHGFGLLF@unknown?5match?5type?6?$AA@ 200678a4     ai_cmd.obj
 0002:000008b8       ??_C@_0DL@ENJHCNMJ@the?5part?5of?5my?5brain?5to?5create?5f@ 200678b8     ai_cmd.obj
 0002:000008f4       ??_C@_0CM@FBOPNIPA@?$CFs?5at?5?$CF1?41f?5switched?5more?5than?5?$CF@ 200678f4     ai_dmnet.obj
 0002:00000920       ??_C@_0CE@EJLGIIOB@?$CFs?5at?5?$CF2?41f?5entered?5?$CFs?3?5?$CFs?5from?5@ 20067920     ai_dmnet.obj
 0002:00000944       __real@447a0000            20067944     ai_dmnet.obj
 0002:00000948       __real@40c00000            20067948     ai_dmnet.obj
 0002:0000094c       ??_C@_0CD@NJJLHGEF@?$CFs?3?5no?5valid?5ltg?5?$CIprobably?5stuck@ 2006794c     ai_dmnet.obj
 0002:00000970       __real@41a00000            20067970     ai_dmnet.obj
 0002:00000974       ??_C@_0N@INDGBJCC@onreturnflag?$AA@ 20067974     ai_dmnet.obj
 0002:00000984       ??_C@_0BB@BFOOKAAN@returnflag_start?$AA@ 20067984     ai_dmnet.obj
 0002:00000998       ??_C@_09DPAAIBFE@ongetflag?$AA@ 20067998     ai_dmnet.obj
 0002:000009a4       ??_C@_0BC@BPHAAOLA@captureflag_start?$AA@ 200679a4     ai_dmnet.obj
 0002:000009b8       ??_C@_0M@JOFDEJLG@patrol_stop?$AA@ 200679b8     ai_dmnet.obj
 0002:000009c4       ??_C@_0N@IKJEFKFP@patrol_start?$AA@ 200679c4     ai_dmnet.obj
 0002:000009d4       ??_C@_04MKEOLIJC@?5to?5?$AA@ 200679d4     ai_dmnet.obj
 0002:000009dc       ??_C@_0L@IJFFADDJ@inposition?$AA@ 200679dc     ai_dmnet.obj
 0002:000009e8       ??_C@_0M@PEOBAIFC@camp_arrive?$AA@ 200679e8     ai_dmnet.obj
 0002:000009f4       __real@45610000            200679f4     ai_dmnet.obj
 0002:000009f8       ??_C@_09BHIDKEB@camp_stop?$AA@ 200679f8     ai_dmnet.obj
 0002:00000a04       ??_C@_0L@KJNCBGJD@camp_start?$AA@ 20067a04     ai_dmnet.obj
 0002:00000a10       ??_C@_0O@EJODLBHP@getitem_gotit?$AA@ 20067a10     ai_dmnet.obj
 0002:00000a20       ??_C@_0BB@GOIMPKGP@getitem_notthere?$AA@ 20067a20     ai_dmnet.obj
 0002:00000a34       ??_C@_0O@LBCALMFN@getitem_start?$AA@ 20067a34     ai_dmnet.obj
 0002:00000a44       ??_C@_09KGAMDJKG@kill_done?$AA@ 20067a44     ai_dmnet.obj
 0002:00000a50       ??_C@_0L@DMKJIHAF@kill_start?$AA@ 20067a50     ai_dmnet.obj
 0002:00000a5c       __real@40400000            20067a5c     ai_dmnet.obj
 0002:00000a60       __real@45992000            20067a60     ai_dmnet.obj
 0002:00000a64       ??_C@_0M@DFCLNMCD@defend_stop?$AA@ 20067a64     ai_dmnet.obj
 0002:00000a70       ??_C@_09DPKMICOA@ondefense?$AA@ 20067a70     ai_dmnet.obj
 0002:00000a7c       ??_C@_0N@KFKEFAB@defend_start?$AA@ 20067a7c     ai_dmnet.obj
 0002:00000a8c       ??_C@_0BF@DCOBNKPB@accompany_cannotfind?$AA@ 20067a8c     ai_dmnet.obj
 0002:00000aa4       ??_C@_0BM@KDEEGPGK@BotLongTermGoal?3?5go?5for?5air?$AA@ 20067aa4     ai_dmnet.obj
 0002:00000ac0       __real@41000000            20067ac0     ai_dmnet.obj
 0002:00000ac8       __real@3fe999999999999a    20067ac8     ai_dmnet.obj
 0002:00000ad0       __real@3fa999999999999a    20067ad0     ai_dmnet.obj
 0002:00000ad8       ??_C@_0BB@FONGAGIJ@accompany_arrive?$AA@ 20067ad8     ai_dmnet.obj
 0002:00000aec       __real@41700000            20067aec     ai_dmnet.obj
 0002:00000af0       __real@40a00000            20067af0     ai_dmnet.obj
 0002:00000af8       __real@3fe6666666666666    20067af8     ai_dmnet.obj
 0002:00000b00       __real@40800000            20067b00     ai_dmnet.obj
 0002:00000b04       ??_C@_0P@JLGJIDCE@accompany_stop?$AA@ 20067b04     ai_dmnet.obj
 0002:00000b14       ??_C@_0BA@JEJAJCPN@accompany_start?$AA@ 20067b14     ai_dmnet.obj
 0002:00000b24       __real@461c4000            20067b24     ai_dmnet.obj
 0002:00000b28       ??_C@_0L@JEGDCFOO@help_start?$AA@ 20067b28     ai_dmnet.obj
 0002:00000b34       __real@48742400            20067b34     ai_dmnet.obj
 0002:00000b38       ??_C@_08LJGLPHPA@followme?$AA@ 20067b38     ai_dmnet.obj
 0002:00000b44       ??_C@_09GJKBJNFC@lead_stop?$AA@ 20067b44     ai_dmnet.obj
 0002:00000b50       ??_C@_0N@IHDBPIFK@intermission?$AA@ 20067b50     ai_dmnet.obj
 0002:00000b60       ??_C@_0BD@FAEFJCHC@intermission?3?5chat?$AA@ 20067b60     ai_dmnet.obj
 0002:00000b74       ??_C@_08BDAIAION@observer?$AA@ 20067b74     ai_dmnet.obj
 0002:00000b80       ??_C@_0BI@BGMGILOO@observer?3?5left?5observer?$AA@ 20067b80     ai_dmnet.obj
 0002:00000b98       ??_C@_05PJLLPND@stand?$AA@ 20067b98     ai_dmnet.obj
 0002:00000ba0       ??_C@_0BA@EJJPLHJN@stand?3?5time?5out?$AA@ 20067ba0     ai_dmnet.obj
 0002:00000bb0       ??_C@_0BD@EFNKCGD@stand?3?5found?5enemy?$AA@ 20067bb0     ai_dmnet.obj
 0002:00000bc4       ??_C@_07PABIOCAD@respawn?$AA@ 20067bc4     ai_dmnet.obj
 0002:00000bcc       ??_C@_0BD@MNFAOLC@respawn?3?5respawned?$AA@ 20067bcc     ai_dmnet.obj
 0002:00000be0       ??_C@_0BA@OLIPHEKA@activate?5entity?$AA@ 20067be0     ai_dmnet.obj
 0002:00000bf0       ??_C@_0BN@CHDNEHF@activate?5entity?3?5found?5enemy?$AA@ 20067bf0     ai_dmnet.obj
 0002:00000c10       ??_C@_0BL@KOANFMEA@activate?5entity?3?5activated?$AA@ 20067c10     ai_dmnet.obj
 0002:00000c2c       ??_C@_0BL@FHEEABKA@touched?5button?5or?5trigger?6?$AA@ 20067c2c     ai_dmnet.obj
 0002:00000c48       ??_C@_0BK@GBGNKJEG@activate?5entity?3?5time?5out?$AA@ 20067c48     ai_dmnet.obj
 0002:00000c64       ??_C@_0CB@NJIIFLCC@hit?5shootable?5button?5or?5trigger?6@ 20067c64     ai_dmnet.obj
 0002:00000c88       ??_C@_0BJ@EEHKLOIJ@activate?5entity?3?5no?5goal?$AA@ 20067c88     ai_dmnet.obj
 0002:00000ca4       ??_C@_0BK@EGCINOOI@activate?5entity?3?5bot?5dead?$AA@ 20067ca4     ai_dmnet.obj
 0002:00000cc0       ??_C@_0BO@DDGLLAGC@activate?5entity?3?5intermission?$AA@ 20067cc0     ai_dmnet.obj
 0002:00000ce0       ??_C@_0BI@CFBHMKPG@active?5entity?3?5observer?$AA@ 20067ce0     ai_dmnet.obj
 0002:00000cf8       ??_C@_07ONOEGCJB@no?5goal?$AA@ 20067cf8     ai_dmnet.obj
 0002:00000d00       ??_C@_08IFECKGCD@seek?5NBG?$AA@ 20067d00     ai_dmnet.obj
 0002:00000d0c       ??_C@_0BG@LLBOBEHC@seek?5nbg?3?5found?5enemy?$AA@ 20067d0c     ai_dmnet.obj
 0002:00000d24       ??_C@_0BD@KKPPPHA@seek?5nbg?3?5time?5out?$AA@ 20067d24     ai_dmnet.obj
 0002:00000d38       ??_C@_0BD@CNOKIINO@seek?5nbg?3?5bot?5dead?$AA@ 20067d38     ai_dmnet.obj
 0002:00000d4c       ??_C@_0BG@FJPIPBDN@seek?5nbg?3?5intermision?$AA@ 20067d4c     ai_dmnet.obj
 0002:00000d64       ??_C@_0BD@GLAPFIFB@seek?5nbg?3?5observer?$AA@ 20067d64     ai_dmnet.obj
 0002:00000d78       ??_C@_08DHOALBGK@seek?5LTG?$AA@ 20067d78     ai_dmnet.obj
 0002:00000d84       ??_C@_0O@OMHBKBBP@ltg?5seek?3?5nbg?$AA@ 20067d84     ai_dmnet.obj
 0002:00000d98       __real@3f847ae147ae147b    20067d98     ai_dmnet.obj
 0002:00000da0       ??_C@_0BG@NKJENDMP@seek?5ltg?3?5found?5enemy?$AA@ 20067da0     ai_dmnet.obj
 0002:00000db8       ??_C@_0BG@FMPBNGLO@seek?5ltg?3?5random?5chat?$AA@ 20067db8     ai_dmnet.obj
 0002:00000dd0       ??_C@_0BD@NIGGDFHE@seek?5ltg?3?5bot?5dead?$AA@ 20067dd0     ai_dmnet.obj
 0002:00000de4       ??_C@_0BH@BIAHANPH@seek?5ltg?3?5intermission?$AA@ 20067de4     ai_dmnet.obj
 0002:00000dfc       ??_C@_0BD@JOIDOFPL@seek?5ltg?3?5observer?$AA@ 20067dfc     ai_dmnet.obj
 0002:00000e10       ??_C@_0N@JAICAHME@battle?5fight?$AA@ 20067e10     ai_dmnet.obj
 0002:00000e20       ??_C@_0BP@KNHNJPON@battle?5fight?3?5wants?5to?5retreat?$AA@ 20067e20     ai_dmnet.obj
 0002:00000e40       ??_C@_0CB@IGGJLKOL@battle?5fight?3?5enemy?5out?5of?5sight@ 20067e40     ai_dmnet.obj
 0002:00000e64       ??_C@_0BP@NBCPEGCG@battle?5fight?3?5chat?5hit?5someone?$AA@ 20067e64     ai_dmnet.obj
 0002:00000e84       ??_C@_0CE@HNIMDJBG@battle?5fight?3?5chat?5health?5decrea@ 20067e84     ai_dmnet.obj
 0002:00000ea8       ??_C@_0BI@PALDJFNB@battle?5fight?3?5invisible?$AA@ 20067ea8     ai_dmnet.obj
 0002:00000ec0       __real@3fc999999999999a    20067ec0     ai_dmnet.obj
 0002:00000ec8       ??_C@_0BJ@JCMOALOB@battle?5fight?3?5enemy?5dead?$AA@ 20067ec8     ai_dmnet.obj
 0002:00000ee4       ??_C@_0BH@PAJNDMEE@battle?5fight?3?5no?5enemy?$AA@ 20067ee4     ai_dmnet.obj
 0002:00000efc       ??_C@_0BI@BEOBCCFJ@found?5new?5better?5enemy?6?$AA@ 20067efc     ai_dmnet.obj
 0002:00000f14       ??_C@_0BH@CCGABEPC@battle?5fight?3?5bot?5dead?$AA@ 20067f14     ai_dmnet.obj
 0002:00000f2c       ??_C@_0BL@OCIIHEED@battle?5fight?3?5intermission?$AA@ 20067f2c     ai_dmnet.obj
 0002:00000f48       ??_C@_0BH@GEIFMEHN@battle?5fight?3?5observer?$AA@ 20067f48     ai_dmnet.obj
 0002:00000f60       ??_C@_0N@JLOOIPJK@battle?5chase?$AA@ 20067f60     ai_dmnet.obj
 0002:00000f70       ??_C@_0BP@DMHFNNNL@battle?5chase?3?5wants?5to?5retreat?$AA@ 20067f70     ai_dmnet.obj
 0002:00000f90       ??_C@_0BC@MBHDFOHG@battle?5chase?3?5nbg?$AA@ 20067f90     ai_dmnet.obj
 0002:00000fa4       ??_C@_0BH@PKDGJGPO@battle?5chase?3?5time?5out?$AA@ 20067fa4     ai_dmnet.obj
 0002:00000fbc       ??_C@_0BM@JANANJEH@battle?5chase?3?5no?5enemy?5area?$AA@ 20067fbc     ai_dmnet.obj
 0002:00000fd8       ??_C@_0BL@BJLICKPC@battle?5chase?3?5better?5enemy?$AA@ 20067fd8     ai_dmnet.obj
 0002:00000ff4       ??_C@_0BH@PIOMJOG@battle?5chase?3?5no?5enemy?$AA@ 20067ff4     ai_dmnet.obj
 0002:0000100c       ??_C@_0BH@NNHDOBFA@battle?5chase?3?5bot?5dead?$AA@ 2006800c     ai_dmnet.obj
 0002:00001024       ??_C@_0BL@PKAILKOJ@battle?5chase?3?5intermission?$AA@ 20068024     ai_dmnet.obj
 0002:00001040       ??_C@_0BH@JLJGDBNP@battle?5chase?3?5observer?$AA@ 20068040     ai_dmnet.obj
 0002:00001058       ??_C@_0P@ELFCJAMH@battle?5retreat?$AA@ 20068058     ai_dmnet.obj
 0002:00001068       __real@3fd3333333333333    20068068     ai_dmnet.obj
 0002:00001070       ??_C@_0BE@EEPGNAKO@battle?5retreat?3?5nbg?$AA@ 20068070     ai_dmnet.obj
 0002:00001084       __real@42c80000            20068084     ai_dmnet.obj
 0002:00001088       ??_C@_0BL@IFDBGGDM@battle?5retreat?3?5no?5way?5out?$AA@ 20068088     ai_dmnet.obj
 0002:000010a4       ??_C@_0BO@JHDCIIFI@battle?5retreat?3?5another?5enemy?$AA@ 200680a4     ai_dmnet.obj
 0002:000010c4       ??_C@_0BL@KBIAJDEJ@battle?5retreat?3?5lost?5enemy?$AA@ 200680c4     ai_dmnet.obj
 0002:000010e0       ??_C@_0BP@PDKIMDBN@battle?5retreat?3?5wants?5to?5chase?$AA@ 200680e0     ai_dmnet.obj
 0002:00001100       ??_C@_0BL@NMDPGNGL@battle?5retreat?3?5enemy?5dead?$AA@ 20068100     ai_dmnet.obj
 0002:0000111c       ??_C@_0BJ@BKIHIJBD@battle?5retreat?3?5no?5enemy?$AA@ 2006811c     ai_dmnet.obj
 0002:00001138       ??_C@_0BJ@MIHKKBKF@battle?5retreat?3?5bot?5dead?$AA@ 20068138     ai_dmnet.obj
 0002:00001154       ??_C@_0BN@IHDFIOBO@battle?5retreat?3?5intermission?$AA@ 20068154     ai_dmnet.obj
 0002:00001174       ??_C@_0BJ@IOJPHBCK@battle?5retreat?3?5observer?$AA@ 20068174     ai_dmnet.obj
 0002:00001190       ??_C@_0L@EFLDDLAJ@battle?5NBG?$AA@ 20068190     ai_dmnet.obj
 0002:0000119c       ??_C@_0BF@JGNGECFP@battle?5nbg?3?5time?5out?$AA@ 2006819c     ai_dmnet.obj
 0002:000011b4       ??_C@_0BH@PFIKNLIP@battle?5nbg?3?5enemy?5dead?$AA@ 200681b4     ai_dmnet.obj
 0002:000011cc       ??_C@_0BF@GDGOBNEH@battle?5nbg?3?5no?5enemy?$AA@ 200681cc     ai_dmnet.obj
 0002:000011e4       ??_C@_0BF@LBJDDFPB@battle?5nbg?3?5bot?5dead?$AA@ 200681e4     ai_dmnet.obj
 0002:000011fc       ??_C@_0BJ@JPCFIHPK@battle?5nbg?3?5intermission?$AA@ 200681fc     ai_dmnet.obj
 0002:00001218       ??_C@_0BF@PHHGOFHO@battle?5nbg?3?5observer?$AA@ 20068218     ai_dmnet.obj
 0002:00001230       __real@43960000            20068230     ai_dmq3.obj
 0002:00001234       ??_C@_02KAJCLHKP@no?$AA@   20068234     ai_dmq3.obj
 0002:00001238       __real@42480000            20068238     ai_dmq3.obj
 0002:0000123c       ??_C@_08EAEOGCCG@onfollow?$AA@ 2006823c     ai_dmq3.obj
 0002:00001248       ??_C@_09BJNHNGHD@ihaveflag?$AA@ 20068248     ai_dmq3.obj
 0002:00001254       ??_C@_08OKGPDOIO@teamtask?$AA@ 20068254     ai_dmq3.obj
 0002:00001260       ??_C@_02DPKJAMEF@?$CFd?$AA@ 20068260     ai_dmq3.obj
 0002:00001264       __real@43000000            20068264     ai_dmq3.obj
 0002:00001268       ??_C@_0BG@EPIHOAD@?$FLclient?5out?5of?5range?$FN?$AA@ 20068268     ai_dmq3.obj
 0002:00001280       ??_C@_0CB@FEANAAEF@ClientName?3?5client?5out?5of?5range?6@ 20068280     ai_dmq3.obj
 0002:000012a4       ??_C@_05NCCFOPHA@model?$AA@ 200682a4     ai_dmq3.obj
 0002:000012ac       ??_C@_0CB@PGPLLECA@ClientSkin?3?5client?5out?5of?5range?6@ 200682ac     ai_dmq3.obj
 0002:000012d0       ??_C@_01LBDDMOBJ@?$FN?$AA@ 200682d0     ai_dmq3.obj
 0002:000012d4       ??_C@_01OHGJGJJP@?$FL?$AA@ 200682d4     ai_dmq3.obj
 0002:000012d8       ??_C@_01CLKCMJKC@?5?$AA@   200682d8     ai_dmq3.obj
 0002:000012dc       __real@41b80000            200682dc     ai_dmq3.obj
 0002:000012e0       ??_C@_0CF@BEIOCA@BotCreateWayPoint?3?5Out?5of?5waypoi@ 200682e0     ai_dmq3.obj
 0002:00001308       __real@42a00000            20068308     ai_dmq3.obj
 0002:0000130c       __real@42aa0000            2006830c     ai_dmq3.obj
 0002:00001310       __real@42b40000            20068310     ai_dmq3.obj
 0002:00001314       __real@42be0000            20068314     ai_dmq3.obj
 0002:00001318       __real@428c0000            20068318     ai_dmq3.obj
 0002:0000131c       __real@47c34f80            2006831c     ai_dmq3.obj
 0002:00001320       __real@3fefae147ae147ae    20068320     ai_dmq3.obj
 0002:00001328       __real@42200000            20068328     ai_dmq3.obj
 0002:0000132c       __real@43480000            2006832c     ai_dmq3.obj
 0002:00001330       __real@4058000000000000    20068330     ai_dmq3.obj
 0002:00001338       __real@3fe8000000000000    20068338     ai_dmq3.obj
 0002:00001340       __real@44480000            20068340     ai_dmq3.obj
 0002:00001348       __real@3feccccccccccccd    20068348     ai_dmq3.obj
 0002:00001350       __real@3fedeb851eb851ec    20068350     ai_dmq3.obj
 0002:00001358       __real@c066800000000000    20068358     ai_dmq3.obj
 0002:00001360       __real@4076800000000000    20068360     ai_dmq3.obj
 0002:00001368       __real@4066800000000000    20068368     ai_dmq3.obj
 0002:00001370       __real@3fee666666666666    20068370     ai_dmq3.obj
 0002:00001378       __real@3f50624dd2f1a9fc    20068378     ai_dmq3.obj
 0002:00001380       __real@45e3d000            20068380     ai_dmq3.obj
 0002:00001384       __real@49202e40            20068384     ai_dmq3.obj
 0002:00001388       __real@408c200000000000    20068388     ai_dmq3.obj
 0002:00001390       __real@40af400000000000    20068390     ai_dmq3.obj
 0002:00001398       __real@43b40000            20068398     ai_dmq3.obj
 0002:0000139c       __real@43160000            2006839c     ai_dmq3.obj
 0002:000013a0       __real@45c80000            200683a0     ai_dmq3.obj
 0002:000013a8       __real@4024000000000000    200683a8     ai_dmq3.obj
 0002:000013b0       __real@4034000000000000    200683b0     ai_dmq3.obj
 0002:000013b8       __real@4049000000000000    200683b8     ai_dmq3.obj
 0002:000013c0       __real@42800000            200683c0     ai_dmq3.obj
 0002:000013c8       __real@3fe3333333333333    200683c8     ai_dmq3.obj
 0002:000013d0       __real@44800000            200683d0     ai_dmq3.obj
 0002:000013d4       __real@41800000            200683d4     ai_dmq3.obj
 0002:000013d8       __real@3f333333            200683d8     ai_dmq3.obj
 0002:000013dc       __real@45100000            200683dc     ai_dmq3.obj
 0002:000013e0       __real@3ecccccd            200683e0     ai_dmq3.obj
 0002:000013e8       __real@408f400000000000    200683e8     ai_dmq3.obj
 0002:000013f0       __real@c1400000            200683f0     ai_dmq3.obj
 0002:000013f4       ??_C@_0N@IFIOEJJO@mpq3tourney6?$AA@ 200683f4     ai_dmq3.obj
 0002:00001408       __real@4020000000000000    20068408     ai_dmq3.obj
 0002:00001410       ??_C@_0L@IMOIIFCE@q3tourney6?$AA@ 20068410     ai_dmq3.obj
 0002:0000141c       __real@44000000            2006841c     ai_dmq3.obj
 0002:00001420       ??_C@_06KJINILIP@health?$AA@ 20068420     ai_dmq3.obj
 0002:00001428       ??_C@_05FECBCJJD@angle?$AA@ 20068428     ai_dmq3.obj
 0002:00001430       ??_C@_03MHHCOBAB@lip?$AA@  20068430     ai_dmq3.obj
 0002:00001434       __real@461c3c00            20068434     ai_dmq3.obj
 0002:00001438       ??_C@_0N@EDJICHIO@target_delay?$AA@ 20068438     ai_dmq3.obj
 0002:00001448       ??_C@_0N@JGBHMGAI@target_relay?$AA@ 20068448     ai_dmq3.obj
 0002:00001458       ??_C@_0L@LNOJFPAO@func_timer?$AA@ 20068458     ai_dmq3.obj
 0002:00001464       ??_C@_0BB@LKHFHPEP@trigger_multiple?$AA@ 20068464     ai_dmq3.obj
 0002:00001478       __real@4014000000000000    20068478     ai_dmq3.obj
 0002:00001480       ??_C@_0DO@JNGNHOKO@BotGetActivateGoal?3?5entity?5with?5@ 20068480     ai_dmq3.obj
 0002:000014c0       ??_C@_0DA@LAOMJDKC@BotGetActivateGoal?3?5no?5entity?5wi@ 200684c0     ai_dmq3.obj
 0002:000014f0       ??_C@_06JJLAMBGK@target?$AA@ 200684f0     ai_dmq3.obj
 0002:000014f8       ??_C@_0DO@HIKLPKA@BotGetActivateGoal?3?5entity?5with?5@ 200684f8     ai_dmq3.obj
 0002:00001538       ??_C@_0L@FEPNPAJD@targetname?$AA@ 20068538     ai_dmq3.obj
 0002:00001544       ??_C@_0M@PNMKBMEP@func_button?$AA@ 20068544     ai_dmq3.obj
 0002:00001550       ??_C@_06NHCMNMEH@origin?$AA@ 20068550     ai_dmq3.obj
 0002:00001558       ??_C@_0L@HLIKNEFC@spawnflags?$AA@ 20068558     ai_dmq3.obj
 0002:00001564       ??_C@_09KJCKJKEG@func_door?$AA@ 20068564     ai_dmq3.obj
 0002:00001570       ??_C@_0DL@MEHLMGEE@BotGetActivateGoal?3?5entity?5with?5@ 20068570     ai_dmq3.obj
 0002:000015ac       ??_C@_09CNJINBGN@classname?$AA@ 200685ac     ai_dmq3.obj
 0002:000015b8       ??_C@_0DD@KCKJBPAH@BotGetActivateGoal?3?5no?5entity?5fo@ 200685b8     ai_dmq3.obj
 0002:000015ec       ??_C@_03COCDEFBB@?$CK?$CFd?$AA@ 200685ec     ai_dmq3.obj
 0002:000015f0       ??_C@_0BF@GIIMEEEB@BotGoForActivateGoal?$AA@ 200685f0     ai_dmq3.obj
 0002:00001608       ??_C@_0DN@EJIKMLHL@?$CFs?3?5I?5have?5to?5activate?5a?5?$CFs?5at?5?$CF@ 20068608     ai_dmq3.obj
 0002:00001648       ??_C@_0DP@PANKMLEN@?$CFs?3?5I?5have?5to?5shoot?5at?5a?5?$CFs?5from@ 20068648     ai_dmq3.obj
 0002:00001688       __real@bf800000            20068688     ai_dmq3.obj
 0002:0000168c       __real@41900000            2006868c     ai_dmq3.obj
 0002:00001690       ??_C@_0CE@HJEADBFH@BotCheckConsoleMessages?3?5reply?5c@ 20068690     ai_dmq3.obj
 0002:000016b8       __real@3ff8000000000000    200686b8     ai_dmq3.obj
 0002:000016c0       ??_C@_0BK@IPGPBJPO@?$CK?$CK?$CK?$CK?5no?5valid?5reply?5?$CK?$CK?$CK?$CK?6?$AA@ 200686c0     ai_dmq3.obj
 0002:000016dc       ??_C@_0BK@ICOBFDNE@?9?9?9?9?9?9?9?9?9?9?9?9?9?9?9?9?9?9?9?9?9?9?9?9?6?$AA@ 200686dc     ai_dmq3.obj
 0002:000016f8       ??_C@_0O@BBHMLBKC@bot_testrchat?$AA@ 200686f8     ai_dmq3.obj
 0002:00001708       ??_C@_01HIHLOKLC@1?$AA@    20068708     ai_dmq3.obj
 0002:0000170c       ??_C@_0O@LBBMLEKM@?$CKfalling1?4wav?$AA@ 2006870c     ai_dmq3.obj
 0002:0000171c       ??_C@_0CP@JEHKHMIG@EV_GENERAL_SOUND?3?5eventParm?5?$CI?$CFd?$CJ@ 2006871c     ai_dmq3.obj
 0002:0000174c       ??_C@_0BP@NBLBCCPC@sound?1items?1poweruprespawn?4wav?$AA@ 2006874c     ai_dmq3.obj
 0002:0000176c       ??_C@_0CO@MPBFDNLO@EV_GLOBAL_SOUND?3?5eventParm?5?$CI?$CFd?$CJ?5@ 2006876c     ai_dmq3.obj
 0002:0000179c       ??_C@_0CB@MGIHMDHM@BotDeathmatchAI?3?5chat?5enter?5game@ 2006879c     ai_dmq3.obj
 0002:000017c0       ??_C@_0BM@EKLHMNBH@BotDeathmatchAI?3?5no?5ai?5node?$AA@ 200687c0     ai_dmq3.obj
 0002:000017dc       ??_C@_07FDOFLCLN@team?5?$CFs?$AA@ 200687dc     ai_dmq3.obj
 0002:000017e4       ??_C@_03OMLNFKE@sex?$AA@   200687e4     ai_dmq3.obj
 0002:000017e8       ??_C@_0BH@KKMLANHJ@CTF?5without?5Blue?5Flag?6?$AA@ 200687e8     ai_dmq3.obj
 0002:00001800       ??_C@_0BG@HPNDPJMP@CTF?5without?5Red?5Flag?6?$AA@ 20068800     ai_dmq3.obj
 0002:00001818       ??_C@_09OGEBNCBM@g_spSkill?$AA@ 20068818     ai_dmq3.obj
 0002:00001824       ??_C@_01FDFGLJHB@2?$AA@    20068824     ai_dmq3.obj
 0002:00001828       ??_C@_0BF@JHNEDFAH@bot_predictobstacles?$AA@ 20068828     ai_dmq3.obj
 0002:00001840       ??_C@_0O@ILENLOKO@bot_challenge?$AA@ 20068840     ai_dmq3.obj
 0002:00001850       ??_C@_0L@JNAIAIAH@bot_nochat?$AA@ 20068850     ai_dmq3.obj
 0002:0000185c       ??_C@_0N@JOELMLFL@bot_fastchat?$AA@ 2006885c     ai_dmq3.obj
 0002:0000186c       ??_C@_0M@HIPNFLBG@bot_grapple?$AA@ 2006886c     ai_dmq3.obj
 0002:00001878       ??_C@_01GBGANLPD@0?$AA@    20068878     ai_dmq3.obj
 0002:0000187c       ??_C@_0P@OLNMGHML@bot_rocketjump?$AA@ 2006887c     ai_dmq3.obj
 0002:0000188c       ??_C@_0L@GFINLBEC@g_gametype?$AA@ 2006888c     ai_dmq3.obj
 0002:00001898       ??_C@_0BE@HKMNOMAG@unknown?5print?5type?6?$AA@ 20068898     ai_main.obj
 0002:000018ac       ??_C@_0L@CNJLHKJM@?$FO1Exit?3?5?$CFs?$AA@ 200688ac     ai_main.obj
 0002:000018b8       ??_C@_0M@GLOCHAGD@?$FO1Fatal?3?5?$CFs?$AA@ 200688b8     ai_main.obj
 0002:000018c4       ??_C@_0M@LKBEKEOF@?$FO1Error?3?5?$CFs?$AA@ 200688c4     ai_main.obj
 0002:000018d0       ??_C@_0O@LHCIHOMB@?$FO3Warning?3?5?$CFs?$AA@ 200688d0     ai_main.obj
 0002:000018e0       ??_C@_02DKCKIIND@?$CFs?$AA@ 200688e0     ai_main.obj
 0002:000018e4       ??_C@_0BM@BOKNIJ@?$ANarea?5?$CFd?0?5cluster?5?$CFd?5?5?5?5?5?5?5?$AA@ 200688e4     ai_main.obj
 0002:00001900       ??_C@_0CI@JOJDDOJC@?$AN?$FO1Solid?$CB?5?5?5?5?5?5?5?5?5?5?5?5?5?5?5?5?5?5?5?5?5?5?5@ 20068900     ai_main.obj
 0002:00001928       ??_C@_0O@IFLBEIIP@?$AN?$FO1SOLID?5area?$AA@ 20068928     ai_main.obj
 0002:00001938       ??_C@_0M@DHMCHLIE@?$ANemtpy?5area?$AA@ 20068938     ai_main.obj
 0002:00001944       ??_C@_0BE@IKFGCOBJ@?$CF?920s?$CFs?$CFs?3?5roaming?6?$AA@ 20068944     ai_main.obj
 0002:00001958       ??_C@_0BH@KKFFINLC@?$CF?920s?$CFs?$CFs?3?5harvesting?6?$AA@ 20068958     ai_main.obj
 0002:00001970       ??_C@_0CF@NOKKHNPF@?$CF?920s?$CFs?$CFs?3?5attacking?5the?5enemy?5b@ 20068970     ai_main.obj
 0002:00001998       ??_C@_0BL@FAJAGBFK@?$CF?920s?$CFs?$CFs?3?5returning?5flag?6?$AA@ 20068998     ai_main.obj
 0002:000019b4       ??_C@_0BJ@NMLGGIKN@?$CF?920s?$CFs?$CFs?3?5rushing?5base?6?$AA@ 200689b4     ai_main.obj
 0002:000019d0       ??_C@_0BL@IGONECCL@?$CF?920s?$CFs?$CFs?3?5capturing?5flag?6?$AA@ 200689d0     ai_main.obj
 0002:000019ec       ??_C@_0BH@BPGAEHOC@?$CF?920s?$CFs?$CFs?3?5patrolling?6?$AA@ 200689ec     ai_main.obj
 0002:00001a04       ??_C@_0BE@FMIPBBCI@?$CF?920s?$CFs?$CFs?3?5camping?6?$AA@ 20068a04     ai_main.obj
 0002:00001a18       ??_C@_0BH@LBLMLBGP@?$CF?920s?$CFs?$CFs?3?5killing?5?$CFs?6?$AA@ 20068a18     ai_main.obj
 0002:00001a30       ??_C@_0BM@GCIOAMOM@?$CF?920s?$CFs?$CFs?3?5getting?5item?5?$CFs?6?$AA@ 20068a30     ai_main.obj
 0002:00001a4c       ??_C@_0BJ@BMDBIMEB@?$CF?920s?$CFs?$CFs?3?5defending?5?$CFs?6?$AA@ 20068a4c     ai_main.obj
 0002:00001a68       ??_C@_0BM@MFHGPNOH@?$CF?920s?$CFs?$CFs?3?5accompanying?5?$CFs?6?$AA@ 20068a68     ai_main.obj
 0002:00001a84       ??_C@_0BH@IGMMEADN@?$CF?920s?$CFs?$CFs?3?5helping?5?$CFs?6?$AA@ 20068a84     ai_main.obj
 0002:00001a9c       ??_C@_04CACEMDGO@?$FO4F?5?$AA@ 20068a9c     ai_main.obj
 0002:00001aa4       ??_C@_04BHPKDDFM@?$FO1F?5?$AA@ 20068aa4     ai_main.obj
 0002:00001aac       ??_C@_02KNHHEEKP@?5?5?$AA@ 20068aac     ai_main.obj
 0002:00001ab0       ??_C@_01OCOKONAJ@L?$AA@    20068ab0     ai_main.obj
 0002:00001ab4       ??_C@_07CJKDAGDN@?$FO4BLUE?6?$AA@ 20068ab4     ai_main.obj
 0002:00001abc       ??_C@_06LNDKJPFB@?$FO1RED?6?$AA@ 20068abc     ai_main.obj
 0002:00001ac4       ??_C@_0P@LMJINGO@l?2?$CFs?2c?2?$CFs?2a?2?$CFs?$AA@ 20068ac4     ai_main.obj
 0002:00001ad4       ??_C@_0L@IPEIBHBA@roaming?5?$CFs?$AA@ 20068ad4     ai_main.obj
 0002:00001ae0       ??_C@_0L@ICJBNMIF@harvesting?$AA@ 20068ae0     ai_main.obj
 0002:00001aec       ??_C@_0BJ@PEPADENJ@attacking?5the?5enemy?5base?$AA@ 20068aec     ai_main.obj
 0002:00001b08       ??_C@_0P@FJHLCNGM@returning?5flag?$AA@ 20068b08     ai_main.obj
 0002:00001b18       ??_C@_0N@GBHDPJKL@rushing?5base?$AA@ 20068b18     ai_main.obj
 0002:00001b28       ??_C@_0P@PCPLLEMM@capturing?5flag?$AA@ 20068b28     ai_main.obj
 0002:00001b38       ??_C@_0L@GKAIHKNA@killing?5?$CFs?$AA@ 20068b38     ai_main.obj
 0002:00001b44       ??_C@_0BA@FNOGAFMM@getting?5item?5?$CFs?$AA@ 20068b44     ai_main.obj
 0002:00001b54       ??_C@_0N@FMPLLINE@defending?5?$CFs?$AA@ 20068b54     ai_main.obj
 0002:00001b64       ??_C@_0BA@MCDBGPCI@accompanying?5?$CFs?$AA@ 20068b64     ai_main.obj
 0002:00001b74       ??_C@_0L@MCMCNIDL@helping?5?$CFs?$AA@ 20068b74     ai_main.obj
 0002:00001b80       ??_C@_02OBCNPDDN@F?5?$AA@  20068b80     ai_main.obj
 0002:00001b84       ??_C@_0BE@IDNEOHBL@bot_interbreedwrite?$AA@ 20068b84     ai_main.obj
 0002:00001b98       ??_C@_0BD@MIDHDJEH@bot_interbreedchar?$AA@ 20068b98     ai_main.obj
 0002:00001bac       ??_C@_0BK@CCAPHDJA@addbot?5?$CFs?54?5free?5?$CFi?5?$CFs?$CFd?6?$AA@ 20068bac     ai_main.obj
 0002:00001bc8       ??_C@_0BF@BBFOCAKO@bot_reloadcharacters?$AA@ 20068bc8     ai_main.obj
 0002:00001be0       __real@3fdccccccccccccd    20068be0     ai_main.obj
 0002:00001be8       __real@c3340000            20068be8     ai_main.obj
 0002:00001bec       __real@43700000            20068bec     ai_main.obj
 0002:00001bf0       __real@43c80000            20068bf0     ai_main.obj
 0002:00001bf4       __real@42fe0000            20068bf4     ai_main.obj
 0002:00001bf8       __real@47800000            20068bf8     ai_main.obj
 0002:00001c00       __real@3f76800000000000    20068c00     ai_main.obj
 0002:00001c08       ??_C@_0BA@GNMFKLDC@clientLevelShot?$AA@ 20068c08     ai_main.obj
 0002:00001c18       ??_C@_06KBCJDMLG@scores?$AA@ 20068c18     ai_main.obj
 0002:00001c20       ??_C@_05PMMINOBP@tchat?$AA@ 20068c20     ai_main.obj
 0002:00001c28       ??_C@_04BLJLMHHG@chat?$AA@ 20068c28     ai_main.obj
 0002:00001c30       ??_C@_05IJDJACGD@print?$AA@ 20068c30     ai_main.obj
 0002:00001c38       ??_C@_02EODNHJKB@cs?$AA@   20068c38     ai_main.obj
 0002:00001c3c       ??_C@_03DGFNDEPM@cp?5?$AA@ 20068c3c     ai_main.obj
 0002:00001c40       ??_C@_0BP@MGBLPCKB@BotAI?3?5client?5?$CFd?5is?5not?5setup?6?$AA@ 20068c40     ai_main.obj
 0002:00001c60       ??_C@_0N@BLBFMIAO@botsession?$CFi?$AA@ 20068c60     ai_main.obj
 0002:00001c70       ??_C@_0DD@CAOHNHKP@?$CFi?5?$CFi?5?$CFi?5?$CFi?5?$CFi?5?$CFi?5?$CFi?5?$CFi?5?$CFf?5?$CFf?5?$CFf@ 20068c70     ai_main.obj
 0002:00001ca4       ??_C@_0O@HIGNEDPK@bot_testichat?$AA@ 20068ca4     ai_main.obj
 0002:00001cb4       ??_C@_0CA@KCEBJEJI@couldn?8t?5load?5skill?5?$CFf?5from?5?$CFs?6?$AA@ 20068cb4     ai_main.obj
 0002:00001cd4       ??_C@_0BF@PINCHNMN@AAS?5not?5initialized?6?$AA@ 20068cd4     ai_main.obj
 0002:00001cec       ??_C@_0CL@MOACODCL@BotAISetupClient?3?5client?5?$CFd?5alre@ 20068cec     ai_main.obj
 0002:00001d18       ??_C@_0O@NKIABNEG@bot_thinktime?$AA@ 20068d18     ai_main.obj
 0002:00001d28       ??_C@_03HPLEMDKK@200?$AA@  20068d28     ai_main.obj
 0002:00001d2c       ??_C@_0BF@MDEDPJEF@bot_saveroutingcache?$AA@ 20068d2c     ai_main.obj
 0002:00001d44       ??_C@_0BB@GMCJAANP@saveroutingcache?$AA@ 20068d44     ai_main.obj
 0002:00001d58       ??_C@_0P@CMKPBNJI@bot_memorydump?$AA@ 20068d58     ai_main.obj
 0002:00001d68       ??_C@_0L@JEKILDFB@memorydump?$AA@ 20068d68     ai_main.obj
 0002:00001d74       ??_C@_05ECKEHJKK@cddir?$AA@ 20068d74     ai_main.obj
 0002:00001d7c       ??_C@_09CIALLHHK@fs_cdpath?$AA@ 20068d7c     ai_main.obj
 0002:00001d88       ??_C@_07GGMBKBFD@gamedir?$AA@ 20068d88     ai_main.obj
 0002:00001d90       ??_C@_07FMAMAFJE@fs_game?$AA@ 20068d90     ai_main.obj
 0002:00001d98       ??_C@_07BHPNMMNM@basedir?$AA@ 20068d98     ai_main.obj
 0002:00001da0       ??_C@_0M@DGDBFJN@fs_basepath?$AA@ 20068da0     ai_main.obj
 0002:00001dac       ??_C@_0M@MFMPGCMK@aasoptimize?$AA@ 20068dac     ai_main.obj
 0002:00001db8       ??_C@_0BA@CHMPBPHA@bot_aasoptimize?$AA@ 20068db8     ai_main.obj
 0002:00001dc8       ??_C@_0L@MNCDALON@forcewrite?$AA@ 20068dc8     ai_main.obj
 0002:00001dd4       ??_C@_0P@HFCEKFCE@bot_forcewrite?$AA@ 20068dd4     ai_main.obj
 0002:00001de4       ??_C@_0BC@HJNNPMHF@forcereachability?$AA@ 20068de4     ai_main.obj
 0002:00001df8       ??_C@_0BG@GJKIOMNG@bot_forcereachability?$AA@ 20068df8     ai_main.obj
 0002:00001e10       ??_C@_0BA@BADKHCEE@forceclustering?$AA@ 20068e10     ai_main.obj
 0002:00001e20       ??_C@_0BE@HANIKEON@bot_forceclustering?$AA@ 20068e20     ai_main.obj
 0002:00001e34       ??_C@_0BG@HILKKLKJ@bot_visualizejumppads?$AA@ 20068e34     ai_main.obj
 0002:00001e4c       ??_C@_06GCPOGFCC@nochat?$AA@ 20068e4c     ai_main.obj
 0002:00001e54       ??_C@_03MGHMBJCF@log?$AA@  20068e54     ai_main.obj
 0002:00001e58       ??_C@_0O@IHEJFHJE@bot_developer?$AA@ 20068e58     ai_main.obj
 0002:00001e68       ??_C@_0P@HIDOFLAM@max_levelitems?$AA@ 20068e68     ai_main.obj
 0002:00001e78       ??_C@_0N@PMPJOGOE@max_aaslinks?$AA@ 20068e78     ai_main.obj
 0002:00001e88       ??_C@_0P@HEEKJLPJ@sv_mapChecksum?$AA@ 20068e88     ai_main.obj
 0002:00001e98       ??_C@_0M@KCCINJFC@maxentities?$AA@ 20068e98     ai_main.obj
 0002:00001ea4       ??_C@_0L@JKCONGEA@maxclients?$AA@ 20068ea4     ai_main.obj
 0002:00001eb0       ??_C@_01KJLJFBPL@8?$AA@    20068eb0     ai_main.obj
 0002:00001eb4       ??_C@_0BE@BBMLIECL@bot_interbreedcycle?$AA@ 20068eb4     ai_main.obj
 0002:00001ec8       ??_C@_02PIBHCBOA@20?$AA@   20068ec8     ai_main.obj
 0002:00001ecc       ??_C@_0BD@GLHGHIJE@bot_interbreedbots?$AA@ 20068ecc     ai_main.obj
 0002:00001ee0       ??_C@_02PKFBJPLJ@10?$AA@   20068ee0     ai_main.obj
 0002:00001ee4       ??_C@_0BB@LICKAML@bot_testclusters?$AA@ 20068ee4     ai_main.obj
 0002:00001ef8       ??_C@_0O@NEGDFLLI@bot_testsolid?$AA@ 20068ef8     ai_main.obj
 0002:00001f08       ??_C@_0L@DIBKBFBJ@bot_report?$AA@ 20068f08     ai_main.obj
 0002:00001f14       ??_C@_09KJGEBPM@bot_pause?$AA@ 20068f14     ai_main.obj
 0002:00001f20       ??_C@_03GNABGMEE@100?$AA@  20068f20     ai_main.obj
 0002:00001f24       ??_C@_0M@CFKBBDNA@?$BJ?$CI?$CFs?$BJ?$CJ?$BJ?3?5?$CFs?$AA@ 20068f24     ai_team.obj
 0002:00001f30       ??_C@_0L@BCFFODB@returnflag?$AA@ 20068f30     ai_team.obj
 0002:00001f3c       ??_C@_0BC@HILCMIJJ@followflagcarrier?$AA@ 20068f3c     ai_team.obj
 0002:00001f50       ??_C@_0O@FNPCOJLM@cmd_accompany?$AA@ 20068f50     ai_team.obj
 0002:00001f60       ??_C@_0BA@MJCDCBAL@cmd_accompanyme?$AA@ 20068f60     ai_team.obj
 0002:00001f70       ??_C@_07NOFDDIA@getflag?$AA@ 20068f70     ai_team.obj
 0002:00001f78       ??_C@_0M@KCHJGFOM@cmd_getflag?$AA@ 20068f78     ai_team.obj
 0002:00001f84       ??_C@_06BMABBLML@defend?$AA@ 20068f84     ai_team.obj
 0002:00001f8c       ??_C@_0P@MGOFKCGO@cmd_defendbase?$AA@ 20068f8c     ai_team.obj
 0002:00001f9c       ??_C@_0M@GEDMEPM@startleader?$AA@ 20068f9c     ai_team.obj
 0002:00001fa8       ??_C@_0O@EHLIMCMK@iamteamleader?$AA@ 20068fa8     ai_team.obj
 0002:00001fb8       ??_C@_0BA@JCHIJEGJ@whoisteamleader?$AA@ 20068fb8     ai_team.obj
 0002:00001fc8       ??_C@_0O@LCEABBKD@wantonoffense?$AA@ 20068fc8     ai_vcmd.obj
 0002:00001fd8       ??_C@_0O@NOMCBHGI@wantondefense?$AA@ 20068fd8     ai_vcmd.obj
 0002:00001fe8       ??_C@_0M@JLDAEMIJ@whoisleader?$AA@ 20068fe8     ai_vcmd.obj
 0002:00001ff4       ??_C@_0L@HELMBEII@stopleader?$AA@ 20068ff4     ai_vcmd.obj
 0002:00002000       ??_C@_04LOFLEJM@camp?$AA@  20069000     ai_vcmd.obj
 0002:00002008       ??_C@_06KPEKKPL@patrol?$AA@ 20069008     ai_vcmd.obj
 0002:00002010       ??_C@_0L@LIAONOLJ@defendflag?$AA@ 20069010     ai_vcmd.obj
 0002:0000201c       ??_C@_07GBMLDGPP@offense?$AA@ 2006901c     ai_vcmd.obj
 0002:00002024       ??_C@_08DHCKJNNH@onpatrol?$AA@ 20069024     ai_vcmd.obj
 0002:00002030       ??_C@_08GBKLDCBE@EV_TAUNT?$AA@ 20069030     bg_misc.obj
 0002:0000203c       ??_C@_0BE@OHJHDFJH@EV_STOPLOOPINGSOUND?$AA@ 2006903c     bg_misc.obj
 0002:00002050       ??_C@_0O@PBPAKHP@EV_DEBUG_LINE?$AA@ 20069050     bg_misc.obj
 0002:00002060       ??_C@_0BB@HHACOGHI@EV_LIGHTNINGBOLT?$AA@ 20069060     bg_misc.obj
 0002:00002074       ??_C@_09GLJGDJEJ@EV_JUICED?$AA@ 20069074     bg_misc.obj
 0002:00002080       ??_C@_0BA@NHKGBGBA@EV_INVUL_IMPACT?$AA@ 20069080     bg_misc.obj
 0002:00002090       ??_C@_0BC@LMKNBBLF@EV_OBELISKEXPLODE?$AA@ 20069090     bg_misc.obj
 0002:000020a4       ??_C@_0M@KACLGFEA@EV_KAMIKAZE?$AA@ 200690a4     bg_misc.obj
 0002:000020b0       ??_C@_0BK@PIFCIJEJ@EV_PROXIMITY_MINE_TRIGGER?$AA@ 200690b0     bg_misc.obj
 0002:000020cc       ??_C@_0BI@KNJAKDGK@EV_PROXIMITY_MINE_STICK?$AA@ 200690cc     bg_misc.obj
 0002:000020e4       ??_C@_0N@GAJBP@EV_SCOREPLUM?$AA@ 200690e4     bg_misc.obj
 0002:000020f4       ??_C@_0O@JLGFLKBE@EV_GIB_PLAYER?$AA@ 200690f4     bg_misc.obj
 0002:00002104       ??_C@_0BB@EGIJIDAN@EV_POWERUP_REGEN?$AA@ 20069104     bg_misc.obj
 0002:00002118       ??_C@_0BG@CHAMNADK@EV_POWERUP_BATTLESUIT?$AA@ 20069118     bg_misc.obj
 0002:00002130       ??_C@_0BA@HLHGHIIE@EV_POWERUP_QUAD?$AA@ 20069130     bg_misc.obj
 0002:00002140       ??_C@_0M@PPLCDPP@EV_OBITUARY?$AA@ 20069140     bg_misc.obj
 0002:0000214c       ??_C@_09KNGHBIAK@EV_DEATH3?$AA@ 2006914c     bg_misc.obj
 0002:00002158       ??_C@_09LEHMCJEL@EV_DEATH2?$AA@ 20069158     bg_misc.obj
 0002:00002164       ??_C@_09JPFBHKII@EV_DEATH1?$AA@ 20069164     bg_misc.obj
 0002:00002170       ??_C@_07EMHHKOOH@EV_PAIN?$AA@ 20069170     bg_misc.obj
 0002:00002178       ??_C@_09ICDIPKFJ@EV_BULLET?$AA@ 20069178     bg_misc.obj
 0002:00002184       ??_C@_0L@LHBIHDML@EV_SHOTGUN?$AA@ 20069184     bg_misc.obj
 0002:00002190       ??_C@_0N@HMLLJFGF@EV_RAILTRAIL?$AA@ 20069190     bg_misc.obj
 0002:000021a0       ??_C@_0BG@LPAHEABB@EV_MISSILE_MISS_METAL?$AA@ 200691a0     bg_misc.obj
 0002:000021b8       ??_C@_0BA@CAHALNAE@EV_MISSILE_MISS?$AA@ 200691b8     bg_misc.obj
 0002:000021c8       ??_C@_0P@JFMFNBMO@EV_MISSILE_HIT?$AA@ 200691c8     bg_misc.obj
 0002:000021d8       ??_C@_0BD@MFLMCLPN@EV_BULLET_HIT_WALL?$AA@ 200691d8     bg_misc.obj
 0002:000021ec       ??_C@_0BE@KBABEJMP@EV_BULLET_HIT_FLESH?$AA@ 200691ec     bg_misc.obj
 0002:00002200       ??_C@_0BF@DDOIKLHD@EV_GLOBAL_TEAM_SOUND?$AA@ 20069200     bg_misc.obj
 0002:00002218       ??_C@_0BA@JAMKLOPJ@EV_GLOBAL_SOUND?$AA@ 20069218     bg_misc.obj
 0002:00002228       ??_C@_0BB@LJGGMAII@EV_GENERAL_SOUND?$AA@ 20069228     bg_misc.obj
 0002:0000223c       ??_C@_0BC@ECIIAFLJ@EV_GRENADE_BOUNCE?$AA@ 2006923c     bg_misc.obj
 0002:00002250       ??_C@_0BH@FNNILPIN@EV_PLAYER_TELEPORT_OUT?$AA@ 20069250     bg_misc.obj
 0002:00002268       ??_C@_0BG@HBBJKNDP@EV_PLAYER_TELEPORT_IN?$AA@ 20069268     bg_misc.obj
 0002:00002280       ??_C@_0M@ECGFPIMP@EV_ITEM_POP?$AA@ 20069280     bg_misc.obj
 0002:0000228c       ??_C@_0BA@GJNCODNG@EV_ITEM_RESPAWN?$AA@ 2006928c     bg_misc.obj
 0002:0000229c       ??_C@_0O@HHGOLJPJ@EV_USE_ITEM15?$AA@ 2006929c     bg_misc.obj
 0002:000022ac       ??_C@_0O@GOHFIILI@EV_USE_ITEM14?$AA@ 200692ac     bg_misc.obj
 0002:000022bc       ??_C@_0O@CBDEBOHP@EV_USE_ITEM13?$AA@ 200692bc     bg_misc.obj
 0002:000022cc       ??_C@_0O@DICPCPDO@EV_USE_ITEM12?$AA@ 200692cc     bg_misc.obj
 0002:000022dc       ??_C@_0O@BDACHMPN@EV_USE_ITEM11?$AA@ 200692dc     bg_misc.obj
 0002:000022ec       ??_C@_0O@KBJENLM@EV_USE_ITEM10?$AA@ 200692ec     bg_misc.obj
 0002:000022fc       ??_C@_0N@PHODCBCK@EV_USE_ITEM9?$AA@ 200692fc     bg_misc.obj
 0002:0000230c       ??_C@_0N@OOPIBAGL@EV_USE_ITEM8?$AA@ 2006930c     bg_misc.obj
 0002:0000231c       ??_C@_0N@GJGAAMKE@EV_USE_ITEM7?$AA@ 2006931c     bg_misc.obj
 0002:0000232c       ??_C@_0N@HAHLDNOF@EV_USE_ITEM6?$AA@ 2006932c     bg_misc.obj
 0002:0000233c       ??_C@_0N@FLFGGOCG@EV_USE_ITEM5?$AA@ 2006933c     bg_misc.obj
 0002:0000234c       ??_C@_0N@ECENFPGH@EV_USE_ITEM4?$AA@ 2006934c     bg_misc.obj
 0002:0000235c       ??_C@_0N@NAMMJKA@EV_USE_ITEM3?$AA@ 2006935c     bg_misc.obj
 0002:0000236c       ??_C@_0N@BEBHPIOB@EV_USE_ITEM2?$AA@ 2006936c     bg_misc.obj
 0002:0000237c       ??_C@_0N@DPDKKLCC@EV_USE_ITEM1?$AA@ 2006937c     bg_misc.obj
 0002:0000238c       ??_C@_0N@CGCBJKGD@EV_USE_ITEM0?$AA@ 2006938c     bg_misc.obj
 0002:0000239c       ??_C@_0P@PFJPAFGH@EV_FIRE_WEAPON?$AA@ 2006939c     bg_misc.obj
 0002:000023ac       ??_C@_0BB@ENKPHJLP@EV_CHANGE_WEAPON?$AA@ 200693ac     bg_misc.obj
 0002:000023c0       ??_C@_09NMIICG@EV_NOAMMO?$AA@ 200693c0     bg_misc.obj
 0002:000023cc       ??_C@_0BG@KFILGAMN@EV_GLOBAL_ITEM_PICKUP?$AA@ 200693cc     bg_misc.obj
 0002:000023e4       ??_C@_0P@BGIOEPCB@EV_ITEM_PICKUP?$AA@ 200693e4     bg_misc.obj
 0002:000023f4       ??_C@_0P@NIPCJOBG@EV_WATER_CLEAR?$AA@ 200693f4     bg_misc.obj
 0002:00002404       ??_C@_0P@MIAIODEJ@EV_WATER_UNDER?$AA@ 20069404     bg_misc.obj
 0002:00002414       ??_C@_0P@LHDMOIIG@EV_WATER_LEAVE?$AA@ 20069414     bg_misc.obj
 0002:00002424       ??_C@_0P@GCDBKPMP@EV_WATER_TOUCH?$AA@ 20069424     bg_misc.obj
 0002:00002434       ??_C@_07GKBEHGAP@EV_JUMP?$AA@ 20069434     bg_misc.obj
 0002:0000243c       ??_C@_0M@BPNFGBOJ@EV_JUMP_PAD?$AA@ 2006943c     bg_misc.obj
 0002:00002448       ??_C@_0M@LKJJNJOM@EV_FALL_FAR?$AA@ 20069448     bg_misc.obj
 0002:00002454       ??_C@_0P@MGFLMCKC@EV_FALL_MEDIUM?$AA@ 20069454     bg_misc.obj
 0002:00002464       ??_C@_0O@EAFDHAJM@EV_FALL_SHORT?$AA@ 20069464     bg_misc.obj
 0002:00002474       ??_C@_0L@HOOIOPKF@EV_STEP_16?$AA@ 20069474     bg_misc.obj
 0002:00002480       ??_C@_0L@BKIECKKB@EV_STEP_12?$AA@ 20069480     bg_misc.obj
 0002:0000248c       ??_C@_09EHOLDGNN@EV_STEP_8?$AA@ 2006948c     bg_misc.obj
 0002:00002498       ??_C@_09OLFOHJNB@EV_STEP_4?$AA@ 20069498     bg_misc.obj
 0002:000024a4       ??_C@_07FFIIIPLH@EV_SWIM?$AA@ 200694a4     bg_misc.obj
 0002:000024ac       ??_C@_0M@NPJBGELA@EV_FOOTWADE?$AA@ 200694ac     bg_misc.obj
 0002:000024b8       ??_C@_0O@HLJHKIDH@EV_FOOTSPLASH?$AA@ 200694b8     bg_misc.obj
 0002:000024c8       ??_C@_0BC@DIJMAMMI@EV_FOOTSTEP_METAL?$AA@ 200694c8     bg_misc.obj
 0002:000024dc       ??_C@_0M@HLKBOJPO@EV_FOOTSTEP?$AA@ 200694dc     bg_misc.obj
 0002:000024e8       ??_C@_07JFMDDPHJ@EV_NONE?$AA@ 200694e8     bg_misc.obj
 0002:000024f0       ??_C@_0BB@EMIIAFKA@icons?1iconf_blu1?$AA@ 200694f0     bg_misc.obj
 0002:00002504       ??_C@_0BI@FKICCNIF@models?1flags?1b_flag?4md3?$AA@ 20069504     bg_misc.obj
 0002:0000251c       ??_C@_0BC@NLKCOFAB@team_CTF_blueflag?$AA@ 2006951c     bg_misc.obj
 0002:00002530       ??_C@_0BB@EMIEBEOP@icons?1iconf_red1?$AA@ 20069530     bg_misc.obj
 0002:00002544       ??_C@_0BI@PEHEOJEO@models?1flags?1r_flag?4md3?$AA@ 20069544     bg_misc.obj
 0002:0000255c       ??_C@_0BB@JNMMCIHG@team_CTF_redflag?$AA@ 2006955c     bg_misc.obj
 0002:00002570       ??_C@_0N@GLEPEEPG@icons?1flight?$AA@ 20069570     bg_misc.obj
 0002:00002580       ??_C@_0CI@IADFFEDP@models?1powerups?1instant?1flight_r@ 20069580     bg_misc.obj
 0002:000025a8       ??_C@_0CD@MKDGJOMG@models?1powerups?1instant?1flight?4m@ 200695a8     bg_misc.obj
 0002:000025cc       ??_C@_0BH@COLFHEAE@sound?1items?1flight?4wav?$AA@ 200695cc     bg_misc.obj
 0002:000025e4       ??_C@_0M@MBNKEMMH@item_flight?$AA@ 200695e4     bg_misc.obj
 0002:000025f0       ??_C@_0BG@LHDLOKKN@sound?1items?1regen?4wav?$AA@ 200695f0     bg_misc.obj
 0002:00002608       ??_C@_0M@FDCLJBFC@icons?1regen?$AA@ 20069608     bg_misc.obj
 0002:00002614       ??_C@_0CH@FANACKJM@models?1powerups?1instant?1regen_ri@ 20069614     bg_misc.obj
 0002:0000263c       ??_C@_0CC@OEAPIKIN@models?1powerups?1instant?1regen?4md@ 2006963c     bg_misc.obj
 0002:00002660       ??_C@_0BN@OBGKHNFF@sound?1items?1regeneration?4wav?$AA@ 20069660     bg_misc.obj
 0002:00002680       ??_C@_0L@MMGPPPDM@item_regen?$AA@ 20069680     bg_misc.obj
 0002:0000268c       ??_C@_0M@FDDJPHJJ@icons?1invis?$AA@ 2006968c     bg_misc.obj
 0002:00002698       ??_C@_0CH@IMIHJDNC@models?1powerups?1instant?1invis_ri@ 20069698     bg_misc.obj
 0002:000026c0       ??_C@_0CC@HBONCEML@models?1powerups?1instant?1invis?4md@ 200696c0     bg_misc.obj
 0002:000026e4       ??_C@_0BN@OJBEBLGB@sound?1items?1invisibility?4wav?$AA@ 200696e4     bg_misc.obj
 0002:00002704       ??_C@_0L@MMHNJJPH@item_invis?$AA@ 20069704     bg_misc.obj
 0002:00002710       ??_C@_0M@CFINMGCL@icons?1haste?$AA@ 20069710     bg_misc.obj
 0002:0000271c       ??_C@_0CH@KKDDKNEF@models?1powerups?1instant?1haste_ri@ 2006971c     bg_misc.obj
 0002:00002744       ??_C@_0CC@NKPAJCMI@models?1powerups?1instant?1haste?4md@ 20069744     bg_misc.obj
 0002:00002768       ??_C@_0BG@IJMEPCOI@sound?1items?1haste?4wav?$AA@ 20069768     bg_misc.obj
 0002:00002780       ??_C@_0L@LKMJKIEF@item_haste?$AA@ 20069780     bg_misc.obj
 0002:0000278c       ??_C@_0DA@OCPACKGN@sound?1items?1airout?4wav?5sound?1ite@ 2006978c     bg_misc.obj
 0002:000027bc       ??_C@_0BB@MGICBJOH@icons?1envirosuit?$AA@ 200697bc     bg_misc.obj
 0002:000027d0       ??_C@_0CI@KAEDJDGE@models?1powerups?1instant?1enviro_r@ 200697d0     bg_misc.obj
 0002:000027f8       ??_C@_0CD@JLGNIGLA@models?1powerups?1instant?1enviro?4m@ 200697f8     bg_misc.obj
 0002:0000281c       ??_C@_0BI@DEKBIKDD@sound?1items?1protect?4wav?$AA@ 2006981c     bg_misc.obj
 0002:00002834       ??_C@_0M@HBCGNAN@item_enviro?$AA@ 20069834     bg_misc.obj
 0002:00002840       ??_C@_0DA@PPPPKFJI@sound?1items?1damage2?4wav?5sound?1it@ 20069840     bg_misc.obj
 0002:00002870       ??_C@_0L@DICHEOBB@icons?1quad?$AA@ 20069870     bg_misc.obj
 0002:0000287c       ??_C@_0CG@JNMBMLHJ@models?1powerups?1instant?1quad_rin@ 2006987c     bg_misc.obj
 0002:000028a4       ??_C@_0CB@HIFGFDGN@models?1powerups?1instant?1quad?4md3@ 200698a4     bg_misc.obj
 0002:000028c8       ??_C@_0BL@GLEJLOCA@sound?1items?1quaddamage?4wav?$AA@ 200698c8     bg_misc.obj
 0002:000028e4       ??_C@_09MDKNIFFH@item_quad?$AA@ 200698e4     bg_misc.obj
 0002:000028f0       ??_C@_0BL@GLIFPGGG@sound?1items?1use_medkit?4wav?$AA@ 200698f0     bg_misc.obj
 0002:0000290c       ??_C@_06JDLGEHAD@Medkit?$AA@ 2006990c     bg_misc.obj
 0002:00002914       ??_C@_0N@PNMDFAPK@icons?1medkit?$AA@ 20069914     bg_misc.obj
 0002:00002924       ??_C@_0CL@LOBKLABC@models?1powerups?1holdable?1medkit_@ 20069924     bg_misc.obj
 0002:00002950       ??_C@_0CE@NKMJILL@models?1powerups?1holdable?1medkit?4@ 20069950     bg_misc.obj
 0002:00002974       ??_C@_0BA@PDDMBOCP@holdable_medkit?$AA@ 20069974     bg_misc.obj
 0002:00002984       ??_C@_0BE@PCKJDFFA@Personal?5Teleporter?$AA@ 20069984     bg_misc.obj
 0002:00002998       ??_C@_0BB@HCFICFKF@icons?1teleporter?$AA@ 20069998     bg_misc.obj
 0002:000029ac       ??_C@_0CI@FHEOFFOB@models?1powerups?1holdable?1telepor@ 200699ac     bg_misc.obj
 0002:000029d4       ??_C@_0BJ@PNIOAJDI@sound?1items?1holdable?4wav?$AA@ 200699d4     bg_misc.obj
 0002:000029f0       ??_C@_0BE@GNEKBMLB@holdable_teleporter?$AA@ 200699f0     bg_misc.obj
 0002:00002a04       ??_C@_08LIBOGPIN@Bfg?5Ammo?$AA@ 20069a04     bg_misc.obj
 0002:00002a10       ??_C@_0BA@NIKNDLKG@icons?1icona_bfg?$AA@ 20069a10     bg_misc.obj
 0002:00002a20       ??_C@_0BP@BOBKFIKJ@models?1powerups?1ammo?1bfgam?4md3?$AA@ 20069a20     bg_misc.obj
 0002:00002a40       ??_C@_08EHEJHGBG@ammo_bfg?$AA@ 20069a40     bg_misc.obj
 0002:00002a4c       ??_C@_05INIOBJHH@Slugs?$AA@ 20069a4c     bg_misc.obj
 0002:00002a54       ??_C@_0BE@DPOADFL@icons?1icona_railgun?$AA@ 20069a54     bg_misc.obj
 0002:00002a68       ??_C@_0CD@CAJEPMME@models?1powerups?1ammo?1railgunam?4m@ 20069a68     bg_misc.obj
 0002:00002a8c       ??_C@_0L@JEFOIHIM@ammo_slugs?$AA@ 20069a8c     bg_misc.obj
 0002:00002a98       ??_C@_07MLLADOAB@Rockets?$AA@ 20069a98     bg_misc.obj
 0002:00002aa0       ??_C@_0BD@BFBJLPJK@icons?1icona_rocket?$AA@ 20069aa0     bg_misc.obj
 0002:00002ab4       ??_C@_0CC@KCOEDLFM@models?1powerups?1ammo?1rocketam?4md@ 20069ab4     bg_misc.obj
 0002:00002ad8       ??_C@_0N@CLEPKBOE@ammo_rockets?$AA@ 20069ad8     bg_misc.obj
 0002:00002ae8       ??_C@_09JCCOMJEA@Lightning?$AA@ 20069ae8     bg_misc.obj
 0002:00002af4       ??_C@_0BG@MEGMAGOM@icons?1icona_lightning?$AA@ 20069af4     bg_misc.obj
 0002:00002b0c       ??_C@_0CF@HDAADIIL@models?1powerups?1ammo?1lightningam@ 20069b0c     bg_misc.obj
 0002:00002b34       ??_C@_0P@NBJHKAMD@ammo_lightning?$AA@ 20069b34     bg_misc.obj
 0002:00002b44       ??_C@_05KCAMIOGJ@Cells?$AA@ 20069b44     bg_misc.obj
 0002:00002b4c       ??_C@_0BD@NCNJEHKB@icons?1icona_plasma?$AA@ 20069b4c     bg_misc.obj
 0002:00002b60       ??_C@_0CC@FGLALJGN@models?1powerups?1ammo?1plasmaam?4md@ 20069b60     bg_misc.obj
 0002:00002b84       ??_C@_0L@LLNMBAJC@ammo_cells?$AA@ 20069b84     bg_misc.obj
 0002:00002b90       ??_C@_08PMBIADEN@Grenades?$AA@ 20069b90     bg_misc.obj
 0002:00002b9c       ??_C@_0BE@LHOKGGAM@icons?1icona_grenade?$AA@ 20069b9c     bg_misc.obj
 0002:00002bb0       ??_C@_0CD@HNOBKKLC@models?1powerups?1ammo?1grenadeam?4m@ 20069bb0     bg_misc.obj
 0002:00002bd4       ??_C@_0O@CMJIOKCF@ammo_grenades?$AA@ 20069bd4     bg_misc.obj
 0002:00002be4       ??_C@_07DHNDKCGP@Bullets?$AA@ 20069be4     bg_misc.obj
 0002:00002bec       ??_C@_0BH@HMOAGCNP@icons?1icona_machinegun?$AA@ 20069bec     bg_misc.obj
 0002:00002c04       ??_C@_0CG@OLENEOKN@models?1powerups?1ammo?1machineguna@ 20069c04     bg_misc.obj
 0002:00002c2c       ??_C@_0N@NHCMDNIK@ammo_bullets?$AA@ 20069c2c     bg_misc.obj
 0002:00002c3c       ??_C@_06PBPEPGGL@Shells?$AA@ 20069c3c     bg_misc.obj
 0002:00002c44       ??_C@_0BE@NMAFHJEI@icons?1icona_shotgun?$AA@ 20069c44     bg_misc.obj
 0002:00002c58       ??_C@_0CD@MBAGJHDE@models?1powerups?1ammo?1shotgunam?4m@ 20069c58     bg_misc.obj
 0002:00002c7c       ??_C@_0BH@DPAADLFH@sound?1misc?1am_pkup?4wav?$AA@ 20069c7c     bg_misc.obj
 0002:00002c94       ??_C@_0M@NLICANGB@ammo_shells?$AA@ 20069c94     bg_misc.obj
 0002:00002ca0       ??_C@_0P@CFJPDDC@Grappling?5Hook?$AA@ 20069ca0     bg_misc.obj
 0002:00002cb0       ??_C@_0BE@DPKNJNBE@icons?1iconw_grapple?$AA@ 20069cb0     bg_misc.obj
 0002:00002cc4       ??_C@_0CE@LFAGANA@models?1weapons2?1grapple?1grapple?4@ 20069cc4     bg_misc.obj
 0002:00002ce8       ??_C@_0BF@MEMGGPGH@weapon_grapplinghook?$AA@ 20069ce8     bg_misc.obj
 0002:00002d00       ??_C@_0BA@NCCNKCA@icons?1iconw_bfg?$AA@ 20069d00     bg_misc.obj
 0002:00002d10       ??_C@_0BM@HHDGGOHP@models?1weapons2?1bfg?1bfg?4md3?$AA@ 20069d10     bg_misc.obj
 0002:00002d2c       ??_C@_0L@JBGNLNGG@weapon_bfg?$AA@ 20069d2c     bg_misc.obj
 0002:00002d38       ??_C@_0L@JFFCGJF@Plasma?5Gun?$AA@ 20069d38     bg_misc.obj
 0002:00002d44       ??_C@_0BD@NADHMFK@icons?1iconw_plasma?$AA@ 20069d44     bg_misc.obj
 0002:00002d58       ??_C@_0CC@EHGHEDND@models?1weapons2?1plasma?1plasma?4md@ 20069d58     bg_misc.obj
 0002:00002d7c       ??_C@_0BB@LBHAKENA@weapon_plasmagun?$AA@ 20069d7c     bg_misc.obj
 0002:00002d90       ??_C@_0BE@CJEOPCPE@icons?1iconw_railgun?$AA@ 20069d90     bg_misc.obj
 0002:00002da4       ??_C@_0CE@JHJFFEBE@models?1weapons2?1railgun?1railgun?4@ 20069da4     bg_misc.obj
 0002:00002dc8       ??_C@_0P@FEPBKEBF@weapon_railgun?$AA@ 20069dc8     bg_misc.obj
 0002:00002dd8       ??_C@_0BG@CHEJEOPA@icons?1iconw_lightning?$AA@ 20069dd8     bg_misc.obj
 0002:00002df0       ??_C@_0CI@MNAFJDPO@models?1weapons2?1lightning?1lightn@ 20069df0     bg_misc.obj
 0002:00002e18       ??_C@_0BB@OCCEAFCD@weapon_lightning?$AA@ 20069e18     bg_misc.obj
 0002:00002e2c       ??_C@_0BD@MKMDIEGB@icons?1iconw_rocket?$AA@ 20069e2c     bg_misc.obj
 0002:00002e40       ??_C@_0CE@GGGFLKKE@models?1weapons2?1rocketl?1rocketl?4@ 20069e40     bg_misc.obj
 0002:00002e64       ??_C@_0BG@HJKONAJE@weapon_rocketlauncher?$AA@ 20069e64     bg_misc.obj
 0002:00002e80       ??_C@_0EG@LFEMOCGK@sound?1weapons?1grenade?1hgrenb1a?4w@ 20069e80     bg_misc.obj
 0002:00002ec8       ??_C@_0BE@JNFKJHKD@icons?1iconw_grenade?$AA@ 20069ec8     bg_misc.obj
 0002:00002edc       ??_C@_0CG@INCGOMDL@models?1weapons2?1grenadel?1grenade@ 20069edc     bg_misc.obj
 0002:00002f04       ??_C@_0BH@DGCCJPLM@weapon_grenadelauncher?$AA@ 20069f04     bg_misc.obj
 0002:00002f1c       ??_C@_0BH@GIACBLNI@icons?1iconw_machinegun?$AA@ 20069f1c     bg_misc.obj
 0002:00002f34       ??_C@_0CK@BBPFNIFO@models?1weapons2?1machinegun?1machi@ 20069f34     bg_misc.obj
 0002:00002f60       ??_C@_0BC@HHBNPFPN@weapon_machinegun?$AA@ 20069f60     bg_misc.obj
 0002:00002f74       ??_C@_0BE@PGLFIIOH@icons?1iconw_shotgun?$AA@ 20069f74     bg_misc.obj
 0002:00002f88       ??_C@_0CE@CJGCHKCN@models?1weapons2?1shotgun?1shotgun?4@ 20069f88     bg_misc.obj
 0002:00002fac       ??_C@_0P@ILAKNOAG@weapon_shotgun?$AA@ 20069fac     bg_misc.obj
 0002:00002fbc       ??_C@_0BF@PMEPIOCM@icons?1iconw_gauntlet?$AA@ 20069fbc     bg_misc.obj
 0002:00002fd4       ??_C@_0CG@PFPPJBAC@models?1weapons2?1gauntlet?1gauntle@ 20069fd4     bg_misc.obj
 0002:00002ffc       ??_C@_0BG@BBKFHONL@sound?1misc?1w_pkup?4wav?$AA@ 20069ffc     bg_misc.obj
 0002:00003014       ??_C@_0BA@CLDPODJE@weapon_gauntlet?$AA@ 2006a014     bg_misc.obj
 0002:00003024       ??_C@_0M@IOJDMPNO@Mega?5Health?$AA@ 2006a024     bg_misc.obj
 0002:00003030       ??_C@_0BB@EGPGIMOM@icons?1iconh_mega?$AA@ 2006a030     bg_misc.obj
 0002:00003044       ??_C@_0CH@NEGHBKPB@models?1powerups?1health?1mega_sphe@ 2006a044     bg_misc.obj
 0002:0000306c       ??_C@_0CG@PDJMMGME@models?1powerups?1health?1mega_cros@ 2006a06c     bg_misc.obj
 0002:00003094       ??_C@_0BJ@FGLGEHNG@sound?1items?1m_health?4wav?$AA@ 2006a094     bg_misc.obj
 0002:000030b0       ??_C@_0BB@PBGAONGH@item_health_mega?$AA@ 2006a0b0     bg_misc.obj
 0002:000030c4       ??_C@_09EBELOOOD@50?5Health?$AA@ 2006a0c4     bg_misc.obj
 0002:000030d0       ??_C@_0BA@IGNANAGL@icons?1iconh_red?$AA@ 2006a0d0     bg_misc.obj
 0002:000030e0       ??_C@_0CI@CEEMEFNH@models?1powerups?1health?1large_sph@ 2006a0e0     bg_misc.obj
 0002:00003108       ??_C@_0CH@NHFAKEFE@models?1powerups?1health?1large_cro@ 2006a108     bg_misc.obj
 0002:00003130       ??_C@_0BJ@ILCAJOFD@sound?1items?1l_health?4wav?$AA@ 2006a130     bg_misc.obj
 0002:0000314c       ??_C@_0BC@JGDLKFIO@item_health_large?$AA@ 2006a14c     bg_misc.obj
 0002:00003160       ??_C@_09OJAALANF@25?5Health?$AA@ 2006a160     bg_misc.obj
 0002:0000316c       ??_C@_0BD@CDBLAHCA@icons?1iconh_yellow?$AA@ 2006a16c     bg_misc.obj
 0002:00003180       ??_C@_0CJ@NCCPDHOD@models?1powerups?1health?1medium_sp@ 2006a180     bg_misc.obj
 0002:000031ac       ??_C@_0CI@NAEMLIB@models?1powerups?1health?1medium_cr@ 2006a1ac     bg_misc.obj
 0002:000031d4       ??_C@_0BJ@OLHMCLBI@sound?1items?1n_health?4wav?$AA@ 2006a1d4     bg_misc.obj
 0002:000031f0       ??_C@_0M@KCNAKNNL@item_health?$AA@ 2006a1f0     bg_misc.obj
 0002:000031fc       ??_C@_08IAIFJOAI@5?5Health?$AA@ 2006a1fc     bg_misc.obj
 0002:00003208       ??_C@_0BC@IMNPBGFF@icons?1iconh_green?$AA@ 2006a208     bg_misc.obj
 0002:0000321c       ??_C@_0CI@MPAPPIIE@models?1powerups?1health?1small_sph@ 2006a21c     bg_misc.obj
 0002:00003244       ??_C@_0CH@JKNLMIJB@models?1powerups?1health?1small_cro@ 2006a244     bg_misc.obj
 0002:0000326c       ??_C@_0BJ@BIFHONLM@sound?1items?1s_health?4wav?$AA@ 2006a26c     bg_misc.obj
 0002:00003288       ??_C@_0BC@DOHAFEBI@item_health_small?$AA@ 2006a288     bg_misc.obj
 0002:0000329c       ??_C@_0BA@CEJNPBJG@icons?1iconr_red?$AA@ 2006a29c     bg_misc.obj
 0002:000032ac       ??_C@_0CE@EGJFDJJK@models?1powerups?1armor?1armor_red?4@ 2006a2ac     bg_misc.obj
 0002:000032d0       ??_C@_0BA@EKKMHIH@item_armor_body?$AA@ 2006a2d0     bg_misc.obj
 0002:000032e0       ??_C@_0BD@BKPFMPMP@icons?1iconr_yellow?$AA@ 2006a2e0     bg_misc.obj
 0002:000032f4       ??_C@_0CE@PHKMKHKB@models?1powerups?1armor?1armor_yel?4@ 2006a2f4     bg_misc.obj
 0002:00003318       ??_C@_0BI@KNMPECGK@sound?1misc?1ar2_pkup?4wav?$AA@ 2006a318     bg_misc.obj
 0002:00003330       ??_C@_0BC@FPPLPJIL@item_armor_combat?$AA@ 2006a330     bg_misc.obj
 0002:00003344       ??_C@_0M@PJIPIDNH@Armor?5Shard?$AA@ 2006a344     bg_misc.obj
 0002:00003350       ??_C@_0BC@LPFHDODA@icons?1iconr_shard?$AA@ 2006a350     bg_misc.obj
 0002:00003364       ??_C@_0CH@NEKDLKN@models?1powerups?1armor?1shard_sphe@ 2006a364     bg_misc.obj
 0002:0000338c       ??_C@_0CA@NOFOCCIK@models?1powerups?1armor?1shard?4md3?$AA@ 2006a38c     bg_misc.obj
 0002:000033ac       ??_C@_0BI@DECNCEGL@sound?1misc?1ar1_pkup?4wav?$AA@ 2006a3ac     bg_misc.obj
 0002:000033c4       ??_C@_0BB@DDGIAABK@item_armor_shard?$AA@ 2006a3c4     bg_misc.obj
 0002:000033d8       ??_C@_0BH@MFGKJDLM@HoldableItem?5not?5found?$AA@ 2006a3d8     bg_misc.obj
 0002:000033f0       ??_C@_0CB@DEACFJO@Couldn?8t?5find?5item?5for?5weapon?5?$CFi@ 2006a3f0     bg_misc.obj
 0002:00003414       __real@c2100000            2006a414     bg_misc.obj
 0002:00003418       __real@42100000            2006a418     bg_misc.obj
 0002:0000341c       __real@c2480000            2006a41c     bg_misc.obj
 0002:00003420       __real@42300000            2006a420     bg_misc.obj
 0002:00003424       ??_C@_0CG@HNLFCMEK@BG_CanItemBeGrabbed?3?5unknown?5enu@ 2006a424     bg_misc.obj
 0002:0000344c       ??_C@_0BM@NECGLAIF@BG_CanItemBeGrabbed?3?5IT_BAD?$AA@ 2006a44c     bg_misc.obj
 0002:00003468       ??_C@_0CI@MFONMA@BG_CanItemBeGrabbed?3?5index?5out?5o@ 2006a468     bg_misc.obj
 0002:00003490       ??_C@_0CK@DNBGNAED@BG_EvaluateTrajectory?3?5unknown?5t@ 2006a490     bg_misc.obj
 0002:000034c0       __real@4079000000000000    2006a4c0     bg_misc.obj
 0002:000034c8       __real@40490fdb            2006a4c8     bg_misc.obj
 0002:000034cc       ??_C@_0CP@MCFPOIMF@BG_EvaluateTrajectoryDelta?3?5unkn@ 2006a4cc     bg_misc.obj
 0002:000034fc       ??_C@_0DA@KOPJLGJF@Cgame?5event?5svt?5?$CF5d?5?9?$DO?5?$CF5d?3?5num?5@ 2006a4fc     bg_misc.obj
 0002:00003530       __real@0000000000000000    2006a530     bg_misc.obj
 0002:00003538       ??_C@_0L@MNPDPHLD@showevents?$AA@ 2006a538     bg_misc.obj
 0002:00003544       __real@42340000            2006a544     bg_misc.obj
 0002:00003548       __real@405fc00000000000    2006a548     bg_pmove.obj
 0002:00003550       __real@41f00000            2006a550     bg_pmove.obj
 0002:00003554       __real@c1800000            2006a554     bg_pmove.obj
 0002:00003558       __real@4008000000000000    2006a558     bg_pmove.obj
 0002:00003560       __real@c3480000            2006a560     bg_pmove.obj
 0002:00003564       ??_C@_08KACHPCJN@?$CFi?3Land?6?$AA@ 2006a564     bg_pmove.obj
 0002:00003570       ??_C@_09OPMLNNOA@?$CFi?3steep?6?$AA@ 2006a570     bg_pmove.obj
 0002:0000357c       ??_C@_0M@CKJFDFGH@?$CFi?3kickoff?6?$AA@ 2006a57c     bg_pmove.obj
 0002:00003588       __real@40e00000            2006a588     bg_pmove.obj
 0002:00003590       __real@3f1a36e2eb1c432d    2006a590     bg_pmove.obj
 0002:00003598       ??_C@_0N@KJCNHCBK@?$CFi?3allsolid?6?$AA@ 2006a598     bg_pmove.obj
 0002:000035a8       ??_C@_08EOGJDHPF@?$CFi?3lift?6?$AA@ 2006a5a8     bg_pmove.obj
 0002:000035b4       __real@c1c00000            2006a5b4     bg_pmove.obj
 0002:000035b8       __real@3ff4cccccccccccd    2006a5b8     bg_pmove.obj
 0002:000035c0       ??_C@_0M@CDHDENEF@?$CFi?3stepped?6?$AA@ 2006a5c0     bg_slidemove.obj
 0002:000035cc       __real@41300000            2006a5cc     bg_slidemove.obj
 0002:000035d0       ??_C@_0BE@FLPNHHPN@?$CFi?3bend?5can?8t?5step?6?$AA@ 2006a5d0     bg_slidemove.obj
 0002:000035e8       __real@4070000000000000    2006a5e8     g_active.obj
 0002:000035f0       __real@437f0000            2006a5f0     g_active.obj
 0002:000035f4       ??_C@_0BH@CIEIFFOL@sound?1player?1gurp2?4wav?$AA@ 2006a5f4     g_active.obj
 0002:0000360c       ??_C@_0BH@KONMCHEF@sound?1player?1gurp1?4wav?$AA@ 2006a60c     g_active.obj
 0002:00003624       ??_C@_0L@FMIBJCKG@?$CKdrown?4wav?$AA@ 2006a624     g_active.obj
 0002:00003630       ??_C@_0CJ@OOBJBOCC@cp?5?$CCTen?5seconds?5until?5inactivity@ 2006a630     g_active.obj
 0002:0000365c       ??_C@_0BK@CMFHJBAI@Dropped?5due?5to?5inactivity?$AA@ 2006a65c     g_active.obj
 0002:00003678       __real@3ff199999999999a    2006a678     g_active.obj
 0002:00003680       ??_C@_02NCPIBIBE@33?$AA@   2006a680     g_active.obj
 0002:00003684       ??_C@_0L@JLBEBBAD@pmove_msec?$AA@ 2006a684     g_active.obj
 0002:00003690       ??_C@_09HCJPKLNL@?5?$CFi?5?$CFi?5?$CFi?$AA@ 2006a690     g_arenas.obj
 0002:0000369c       ??_C@_0CB@CLLCPLDB@postgame?5?$CFi?5?$CFi?5?$CFi?5?$CFi?5?$CFi?5?$CFi?5?$CFi?5?$CFi@ 2006a69c     g_arenas.obj
 0002:000036c0       ??_C@_0BL@HAGGIKPH@postgame?5?$CFi?5?$CFi?50?50?50?50?50?50?$AA@ 2006a6c0     g_arenas.obj
 0002:000036dc       ??_C@_0BL@MJMDOODN@?$FO1ERROR?3?5out?5of?5gentities?6?$AA@ 2006a6dc     g_arenas.obj
 0002:000036f8       ??_C@_0N@NHMKEGEN@g_podiumDrop?$AA@ 2006a6f8     g_arenas.obj
 0002:00003708       ??_C@_0N@CBICAJMD@g_podiumDist?$AA@ 2006a708     g_arenas.obj
 0002:00003718       ??_C@_0CF@MDONDONI@models?1mapobjects?1podium?1podium4@ 2006a718     g_arenas.obj
 0002:00003740       ??_C@_06NPKMJLHA@podium?$AA@ 2006a740     g_arenas.obj
 0002:00003748       ??_C@_05BJJDEFHJ@?2num?2?$AA@ 2006a748     g_bot.obj
 0002:00003750       ??_C@_06CBHGEMFM@?$DMNULL?$DO?$AA@ 2006a750     g_bot.obj
 0002:00003758       ??_C@_01CELHOKLL@?$HN?$AA@ 2006a758     g_bot.obj
 0002:0000375c       ??_C@_0BN@HAJDHEGK@Unexpected?5end?5of?5info?5file?6?$AA@ 2006a75c     g_bot.obj
 0002:0000377c       ??_C@_0BE@IKMJLADL@Max?5infos?5exceeded?6?$AA@ 2006a77c     g_bot.obj
 0002:00003790       ??_C@_0BI@BMEIBPEH@Missing?5?$HL?5in?5info?5file?6?$AA@ 2006a790     g_bot.obj
 0002:000037a8       ??_C@_01HCONENDN@?$HL?$AA@ 2006a7a8     g_bot.obj
 0002:000037ac       ??_C@_03HBNNNHNM@map?$AA@  2006a7ac     g_bot.obj
 0002:000037b0       ??_C@_0BE@HKGNLKGC@addbot?5?$CFs?5?$CFf?5?$CFs?5?$CFi?6?$AA@ 2006a7b0     g_bot.obj
 0002:000037c4       ??_C@_04MEMAJGDJ@name?$AA@ 2006a7c4     g_bot.obj
 0002:000037cc       ??_C@_08CKHMKINC@kick?5?$CFs?6?$AA@ 2006a7cc     g_bot.obj
 0002:000037d8       ??_C@_0CD@DFNICLKJ@play?5sound?1player?1announce?1?$CFs?4wa@ 2006a7d8     g_bot.obj
 0002:000037fc       ??_C@_07DLHCIBDH@default?$AA@ 2006a7fc     g_bot.obj
 0002:00003804       ??_C@_0BI@KOJDMFEB@BotAISetupClient?5failed?$AA@ 2006a804     g_bot.obj
 0002:0000381c       ??_C@_04KADBPNCB@team?$AA@ 2006a81c     g_bot.obj
 0002:00003824       ??_C@_05ODMCMJAJ@skill?$AA@ 2006a824     g_bot.obj
 0002:0000382c       ??_C@_0O@HKBPPLKD@characterfile?$AA@ 2006a82c     g_bot.obj
 0002:0000383c       ??_C@_0N@GEFCGCPK@loaddefered?6?$AA@ 2006a83c     g_bot.obj
 0002:0000384c       ??_C@_0L@FBHMLJNH@cl_running?$AA@ 2006a84c     g_bot.obj
 0002:00003858       ??_C@_0ED@LBGLLNI@Usage?3?5Addbot?5?$DMbotname?$DO?5?$FLskill?51@ 2006a858     g_bot.obj
 0002:0000389c       ??_C@_0L@BKCPIMBP@bot_enable?$AA@ 2006a89c     g_bot.obj
 0002:000038a8       ??_C@_05CEDINIPN@?$CF5?42f?$AA@ 2006a8a8     g_bot.obj
 0002:000038b0       ??_C@_0FB@BKCBGING@?$FO1Start?5server?5with?5more?5?8open?8?5@ 2006a8b0     g_bot.obj
 0002:00003904       ??_C@_0DE@MKFCEMGM@?$FO1Unable?5to?5add?5bot?4?5?5All?5player@ 2006a904     g_bot.obj
 0002:00003938       ??_C@_0CG@GFPKDAFH@?$FO1Error?3?5bot?5has?5no?5aifile?5speci@ 2006a938     g_bot.obj
 0002:00003960       ??_C@_06GJLCKOIA@aifile?$AA@ 2006a960     g_bot.obj
 0002:00003968       ??_C@_01BMBHCPLG@5?$AA@    2006a968     g_bot.obj
 0002:0000396c       ??_C@_06KEONFOCA@color2?$AA@ 2006a96c     g_bot.obj
 0002:00003974       ??_C@_01FAMBOPH@4?$AA@     2006a974     g_bot.obj
 0002:00003978       ??_C@_06IPMAANOD@color1?$AA@ 2006a978     g_bot.obj
 0002:00003980       ??_C@_04ICKCIGNO@male?$AA@ 2006a980     g_bot.obj
 0002:00003988       ??_C@_06LFOIHHME@gender?$AA@ 2006a988     g_bot.obj
 0002:00003990       ??_C@_0P@JMIBMNM@team_headmodel?$AA@ 2006a990     g_bot.obj
 0002:000039a0       ??_C@_09DHBBGOBJ@headmodel?$AA@ 2006a9a0     g_bot.obj
 0002:000039ac       ??_C@_0L@KEDOKIKJ@team_model?$AA@ 2006a9ac     g_bot.obj
 0002:000039b8       ??_C@_0O@CLCMCGPB@visor?1default?$AA@ 2006a9b8     g_bot.obj
 0002:000039c8       ??_C@_02PEECMOAB@90?$AA@   2006a9c8     g_bot.obj
 0002:000039cc       ??_C@_02PONMODAL@70?$AA@   2006a9cc     g_bot.obj
 0002:000039d0       ??_C@_08HBHLIHAM@handicap?$AA@ 2006a9d0     g_bot.obj
 0002:000039dc       ??_C@_02PNFIDHGF@50?$AA@   2006a9dc     g_bot.obj
 0002:000039e0       ??_C@_05NBLIHODN@?$CF1?42f?$AA@ 2006a9e0     g_bot.obj
 0002:000039e8       ??_C@_05DGPADKBM@snaps?$AA@ 2006a9e8     g_bot.obj
 0002:000039f0       ??_C@_04HCCHHEEF@rate?$AA@ 2006a9f0     g_bot.obj
 0002:000039f8       ??_C@_05GFEIOEMO@25000?$AA@ 2006a9f8     g_bot.obj
 0002:00003a00       ??_C@_07PNOKIGNH@funname?$AA@ 2006aa00     g_bot.obj
 0002:00003a08       ??_C@_0BP@NGBNIFAK@?$FO1Error?3?5Bot?5?8?$CFs?8?5not?5defined?6?$AA@ 2006aa08     g_bot.obj
 0002:00003a28       ??_C@_0BJ@JBHOCGJI@?$FO3Unable?5to?5delay?5spawn?6?$AA@ 2006aa28     g_bot.obj
 0002:00003a44       ??_C@_0BJ@GPLOPMDF@?$CF?916s?5?$CF?916s?5?$CF?920s?5?$CF?920s?6?$AA@ 2006aa44     g_bot.obj
 0002:00003a60       ??_C@_0BB@OCLCLNLB@bots?1default_c?4c?$AA@ 2006aa60     g_bot.obj
 0002:00003a74       ??_C@_0O@PCBPGDGA@UnnamedPlayer?$AA@ 2006aa74     g_bot.obj
 0002:00003a88       ??_C@_0EB@OHFELCCO@?$FO1name?5?5?5?5?5?5?5?5?5?5?5?5?5model?5?5?5?5?5?5?5?5@ 2006aa88     g_bot.obj
 0002:00003acc       ??_C@_0BK@DFMGEDHJ@?$FO1Invalid?5bot?5number?3?5?$CFi?6?$AA@ 2006aacc     g_bot.obj
 0002:00003ae8       ??_C@_04OOIACBCD@bots?$AA@ 2006aae8     g_bot.obj
 0002:00003af0       ??_C@_08FACPJMEJ@training?$AA@ 2006aaf0     g_bot.obj
 0002:00003afc       ??_C@_07BELCMIIP@special?$AA@ 2006aafc     g_bot.obj
 0002:00003b04       ??_C@_09KPHKOKCC@timelimit?$AA@ 2006ab04     g_bot.obj
 0002:00003b10       ??_C@_09GCIEGDDN@fraglimit?$AA@ 2006ab10     g_bot.obj
 0002:00003b1c       ??_C@_0P@IGNPDGBD@bot_minplayers?$AA@ 2006ab1c     g_bot.obj
 0002:00003b2c       ??_C@_03IHCLBPIC@num?$AA@  2006ab2c     g_bot.obj
 0002:00003b30       ??_C@_02IKAHHCAI@?$CFi?$AA@ 2006ab30     g_bot.obj
 0002:00003b34       ??_C@_0BC@MIFKOHOA@?$CFi?5arenas?5parsed?6?$AA@ 2006ab34     g_bot.obj
 0002:00003b48       ??_C@_08IDJEBFOJ@scripts?1?$AA@ 2006ab48     g_bot.obj
 0002:00003b54       ??_C@_07OMEBBDEO@scripts?$AA@ 2006ab54     g_bot.obj
 0002:00003b5c       ??_C@_06IPPMLGON@?4arena?$AA@ 2006ab5c     g_bot.obj
 0002:00003b64       ??_C@_0BD@KEINBKFE@scripts?1arenas?4txt?$AA@ 2006ab64     g_bot.obj
 0002:00003b78       ??_C@_0N@BFDKEKMB@g_arenasFile?$AA@ 2006ab78     g_bot.obj
 0002:00003b88       ??_C@_0CO@OKDDPLPD@?$FO1file?5too?5large?3?5?$CFs?5is?5?$CFi?0?5max?5@ 2006ab88     g_bot.obj
 0002:00003bb8       ??_C@_0BG@BJEIGKLP@?$FO1file?5not?5found?3?5?$CFs?6?$AA@ 2006abb8     g_bot.obj
 0002:00003bd0       ??_C@_0BG@FOPKNLEB@addbot?5?$CFs?5?$CFf?5free?5?$CFi?6?$AA@ 2006abd0     g_bot.obj
 0002:00003be8       ??_C@_0BA@KCNHFFOD@?$CFi?5bots?5parsed?6?$AA@ 2006abe8     g_bot.obj
 0002:00003bf8       ??_C@_04NONLJGOA@?4bot?$AA@ 2006abf8     g_bot.obj
 0002:00003c00       ??_C@_0BB@LMBKKAOC@scripts?1bots?4txt?$AA@ 2006ac00     g_bot.obj
 0002:00003c14       ??_C@_0L@IDJNDIMJ@g_botsFile?$AA@ 2006ac14     g_bot.obj
 0002:00003c20       ??_C@_08MDEJHCAF@nohumans?$AA@ 2006ac20     g_client.obj
 0002:00003c2c       ??_C@_06JHOFIDHH@nobots?$AA@ 2006ac2c     g_client.obj
 0002:00003c34       ??_C@_0BH@IGAFCIL@info_player_deathmatch?$AA@ 2006ac34     g_client.obj
 0002:00003c4c       __real@41100000            2006ac4c     g_client.obj
 0002:00003c50       ??_C@_0BM@DGHFFJBI@Couldn?8t?5find?5a?5spawn?5point?$AA@ 2006ac50     g_client.obj
 0002:00003c6c       ??_C@_07ILHJIGAO@bodyque?$AA@ 2006ac6c     g_client.obj
 0002:00003c74       ??_C@_0BO@IFHBFKHP@ClientUserinfoChanged?3?5?$CFi?5?$CFs?6?$AA@ 2006ac74     g_client.obj
 0002:00003c98       ??_C@_0GA@GJMCBBDN@n?2?$CFs?2t?2?$CFi?2model?2?$CFs?2hmodel?2?$CFs?2g_r@ 2006ac98     g_client.obj
 0002:00003cf8       ??_C@_0EO@IELCCCFM@n?2?$CFs?2t?2?$CFi?2model?2?$CFs?2hmodel?2?$CFs?2c1?2@ 2006acf8     g_client.obj
 0002:00003d48       ??_C@_0L@CPNMJIBN@g_blueteam?$AA@ 2006ad48     g_client.obj
 0002:00003d54       ??_C@_09LPNHELAH@g_redteam?$AA@ 2006ad54     g_client.obj
 0002:00003d60       ??_C@_0M@IKKMOBIP@teamoverlay?$AA@ 2006ad60     g_client.obj
 0002:00003d6c       ??_C@_01OJONOECF@b?$AA@    2006ad6c     g_client.obj
 0002:00003d70       ??_C@_01KDCPPGHE@r?$AA@    2006ad70     g_client.obj
 0002:00003d74       ??_C@_0BM@IJFFLPEN@print?5?$CC?$CFs?$FO7?5renamed?5to?5?$CFs?6?$CC?$AA@ 2006ad74     g_client.obj
 0002:00003d90       ??_C@_0L@PGGJLCHO@scoreboard?$AA@ 2006ad90     g_client.obj
 0002:00003d9c       ??_C@_0BA@PKAEEJJB@cg_predictItems?$AA@ 2006ad9c     g_client.obj
 0002:00003dac       ??_C@_09IPAEKDAI@localhost?$AA@ 2006adac     g_client.obj
 0002:00003db8       ??_C@_02GIIHKPLE@ip?$AA@   2006adb8     g_client.obj
 0002:00003dbc       ??_C@_0O@JBDOHEEF@?2name?2badinfo?$AA@ 2006adbc     g_client.obj
 0002:00003dcc       ??_C@_0BI@LLOHFCPM@print?5?$CC?$CFs?$FO7?5connected?6?$CC?$AA@ 2006adcc     g_client.obj
 0002:00003de4       ??_C@_0BD@LEMBFDEN@ClientConnect?3?5?$CFi?6?$AA@ 2006ade4     g_client.obj
 0002:00003df8       ??_C@_0BB@KINAMDJK@BotConnectfailed?$AA@ 2006adf8     g_client.obj
 0002:00003e0c       ??_C@_0BB@GKDCDICO@Invalid?5password?$AA@ 2006ae0c     g_client.obj
 0002:00003e20       ??_C@_04CGFJFPFD@none?$AA@ 2006ae20     g_client.obj
 0002:00003e28       ??_C@_08NLHBPEGP@password?$AA@ 2006ae28     g_client.obj
 0002:00003e34       ??_C@_0CB@BAJJGAM@You?5are?5banned?5from?5this?5server?4@ 2006ae34     g_client.obj
 0002:00003e58       ??_C@_0BB@JCCEPCGJ@ClientBegin?3?5?$CFi?6?$AA@ 2006ae58     g_client.obj
 0002:00003e6c       ??_C@_0BP@PGPGIDAG@print?5?$CC?$CFs?$FO7?5entered?5the?5game?6?$CC?$AA@ 2006ae6c     g_client.obj
 0002:00003e8c       ??_C@_06BALNJMNP@player?$AA@ 2006ae8c     g_client.obj
 0002:00003e94       ??_C@_0N@GGGDBMDO@disconnected?$AA@ 2006ae94     g_client.obj
 0002:00003ea4       ??_C@_0BG@PJMKPFGA@ClientDisconnect?3?5?$CFi?6?$AA@ 2006aea4     g_client.obj
 0002:00003ebc       ??_C@_09OKMOBHEE@Harvester?$AA@ 2006aebc     g_cmds.obj
 0002:00003ec8       ??_C@_08JKIFACLF@Overload?$AA@ 2006aec8     g_cmds.obj
 0002:00003ed4       ??_C@_0N@FCMBHKKN@One?5Flag?5CTF?$AA@ 2006aed4     g_cmds.obj
 0002:00003ee4       ??_C@_0BB@OOIHNFAG@Capture?5the?5Flag?$AA@ 2006aee4     g_cmds.obj
 0002:00003ef8       ??_C@_0BA@KHHNIIJE@Team?5Deathmatch?$AA@ 2006aef8     g_cmds.obj
 0002:00003f08       ??_C@_0O@NNAOEDOE@Single?5Player?$AA@ 2006af08     g_cmds.obj
 0002:00003f18       ??_C@_0L@FENDKKGN@Tournament?$AA@ 2006af18     g_cmds.obj
 0002:00003f24       ??_C@_0N@PCEMCJC@Free?5For?5All?$AA@ 2006af24     g_cmds.obj
 0002:00003f34       ??_C@_06MHOMHIDM@report?$AA@ 2006af34     g_cmds.obj
 0002:00003f3c       ??_C@_0BD@JFEBCONJ@search?5and?5destroy?$AA@ 2006af3c     g_cmds.obj
 0002:00003f50       ??_C@_0P@BDHIOPIB@guard?5location?$AA@ 2006af50     g_cmds.obj
 0002:00003f60       ??_C@_08NJPHEENP@cover?5me?$AA@ 2006af60     g_cmds.obj
 0002:00003f6c       ??_C@_09NKPGKNPA@come?5here?$AA@ 2006af6c     g_cmds.obj
 0002:00003f78       ??_C@_0BD@BGOJJIFC@hold?5this?5position?$AA@ 2006af78     g_cmds.obj
 0002:00003f8c       ??_C@_0BD@BEPMJBOM@hold?5your?5position?$AA@ 2006af8c     g_cmds.obj
 0002:00003fa0       ??_C@_0BC@BADCIGBJ@scores?5?$CFi?5?$CFi?5?$CFi?$CFs?$AA@ 2006afa0     g_cmds.obj
 0002:00003fb4       ??_C@_0CL@EAFNPFGA@?5?$CFi?5?$CFi?5?$CFi?5?$CFi?5?$CFi?5?$CFi?5?$CFi?5?$CFi?5?$CFi?5?$CFi?5?$CF@ 2006afb4     g_cmds.obj
 0002:00003fe0       ??_C@_0DA@KHFNLLBI@print?5?$CCYou?5must?5be?5alive?5to?5use?5@ 2006afe0     g_cmds.obj
 0002:00004010       ??_C@_0DA@DLJNDFCJ@print?5?$CCCheats?5are?5not?5enabled?5on@ 2006b010     g_cmds.obj
 0002:00004040       ??_C@_0CG@OFMIDLCG@print?5?$CCUser?5?$CFs?5is?5not?5on?5the?5ser@ 2006b040     g_cmds.obj
 0002:00004068       ??_C@_0CB@IOMDOEKP@print?5?$CCClient?5?$CFi?5is?5not?5active?6?$CC@ 2006b068     g_cmds.obj
 0002:0000408c       ??_C@_0BN@FGLBNIJH@print?5?$CCBad?5client?5slot?3?5?$CFi?6?$CC?$AA@ 2006b08c     g_cmds.obj
 0002:000040ac       ??_C@_06CHFMFANC@assist?$AA@ 2006b0ac     g_cmds.obj
 0002:000040b4       ??_C@_0O@DCIHIELO@gauntletaward?$AA@ 2006b0b4     g_cmds.obj
 0002:000040c4       ??_C@_0L@GBLMIJON@impressive?$AA@ 2006b0c4     g_cmds.obj
 0002:000040d0       ??_C@_09MBDMPFOO@excellent?$AA@ 2006b0d0     g_cmds.obj
 0002:000040dc       ??_C@_05JJEJIJLL@armor?$AA@ 2006b0dc     g_cmds.obj
 0002:000040e4       ??_C@_04PGKJFGNK@ammo?$AA@ 2006b0e4     g_cmds.obj
 0002:000040ec       ??_C@_07PKKCMMCH@weapons?$AA@ 2006b0ec     g_cmds.obj
 0002:000040f4       ??_C@_03NFKEKGGK@all?$AA@  2006b0f4     g_cmds.obj
 0002:000040f8       ??_C@_0L@GPCEIOHM@print?5?$CC?$CFs?$CC?$AA@ 2006b0f8     g_cmds.obj
 0002:00004104       ??_C@_0M@MCLKHHDH@godmode?5ON?6?$AA@ 2006b104     g_cmds.obj
 0002:00004110       ??_C@_0N@POKEKLLJ@godmode?5OFF?6?$AA@ 2006b110     g_cmds.obj
 0002:00004120       ??_C@_0N@OBJNJDJO@notarget?5ON?6?$AA@ 2006b120     g_cmds.obj
 0002:00004130       ??_C@_0O@FBINJHBB@notarget?5OFF?6?$AA@ 2006b130     g_cmds.obj
 0002:00004140       ??_C@_0L@MDMNIPJN@noclip?5ON?6?$AA@ 2006b140     g_cmds.obj
 0002:0000414c       ??_C@_0M@MIKGJGLH@noclip?5OFF?6?$AA@ 2006b14c     g_cmds.obj
 0002:00004158       ??_C@_0CP@EMMMGMNN@print?5?$CCMust?5be?5in?5g_gametype?50?5f@ 2006b158     g_cmds.obj
 0002:00004188       ??_C@_0BO@HCBBHHLG@cp?5?$CC?$CFs?$FO7?5joined?5the?5battle?4?6?$CC?$AA@ 2006b188     g_cmds.obj
 0002:000041a8       ??_C@_0CC@CKOABLEC@cp?5?$CC?$CFs?$FO7?5joined?5the?5spectators?4?6@ 2006b1a8     g_cmds.obj
 0002:000041cc       ??_C@_0CB@MALDLCDE@cp?5?$CC?$CFs?$FO7?5joined?5the?5blue?5team?4?6?$CC@ 2006b1cc     g_cmds.obj
 0002:000041f0       ??_C@_0CA@FCJONFGI@cp?5?$CC?$CFs?$FO7?5joined?5the?5red?5team?4?6?$CC?$AA@ 2006b1f0     g_cmds.obj
 0002:00004210       ??_C@_0CG@BNBAGBGM@cp?5?$CCBlue?5team?5has?5too?5many?5playe@ 2006b210     g_cmds.obj
 0002:00004238       ??_C@_0CF@OMMGDNAE@cp?5?$CCRed?5team?5has?5too?5many?5player@ 2006b238     g_cmds.obj
 0002:00004260       ??_C@_01LKDEMHDF@s?$AA@    2006b260     g_cmds.obj
 0002:00004264       ??_C@_09FNMDCDOI@spectator?$AA@ 2006b264     g_cmds.obj
 0002:00004270       ??_C@_07NNICNDK@follow2?$AA@ 2006b270     g_cmds.obj
 0002:00004278       ??_C@_07CGPFHOPJ@follow1?$AA@ 2006b278     g_cmds.obj
 0002:00004280       ??_C@_05DBKDOICH@score?$AA@ 2006b280     g_cmds.obj
 0002:00004288       ??_C@_0DM@NEIAOCHE@print?5?$CCMay?5not?5switch?5teams?5more@ 2006b288     g_cmds.obj
 0002:000042c4       ??_C@_0BI@PDLENAMN@print?5?$CCSpectator?5team?6?$CC?$AA@ 2006b2c4     g_cmds.obj
 0002:000042dc       ??_C@_0BD@COAKLBJE@print?5?$CCFree?5team?6?$CC?$AA@ 2006b2dc     g_cmds.obj
 0002:000042f0       ??_C@_0BC@HGAENHGG@print?5?$CCRed?5team?6?$CC?$AA@ 2006b2f0     g_cmds.obj
 0002:00004304       ??_C@_0BD@PGCCOEMO@print?5?$CCBlue?5team?6?$CC?$AA@ 2006b304     g_cmds.obj
 0002:00004318       ??_C@_0BO@KJIMFOBJ@Cmd_FollowCycle_f?3?5bad?5dir?5?$CFi?$AA@ 2006b318     g_cmds.obj
 0002:00004338       ??_C@_05JMJKDBEJ@?$CFs?$CFs?6?$AA@ 2006b338     g_cmds.obj
 0002:00004340       ??_C@_0O@FNNABOLL@?$BJ?$FL?$CFs?$CFc?$CFc?$BJ?$FN?$BJ?3?5?$AA@ 2006b340     g_cmds.obj
 0002:00004350       ??_C@_0BD@GLHHAOBD@?$BJ?$FL?$CFs?$CFc?$CFc?$BJ?$FN?5?$CI?$CFs?$CJ?$BJ?3?5?$AA@ 2006b350     g_cmds.obj
 0002:00004364       ??_C@_0O@FGLMEIPO@?$BJ?$CI?$CFs?$CFc?$CFc?$BJ?$CJ?$BJ?3?5?$AA@ 2006b364     g_cmds.obj
 0002:00004374       ??_C@_0BD@LHDLGCNL@?$BJ?$CI?$CFs?$CFc?$CFc?$BJ?$CJ?5?$CI?$CFs?$CJ?$BJ?3?5?$AA@ 2006b374     g_cmds.obj
 0002:00004388       ??_C@_0BB@OADDLILN@sayteam?3?5?$CFs?3?5?$CFs?6?$AA@ 2006b388     g_cmds.obj
 0002:0000439c       ??_C@_09GPHNFPKO@?$CFs?$CFc?$CFc?$BJ?3?5?$AA@ 2006b39c     g_cmds.obj
 0002:000043a8       ??_C@_0N@PIPLJLA@say?3?5?$CFs?3?5?$CFs?6?$AA@ 2006b3a8     g_cmds.obj
 0002:000043b8       ??_C@_0O@CCPEDGNK@?$CFs?5?$CC?$CFs?$CFc?$CFc?$CFs?$CC?$AA@ 2006b3b8     g_cmds.obj
 0002:000043c8       ??_C@_0O@PGEGBHPB@voice?3?5?$CFs?5?$CFs?6?$AA@ 2006b3c8     g_cmds.obj
 0002:000043d8       ??_C@_0P@GLNDPPNN@?$CFs?5?$CFd?5?$CFd?5?$CFd?5?$CFs?$AA@ 2006b3d8     g_cmds.obj
 0002:000043e8       ??_C@_05LBAAHPBE@vchat?$AA@ 2006b3e8     g_cmds.obj
 0002:000043f0       ??_C@_05BLGJOHFB@vtell?$AA@ 2006b3f0     g_cmds.obj
 0002:000043f8       ??_C@_06FPNOEFND@vtchat?$AA@ 2006b3f8     g_cmds.obj
 0002:00004400       ??_C@_0M@MIDAEIOB@print?5?$CC?$CFs?6?$CC?$AA@ 2006b400     g_cmds.obj
 0002:0000440c       ??_C@_0BL@LDCKNKB@print?5?$CC?$CFs?5called?5a?5vote?4?6?$CC?$AA@ 2006b40c     g_cmds.obj
 0002:00004428       ??_C@_07CMIPDAGF@?$CFs?5?$CC?$CFs?$CC?$AA@ 2006b428     g_cmds.obj
 0002:00004430       ??_C@_0N@NPFCFAAA@vstr?5nextmap?$AA@ 2006b430     g_cmds.obj
 0002:00004440       ??_C@_0BK@IOHPLFMM@print?5?$CCnextmap?5not?5set?4?6?$CC?$AA@ 2006b440     g_cmds.obj
 0002:0000445c       ??_C@_0BI@EHIPCLJD@?$CFs?5?$CFs?$DL?5set?5nextmap?5?$CC?$CFs?$CC?$AA@ 2006b45c     g_cmds.obj
 0002:00004474       ??_C@_05DNIIFBMG@?$CFs?5?$CFs?$AA@ 2006b474     g_cmds.obj
 0002:0000447c       ??_C@_05DIALNFFA@?$CFs?5?$CFd?$AA@ 2006b47c     g_cmds.obj
 0002:00004484       ??_C@_0BL@HOKFFIC@print?5?$CCInvalid?5gametype?4?6?$CC?$AA@ 2006b484     g_cmds.obj
 0002:000044a0       ??_C@_03OFAPEBGM@?$CFs?6?$AA@ 2006b4a0     g_cmds.obj
 0002:000044a8       ??_C@_0KJ@BAKDCPAJ@print?5?$CCVote?5commands?5are?3?5map_re@ 2006b4a8     g_cmds.obj
 0002:00004554       ??_C@_0L@LPENDGCI@g_doWarmup?$AA@ 2006b554     g_cmds.obj
 0002:00004560       ??_C@_0L@NBDAICFL@clientkick?$AA@ 2006b560     g_cmds.obj
 0002:0000456c       ??_C@_04FNIJDBCC@kick?$AA@ 2006b56c     g_cmds.obj
 0002:00004574       ??_C@_07MCHHMPMB@nextmap?$AA@ 2006b574     g_cmds.obj
 0002:0000457c       ??_C@_0M@NBIMEKNE@map_restart?$AA@ 2006b57c     g_cmds.obj
 0002:00004588       ??_C@_0BO@PMPHENKD@print?5?$CCInvalid?5vote?5string?4?6?$CC?$AA@ 2006b588     g_cmds.obj
 0002:000045a8       ??_C@_0DC@KBNBHNDJ@print?5?$CCNot?5allowed?5to?5call?5a?5vot@ 2006b5a8     g_cmds.obj
 0002:000045dc       ??_C@_0DG@PHEGLJKA@print?5?$CCYou?5have?5called?5the?5maxim@ 2006b5dc     g_cmds.obj
 0002:00004614       ??_C@_0CI@IOOGHLKJ@print?5?$CCA?5vote?5is?5already?5in?5prog@ 2006b614     g_cmds.obj
 0002:0000463c       ??_C@_0CC@MKEOLBNH@print?5?$CCVoting?5not?5allowed?5here?4?6@ 2006b63c     g_cmds.obj
 0002:00004660       ??_C@_0BE@KBOHCPHM@print?5?$CCVote?5cast?4?6?$CC?$AA@ 2006b660     g_cmds.obj
 0002:00004674       ??_C@_0CL@KIACKMGK@print?5?$CCNot?5allowed?5to?5vote?5as?5sp@ 2006b674     g_cmds.obj
 0002:000046a0       ??_C@_0BM@JAOFDBMB@print?5?$CCVote?5already?5cast?4?6?$CC?$AA@ 2006b6a0     g_cmds.obj
 0002:000046bc       ??_C@_0BO@JJMMHDFC@print?5?$CCNo?5vote?5in?5progress?4?6?$CC?$AA@ 2006b6bc     g_cmds.obj
 0002:000046dc       ??_C@_0CA@ENAIANHJ@print?5?$CC?$CFs?5called?5a?5team?5vote?4?6?$CC?$AA@ 2006b6dc     g_cmds.obj
 0002:000046fc       ??_C@_0DC@JMKMFJGE@print?5?$CCTeam?5vote?5commands?5are?3?5l@ 2006b6fc     g_cmds.obj
 0002:00004730       ??_C@_0DA@BDICJJF@print?5?$CC?$CFs?5is?5not?5a?5valid?5player?5@ 2006b730     g_cmds.obj
 0002:00004760       ??_C@_06DFLPLEOP@leader?$AA@ 2006b760     g_cmds.obj
 0002:00004768       ??_C@_0DL@IFNKHCNG@print?5?$CCYou?5have?5called?5the?5maxim@ 2006b768     g_cmds.obj
 0002:000047a4       ??_C@_0CN@INNKCADJ@print?5?$CCA?5team?5vote?5is?5already?5in@ 2006b7a4     g_cmds.obj
 0002:000047d4       ??_C@_0BJ@DCKHGAB@print?5?$CCTeam?5vote?5cast?4?6?$CC?$AA@ 2006b7d4     g_cmds.obj
 0002:000047f0       ??_C@_0CB@LGGMNIHI@print?5?$CCTeam?5vote?5already?5cast?4?6?$CC@ 2006b7f0     g_cmds.obj
 0002:00004814       ??_C@_0CD@BLODMPFK@print?5?$CCNo?5team?5vote?5in?5progress?4@ 2006b814     g_cmds.obj
 0002:00004838       ??_C@_0CF@GJFHLKOA@print?5?$CCusage?3?5setviewpos?5x?5y?5z?5y@ 2006b838     g_cmds.obj
 0002:00004860       ??_C@_0BI@FJNBDMBJ@print?5?$CCunknown?5cmd?5?$CFs?6?$CC?$AA@ 2006b860     g_cmds.obj
 0002:00004878       ??_C@_05BLKJBNOD@stats?$AA@ 2006b878     g_cmds.obj
 0002:00004880       ??_C@_0L@CCEFBCKP@setviewpos?$AA@ 2006b880     g_cmds.obj
 0002:0000488c       ??_C@_02DPGMDCM@gc?$AA@    2006b88c     g_cmds.obj
 0002:00004890       ??_C@_08OLLMCBNG@teamvote?$AA@ 2006b890     g_cmds.obj
 0002:0000489c       ??_C@_0N@JDBKAFAM@callteamvote?$AA@ 2006b89c     g_cmds.obj
 0002:000048ac       ??_C@_04GHHIKFLG@vote?$AA@ 2006b8ac     g_cmds.obj
 0002:000048b4       ??_C@_08NNMLCPB@callvote?$AA@ 2006b8b4     g_cmds.obj
 0002:000048c0       ??_C@_05LCFPHLEE@where?$AA@ 2006b8c0     g_cmds.obj
 0002:000048c8       ??_C@_0L@FFKCNEMH@followprev?$AA@ 2006b8c8     g_cmds.obj
 0002:000048d4       ??_C@_0L@GBHEMAKD@follownext?$AA@ 2006b8d4     g_cmds.obj
 0002:000048e0       ??_C@_06HNJAFFAK@follow?$AA@ 2006b8e0     g_cmds.obj
 0002:000048e8       ??_C@_09EFOFPGPE@levelshot?$AA@ 2006b8e8     g_cmds.obj
 0002:000048f4       ??_C@_06IHODGGMJ@noclip?$AA@ 2006b8f4     g_cmds.obj
 0002:000048fc       ??_C@_08HPLPOCJL@notarget?$AA@ 2006b8fc     g_cmds.obj
 0002:00004908       ??_C@_03DKFAMNOH@god?$AA@  2006b908     g_cmds.obj
 0002:0000490c       ??_C@_04BMBHJADG@give?$AA@ 2006b90c     g_cmds.obj
 0002:00004914       ??_C@_06JMKGCPMO@votell?$AA@ 2006b914     g_cmds.obj
 0002:0000491c       ??_C@_0L@GKKIAMHC@vosay_team?$AA@ 2006b91c     g_cmds.obj
 0002:00004928       ??_C@_05EGEGDMMG@vosay?$AA@ 2006b928     g_cmds.obj
 0002:00004930       ??_C@_09CPIJOHHK@vsay_team?$AA@ 2006b930     g_cmds.obj
 0002:0000493c       ??_C@_04IBCNHBFH@vsay?$AA@ 2006b93c     g_cmds.obj
 0002:00004944       ??_C@_04LBPCFPDD@tell?$AA@ 2006b944     g_cmds.obj
 0002:0000494c       ??_C@_08NBFNGOHN@say_team?$AA@ 2006b94c     g_cmds.obj
 0002:00004958       ??_C@_03BANJEMDJ@say?$AA@  2006b958     g_cmds.obj
 0002:0000495c       ??_C@_0BE@DNAOGBCN@tell?3?5?$CFs?5to?5?$CFs?3?5?$CFs?6?$AA@ 2006b95c     g_cmds.obj
 0002:00004970       ??_C@_0BF@KNCPEACI@vtell?3?5?$CFs?5to?5?$CFs?3?5?$CFs?6?$AA@ 2006b970     g_cmds.obj
 0002:00004988       ??_C@_06GEFAPDPP@praise?$AA@ 2006b988     g_cmds.obj
 0002:00004990       ??_C@_0M@BGKKOPE@MOD_GRAPPLE?$AA@ 2006b990     g_combat.obj
 0002:0000499c       ??_C@_0BB@JHNHPELL@MOD_TRIGGER_HURT?$AA@ 2006b99c     g_combat.obj
 0002:000049b0       ??_C@_0BB@HMLMKPCA@MOD_TARGET_LASER?$AA@ 2006b9b0     g_combat.obj
 0002:000049c4       ??_C@_0M@NECNIJDJ@MOD_SUICIDE?$AA@ 2006b9c4     g_combat.obj
 0002:000049d0       ??_C@_0M@JONLOPJN@MOD_FALLING?$AA@ 2006b9d0     g_combat.obj
 0002:000049dc       ??_C@_0N@IMHJNLFF@MOD_TELEFRAG?$AA@ 2006b9dc     g_combat.obj
 0002:000049ec       ??_C@_09GPMGMMBL@MOD_CRUSH?$AA@ 2006b9ec     g_combat.obj
 0002:000049f8       ??_C@_08LEPCJCFO@MOD_LAVA?$AA@ 2006b9f8     g_combat.obj
 0002:00004a04       ??_C@_09KBJPPHD@MOD_SLIME?$AA@ 2006ba04     g_combat.obj
 0002:00004a10       ??_C@_09MAPLCDLI@MOD_WATER?$AA@ 2006ba10     g_combat.obj
 0002:00004a1c       ??_C@_0P@OHBIPEGK@MOD_BFG_SPLASH?$AA@ 2006ba1c     g_combat.obj
 0002:00004a2c       ??_C@_07EOLOFKFM@MOD_BFG?$AA@ 2006ba2c     g_combat.obj
 0002:00004a34       ??_C@_0O@GLCOIAIP@MOD_LIGHTNING?$AA@ 2006ba34     g_combat.obj
 0002:00004a44       ??_C@_0M@BHIJMBBE@MOD_RAILGUN?$AA@ 2006ba44     g_combat.obj
 0002:00004a50       ??_C@_0BC@PIBHLJKK@MOD_PLASMA_SPLASH?$AA@ 2006ba50     g_combat.obj
 0002:00004a64       ??_C@_0L@JPCJGHHF@MOD_PLASMA?$AA@ 2006ba64     g_combat.obj
 0002:00004a70       ??_C@_0BC@KJDNONBC@MOD_ROCKET_SPLASH?$AA@ 2006ba70     g_combat.obj
 0002:00004a84       ??_C@_0L@FIOJJPEO@MOD_ROCKET?$AA@ 2006ba84     g_combat.obj
 0002:00004a90       ??_C@_0BD@PLGCKMBF@MOD_GRENADE_SPLASH?$AA@ 2006ba90     g_combat.obj
 0002:00004aa4       ??_C@_0M@KDJNKEED@MOD_GRENADE?$AA@ 2006baa4     g_combat.obj
 0002:00004ab0       ??_C@_0P@DNHADEBJ@MOD_MACHINEGUN?$AA@ 2006bab0     g_combat.obj
 0002:00004ac0       ??_C@_0N@MJPPIPMF@MOD_GAUNTLET?$AA@ 2006bac0     g_combat.obj
 0002:00004ad0       ??_C@_0M@MIHCLLAH@MOD_SHOTGUN?$AA@ 2006bad0     g_combat.obj
 0002:00004adc       ??_C@_0M@BKDMLGAO@MOD_UNKNOWN?$AA@ 2006badc     g_combat.obj
 0002:00004ae8       ??_C@_0P@LIDDFKFD@kamikaze?5timer?$AA@ 2006bae8     g_combat.obj
 0002:00004af8       ??_C@_0BB@JDBGHPJP@team_blueobelisk?$AA@ 2006baf8     g_combat.obj
 0002:00004b0c       ??_C@_0BA@GIMOGCGC@team_redobelisk?$AA@ 2006bb0c     g_combat.obj
 0002:00004b1c       ??_C@_0CE@HGPMHBOH@Kill?3?5?$CFi?5?$CFi?5?$CFi?3?5?$CFs?5killed?5?$CFs?5by?5@ 2006bb1c     g_combat.obj
 0002:00004b40       ??_C@_0P@BDPEDPJP@?$DMbad?5obituary?$DO?$AA@ 2006bb40     g_combat.obj
 0002:00004b50       ??_C@_07GECLLGBL@?$DMworld?$DO?$AA@ 2006bb50     g_combat.obj
 0002:00004b58       ??_C@_0N@HGAIBNNB@?$DMnon?9client?$DO?$AA@ 2006bb58     g_combat.obj
 0002:00004b68       __real@3fe51eb851eb851f    2006bb68     g_combat.obj
 0002:00004b70       __real@4000000000000000    2006bb70     g_combat.obj
 0002:00004b78       ??_C@_0CM@LEIIGBFN@?$CFi?3?5client?3?$CFi?5health?3?$CFi?5damage?3?$CF@ 2006bb78     g_combat.obj
 0002:00004ba8       __real@402e000000000000    2006bba8     g_combat.obj
 0002:00004bb0       __real@43400000            2006bbb0     g_items.obj
 0002:00004bb4       ??_C@_0CA@FLGMIHAB@sound?1items?1kamikazerespawn?4wav?$AA@ 2006bbb4     g_items.obj
 0002:00004bd4       ??_C@_0BM@BNLFEEPK@RespawnItem?3?5bad?5teammaster?$AA@ 2006bbd4     g_items.obj
 0002:00004bf0       ??_C@_0N@OCCHADDH@Item?3?5?$CFi?5?$CFs?6?$AA@ 2006bbf0     g_items.obj
 0002:00004c00       __real@4069000000000000    2006bc00     g_items.obj
 0002:00004c08       __real@4046800000000000    2006bc08     g_items.obj
 0002:00004c10       ??_C@_0CJ@EMOANFCC@FinishSpawningItem?3?5?$CFs?5startsoli@ 2006bc10     g_items.obj
 0002:00004c3c       __real@45800000            2006bc3c     g_items.obj
 0002:00004c40       ??_C@_0CH@HHMBIMLK@?$FO3WARNING?3?5No?5team_CTF_blueflag?5@ 2006bc40     g_items.obj
 0002:00004c68       ??_C@_0CG@DNHJENHJ@?$FO3WARNING?3?5No?5team_CTF_redflag?5i@ 2006bc68     g_items.obj
 0002:00004c90       ??_C@_0BD@LOGEPNHD@RegisterItem?3?5NULL?$AA@ 2006bc90     g_items.obj
 0002:00004ca4       ??_C@_0BF@PHBDLOMN@?$CFi?5items?5registered?6?$AA@ 2006bca4     g_items.obj
 0002:00004cbc       ??_C@_0L@BHNPAADM@disable_?$CFs?$AA@ 2006bcbc     g_items.obj
 0002:00004cc8       ??_C@_0O@MNEGCFDN@noglobalsound?$AA@ 2006bcc8     g_items.obj
 0002:00004cd8       ??_C@_04PNOAOIAG@wait?$AA@ 2006bcd8     g_items.obj
 0002:00004ce0       ??_C@_06NLFCANPD@random?$AA@ 2006bce0     g_items.obj
 0002:00004ce8       __real@c0000000            2006bce8     g_items.obj
 0002:00004cec       ??_C@_0L@NIHHPBKG@g_rankings?$AA@ 2006bcec     g_main.obj
 0002:00004cf8       ??_C@_0M@HOGKGHBI@pmove_fixed?$AA@ 2006bcf8     g_main.obj
 0002:00004d04       ??_C@_0BA@EKPBHCCJ@g_smoothClients?$AA@ 2006bd04     g_main.obj
 0002:00004d14       ??_C@_0N@JIFICDHI@g_listEntity?$AA@ 2006bd14     g_main.obj
 0002:00004d24       ??_C@_0M@MECNLONK@g_allowVote?$AA@ 2006bd24     g_main.obj
 0002:00004d30       ??_C@_02PFIAKEDG@80?$AA@   2006bd30     g_main.obj
 0002:00004d34       ??_C@_09DKNLLEN@com_blood?$AA@ 2006bd34     g_main.obj
 0002:00004d40       ??_C@_06IBNENCEO@g_motd?$AA@ 2006bd40     g_main.obj
 0002:00004d48       ??_C@_0N@CGHOHBHC@g_debugAlloc?$AA@ 2006bd48     g_main.obj
 0002:00004d58       ??_C@_0O@JCLHDLKF@g_debugDamage?$AA@ 2006bd58     g_main.obj
 0002:00004d68       ??_C@_0M@EPOBGCBB@g_debugMove?$AA@ 2006bd68     g_main.obj
 0002:00004d74       ??_C@_0N@JGEKALLI@g_inactivity?$AA@ 2006bd74     g_main.obj
 0002:00004d84       ??_C@_0P@JEPDGNEP@g_forcerespawn?$AA@ 2006bd84     g_main.obj
 0002:00004d94       ??_C@_02PJNFELNH@30?$AA@   2006bd94     g_main.obj
 0002:00004d98       ??_C@_0BE@CNNPIPEC@g_weaponTeamRespawn?$AA@ 2006bd98     g_main.obj
 0002:00004dac       ??_C@_0BA@CMOCDPF@g_weaponrespawn?$AA@ 2006bdac     g_main.obj
 0002:00004dbc       ??_C@_01EKENIIDA@3?$AA@    2006bdbc     g_main.obj
 0002:00004dc0       ??_C@_0N@LCBCFAFA@g_quadfactor?$AA@ 2006bdc0     g_main.obj
 0002:00004dd0       ??_C@_04KOJKLCBG@1000?$AA@ 2006bdd0     g_main.obj
 0002:00004dd8       ??_C@_0M@PDFGFIOM@g_knockback?$AA@ 2006bdd8     g_main.obj
 0002:00004de4       ??_C@_03BAAJCDMO@800?$AA@  2006bde4     g_main.obj
 0002:00004de8       ??_C@_09HNGNBNKN@g_gravity?$AA@ 2006bde8     g_main.obj
 0002:00004df4       ??_C@_03MEIMHAKB@320?$AA@  2006bdf4     g_main.obj
 0002:00004df8       ??_C@_07KCHPCPJD@g_speed?$AA@ 2006bdf8     g_main.obj
 0002:00004e00       ??_C@_09BJOAODLF@dedicated?$AA@ 2006be00     g_main.obj
 0002:00004e0c       ??_C@_0L@MLCEEGBP@g_needpass?$AA@ 2006be0c     g_main.obj
 0002:00004e18       ??_C@_0M@NIKBMNDP@g_filterBan?$AA@ 2006be18     g_main.obj
 0002:00004e24       ??_C@_08NKMDLNHL@g_banIPs?$AA@ 2006be24     g_main.obj
 0002:00004e30       ??_C@_0L@GHAPAPFD@g_password?$AA@ 2006be30     g_main.obj
 0002:00004e3c       ??_C@_09IPDDEHO@g_logSync?$AA@ 2006be3c     g_main.obj
 0002:00004e48       ??_C@_09BNLGBMID@games?4log?$AA@ 2006be48     g_main.obj
 0002:00004e54       ??_C@_05PJEIAAGC@g_log?$AA@ 2006be54     g_main.obj
 0002:00004e5c       ??_C@_08HAMOJLDA@g_warmup?$AA@ 2006be5c     g_main.obj
 0002:00004e68       ??_C@_0BD@CLGJCDLA@g_teamForceBalance?$AA@ 2006be68     g_main.obj
 0002:00004e7c       ??_C@_0P@PONBNCIE@g_teamAutoJoin?$AA@ 2006be7c     g_main.obj
 0002:00004e8c       ??_C@_0P@IEOFAMLI@g_friendlyFire?$AA@ 2006be8c     g_main.obj
 0002:00004e9c       ??_C@_0BF@LICFCALK@g_synchronousClients?$AA@ 2006be9c     g_main.obj
 0002:00004eb4       ??_C@_0N@FCAHJCDA@capturelimit?$AA@ 2006beb4     g_main.obj
 0002:00004ec4       ??_C@_07GMGCLCAP@dmflags?$AA@ 2006bec4     g_main.obj
 0002:00004ecc       ??_C@_0BB@JCLDAPBF@g_maxGameClients?$AA@ 2006becc     g_main.obj
 0002:00004ee0       ??_C@_0L@DFBEGALI@sv_mapname?$AA@ 2006bee0     g_main.obj
 0002:00004eec       ??_C@_0M@GHMJJAD@g_restarted?$AA@ 2006beec     g_main.obj
 0002:00004ef8       ??_C@_0M@BBDAHLGI@May?525?52008?$AA@ 2006bef8     g_main.obj
 0002:00004f04       ??_C@_08CLLHAKFA@gamedate?$AA@ 2006bf04     g_main.obj
 0002:00004f10       ??_C@_06KOMAFLML@baseq3?$AA@ 2006bf10     g_main.obj
 0002:00004f18       ??_C@_08HCPAIKAO@gamename?$AA@ 2006bf18     g_main.obj
 0002:00004f24       ??_C@_09NFOPKLIK@sv_cheats?$AA@ 2006bf24     g_main.obj
 0002:00004f30       ??_C@_0BL@EIPAHDOP@?$CFi?5teams?5with?5?$CFi?5entities?6?$AA@ 2006bf30     g_main.obj
 0002:00004f4c       ??_C@_0DA@HFHMPEPI@g_gametype?5?$CFi?5is?5out?5of?5range?0?5d@ 2006bf4c     g_main.obj
 0002:00004f7c       ??_C@_0CC@FFJICNKE@print?5?$CCServer?3?5?$CFs?5changed?5to?5?$CFs?6@ 2006bf7c     g_main.obj
 0002:00004fa0       ??_C@_0BA@MOHNLIKA@com_buildScript?$AA@ 2006bfa0     g_main.obj
 0002:00004fb0       ??_C@_0CF@MLCIJBNO@?9?9?9?9?9?9?9?9?9?9?9?9?9?9?9?9?9?9?9?9?9?9?9?9?9?9?9?9?9?9?9?9@ 2006bfb0     g_main.obj
 0002:00004fd8       ??_C@_0BG@MOMCCAKP@Not?5logging?5to?5disk?4?6?$AA@ 2006bfd8     g_main.obj
 0002:00004ff0       ??_C@_0O@DEDEBKNJ@InitGame?3?5?$CFs?6?$AA@ 2006bff0     g_main.obj
 0002:00005000       ??_C@_0DO@BDNDJIG@?9?9?9?9?9?9?9?9?9?9?9?9?9?9?9?9?9?9?9?9?9?9?9?9?9?9?9?9?9?9?9?9@ 2006c000     g_main.obj
 0002:00005040       ??_C@_0CE@PLBPIHPI@WARNING?3?5Couldn?8t?5open?5logfile?3?5@ 2006c040     g_main.obj
 0002:00005064       ??_C@_0BF@CCJLMEBG@sound?1player?1fry?4wav?$AA@ 2006c064     g_main.obj
 0002:0000507c       ??_C@_0O@LOFLFABD@gamedate?3?5?$CFs?6?$AA@ 2006c07c     g_main.obj
 0002:0000508c       ??_C@_0O@MKINOKNK@gamename?3?5?$CFs?6?$AA@ 2006c08c     g_main.obj
 0002:0000509c       ??_C@_0CF@FDKFKNJ@?9?9?9?9?9?9?9?5Game?5Initialization?5?9?9?9?9@ 2006c09c     g_main.obj
 0002:000050c4       ??_C@_0P@OFNEJLIL@ShutdownGame?3?6?$AA@ 2006c0c4     g_main.obj
 0002:000050d4       ??_C@_0BI@EOKPGBAF@?$DN?$DN?$DN?$DN?5ShutdownGame?5?$DN?$DN?$DN?$DN?6?$AA@ 2006c0d4     g_main.obj
 0002:000050ec       ??_C@_01INIBCBCB@f?$AA@    2006c0ec     g_main.obj
 0002:000050f0       ??_C@_0BJ@LMMLDPE@info_player_intermission?$AA@ 2006c0f0     g_main.obj
 0002:0000510c       ??_C@_0O@PKDALKNK@vstr?5nextmap?6?$AA@ 2006c10c     g_main.obj
 0002:0000511c       ??_C@_0P@BKKOFHJN@map_restart?50?6?$AA@ 2006c11c     g_main.obj
 0002:0000512c       ??_C@_09OHCHOIDO@?$CF3i?3?$CFi?$CFi?5?$AA@ 2006c12c     g_main.obj
 0002:00005138       ??_C@_0CE@CGGOAMCD@score?3?5?$CFi?5?5ping?3?5?$CFi?5?5client?3?5?$CFi?5@ 2006c138     g_main.obj
 0002:0000515c       ??_C@_0BB@HEGEAGAN@red?3?$CFi?5?5blue?3?$CFi?6?$AA@ 2006c15c     g_main.obj
 0002:00005170       ??_C@_09KHIKBPEI@Exit?3?5?$CFs?6?$AA@ 2006c170     g_main.obj
 0002:0000517c       ??_C@_0CE@BHHEOIMM@print?5?$CCBlue?5hit?5the?5capturelimit@ 2006c17c     g_main.obj
 0002:000051a0       ??_C@_0BC@NGNDEIFJ@Capturelimit?5hit?4?$AA@ 2006c1a0     g_main.obj
 0002:000051b4       ??_C@_0CD@JENHKKNP@print?5?$CCRed?5hit?5the?5capturelimit?4@ 2006c1b4     g_main.obj
 0002:000051d8       ??_C@_0CB@FMCEIKLA@print?5?$CC?$CFs?$FO7?5hit?5the?5fraglimit?4?6?$CC@ 2006c1d8     g_main.obj
 0002:000051fc       ??_C@_0CB@OIEPEJAM@print?5?$CCBlue?5hit?5the?5fraglimit?4?6?$CC@ 2006c1fc     g_main.obj
 0002:00005220       ??_C@_0P@PJCPOIKO@Fraglimit?5hit?4?$AA@ 2006c220     g_main.obj
 0002:00005230       ??_C@_0CA@KPFPAKGG@print?5?$CCRed?5hit?5the?5fraglimit?4?6?$CC?$AA@ 2006c230     g_main.obj
 0002:00005250       ??_C@_0P@EKMAOGJF@Timelimit?5hit?4?$AA@ 2006c250     g_main.obj
 0002:00005260       ??_C@_0BI@GKJLDCNN@print?5?$CCTimelimit?5hit?4?6?$CC?$AA@ 2006c260     g_main.obj
 0002:00005278       ??_C@_08FFAHPNKC@Warmup?3?6?$AA@ 2006c278     g_main.obj
 0002:00005284       ??_C@_0BG@ICALOBOM@print?5?$CCVote?5passed?4?6?$CC?$AA@ 2006c284     g_main.obj
 0002:0000529c       ??_C@_0BG@NEFGNBIH@print?5?$CCVote?5failed?4?6?$CC?$AA@ 2006c29c     g_main.obj
 0002:000052b4       ??_C@_0CD@EKLBBMMK@print?5?$CC?$CFs?5is?5the?5new?5team?5leader@ 2006c2b4     g_main.obj
 0002:000052d8       ??_C@_0CH@IFAGPGDJ@print?5?$CC?$CFs?5is?5not?5on?5the?5team?5any@ 2006c2d8     g_main.obj
 0002:00005300       ??_C@_0BN@PMDPLBOA@print?5?$CC?$CFs?5is?5not?5connected?6?$CC?$AA@ 2006c300     g_main.obj
 0002:00005320       ??_C@_0BL@KCNKNMK@print?5?$CCTeam?5vote?5passed?4?6?$CC?$AA@ 2006c320     g_main.obj
 0002:0000533c       ??_C@_0BL@FMHAJNKB@print?5?$CCTeam?5vote?5failed?4?6?$CC?$AA@ 2006c33c     g_main.obj
 0002:00005358       ??_C@_0BA@JGLONBEK@NULL?5ent?9?$DOthink?$AA@ 2006c358     g_main.obj
 0002:00005368       ??_C@_08JBKNBCEM@?$CF4i?3?5?$CFs?6?$AA@ 2006c368     g_main.obj
 0002:00005374       ??_C@_0CL@HPAAECKJ@G_Alloc?3?5failed?5on?5allocation?5of@ 2006c374     g_mem.obj
 0002:000053a0       ??_C@_0BP@CMDJHEKJ@G_Alloc?5of?5?$CFi?5bytes?5?$CI?$CFi?5left?$CJ?6?$AA@ 2006c3a0     g_mem.obj
 0002:000053c0       ??_C@_0DC@GFNDCLPP@Game?5memory?5status?3?5?$CFi?5out?5of?5?$CFi@ 2006c3c0     g_mem.obj
 0002:000053f4       ??_C@_0CO@BGNILIGB@Couldn?8t?5find?5target?5for?5misc_pa@ 2006c3f4     g_misc.obj
 0002:00005424       ??_C@_04FBAPEKPH@roll?$AA@ 2006c424     g_misc.obj
 0002:00005430       __real@3fe4cccccccccccd    2006c430     g_missile.obj
 0002:00005438       ??_C@_04DGFIONEK@hook?$AA@ 2006c438     g_missile.obj
 0002:00005440       __real@44fa0000            2006c440     g_missile.obj
 0002:00005444       ??_C@_06BAPMGMJB@plasma?$AA@ 2006c444     g_missile.obj
 0002:0000544c       __real@442f0000            2006c44c     g_missile.obj
 0002:00005450       ??_C@_07JBPBHDIL@grenade?$AA@ 2006c450     g_missile.obj
 0002:00005458       ??_C@_03CJHCFFJJ@bfg?$AA@  2006c458     g_missile.obj
 0002:0000545c       __real@44610000            2006c45c     g_missile.obj
 0002:00005460       ??_C@_06NHDMJEKK@rocket?$AA@ 2006c460     g_missile.obj
 0002:00005468       ??_C@_0CC@FGLHJPEN@pushed_p?5?$DO?5?$CGpushed?$FLMAX_GENTITIES@ 2006c468     g_mover.obj
 0002:00005490       __real@3fc0000000000000    2006c490     g_mover.obj
 0002:00005498       ??_C@_0CE@HFNOCNBN@Reached_BinaryMover?3?5bad?5moverSt@ 2006c498     g_mover.obj
 0002:000054bc       ??_C@_05PEENBMOG@color?$AA@ 2006c4bc     g_mover.obj
 0002:000054c4       ??_C@_05PGFNHLMG@1?51?51?$AA@ 2006c4c4     g_mover.obj
 0002:000054cc       ??_C@_05OEPGNJB@light?$AA@ 2006c4cc     g_mover.obj
 0002:000054d4       ??_C@_05GPLCCBII@noise?$AA@ 2006c4d4     g_mover.obj
 0002:000054dc       ??_C@_0N@FKJMDFJC@door_trigger?$AA@ 2006c4dc     g_mover.obj
 0002:000054ec       ??_C@_03EMOFKE@dmg?$AA@    2006c4ec     g_mover.obj
 0002:000054f0       ??_C@_0BP@MPMCKOBA@sound?1movers?1doors?1dr1_end?4wav?$AA@ 2006c4f0     g_mover.obj
 0002:00005510       ??_C@_0CA@KGLPIIML@sound?1movers?1doors?1dr1_strt?4wav?$AA@ 2006c510     g_mover.obj
 0002:00005530       __real@42040000            2006c530     g_mover.obj
 0002:00005534       ??_C@_0N@GNEHAGP@plat_trigger?$AA@ 2006c534     g_mover.obj
 0002:00005544       ??_C@_06LNLHEAAG@height?$AA@ 2006c544     g_mover.obj
 0002:0000554c       ??_C@_05HJCMGBKF@speed?$AA@ 2006c54c     g_mover.obj
 0002:00005554       ??_C@_0BP@FMIAEABD@sound?1movers?1plats?1pt1_end?4wav?$AA@ 2006c554     g_mover.obj
 0002:00005574       ??_C@_0CA@DPCFJLJP@sound?1movers?1plats?1pt1_strt?4wav?$AA@ 2006c574     g_mover.obj
 0002:00005594       ??_C@_0CA@HPFJMDOC@sound?1movers?1switches?1butn2?4wav?$AA@ 2006c594     g_mover.obj
 0002:000055b4       ??_C@_0M@ONCHNMHP@path_corner?$AA@ 2006c5b4     g_mover.obj
 0002:000055c0       ??_C@_0DB@KEBMPPOD@Train?5corner?5at?5?$CFs?5without?5a?5tar@ 2006c5c0     g_mover.obj
 0002:000055f4       ??_C@_0CF@EGOCJBJB@Train?5corner?5at?5?$CFs?5without?5a?5tar@ 2006c5f4     g_mover.obj
 0002:0000561c       ??_C@_0CJ@BMOHOFCP@func_train?5at?5?$CFs?5with?5an?5unfound@ 2006c61c     g_mover.obj
 0002:00005648       ??_C@_0CG@DHHNMBFP@path_corner?5with?5no?5targetname?5a@ 2006c648     g_mover.obj
 0002:00005670       ??_C@_0CD@BNKPEMCB@func_train?5without?5a?5target?5at?5?$CF@ 2006c670     g_mover.obj
 0002:00005694       ??_C@_05CBPKLGJM@phase?$AA@ 2006c694     g_mover.obj
 0002:0000569c       ??_C@_02MLODCJFF@32?$AA@   2006c69c     g_mover.obj
 0002:000056a0       __real@3fc45f306446f9b4    2006c6a0     g_mover.obj
 0002:000056a8       ??_C@_09INHJFLOH@session?$CFi?$AA@ 2006c6a8     g_session.obj
 0002:000056b4       ??_C@_0BF@GKKABID@?$CFi?5?$CFi?5?$CFi?5?$CFi?5?$CFi?5?$CFi?5?$CFi?$AA@ 2006c6b4     g_session.obj
 0002:000056cc       ??_C@_0CK@FAAHDCAM@Gametype?5changed?0?5clearing?5sessi@ 2006c6cc     g_session.obj
 0002:000056f8       ??_C@_07KMJDECGK@session?$AA@ 2006c6f8     g_session.obj
 0002:00005700       ??_C@_0P@IPNNKHAH@teamtournament?$AA@ 2006c700     g_spawn.obj
 0002:00005710       ??_C@_09KFJDBEJE@harvester?$AA@ 2006c710     g_spawn.obj
 0002:0000571c       ??_C@_07BNFEBHAE@obelisk?$AA@ 2006c71c     g_spawn.obj
 0002:00005724       ??_C@_07BEINKNPB@oneflag?$AA@ 2006c724     g_spawn.obj
 0002:0000572c       ??_C@_03JHHHHEKD@ctf?$AA@  2006c72c     g_spawn.obj
 0002:00005730       ??_C@_06EJFMBPJF@single?$AA@ 2006c730     g_spawn.obj
 0002:00005738       ??_C@_0L@NCEPCFLK@tournament?$AA@ 2006c738     g_spawn.obj
 0002:00005744       ??_C@_03PAEKGFEI@ffa?$AA@  2006c744     g_spawn.obj
 0002:00005748       ??_C@_0N@PAECNMEH@item_botroam?$AA@ 2006c748     g_spawn.obj
 0002:00005758       ??_C@_0BD@GGIPJOIB@team_CTF_bluespawn?$AA@ 2006c758     g_spawn.obj
 0002:0000576c       ??_C@_0BC@KIKIBEND@team_CTF_redspawn?$AA@ 2006c76c     g_spawn.obj
 0002:00005780       ??_C@_0BE@COKGGHPD@team_CTF_blueplayer?$AA@ 2006c780     g_spawn.obj
 0002:00005794       ??_C@_0BD@KLANHAKB@team_CTF_redplayer?$AA@ 2006c794     g_spawn.obj
 0002:000057a8       ??_C@_0P@KKMFIJKM@shooter_plasma?$AA@ 2006c7a8     g_spawn.obj
 0002:000057b8       ??_C@_0BA@MJCDAGHP@shooter_grenade?$AA@ 2006c7b8     g_spawn.obj
 0002:000057c8       ??_C@_0P@GNAFHBJH@shooter_rocket?$AA@ 2006c7c8     g_spawn.obj
 0002:000057d8       ??_C@_0BD@OJADMBDB@misc_portal_camera?$AA@ 2006c7d8     g_spawn.obj
 0002:000057ec       ??_C@_0BE@FCJPPDGO@misc_portal_surface?$AA@ 2006c7ec     g_spawn.obj
 0002:00005800       ??_C@_0L@PMAFMKKM@misc_model?$AA@ 2006c800     g_spawn.obj
 0002:0000580c       ??_C@_0BF@OMPOACGH@misc_teleporter_dest?$AA@ 2006c80c     g_spawn.obj
 0002:00005824       ??_C@_0M@NLNGBECJ@target_push?$AA@ 2006c824     g_spawn.obj
 0002:00005830       ??_C@_0BA@BFKBOHOP@target_location?$AA@ 2006c830     g_spawn.obj
 0002:00005840       ??_C@_0BA@NENIEICJ@target_position?$AA@ 2006c840     g_spawn.obj
 0002:00005850       ??_C@_0M@KFDPHLNE@target_kill?$AA@ 2006c850     g_spawn.obj
 0002:0000585c       ??_C@_0BC@GJLLMIEM@target_teleporter?$AA@ 2006c85c     g_spawn.obj
 0002:00005870       ??_C@_0N@DIKJAPJH@target_score?$AA@ 2006c870     g_spawn.obj
 0002:00005880       ??_C@_0N@LGMMDFPN@target_laser?$AA@ 2006c880     g_spawn.obj
 0002:00005890       ??_C@_0N@IADDOFND@target_print?$AA@ 2006c890     g_spawn.obj
 0002:000058a0       ??_C@_0P@MNJIBEAO@target_speaker?$AA@ 2006c8a0     g_spawn.obj
 0002:000058b0       ??_C@_0BH@FJADHEOA@target_remove_powerups?$AA@ 2006c8b0     g_spawn.obj
 0002:000058c8       ??_C@_0M@KALMALDK@target_give?$AA@ 2006c8c8     g_spawn.obj
 0002:000058d4       ??_C@_0N@JFLGFCMM@trigger_hurt?$AA@ 2006c8d4     g_spawn.obj
 0002:000058e4       ??_C@_0BB@COMMHECA@trigger_teleport?$AA@ 2006c8e4     g_spawn.obj
 0002:000058f8       ??_C@_0N@CCJDLJOF@trigger_push?$AA@ 2006c8f8     g_spawn.obj
 0002:00005908       ??_C@_0P@KDHOHKJL@trigger_always?$AA@ 2006c908     g_spawn.obj
 0002:00005918       ??_C@_0L@KLICIANB@func_group?$AA@ 2006c918     g_spawn.obj
 0002:00005924       ??_C@_0L@PGCOCBM@func_train?$AA@ 2006c924     g_spawn.obj
 0002:00005930       ??_C@_0O@FPCFJAHB@func_pendulum?$AA@ 2006c930     g_spawn.obj
 0002:00005940       ??_C@_0N@BAMIHEIF@func_bobbing?$AA@ 2006c940     g_spawn.obj
 0002:00005950       ??_C@_0O@JDFCILJF@func_rotating?$AA@ 2006c950     g_spawn.obj
 0002:00005960       ??_C@_0M@OOBMECJN@func_static?$AA@ 2006c960     g_spawn.obj
 0002:0000596c       ??_C@_09HCDLIOGG@func_plat?$AA@ 2006c96c     g_spawn.obj
 0002:00005978       ??_C@_09BLMHBGJ@info_camp?$AA@ 2006c978     g_spawn.obj
 0002:00005984       ??_C@_0N@FHKCBFMD@info_notnull?$AA@ 2006c984     g_spawn.obj
 0002:00005994       ??_C@_09MBOCECHK@info_null?$AA@ 2006c994     g_spawn.obj
 0002:000059a0       ??_C@_0BC@IHPKIKNE@info_player_start?$AA@ 2006c9a0     g_spawn.obj
 0002:000059b4       ??_C@_0BE@OHABMMFD@targetShaderNewName?$AA@ 2006c9b4     g_spawn.obj
 0002:000059c8       ??_C@_0BB@FKLCNMKK@targetShaderName?$AA@ 2006c9c8     g_spawn.obj
 0002:000059dc       ??_C@_06GNEAMJOC@angles?$AA@ 2006c9dc     g_spawn.obj
 0002:000059e4       ??_C@_05IOMEMJEC@count?$AA@ 2006c9e4     g_spawn.obj
 0002:000059ec       ??_C@_07ONPBMBOP@message?$AA@ 2006c9ec     g_spawn.obj
 0002:000059f4       ??_C@_06LNKHAAKC@model2?$AA@ 2006c9f4     g_spawn.obj
 0002:000059fc       ??_C@_0CC@JNJOINHG@?$CFs?5doesn?8t?5have?5a?5spawn?5function@ 2006c9fc     g_spawn.obj
 0002:00005a20       ??_C@_0BN@EMEGOFNC@G_CallSpawn?3?5NULL?5classname?6?$AA@ 2006ca20     g_spawn.obj
 0002:00005a40       ??_C@_08NJPDEKHO@gametype?$AA@ 2006ca40     g_spawn.obj
 0002:00005a4c       ??_C@_06MFKCCKGP@notq3a?$AA@ 2006ca4c     g_spawn.obj
 0002:00005a54       ??_C@_07DDCDJNBH@notfree?$AA@ 2006ca54     g_spawn.obj
 0002:00005a5c       ??_C@_07CLBNBEAH@notteam?$AA@ 2006ca5c     g_spawn.obj
 0002:00005a64       ??_C@_09FDFEENEB@notsingle?$AA@ 2006ca64     g_spawn.obj
 0002:00005a70       ??_C@_0CE@JHGDANIP@G_AddSpawnVarToken?3?5MAX_SPAWN_CH@ 2006ca70     g_spawn.obj
 0002:00005a94       ??_C@_0CB@JFPBODJK@G_ParseSpawnVars?3?5MAX_SPAWN_VARS@ 2006ca94     g_spawn.obj
 0002:00005ab8       ??_C@_0CN@NMMGIHBC@G_ParseSpawnVars?3?5closing?5brace?5@ 2006cab8     g_spawn.obj
 0002:00005ae8       ??_C@_0CM@DONEEOIH@G_ParseSpawnVars?3?5EOF?5without?5cl@ 2006cae8     g_spawn.obj
 0002:00005b14       ??_C@_0CM@CKLLJIGA@G_ParseSpawnVars?3?5found?5?$CFs?5when?5@ 2006cb14     g_spawn.obj
 0002:00005b40       ??_C@_0P@INMNNPOJ@g_enableBreath?$AA@ 2006cb40     g_spawn.obj
 0002:00005b50       ??_C@_0N@PNMKKPBO@enableBreath?$AA@ 2006cb50     g_spawn.obj
 0002:00005b60       ??_C@_0N@CMGOADK@g_enableDust?$AA@ 2006cb60     g_spawn.obj
 0002:00005b70       ??_C@_0L@FLFKAOCP@enableDust?$AA@ 2006cb70     g_spawn.obj
 0002:00005b7c       ??_C@_07GFBFDLBM@gravity?$AA@ 2006cb7c     g_spawn.obj
 0002:00005b84       ??_C@_05LLDJOKNO@music?$AA@ 2006cb84     g_spawn.obj
 0002:00005b8c       ??_C@_08CCHPPKDI@baseq3?91?$AA@ 2006cb8c     g_spawn.obj
 0002:00005b98       ??_C@_0DD@EBBCPGHA@SP_worldspawn?3?5The?5first?5entity?5@ 2006cb98     g_spawn.obj
 0002:00005bcc       ??_C@_0L@BIFLFHPF@worldspawn?$AA@ 2006cbcc     g_spawn.obj
 0002:00005bd8       ??_C@_0BL@HLOLFMOK@SpawnEntities?3?5no?5entities?$AA@ 2006cbd8     g_spawn.obj
 0002:00005bf4       ??_C@_0BI@LMFPAHLD@IP?5filter?5list?5is?5full?6?$AA@ 2006cbf4     g_svcmds.obj
 0002:00005c0c       ??_C@_0BI@DIECJMKD@Bad?5filter?5address?3?5?$CFs?6?$AA@ 2006cc0c     g_svcmds.obj
 0002:00005c24       ??_C@_0CO@DILFDDOI@g_banIPs?5overflowed?5at?5MAX_CVAR_@ 2006cc24     g_svcmds.obj
 0002:00005c54       ??_C@_01LFCBOECM@?4?$AA@   2006cc54     g_svcmds.obj
 0002:00005c58       ??_C@_01NBENCBCI@?$CK?$AA@ 2006cc58     g_svcmds.obj
 0002:00005c5c       ??_C@_0BJ@LEBLJMPE@Usage?3?5?5addip?5?$DMip?9mask?$DO?6?$AA@ 2006cc5c     g_svcmds.obj
 0002:00005c78       ??_C@_0BB@DFCHPNBP@Didn?8t?5find?5?$CFs?4?6?$AA@ 2006cc78     g_svcmds.obj
 0002:00005c8c       ??_C@_09HBKBHJKE@Removed?4?6?$AA@ 2006cc8c     g_svcmds.obj
 0002:00005c98       ??_C@_0BP@OJMGJOKB@Usage?3?5?5sv?5removeip?5?$DMip?9mask?$DO?6?$AA@ 2006cc98     g_svcmds.obj
 0002:00005cb8       ??_C@_01EEMJAFIK@?6?$AA@   2006ccb8     g_svcmds.obj
 0002:00005cbc       ??_C@_0BF@HIBFLMFA@?$CF3i?5?5?5?5?5?5?5?5?5?5?5?5?5?5?5?5?5?$AA@ 2006ccbc     g_svcmds.obj
 0002:00005cd4       ??_C@_0BF@JEKJFFDI@ET_GRAPPLE?5?5?5?5?5?5?5?5?5?5?$AA@ 2006ccd4     g_svcmds.obj
 0002:00005cec       ??_C@_0BF@FONFEMNK@ET_INVISIBLE?5?5?5?5?5?5?5?5?$AA@ 2006ccec     g_svcmds.obj
 0002:00005d04       ??_C@_0BF@KNGJOHIC@ET_TELEPORT_TRIGGER?5?$AA@ 2006cd04     g_svcmds.obj
 0002:00005d1c       ??_C@_0BF@JCJGMGAM@ET_PUSH_TRIGGER?5?5?5?5?5?$AA@ 2006cd1c     g_svcmds.obj
 0002:00005d34       ??_C@_0BF@JKKJEPNL@ET_SPEAKER?5?5?5?5?5?5?5?5?5?5?$AA@ 2006cd34     g_svcmds.obj
 0002:00005d4c       ??_C@_0BF@FABEBACG@ET_PORTAL?5?5?5?5?5?5?5?5?5?5?5?$AA@ 2006cd4c     g_svcmds.obj
 0002:00005d64       ??_C@_0BF@DBCLPHFC@ET_BEAM?5?5?5?5?5?5?5?5?5?5?5?5?5?$AA@ 2006cd64     g_svcmds.obj
 0002:00005d7c       ??_C@_0BF@CKCOPBOH@ET_MOVER?5?5?5?5?5?5?5?5?5?5?5?5?$AA@ 2006cd7c     g_svcmds.obj
 0002:00005d94       ??_C@_0BF@JMOJKPHI@ET_MISSILE?5?5?5?5?5?5?5?5?5?5?$AA@ 2006cd94     g_svcmds.obj
 0002:00005dac       ??_C@_0BF@IIDKJKIF@ET_ITEM?5?5?5?5?5?5?5?5?5?5?5?5?5?$AA@ 2006cdac     g_svcmds.obj
 0002:00005dc4       ??_C@_0BF@GHCCJGLD@ET_PLAYER?5?5?5?5?5?5?5?5?5?5?5?$AA@ 2006cdc4     g_svcmds.obj
 0002:00005ddc       ??_C@_0BF@GBIOGILC@ET_GENERAL?5?5?5?5?5?5?5?5?5?5?$AA@ 2006cddc     g_svcmds.obj
 0002:00005df4       ??_C@_04LAMNNBAP@?$CF3i?3?$AA@ 2006cdf4     g_svcmds.obj
 0002:00005dfc       ??_C@_0BO@DPIFHGAP@User?5?$CFs?5is?5not?5on?5the?5server?6?$AA@ 2006cdfc     g_svcmds.obj
 0002:00005e1c       ??_C@_0BM@KMBENOOM@Client?5?$CFi?5is?5not?5connected?6?$AA@ 2006ce1c     g_svcmds.obj
 0002:00005e38       ??_C@_0BF@BEBENGBA@Bad?5client?5slot?3?5?$CFi?6?$AA@ 2006ce38     g_svcmds.obj
 0002:00005e50       ??_C@_0BD@OKBENEII@print?5?$CCserver?3?5?$CFs?$CC?$AA@ 2006ce50     g_svcmds.obj
 0002:00005e64       ??_C@_09DNOCIDID@g_banIPs?6?$AA@ 2006ce64     g_svcmds.obj
 0002:00005e70       ??_C@_06DDGIHMAP@listip?$AA@ 2006ce70     g_svcmds.obj
 0002:00005e78       ??_C@_08FODIKFHA@removeip?$AA@ 2006ce78     g_svcmds.obj
 0002:00005e84       ??_C@_05DNFKLKCD@addip?$AA@ 2006ce84     g_svcmds.obj
 0002:00005e8c       ??_C@_0N@EKGBLHCI@abort_podium?$AA@ 2006ce8c     g_svcmds.obj
 0002:00005e9c       ??_C@_07OCFGLMLF@botlist?$AA@ 2006ce9c     g_svcmds.obj
 0002:00005ea4       ??_C@_06CJHCPEHG@addbot?$AA@ 2006cea4     g_svcmds.obj
 0002:00005eac       ??_C@_0M@OOGGMGEK@game_memory?$AA@ 2006ceac     g_svcmds.obj
 0002:00005eb8       ??_C@_09NGKIAGHE@forceteam?$AA@ 2006ceb8     g_svcmds.obj
 0002:00005ec4       ??_C@_0L@CLDMIJOM@entitylist?$AA@ 2006cec4     g_svcmds.obj
 0002:00005ed0       ??_C@_05EKJCMADO@delay?$AA@ 2006ced0     g_target.obj
 0002:00005ed8       ??_C@_07PCJFOBJC@cp?5?$CC?$CFs?$CC?$AA@ 2006ced8     g_target.obj
 0002:00005ee0       ??_C@_06MKMJDPPC@?$CFs?4wav?$AA@ 2006cee0     g_target.obj
 0002:00005ee8       ??_C@_04IBLEHOMF@?4wav?$AA@ 2006cee8     g_target.obj
 0002:00005ef0       ??_C@_0CJ@MCNLAIAG@target_speaker?5without?5a?5noise?5k@ 2006cef0     g_target.obj
 0002:00005f1c       ??_C@_07FGPCJFED@NOSOUND?$AA@ 2006cf1c     g_target.obj
 0002:00005f24       __real@45000000            2006cf24     g_target.obj
 0002:00005f28       ??_C@_0BO@JBAPADMO@?$CFs?5at?5?$CFs?3?5?$CFs?5is?5a?5bad?5target?6?$AA@ 2006cf28     g_target.obj
 0002:00005f48       ??_C@_0CG@NCOEMBAJ@Couldn?8t?5find?5teleporter?5destina@ 2006cf48     g_target.obj
 0002:00005f70       ??_C@_0BF@CCKDOAMJ@untargeted?5?$CFs?5at?5?$CFs?6?$AA@ 2006cf70     g_target.obj
 0002:00005f88       ??_C@_07CIFAGBMG@unknown?$AA@ 2006cf88     g_target.obj
 0002:00005f90       ??_C@_04HEDFJGEJ@FREE?$AA@ 2006cf90     g_team.obj
 0002:00005f98       ??_C@_09GNDCBOBP@SPECTATOR?$AA@ 2006cf98     g_team.obj
 0002:00005fa4       ??_C@_04CNFFLDFF@BLUE?$AA@ 2006cfa4     g_team.obj
 0002:00005fac       ??_C@_03FNPLCCOA@RED?$AA@  2006cfac     g_team.obj
 0002:00005fb0       ??_C@_02PGJLIFGD@?$FO7?$AA@ 2006cfb0     g_team.obj
 0002:00005fb4       ??_C@_02JCPHEAGH@?$FO3?$AA@ 2006cfb4     g_team.obj
 0002:00005fb8       ??_C@_02NNLGNGKA@?$FO4?$AA@ 2006cfb8     g_team.obj
 0002:00005fbc       ??_C@_02KAMBCCOF@?$FO1?$AA@ 2006cfbc     g_team.obj
 0002:00005fc0       ??_C@_0BB@GAGKBLAF@PrintMsg?5overrun?$AA@ 2006cfc0     g_team.obj
 0002:00005fd4       __real@45fa0000            2006cfd4     g_team.obj
 0002:00005fd8       ??_C@_0CC@MJFJLHGN@?$CFs?$FO7?5fragged?5?$CFs?8s?5skull?5carrier?$CB@ 2006cfd8     g_team.obj
 0002:00005ffc       ??_C@_0CB@KOPONFBB@?$CFs?$FO7?5fragged?5?$CFs?8s?5flag?5carrier?$CB?6@ 2006cffc     g_team.obj
 0002:00006020       ??_C@_0BF@NFGOPKAE@team_CTF_neutralflag?$AA@ 2006d020     g_team.obj
 0002:00006038       ??_C@_0CP@OBNDLAL@Warning?3?5?5NULL?5passed?5to?5Team_Re@ 2006d038     g_team.obj
 0002:00006068       ??_C@_0CN@EPFNCNCH@Warning?3?5?5NULL?5passed?5to?5Team_Ta@ 2006d068     g_team.obj
 0002:00006098       ??_C@_0DA@ICMFPMGB@Warning?3?5?5NULL?5passed?5to?5Team_Ca@ 2006d098     g_team.obj
 0002:000060c8       ??_C@_0BL@EJNDMGGL@The?5?$CFs?5flag?5has?5returned?$CB?6?$AA@ 2006d0c8     g_team.obj
 0002:000060e4       ??_C@_0BI@KNNACEDO@The?5flag?5has?5returned?$CB?6?$AA@ 2006d0e4     g_team.obj
 0002:000060fc       ??_C@_0BM@NKAOENPK@?$CFs?$FO7?5captured?5the?5?$CFs?5flag?$CB?6?$AA@ 2006d0fc     g_team.obj
 0002:00006118       ??_C@_0BM@BDFECDMG@?$CFs?$FO7?5returned?5the?5?$CFs?5flag?$CB?6?$AA@ 2006d118     g_team.obj
 0002:00006134       ??_C@_0BH@PJAKMCBO@?$CFs?$FO7?5got?5the?5?$CFs?5flag?$CB?6?$AA@ 2006d134     g_team.obj
 0002:0000614c       ??_C@_0CG@PMIHGLOD@Don?8t?5know?5what?5team?5the?5flag?5is@ 2006d14c     g_team.obj
 0002:00006174       ??_C@_08BKJPOMKC@?$CFc?$CFc?$CFs?$FO7?$AA@ 2006d174     g_team.obj
 0002:00006180       ??_C@_0M@PHDLOMHJ@tinfo?5?$CFi?5?$CFs?$AA@ 2006d180     g_team.obj
 0002:0000618c       ??_C@_0BD@FAPFLCHD@?5?$CFi?5?$CFi?5?$CFi?5?$CFi?5?$CFi?5?$CFi?$AA@ 2006d18c     g_team.obj
 0002:000061a0       ??_C@_0CF@LENMBBGI@trigger_multiple?5has?5random?5?$DO?$DN?5w@ 2006d1a0     g_trigger.obj
 0002:000061c8       ??_C@_03LOHCHBBO@0?45?$AA@ 2006d1c8     g_trigger.obj
 0002:000061cc       ??_C@_0BI@DGLBHPLI@sound?1world?1jumppad?4wav?$AA@ 2006d1cc     g_trigger.obj
 0002:000061e4       ??_C@_0BH@FEKNGHLG@sound?1misc?1windfly?4wav?$AA@ 2006d1e4     g_trigger.obj
 0002:000061fc       ??_C@_0BI@KPLPFMKN@sound?1world?1electro?4wav?$AA@ 2006d1fc     g_trigger.obj
 0002:00006214       ??_C@_0CF@GJKCPHON@func_timer?5at?5?$CFs?5has?5random?5?$DO?$DN?5w@ 2006d214     g_trigger.obj
 0002:0000623c       ??_C@_0N@MLGFLFEI@?$CFs?$DN?$CFs?3?$CF5?42f?$EA?$AA@ 2006d23c     g_utils.obj
 0002:0000624c       ??_C@_0CC@KBENIHEG@G_FindConfigstringIndex?3?5overflo@ 2006d24c     g_utils.obj
 0002:00006270       ??_C@_0CD@HHFHMIIH@G_PickTarget?3?5target?5?$CFs?5not?5foun@ 2006d270     g_utils.obj
 0002:00006294       ??_C@_0CK@JOENGKNM@G_PickTarget?5called?5with?5NULL?5ta@ 2006d294     g_utils.obj
 0002:000062c0       ??_C@_0CI@HMPHOHE@entity?5was?5removed?5while?5using?5t@ 2006d2c0     g_utils.obj
 0002:000062e8       ??_C@_0BO@JIDGNOMJ@WARNING?3?5Entity?5used?5itself?4?6?$AA@ 2006d2e8     g_utils.obj
 0002:00006308       ??_C@_0L@OPPGOKFJ@?$CI?$CFi?5?$CFi?5?$CFi?$CJ?$AA@ 2006d308     g_utils.obj
 0002:00006318       __real@400921fb60000000    2006d318     g_utils.obj
 0002:00006320       ??_C@_07CBNPCFPB@noclass?$AA@ 2006d320     g_utils.obj
 0002:00006328       ??_C@_0BK@OECJBIJE@G_Spawn?3?5no?5free?5entities?$AA@ 2006d328     g_utils.obj
 0002:00006344       ??_C@_05FAPHKBON@freed?$AA@ 2006d344     g_utils.obj
 0002:0000634c       ??_C@_0L@CPIFJPHE@tempEntity?$AA@ 2006d34c     g_utils.obj
 0002:00006358       ??_C@_0CM@MOJHPIKM@G_AddEvent?3?5zero?5event?5added?5for@ 2006d358     g_utils.obj
 0002:00006388       __real@bfefae147ae147ae    2006d388     g_utils.obj
 0002:00006390       __real@46000000            2006d390     g_weapon.obj
 0002:00006394       __real@48000000            2006d394     g_weapon.obj
 0002:00006398       __real@4030000000000000    2006d398     g_weapon.obj
 0002:000063a0       __real@3e4ccccd            2006d3a0     g_weapon.obj
 0002:000063a4       __real@44400000            2006d3a4     g_weapon.obj
 0002:000063a8       __real@41600000            2006d3a8     g_weapon.obj
 0002:000063ac       ??_C@_0BK@JDDBNDOP@Q_fabs?$CIinv_denom?$CJ?5?$CB?$DN?50?40f?$AA@ 2006d3ac     q_math.obj
 0002:000063c8       ??_C@_0DD@HJOIBKLP@d?3?2distr?2games_src?2quake3?91?432b?2@ 2006d3c8     q_math.obj
 0002:000063fc       __real@3f000000            2006d3fc     q_math.obj
 0002:00006400       __real@4066c16c16c16c17    2006d400     q_math.obj
 0002:00006408       __real@3c8efa35            2006d408     q_math.obj
 0002:0000640c       ??_C@_04HDOCAJNK@?$CFs?$CFs?$AA@ 2006d40c     q_shared.obj
 0002:00006414       ??_C@_0BI@KPLEBEJF@ERROR?3?5?$CFs?0?5line?5?$CFd?3?5?$CFs?6?$AA@ 2006d414     q_shared.obj
 0002:0000642c       ??_C@_0BK@DJMKDJBL@WARNING?3?5?$CFs?0?5line?5?$CFd?3?5?$CFs?6?$AA@ 2006d42c     q_shared.obj
 0002:00006448       ??_C@_0BF@BFEJCABG@MatchToken?3?5?$CFs?5?$CB?$DN?5?$CFs?$AA@ 2006d448     q_shared.obj
 0002:00006460       ??_C@_01PKGAHCOL@?$CJ?$AA@ 2006d460     q_shared.obj
 0002:00006464       ??_C@_01ODHLEDKK@?$CI?$AA@ 2006d464     q_shared.obj
 0002:00006468       ??_C@_0BJ@OLBOPICM@Q_strncpyz?3?5destsize?5?$DM?51?$AA@ 2006d468     q_shared.obj
 0002:00006484       ??_C@_0BF@BJHHBLMD@Q_strncpyz?3?5NULL?5src?$AA@ 2006d484     q_shared.obj
 0002:0000649c       ??_C@_0BG@EKAPNPCH@Q_strncpyz?3?5NULL?5dest?$AA@ 2006d49c     q_shared.obj
 0002:000064b4       ??_C@_0BN@EFOOAHFL@Q_strcat?3?5already?5overflowed?$AA@ 2006d4b4     q_shared.obj
 0002:000064d4       ??_C@_0CD@GIPJKOOD@Com_sprintf?3?5overflow?5of?5?$CFi?5in?5?$CF@ 2006d4d4     q_shared.obj
 0002:000064f8       ??_C@_0CC@GMEFDOKA@Com_sprintf?3?5overflowed?5bigbuffe@ 2006d4f8     q_shared.obj
 0002:0000651c       ??_C@_0CG@FLHABLN@Info_ValueForKey?3?5oversize?5infos@ 2006d51c     q_shared.obj
 0002:00006544       ??_C@_0CE@HMPLGKDK@Info_RemoveKey?3?5oversize?5infostr@ 2006d544     q_shared.obj
 0002:00006568       ??_C@_0CI@CPIEPBLO@Info_RemoveKey_Big?3?5oversize?5inf@ 2006d568     q_shared.obj
 0002:00006590       ??_C@_0BN@CAOBGKLE@Info?5string?5length?5exceeded?6?$AA@ 2006d590     q_shared.obj
 0002:000065b0       ??_C@_06NELKLDPM@?2?$CFs?2?$CFs?$AA@ 2006d5b0     q_shared.obj
 0002:000065b8       ??_C@_0CD@MGFMEBLE@Can?8t?5use?5keys?5or?5values?5with?5a?5@ 2006d5b8     q_shared.obj
 0002:000065dc       ??_C@_0CL@JCFAGLFD@Can?8t?5use?5keys?5or?5values?5with?5a?5@ 2006d5dc     q_shared.obj
 0002:00006608       ??_C@_0CD@JIDDAEOO@Can?8t?5use?5keys?5or?5values?5with?5a?5@ 2006d608     q_shared.obj
 0002:0000662c       ??_C@_0CJ@CEEBDGNA@Info_SetValueForKey?3?5oversize?5in@ 2006d62c     q_shared.obj
 0002:00006658       ??_C@_0CB@EMDOOGBI@BIG?5Info?5string?5length?5exceeded?6@ 2006d658     q_shared.obj
 0002:0000667c       ??_C@_0P@NHGFNCDP@format?5?$CB?$DN?5NULL?$AA@ 2006d67c     LIBCMTD:sscanf.obj
 0002:0000668c       ??_C@_08MPLNDKMI@sscanf?4c?$AA@ 2006d68c     LIBCMTD:sscanf.obj
 0002:00006698       ??_C@_0P@NFGNABCI@string?5?$CB?$DN?5NULL?$AA@ 2006d698     LIBCMTD:sscanf.obj
 0002:000066a8       ??_C@_0L@MDILGHEC@vsprintf?4c?$AA@ 2006d6a8     LIBCMTD:vsprintf.obj
 0002:00006708       ??_C@_02PHMGELLB@?6?6?$AA@ 2006d708     LIBCMTD:assert.obj
 0002:0000670c       ??_C@_03KHICJKCI@?4?4?4?$AA@ 2006d70c     LIBCMTD:assert.obj
 0002:00006710       ??_C@_0CF@GOGNBNAK@Microsoft?5Visual?5C?$CL?$CL?5Runtime?5Lib@ 2006d710     LIBCMTD:assert.obj
 0002:00006738       ??_C@_0DN@EBBNMLME@?$CIPress?5Retry?5to?5debug?5the?5applic@ 2006d738     LIBCMTD:assert.obj
 0002:00006778       ??_C@_0HA@OJHAGA@For?5information?5on?5how?5your?5prog@ 2006d778     LIBCMTD:assert.obj
 0002:000067e8       ??_C@_0N@MEECIJGN@Expression?3?5?$AA@ 2006d7e8     LIBCMTD:assert.obj
 0002:000067f8       ??_C@_06FIEBOLOH@Line?3?5?$AA@ 2006d7f8     LIBCMTD:assert.obj
 0002:00006800       ??_C@_06IGPBOHMJ@File?3?5?$AA@ 2006d800     LIBCMTD:assert.obj
 0002:00006808       ??_C@_0BH@DNAGHKFM@?$DMprogram?5name?5unknown?$DO?$AA@ 2006d808     LIBCMTD:assert.obj
 0002:00006820       ??_C@_09KLGCKDOD@Program?3?5?$AA@ 2006d820     LIBCMTD:assert.obj
 0002:0000682c       ??_C@_0BC@LAIDCHCH@Assertion?5failed?$CB?$AA@ 2006d82c     LIBCMTD:assert.obj
 0002:00006840       ??_C@_09IFKEODFF@dllcrt0?4c?$AA@ 2006d840     LIBCMTD:dllcrt0.obj
 0002:0000685c       ??_C@_09BLOOPMDK@isctype?4c?$AA@ 2006d85c     LIBCMTD:isctype.obj
 0002:00006868       ??_C@_0BJ@IAKBGELC@?$CIunsigned?$CJ?$CIc?5?$CL?51?$CJ?5?$DM?$DN?5256?$AA@ 2006d868     LIBCMTD:isctype.obj
 0002:00006a08       ??_C@_07LCBHPJJN@LC_TIME?$AA@ 2006da08     LIBCMTD:setlocal.obj
 0002:00006a10       ??_C@_0L@DLHIECNL@LC_NUMERIC?$AA@ 2006da10     LIBCMTD:setlocal.obj
 0002:00006a1c       ??_C@_0M@MIENIKLA@LC_MONETARY?$AA@ 2006da1c     LIBCMTD:setlocal.obj
 0002:00006a28       ??_C@_08EADHIDAD@LC_CTYPE?$AA@ 2006da28     LIBCMTD:setlocal.obj
 0002:00006a34       ??_C@_0L@KFJHEKIK@LC_COLLATE?$AA@ 2006da34     LIBCMTD:setlocal.obj
 0002:00006a40       ??_C@_06NEFDFEKB@LC_ALL?$AA@ 2006da40     LIBCMTD:setlocal.obj
 0002:00006a54       ??_C@_0L@LEECJGMI@setlocal?4c?$AA@ 2006da54     LIBCMTD:setlocal.obj
 0002:00006a6c       ??_C@_01ICJEACDI@?$DL?$AA@ 2006da6c     LIBCMTD:setlocal.obj
 0002:00006a70       ??_C@_02BALPLPBG@?$DN?$DL?$AA@ 2006da70     LIBCMTD:setlocal.obj
 0002:00006a74       ??_C@_01NEMOKFLO@?$DN?$AA@ 2006da74     LIBCMTD:setlocal.obj
 0002:00006a78       ??_C@_03EGDHDPFD@_?4?0?$AA@ 2006da78     LIBCMTD:setlocal.obj
 0002:00006a7c       ??_C@_01IDAFKMJL@_?$AA@    2006da7c     LIBCMTD:setlocal.obj
 0002:00006a80       ??_C@_0L@JKCACIOJ@tidtable?4c?$AA@ 2006da80     LIBCMTD:tidtable.obj
 0002:00006a8c       ??_C@_07PEJMOBNF@FlsFree?$AA@ 2006da8c     LIBCMTD:tidtable.obj
 0002:00006a94       ??_C@_0M@JCPCPOEF@FlsSetValue?$AA@ 2006da94     LIBCMTD:tidtable.obj
 0002:00006aa0       ??_C@_0M@GDNOONDI@FlsGetValue?$AA@ 2006daa0     LIBCMTD:tidtable.obj
 0002:00006aac       ??_C@_08KNHFBNJ@FlsAlloc?$AA@ 2006daac     LIBCMTD:tidtable.obj
 0002:00006ab8       ??_C@_0N@MDJJJHMB@kernel32?4dll?$AA@ 2006dab8     LIBCMTD:tidtable.obj
 0002:00006ae0       __real@4150017ec0000000    2006dae0     LIBCMTD:testfdiv.obj
 0002:00006ae8       __real@4147ffff80000000    2006dae8     LIBCMTD:testfdiv.obj
 0002:00006af0       ??_C@_0BK@NHEOCAHP@IsProcessorFeaturePresent?$AA@ 2006daf0     LIBCMTD:testfdiv.obj
 0002:00006b0c       ??_C@_08CPNIBGIE@KERNEL32?$AA@ 2006db0c     LIBCMTD:testfdiv.obj
 0002:00006b18       ??_C@_05KLBDPFGC@e?$CL000?$AA@ 2006db18     LIBCMTD:cvt.obj
 0002:00006b20       ??_C@_0P@FELNCIKG@stream?5?$CB?$DN?5NULL?$AA@ 2006db20     LIBCMTD:input.obj
 0002:00006b30       ??_C@_07CMLOKKIF@input?4c?$AA@ 2006db30     LIBCMTD:input.obj
 0002:00006b44       ??_C@_0BB@NAGLCMLI@Assertion?5Failed?$AA@ 2006db44     LIBCMTD:dbgrpt.obj
 0002:00006b58       ??_C@_05NAOIJFC@Error?$AA@ 2006db58     LIBCMTD:dbgrpt.obj
 0002:00006b60       ??_C@_07KGMMFLDN@Warning?$AA@ 2006db60     LIBCMTD:dbgrpt.obj
 0002:00006b68       ??_C@_08ODMAMGBE@dbgrpt?4c?$AA@ 2006db68     LIBCMTD:dbgrpt.obj
 0002:00006b84       ??_C@_0M@IPILFDFN@?$CFs?$CI?$CFd?$CJ?5?3?5?$CFs?$AA@ 2006db84     LIBCMTD:dbgrpt.obj
 0002:00006b90       ??_C@_01LIIJDEN@?$AN?$AA@  2006db90     LIBCMTD:dbgrpt.obj
 0002:00006b94       ??_C@_0BD@CAENFOHP@Assertion?5failed?3?5?$AA@ 2006db94     LIBCMTD:dbgrpt.obj
 0002:00006ba8       ??_C@_0CL@EACFGMNB@_CrtDbgReport?3?5String?5too?5long?5o@ 2006dba8     LIBCMTD:dbgrpt.obj
 0002:00006bd4       ??_C@_0DC@HLHDIIKH@Second?5Chance?5Assertion?5Failed?3?5@ 2006dbd4     LIBCMTD:dbgrpt.obj
 0002:00006c08       ??_C@_09FOPFMPEJ@wsprintfA?$AA@ 2006dc08     LIBCMTD:dbgrpt.obj
 0002:00006c14       ??_C@_0L@GMPLCCII@user32?4dll?$AA@ 2006dc14     LIBCMTD:dbgrpt.obj
 0002:00006c2c       ??_C@_0CD@EBCGLDDL@Microsoft?5Visual?5C?$CL?$CL?5Debug?5Libra@ 2006dc2c     LIBCMTD:dbgrpt.obj
 0002:00006c50       ??_C@_0FD@IIKNDPHJ@Debug?5?$CFs?$CB?6?6Program?3?5?$CFs?$CFs?$CFs?$CFs?$CFs?$CFs@ 2006dc50     LIBCMTD:dbgrpt.obj
 0002:00006ca4       ??_C@_09OFBFHMBK@?6Module?3?5?$AA@ 2006dca4     LIBCMTD:dbgrpt.obj
 0002:00006cb0       ??_C@_07OPHPPLBG@?6File?3?5?$AA@ 2006dcb0     LIBCMTD:dbgrpt.obj
 0002:00006cb8       ??_C@_07DBMPPHDI@?6Line?3?5?$AA@ 2006dcb8     LIBCMTD:dbgrpt.obj
 0002:00006cc0       ??_C@_0HD@GNBNFCCL@?6?6For?5information?5on?5how?5your?5pr@ 2006dcc0     LIBCMTD:dbgrpt.obj
 0002:00006d34       ??_C@_0BG@IHOEIIEJ@szUserMessage?5?$CB?$DN?5NULL?$AA@ 2006dd34     LIBCMTD:dbgrpt.obj
 0002:00006d58       __DEFAULT_CW_in_mem        2006dd58     LIBCMTD:common.obj
 0002:00006d5a       __pi_by_2_to_61            2006dd5a     LIBCMTD:common.obj
 0002:00006d94       ??_C@_07FEAFKIIG@a_map?4c?$AA@ 2006dd94     LIBCMTD:a_map.obj
 0002:00006d9c       ??_C@_13NOLLCAOD@?$AA?$AA?$AA?$AA@ 2006dd9c     LIBCMTD:a_map.obj
 0002:00006dc4       ??_C@_0L@KDOEJCKC@_nextafter?$AA@ 2006ddc4     LIBCMTD:fpexcept.obj
 0002:00006dd0       ??_C@_05JGDBENOH@_logb?$AA@ 2006ddd0     LIBCMTD:fpexcept.obj
 0002:00006dd8       ??_C@_03ONILCKOB@_yn?$AA@  2006ddd8     LIBCMTD:fpexcept.obj
 0002:00006ddc       ??_C@_03NAKIGLHK@_y1?$AA@  2006dddc     LIBCMTD:fpexcept.obj
 0002:00006de0       ??_C@_03MJLDFKDL@_y0?$AA@  2006dde0     LIBCMTD:fpexcept.obj
 0002:00006de4       ??_C@_05GKKHEGJL@frexp?$AA@ 2006dde4     LIBCMTD:fpexcept.obj
 0002:00006dec       ??_C@_04KEPJIHGP@fmod?$AA@ 2006ddec     LIBCMTD:fpexcept.obj
 0002:00006df4       ??_C@_06MEIMCGCF@_hypot?$AA@ 2006ddf4     LIBCMTD:fpexcept.obj
 0002:00006dfc       ??_C@_05KBKMEMPO@_cabs?$AA@ 2006ddfc     LIBCMTD:fpexcept.obj
 0002:00006e04       ??_C@_05CEJMAHNP@ldexp?$AA@ 2006de04     LIBCMTD:fpexcept.obj
 0002:00006e0c       ??_C@_04EHEDPDJG@modf?$AA@ 2006de0c     LIBCMTD:fpexcept.obj
 0002:00006e14       ??_C@_04ODHECPBC@fabs?$AA@ 2006de14     LIBCMTD:fpexcept.obj
 0002:00006e1c       ??_C@_05PBJFFIGL@floor?$AA@ 2006de1c     LIBCMTD:fpexcept.obj
 0002:00006e24       ??_C@_04GFPJNGEK@ceil?$AA@ 2006de24     LIBCMTD:fpexcept.obj
 0002:00006e2c       ??_C@_03IIINPABG@tan?$AA@  2006de2c     LIBCMTD:fpexcept.obj
 0002:00006e30       ??_C@_03LALBNOCG@cos?$AA@  2006de30     LIBCMTD:fpexcept.obj
 0002:00006e34       ??_C@_03BLEJJJBH@sin?$AA@  2006de34     LIBCMTD:fpexcept.obj
 0002:00006e38       ??_C@_04EIAKFFMI@sqrt?$AA@ 2006de38     LIBCMTD:fpexcept.obj
 0002:00006e40       ??_C@_05KNGEOGJB@atan2?$AA@ 2006de40     LIBCMTD:fpexcept.obj
 0002:00006e48       ??_C@_04MLLJIGOK@atan?$AA@ 2006de48     LIBCMTD:fpexcept.obj
 0002:00006e50       ??_C@_04PDIFKINK@acos?$AA@ 2006de50     LIBCMTD:fpexcept.obj
 0002:00006e58       ??_C@_04FIHNOPOL@asin?$AA@ 2006de58     LIBCMTD:fpexcept.obj
 0002:00006e60       ??_C@_04FJHINJAO@tanh?$AA@ 2006de60     LIBCMTD:fpexcept.obj
 0002:00006e68       ??_C@_04HPJJNFIM@cosh?$AA@ 2006de68     LIBCMTD:fpexcept.obj
 0002:00006e70       ??_C@_04COOMCNPB@sinh?$AA@ 2006de70     LIBCMTD:fpexcept.obj
 0002:00006e78       ??_C@_05HGHHAHAP@log10?$AA@ 2006de78     LIBCMTD:fpexcept.obj
 0002:00006e80       ??_C@_03JGHBODFD@pow?$AA@  2006de80     LIBCMTD:fpexcept.obj
 0002:00006e84       ??_C@_03KHJOGHMM@exp?$AA@  2006de84     LIBCMTD:fpexcept.obj
 0002:00006e88       ??_C@_0DP@FICHPIPH@?$CI?$CCinconsistent?5IOB?5fields?$CC?0?5stre@ 2006de88     LIBCMTD:_flsbuf.obj
 0002:00006ec8       ??_C@_09DHJHPHJP@_flsbuf?4c?$AA@ 2006dec8     LIBCMTD:_flsbuf.obj
 0002:00006ed4       ??_C@_0M@CMNAFCJK@str?5?$CB?$DN?5NULL?$AA@ 2006ded4     LIBCMTD:_flsbuf.obj
 0002:00006ee0       ___lookuptable             2006dee0     LIBCMTD:output.obj
 0002:00006f3c       ??_C@_1O@CEDCILHN@?$AA?$CI?$AAn?$AAu?$AAl?$AAl?$AA?$CJ?$AA?$AA@ 2006df3c     LIBCMTD:output.obj
 0002:00006f4c       ??_C@_06OJHGLDPL@?$CInull?$CJ?$AA@ 2006df4c     LIBCMTD:output.obj
 0002:00006f54       ??_C@_08MEPFMIND@output?4c?$AA@ 2006df54     LIBCMTD:output.obj
 0002:00006f60       ??_C@_0P@LGFCLPDP@ch?5?$CB?$DN?5_T?$CI?8?20?8?$CJ?$AA@ 2006df60     LIBCMTD:output.obj
 0002:00006fd8       ??_C@_05EOHGHCHD@exp10?$AA@ 2006dfd8     LIBCMTD:libm_error.obj
 0002:00006fe0       ??_C@_04HPAFEEIN@exp2?$AA@ 2006dfe0     LIBCMTD:libm_error.obj
 0002:00006fe8       ??_C@_04KGLCPMCP@log2?$AA@ 2006dfe8     LIBCMTD:libm_error.obj
 0002:00006ff0       ??_C@_0N@FFJGBINN@AuthenticAMD?$AA@ 2006dff0     LIBCMTD:cpu_disp.obj
 0002:0000704c       ??_C@_0P@MIGLKIOC@CorExitProcess?$AA@ 2006e04c     LIBCMTD:crt0dat.obj
 0002:0000705c       ??_C@_0M@MBOPBNBK@mscoree?4dll?$AA@ 2006e05c     LIBCMTD:crt0dat.obj
 0002:00007068       ??_C@_08FKHPDPAC@winsig?4c?$AA@ 2006e068     LIBCMTD:winsig.obj
 0002:000070a4       ??_C@_0BI@DFKBFLJE@GetProcessWindowStation?$AA@ 2006e0a4     LIBCMTD:crtmbox.obj
 0002:000070bc       ??_C@_0BK@CIDNPOGP@GetUserObjectInformationA?$AA@ 2006e0bc     LIBCMTD:crtmbox.obj
 0002:000070d8       ??_C@_0BD@HHGDFDBJ@GetLastActivePopup?$AA@ 2006e0d8     LIBCMTD:crtmbox.obj
 0002:000070ec       ??_C@_0BA@HNOPNCHB@GetActiveWindow?$AA@ 2006e0ec     LIBCMTD:crtmbox.obj
 0002:000070fc       ??_C@_0M@CHKKJDAI@MessageBoxA?$AA@ 2006e0fc     LIBCMTD:crtmbox.obj
 0002:00007130       ??_C@_09JMJGGMME@fprintf?4c?$AA@ 2006e130     LIBCMTD:fprintf.obj
 0002:0000714c       ??_C@_09KGBNCNDN@setvbuf?4c?$AA@ 2006e14c     LIBCMTD:setvbuf.obj
 0002:00007164       ??_C@_07PNHPCIEC@_file?4c?$AA@ 2006e164     LIBCMTD:_file.obj
 0002:0000717c       ??_C@_06PJIGMIJB@Client?$AA@ 2006e17c     LIBCMTD:dbgheap.obj
 0002:00007184       ??_C@_06KMEJCCGM@Ignore?$AA@ 2006e184     LIBCMTD:dbgheap.obj
 0002:0000718c       ??_C@_03OGPFLFLO@CRT?$AA@  2006e18c     LIBCMTD:dbgheap.obj
 0002:00007190       ??_C@_06EFAGIKOH@Normal?$AA@ 2006e190     LIBCMTD:dbgheap.obj
 0002:00007198       ??_C@_04HJMOFLDF@Free?$AA@ 2006e198     LIBCMTD:dbgheap.obj
 0002:000071ac       ??_C@_0DC@JEMAGEKG@Error?3?5memory?5allocation?3?5bad?5me@ 2006e1ac     LIBCMTD:dbgheap.obj
 0002:000071e0       ??_C@_0CF@BICKFLAF@Invalid?5allocation?5size?3?5?$CFIu?5byt@ 2006e1e0     LIBCMTD:dbgheap.obj
 0002:00007208       ??_C@_0CB@CCLOLAHO@Client?5hook?5allocation?5failure?4?6@ 2006e208     LIBCMTD:dbgheap.obj
 0002:0000722c       ??_C@_0DF@BBEGIFEK@Client?5hook?5allocation?5failure?5a@ 2006e22c     LIBCMTD:dbgheap.obj
 0002:00007264       ??_C@_09DPMMACIH@dbgheap?4c?$AA@ 2006e264     LIBCMTD:dbgheap.obj
 0002:00007270       ??_C@_0BC@FKEPGOPH@_CrtCheckMemory?$CI?$CJ?$AA@ 2006e270     LIBCMTD:dbgheap.obj
 0002:00007294       ??_C@_0BK@DJDKJKNJ@_pFirstBlock?5?$DN?$DN?5pOldBlock?$AA@ 2006e294     LIBCMTD:dbgheap.obj
 0002:000072b0       ??_C@_0BJ@PGMLBCKP@_pLastBlock?5?$DN?$DN?5pOldBlock?$AA@ 2006e2b0     LIBCMTD:dbgheap.obj
 0002:000072cc       ??_C@_0DC@LIEEBBFH@fRealloc?5?$HM?$HM?5?$CI?$CBfRealloc?5?$CG?$CG?5pNewBl@ 2006e2cc     LIBCMTD:dbgheap.obj
 0002:00007300       ??_C@_0EF@BKJNHFDP@pOldBlock?9?$DOnLine?5?$DN?$DN?5IGNORE_LINE?5@ 2006e300     LIBCMTD:dbgheap.obj
 0002:00007348       ??_C@_0CC@MCCNOMLK@_CrtIsValidHeapPointer?$CIpUserData@ 2006e348     LIBCMTD:dbgheap.obj
 0002:00007370       ??_C@_0EM@LGFLMAGJ@The?5Block?5at?50x?$CFp?5was?5allocated?5@ 2006e370     LIBCMTD:dbgheap.obj
 0002:000073bc       ??_C@_0CO@KPNFNEPA@Allocation?5too?5large?5or?5negative@ 2006e3bc     LIBCMTD:dbgheap.obj
 0002:000073ec       ??_C@_0CE@DOFMDOL@Client?5hook?5re?9allocation?5failur@ 2006e3ec     LIBCMTD:dbgheap.obj
 0002:00007410       ??_C@_0DI@KKJPDPGM@Client?5hook?5re?9allocation?5failur@ 2006e410     LIBCMTD:dbgheap.obj
 0002:00007464       ??_C@_0BG@JDINNDDC@_pFirstBlock?5?$DN?$DN?5pHead?$AA@ 2006e464     LIBCMTD:dbgheap.obj
 0002:0000747c       ??_C@_0BF@LMGMGAEG@_pLastBlock?5?$DN?$DN?5pHead?$AA@ 2006e47c     LIBCMTD:dbgheap.obj
 0002:00007494       ??_C@_0BO@LGCGBMOH@pHead?9?$DOnBlockUse?5?$DN?$DN?5nBlockUse?$AA@ 2006e494     LIBCMTD:dbgheap.obj
 0002:000074b4       ??_C@_0DN@GKKPDMLN@pHead?9?$DOnLine?5?$DN?$DN?5IGNORE_LINE?5?$CG?$CG?5p@ 2006e4b4     LIBCMTD:dbgheap.obj
 0002:000074f4       ??_C@_0CI@CMGHMNIC@DAMAGE?3?5after?5?$CFhs?5block?5?$CI?$CD?$CFd?$CJ?5at@ 2006e4f4     LIBCMTD:dbgheap.obj
 0002:0000751c       ??_C@_0CJ@OHOOBLKI@DAMAGE?3?5before?5?$CFhs?5block?5?$CI?$CD?$CFd?$CJ?5a@ 2006e51c     LIBCMTD:dbgheap.obj
 0002:00007548       ??_C@_0CH@IAGMNLOM@_BLOCK_TYPE_IS_VALID?$CIpHead?9?$DOnBlo@ 2006e548     LIBCMTD:dbgheap.obj
 0002:00007570       ??_C@_0BL@KEIPLFAC@Client?5hook?5free?5failure?4?6?$AA@ 2006e570     LIBCMTD:dbgheap.obj
 0002:00007590       ??_C@_0EJ@HEIBCIMJ@The?5Block?5at?50x?$CFp?5was?5allocated?5@ 2006e590     LIBCMTD:dbgheap.obj
 0002:000075fc       ??_C@_0CI@JMLBEDHJ@?$CFhs?5located?5at?50x?$CFp?5is?5?$CFIu?5bytes@ 2006e5fc     LIBCMTD:dbgheap.obj
 0002:00007624       ??_C@_0CA@FGFAGAOM@?$CFhs?5allocated?5at?5file?5?$CFhs?$CI?$CFd?$CJ?4?6?$AA@ 2006e624     LIBCMTD:dbgheap.obj
 0002:00007644       ??_C@_0CH@JKKAOBEK@DAMAGE?3?5on?5top?5of?5Free?5block?5at?5@ 2006e644     LIBCMTD:dbgheap.obj
 0002:0000766c       ??_C@_07OHKEFPKJ@DAMAGED?$AA@ 2006e66c     LIBCMTD:dbgheap.obj
 0002:00007674       ??_C@_0CL@HNNNMKMJ@_heapchk?5fails?5with?5unknown?5retu@ 2006e674     LIBCMTD:dbgheap.obj
 0002:000076a0       ??_C@_0CC@MFFCHFHO@_heapchk?5fails?5with?5_HEAPBADPTR?4@ 2006e6a0     LIBCMTD:dbgheap.obj
 0002:000076c4       ??_C@_0CC@MJGLGBDG@_heapchk?5fails?5with?5_HEAPBADEND?4@ 2006e6c4     LIBCMTD:dbgheap.obj
 0002:000076e8       ??_C@_0CD@CPKEAPBD@_heapchk?5fails?5with?5_HEAPBADNODE@ 2006e6e8     LIBCMTD:dbgheap.obj
 0002:0000770c       ??_C@_0CE@MKKHMBMK@_heapchk?5fails?5with?5_HEAPBADBEGI@ 2006e70c     LIBCMTD:dbgheap.obj
 0002:0000776c       ??_C@_0CB@EAAIGELO@Bad?5memory?5block?5found?5at?50x?$CFp?4?6@ 2006e76c     LIBCMTD:dbgheap.obj
 0002:00007790       ??_C@_0CI@KDKEAJEJ@_CrtMemCheckPoint?3?5NULL?5state?5po@ 2006e790     LIBCMTD:dbgheap.obj
 0002:000077c4       ??_C@_0CI@ENCLCMLG@_CrtMemDifference?3?5NULL?5state?5po@ 2006e7c4     LIBCMTD:dbgheap.obj
 0002:000077ec       ??_C@_0BH@GFGKJDCO@Object?5dump?5complete?4?6?$AA@ 2006e7ec     LIBCMTD:dbgheap.obj
 0002:00007804       ??_C@_0DA@MDLBNIBM@crt?5block?5at?50x?$CFp?0?5subtype?5?$CFx?0?5?$CF@ 2006e804     LIBCMTD:dbgheap.obj
 0002:00007834       ??_C@_0CH@FAGDDGPN@normal?5block?5at?50x?$CFp?0?5?$CFIu?5bytes?5@ 2006e834     LIBCMTD:dbgheap.obj
 0002:0000785c       ??_C@_0DD@GHNAAKBB@client?5block?5at?50x?$CFp?0?5subtype?5?$CFx@ 2006e85c     LIBCMTD:dbgheap.obj
 0002:00007890       ??_C@_06PKLGBFGM@?$HL?$CFld?$HN?5?$AA@ 2006e890     LIBCMTD:dbgheap.obj
 0002:00007898       ??_C@_0L@JMEFFCCJ@?$CFhs?$CI?$CFd?$CJ?5?3?5?$AA@ 2006e898     LIBCMTD:dbgheap.obj
 0002:000078a4       ??_C@_0BE@OIEFNFL@?$CDFile?5Error?$CD?$CI?$CFd?$CJ?5?3?5?$AA@ 2006e8a4     LIBCMTD:dbgheap.obj
 0002:000078b8       ??_C@_0BE@KCIPKCIA@Dumping?5objects?5?9?$DO?6?$AA@ 2006e8b8     LIBCMTD:dbgheap.obj
 0002:000078dc       ??_C@_0BA@HJBKCELP@?5Data?3?5?$DM?$CFs?$DO?5?$CFs?6?$AA@ 2006e8dc     LIBCMTD:dbgheap.obj
 0002:000078ec       ??_C@_05MKKEDADM@?$CF?42X?5?$AA@ 2006e8ec     LIBCMTD:dbgheap.obj
 0002:000078f4       ??_C@_0BI@JBFPOEJA@Detected?5memory?5leaks?$CB?6?$AA@ 2006e8f4     LIBCMTD:dbgheap.obj
 0002:0000790c       ??_C@_0BP@DEDHGGGI@Total?5allocations?3?5?$CFId?5bytes?4?6?$AA@ 2006e90c     LIBCMTD:dbgheap.obj
 0002:0000792c       ??_C@_0CB@BLHDAFNE@Largest?5number?5used?3?5?$CFId?5bytes?4?6@ 2006e92c     LIBCMTD:dbgheap.obj
 0002:00007950       ??_C@_0BO@DACNIABB@?$CFId?5bytes?5in?5?$CFId?5?$CFhs?5Blocks?4?6?$AA@ 2006e950     LIBCMTD:dbgheap.obj
 0002:00007970       ??_C@_0CC@GFBJAAAH@?$CI?$CCoffset?5must?5be?5within?5size?$CC?0?50@ 2006e970     LIBCMTD:dbgheap.obj
 0002:00007994       ??_C@_0CF@PGBEDOC@?$CI?$CCalignment?5must?5be?5a?5power?5of?52@ 2006e994     LIBCMTD:dbgheap.obj
 0002:000079bc       ??_C@_0DL@PGHMMKNE@Damage?5before?50x?$CFp?5which?5was?5all@ 2006e9bc     LIBCMTD:dbgheap.obj
 0002:000079f8       ??_C@_0EI@NDNJMAJK@The?5block?5at?50x?$CFp?5was?5not?5alloca@ 2006e9f8     LIBCMTD:dbgheap.obj
 0002:00007a40       ??_C@_0EF@PGELACII@The?5block?5at?50x?$CFp?5was?5not?5alloca@ 2006ea40     LIBCMTD:dbgheap.obj
 0002:00007a88       ??_C@_08MAFBHINM@ioinit?4c?$AA@ 2006ea88     LIBCMTD:ioinit.obj
 0002:00007a94       ??_C@_09HCDLHOJP@stdenvp?4c?$AA@ 2006ea94     LIBCMTD:stdenvp.obj
 0002:00007aa0       ??_C@_09IKILHJIC@stdargv?4c?$AA@ 2006eaa0     LIBCMTD:stdargv.obj
 0002:00007aac       ??_C@_07BPGNOCOG@a_env?4c?$AA@ 2006eaac     LIBCMTD:a_env.obj
 0002:00007ad4       ??_C@_0P@GGKDKEEG@runtime?5error?5?$AA@ 2006ead4     LIBCMTD:crt0msg.obj
 0002:00007ae4       ??_C@_02PCIJFNDE@?$AN?6?$AA@ 2006eae4     LIBCMTD:crt0msg.obj
 0002:00007ae8       ??_C@_0O@MJNIPGOH@TLOSS?5error?$AN?6?$AA@ 2006eae8     LIBCMTD:crt0msg.obj
 0002:00007af8       ??_C@_0N@BONNPDHF@SING?5error?$AN?6?$AA@ 2006eaf8     LIBCMTD:crt0msg.obj
 0002:00007b08       ??_C@_0P@MBDAJNE@DOMAIN?5error?$AN?6?$AA@ 2006eb08     LIBCMTD:crt0msg.obj
 0002:00007b18       ??_C@_0KC@BDDGGBEJ@R6029?$AN?6?9?5This?5application?5cannot@ 2006eb18     LIBCMTD:crt0msg.obj
 0002:00007bbc       ??_C@_0CF@KJDAIALP@R6028?$AN?6?9?5unable?5to?5initialize?5he@ 2006ebbc     LIBCMTD:crt0msg.obj
 0002:00007be4       ??_C@_0DF@GAKBPDFP@R6027?$AN?6?9?5not?5enough?5space?5for?5lo@ 2006ebe4     LIBCMTD:crt0msg.obj
 0002:00007c1c       ??_C@_0DF@IBLNNAIG@R6026?$AN?6?9?5not?5enough?5space?5for?5st@ 2006ec1c     LIBCMTD:crt0msg.obj
 0002:00007c54       ??_C@_0CG@IOHKGFNJ@R6025?$AN?6?9?5pure?5virtual?5function?5c@ 2006ec54     LIBCMTD:crt0msg.obj
 0002:00007c7c       ??_C@_0DF@JIJJFJDC@R6024?$AN?6?9?5not?5enough?5space?5for?5_o@ 2006ec7c     LIBCMTD:crt0msg.obj
 0002:00007cb4       ??_C@_0CJ@EGEJHFME@R6019?$AN?6?9?5unable?5to?5open?5console?5@ 2006ecb4     LIBCMTD:crt0msg.obj
 0002:00007ce0       ??_C@_0CB@GNHNIELH@R6018?$AN?6?9?5unexpected?5heap?5error?$AN?6@ 2006ece0     LIBCMTD:crt0msg.obj
 0002:00007d04       ??_C@_0CN@FOLDKNG@R6017?$AN?6?9?5unexpected?5multithread?5@ 2006ed04     LIBCMTD:crt0msg.obj
 0002:00007d34       ??_C@_0CM@FAHFJNHO@R6016?$AN?6?9?5not?5enough?5space?5for?5th@ 2006ed34     LIBCMTD:crt0msg.obj
 0002:00007d60       ??_C@_0JG@LBKMGKLD@?$AN?6This?5application?5has?5requested@ 2006ed60     LIBCMTD:crt0msg.obj
 0002:00007df8       ??_C@_0CM@FLCNIPKK@R6009?$AN?6?9?5not?5enough?5space?5for?5en@ 2006edf8     LIBCMTD:crt0msg.obj
 0002:00007e24       ??_C@_0CK@KMMJOAPP@R6008?$AN?6?9?5not?5enough?5space?5for?5ar@ 2006ee24     LIBCMTD:crt0msg.obj
 0002:00007e50       ??_C@_0CF@HOHMHDEK@R6002?$AN?6?9?5floating?5point?5not?5load@ 2006ee50     LIBCMTD:crt0msg.obj
 0002:00007e78       ??_C@_0BK@OFGJDLJJ@Runtime?5Error?$CB?6?6Program?3?5?$AA@ 2006ee78     LIBCMTD:crt0msg.obj
 0002:00007e98       ___newctype                2006ee98     LIBCMTD:ctype.obj
 0002:00008198       __wctype                   2006f198     LIBCMTD:ctype.obj
 0002:0000839c       ??_C@_07GPNABLBE@a_str?4c?$AA@ 2006f39c     LIBCMTD:a_str.obj
 0002:000083b4       ??_C@_08JCCMCCIL@HH?3mm?3ss?$AA@ 2006f3b4     LIBCMTD:strftime.obj
 0002:000083c0       ??_C@_0BE@CKGJFCPC@dddd?0?5MMMM?5dd?0?5yyyy?$AA@ 2006f3c0     LIBCMTD:strftime.obj
 0002:000083d4       ??_C@_08BPBNCDIB@MM?1dd?1yy?$AA@ 2006f3d4     LIBCMTD:strftime.obj
 0002:000083e0       ??_C@_02CJNFDJBF@PM?$AA@   2006f3e0     LIBCMTD:strftime.obj
 0002:000083e4       ??_C@_02DEDBPAFC@AM?$AA@   2006f3e4     LIBCMTD:strftime.obj
 0002:000083e8       ??_C@_08EDHMEBNP@December?$AA@ 2006f3e8     LIBCMTD:strftime.obj
 0002:000083f4       ??_C@_08HCHEGEOA@November?$AA@ 2006f3f4     LIBCMTD:strftime.obj
 0002:00008400       ??_C@_07JJNFCEND@October?$AA@ 2006f400     LIBCMTD:strftime.obj
 0002:00008408       ??_C@_09BHHEALKD@September?$AA@ 2006f408     LIBCMTD:strftime.obj
 0002:00008414       ??_C@_06LBBHFDDG@August?$AA@ 2006f414     LIBCMTD:strftime.obj
 0002:0000841c       ??_C@_04MIEPOIFP@July?$AA@ 2006f41c     LIBCMTD:strftime.obj
 0002:00008424       ??_C@_04CNLMGBGM@June?$AA@ 2006f424     LIBCMTD:strftime.obj
 0002:0000842c       ??_C@_05DMJDNLEJ@April?$AA@ 2006f42c     LIBCMTD:strftime.obj
 0002:00008434       ??_C@_05HPCKOFNC@March?$AA@ 2006f434     LIBCMTD:strftime.obj
 0002:0000843c       ??_C@_08GNJGEPFN@February?$AA@ 2006f43c     LIBCMTD:strftime.obj
 0002:00008448       ??_C@_07CGJPFGJA@January?$AA@ 2006f448     LIBCMTD:strftime.obj
 0002:00008450       ??_C@_03MKABNOCG@Dec?$AA@  2006f450     LIBCMTD:strftime.obj
 0002:00008454       ??_C@_03JPJOFNIA@Nov?$AA@  2006f454     LIBCMTD:strftime.obj
 0002:00008458       ??_C@_03BMAOKBAD@Oct?$AA@  2006f458     LIBCMTD:strftime.obj
 0002:0000845c       ??_C@_03GGCAPAJC@Sep?$AA@  2006f45c     LIBCMTD:strftime.obj
 0002:00008460       ??_C@_03IFJFEIGA@Aug?$AA@  2006f460     LIBCMTD:strftime.obj
 0002:00008464       ??_C@_03LBGABGKK@Jul?$AA@  2006f464     LIBCMTD:strftime.obj
 0002:00008468       ??_C@_03IDFGHECI@Jun?$AA@  2006f468     LIBCMTD:strftime.obj
 0002:0000846c       ??_C@_03CNMDKL@May?$AA@    2006f46c     LIBCMTD:strftime.obj
 0002:00008470       ??_C@_03LEOLGMJP@Apr?$AA@  2006f470     LIBCMTD:strftime.obj
 0002:00008474       ??_C@_03ODNJBKGA@Mar?$AA@  2006f474     LIBCMTD:strftime.obj
 0002:00008478       ??_C@_03HJBDCHOM@Feb?$AA@  2006f478     LIBCMTD:strftime.obj
 0002:0000847c       ??_C@_03JIHJHPIE@Jan?$AA@  2006f47c     LIBCMTD:strftime.obj
 0002:00008480       ??_C@_08INBOOONO@Saturday?$AA@ 2006f480     LIBCMTD:strftime.obj
 0002:0000848c       ??_C@_06JECMNKMI@Friday?$AA@ 2006f48c     LIBCMTD:strftime.obj
 0002:00008494       ??_C@_08HACCIKIA@Thursday?$AA@ 2006f494     LIBCMTD:strftime.obj
 0002:000084a0       ??_C@_09DLIGFAKA@Wednesday?$AA@ 2006f4a0     LIBCMTD:strftime.obj
 0002:000084ac       ??_C@_07BAAGCFCM@Tuesday?$AA@ 2006f4ac     LIBCMTD:strftime.obj
 0002:000084b4       ??_C@_06JLEDEDGH@Monday?$AA@ 2006f4b4     LIBCMTD:strftime.obj
 0002:000084bc       ??_C@_06OOPIFAJ@Sunday?$AA@ 2006f4bc     LIBCMTD:strftime.obj
 0002:000084c4       ??_C@_03FEFJNEK@Sat?$AA@   2006f4c4     LIBCMTD:strftime.obj
 0002:000084c8       ??_C@_03IDIOELNC@Fri?$AA@  2006f4c8     LIBCMTD:strftime.obj
 0002:000084cc       ??_C@_03IOFIKPDN@Thu?$AA@  2006f4cc     LIBCMTD:strftime.obj
 0002:000084d0       ??_C@_03MHOMLAJA@Wed?$AA@  2006f4d0     LIBCMTD:strftime.obj
 0002:000084d4       ??_C@_03NAGEINEP@Tue?$AA@  2006f4d4     LIBCMTD:strftime.obj
 0002:000084d8       ??_C@_03PDAGKDH@Mon?$AA@   2006f4d8     LIBCMTD:strftime.obj
 0002:000084dc       ??_C@_03KOEHGMDN@Sun?$AA@  2006f4dc     LIBCMTD:strftime.obj
 0002:000084e0       ??_C@_0L@OCEOFAIF@strftime?4c?$AA@ 2006f4e0     LIBCMTD:strftime.obj
 0002:000084ec       ??_C@_0DJ@BLPIACFC@?$CI?$CCInvalid?5MBCS?5character?5sequenc@ 2006f4ec     LIBCMTD:strftime.obj
 0002:00008528       ??_C@_0DD@GLPHLKIC@?$CI?$CCZero?5length?5output?5buffer?5pass@ 2006f528     LIBCMTD:strftime.obj
 0002:0000855c       ??_C@_0DL@LLHFCBKO@?$CI?$CCInvalid?5MBCS?5character?5sequenc@ 2006f55c     LIBCMTD:strftime.obj
 0002:00008598       ??_C@_0EC@CJNAOFBG@?$CI?$CCInvalid?5MBCS?5character?5sequenc@ 2006f598     LIBCMTD:strftime.obj
 0002:000085dc       ??_C@_03EBAPMIKO@a?1p?$AA@ 2006f5dc     LIBCMTD:strftime.obj
 0002:000085e0       ??_C@_05JAMEPDIN@am?1pm?$AA@ 2006f5e0     LIBCMTD:strftime.obj
 0002:000085f4       ??_C@_0L@IOJADHBB@inittime?4c?$AA@ 2006f5f4     LIBCMTD:inittime.obj
 0002:00008600       ??_C@_09MECGNAGI@initnum?4c?$AA@ 2006f600     LIBCMTD:initnum.obj
 0002:0000860c       ??_C@_09HKFHICAL@initmon?4c?$AA@ 2006f60c     LIBCMTD:initmon.obj
 0002:00008618       ??_C@_0L@GBAGBCPL@initctyp?4c?$AA@ 2006f618     LIBCMTD:initctyp.obj
 0002:00008624       ??_C@_07CKDBCAPD@mlock?4c?$AA@ 2006f624     LIBCMTD:mlock.obj
 0002:00008640       ___rgLocInfo               2006f640     LIBCMTD:getqloc.obj
 0002:00008ae4       ??_C@_08PKBIPKE@Paraguay?$AA@ 2006fae4     LIBCMTD:getqloc.obj
 0002:00008af0       ??_C@_07GHBIBIBP@Uruguay?$AA@ 2006faf0     LIBCMTD:getqloc.obj
 0002:00008af8       ??_C@_05HBNKAPDN@Chile?$AA@ 2006faf8     LIBCMTD:getqloc.obj
 0002:00008b00       ??_C@_07FEIFIPNF@Ecuador?$AA@ 2006fb00     LIBCMTD:getqloc.obj
 0002:00008b08       ??_C@_09PGNFPGME@Argentina?$AA@ 2006fb08     LIBCMTD:getqloc.obj
 0002:00008b14       ??_C@_04IALPBJF@Peru?$AA@  2006fb14     LIBCMTD:getqloc.obj
 0002:00008b1c       ??_C@_08IJPLNLKH@Colombia?$AA@ 2006fb1c     LIBCMTD:getqloc.obj
 0002:00008b28       ??_C@_09IDMFKCN@Venezuela?$AA@ 2006fb28     LIBCMTD:getqloc.obj
 0002:00008b34       ??_C@_0BD@DNEJOGOK@Dominican?5Republic?$AA@ 2006fb34     LIBCMTD:getqloc.obj
 0002:00008b48       ??_C@_0N@LPINDNDB@South?5Africa?$AA@ 2006fb48     LIBCMTD:getqloc.obj
 0002:00008b58       ??_C@_06BLJPEOBG@Panama?$AA@ 2006fb58     LIBCMTD:getqloc.obj
 0002:00008b60       ??_C@_0L@BOCNDGON@Luxembourg?$AA@ 2006fb60     LIBCMTD:getqloc.obj
 0002:00008b6c       ??_C@_0L@CONEHKA@Costa?5Rica?$AA@ 2006fb6c     LIBCMTD:getqloc.obj
 0002:00008b78       ??_C@_0M@KGBPELAM@Switzerland?$AA@ 2006fb78     LIBCMTD:getqloc.obj
 0002:00008b84       ??_C@_09FJGLIMAG@Guatemala?$AA@ 2006fb84     LIBCMTD:getqloc.obj
 0002:00008b90       ??_C@_06ECHIPDMK@Canada?$AA@ 2006fb90     LIBCMTD:getqloc.obj
 0002:00008b98       ??_C@_0BG@CCEBNPGH@Spanish?5?9?5Modern?5Sort?$AA@ 2006fb98     LIBCMTD:getqloc.obj
 0002:00008bb0       ??_C@_09EFGJAPAD@Australia?$AA@ 2006fbb0     LIBCMTD:getqloc.obj
 0002:00008bbc       ??_C@_07NEKHPBCG@English?$AA@ 2006fbbc     LIBCMTD:getqloc.obj
 0002:00008bc4       ??_C@_07LKIIOGFH@Austria?$AA@ 2006fbc4     LIBCMTD:getqloc.obj
 0002:00008bcc       ??_C@_06EDDDIONA@German?$AA@ 2006fbcc     LIBCMTD:getqloc.obj
 0002:00008bd4       ??_C@_07LIIIOFOA@Belgium?$AA@ 2006fbd4     LIBCMTD:getqloc.obj
 0002:00008bdc       ??_C@_06DIAOLLEH@Mexico?$AA@ 2006fbdc     LIBCMTD:getqloc.obj
 0002:00008be4       ??_C@_07PFALJOGE@Spanish?$AA@ 2006fbe4     LIBCMTD:getqloc.obj
 0002:00008bec       ??_C@_06FFOOPAJB@Basque?$AA@ 2006fbec     LIBCMTD:getqloc.obj
 0002:00008bf4       ??_C@_06DGHNDJFJ@Sweden?$AA@ 2006fbf4     LIBCMTD:getqloc.obj
 0002:00008bfc       ??_C@_07OBINPKFN@Swedish?$AA@ 2006fbfc     LIBCMTD:getqloc.obj
 0002:00008c04       ??_C@_07NCOIHDGC@Iceland?$AA@ 2006fc04     LIBCMTD:getqloc.obj
 0002:00008c0c       ??_C@_09JHBBDDIA@Icelandic?$AA@ 2006fc0c     LIBCMTD:getqloc.obj
 0002:00008c18       ??_C@_06COBCPIFO@France?$AA@ 2006fc18     LIBCMTD:getqloc.obj
 0002:00008c20       ??_C@_06GODMCAND@French?$AA@ 2006fc20     LIBCMTD:getqloc.obj
 0002:00008c28       ??_C@_07MFHPMOED@Finland?$AA@ 2006fc28     LIBCMTD:getqloc.obj
 0002:00008c30       ??_C@_07MCEAMKOD@Finnish?$AA@ 2006fc30     LIBCMTD:getqloc.obj
 0002:00008c38       ??_C@_05CBHOCCK@Spain?$AA@ 2006fc38     LIBCMTD:getqloc.obj
 0002:00008c40       ??_C@_0BL@GIOEGDHB@Spanish?5?9?5Traditional?5Sort?$AA@ 2006fc40     LIBCMTD:getqloc.obj
 0002:00008c5c       ___rglangidNotDefault      2006fc5c     LIBCMTD:getqloc.obj
 0002:00008c70       ___rg_country              2006fc70     LIBCMTD:getqloc.obj
 0002:00008d28       ??_C@_0O@FMJNFNKE@united?9states?$AA@ 2006fd28     LIBCMTD:getqloc.obj
 0002:00008d38       ??_C@_0P@NDHFFKCA@united?9kingdom?$AA@ 2006fd38     LIBCMTD:getqloc.obj
 0002:00008d48       ??_C@_0BC@HHDADLGF@trinidad?5?$CG?5tobago?$AA@ 2006fd48     LIBCMTD:getqloc.obj
 0002:00008d5c       ??_C@_0M@IOAEBDAC@south?9korea?$AA@ 2006fd5c     LIBCMTD:getqloc.obj
 0002:00008d68       ??_C@_0N@FIELFKIJ@south?9africa?$AA@ 2006fd68     LIBCMTD:getqloc.obj
 0002:00008d78       ??_C@_0M@OPNDHCMC@south?5korea?$AA@ 2006fd78     LIBCMTD:getqloc.obj
 0002:00008d84       ??_C@_0N@MDEOEPFI@south?5africa?$AA@ 2006fd84     LIBCMTD:getqloc.obj
 0002:00008d94       ??_C@_06FKAPCJLB@slovak?$AA@ 2006fd94     LIBCMTD:getqloc.obj
 0002:00008d9c       ??_C@_0M@EFJANOAL@puerto?9rico?$AA@ 2006fd9c     LIBCMTD:getqloc.obj
 0002:00008da8       ??_C@_08PGOJKDAI@pr?9china?$AA@ 2006fda8     LIBCMTD:getqloc.obj
 0002:00008db4       ??_C@_08JHDOMCMI@pr?5china?$AA@ 2006fdb4     LIBCMTD:getqloc.obj
 0002:00008dc0       ??_C@_02JHCHFBLL@nz?$AA@   2006fdc0     LIBCMTD:getqloc.obj
 0002:00008dc4       ??_C@_0M@LINHDHKP@new?9zealand?$AA@ 2006fdc4     LIBCMTD:getqloc.obj
 0002:00008dd0       ??_C@_09IIIPPBDB@hong?9kong?$AA@ 2006fdd0     LIBCMTD:getqloc.obj
 0002:00008ddc       ??_C@_07HJLCKBG@holland?$AA@ 2006fddc     LIBCMTD:getqloc.obj
 0002:00008de4       ??_C@_0O@LEHGMHAG@great?5britain?$AA@ 2006fde4     LIBCMTD:getqloc.obj
 0002:00008df4       ??_C@_07FACOMELA@england?$AA@ 2006fdf4     LIBCMTD:getqloc.obj
 0002:00008dfc       ??_C@_05JIHCEICB@czech?$AA@ 2006fdfc     LIBCMTD:getqloc.obj
 0002:00008e04       ??_C@_05BBJOBLGB@china?$AA@ 2006fe04     LIBCMTD:getqloc.obj
 0002:00008e0c       ??_C@_07GPKPHICP@britain?$AA@ 2006fe0c     LIBCMTD:getqloc.obj
 0002:00008e14       ??_C@_07MHIPBHMG@america?$AA@ 2006fe14     LIBCMTD:getqloc.obj
 0002:00008e20       ___rg_language             2006fe20     LIBCMTD:getqloc.obj
 0002:00009028       ??_C@_03KIALPMKC@usa?$AA@  20070028     LIBCMTD:getqloc.obj
 0002:0000902c       ??_C@_02FGJGKGGD@us?$AA@   2007002c     LIBCMTD:getqloc.obj
 0002:00009030       ??_C@_02NEINDODK@uk?$AA@   20070030     LIBCMTD:getqloc.obj
 0002:00009034       ??_C@_05JMPCFJFJ@swiss?$AA@ 20070034     LIBCMTD:getqloc.obj
 0002:0000903c       ??_C@_0BA@HLOCPIOD@swedish?9finland?$AA@ 2007003c     LIBCMTD:getqloc.obj
 0002:0000904c       ??_C@_0BC@PKCNIABK@spanish?9venezuela?$AA@ 2007004c     LIBCMTD:getqloc.obj
 0002:00009060       ??_C@_0BA@GBHHMIJI@spanish?9uruguay?$AA@ 20070060     LIBCMTD:getqloc.obj
 0002:00009070       ??_C@_0BE@BHDOHPMC@spanish?9puerto?5rico?$AA@ 20070070     LIBCMTD:getqloc.obj
 0002:00009084       ??_C@_0N@KMOIDGGN@spanish?9peru?$AA@ 20070084     LIBCMTD:getqloc.obj
 0002:00009094       ??_C@_0BB@HMHLPGPH@spanish?9paraguay?$AA@ 20070094     LIBCMTD:getqloc.obj
 0002:000090a8       ??_C@_0P@MCPKNGFD@spanish?9panama?$AA@ 200700a8     LIBCMTD:getqloc.obj
 0002:000090b8       ??_C@_0BC@IHOHGAIL@spanish?9nicaragua?$AA@ 200700b8     LIBCMTD:getqloc.obj
 0002:000090cc       ??_C@_0P@KLMJDNFJ@spanish?9modern?$AA@ 200700cc     LIBCMTD:getqloc.obj
 0002:000090dc       ??_C@_0BA@BPAPGBCM@spanish?9mexican?$AA@ 200700dc     LIBCMTD:getqloc.obj
 0002:000090ec       ??_C@_0BB@PDECHHHE@spanish?9honduras?$AA@ 200700ec     LIBCMTD:getqloc.obj
 0002:00009100       ??_C@_0BC@KLHKFGDB@spanish?9guatemala?$AA@ 20070100     LIBCMTD:getqloc.obj
 0002:00009114       ??_C@_0BE@MFOOKJAI@spanish?9el?5salvador?$AA@ 20070114     LIBCMTD:getqloc.obj
 0002:00009128       ??_C@_0BA@FCOKFPFC@spanish?9ecuador?$AA@ 20070128     LIBCMTD:getqloc.obj
 0002:00009138       ??_C@_0BL@PLMGIMOO@spanish?9dominican?5republic?$AA@ 20070138     LIBCMTD:getqloc.obj
 0002:00009154       ??_C@_0BD@HLGDNMHB@spanish?9costa?5rica?$AA@ 20070154     LIBCMTD:getqloc.obj
 0002:00009168       ??_C@_0BB@PKCBKCPE@spanish?9colombia?$AA@ 20070168     LIBCMTD:getqloc.obj
 0002:0000917c       ??_C@_0O@MCBIJGNE@spanish?9chile?$AA@ 2007017c     LIBCMTD:getqloc.obj
 0002:0000918c       ??_C@_0BA@BEFEIGJJ@spanish?9bolivia?$AA@ 2007018c     LIBCMTD:getqloc.obj
 0002:0000919c       ??_C@_0BC@EMECMPD@spanish?9argentina?$AA@ 2007019c     LIBCMTD:getqloc.obj
 0002:000091b0       ??_C@_0BF@EALFLENP@portuguese?9brazilian?$AA@ 200701b0     LIBCMTD:getqloc.obj
 0002:000091c8       ??_C@_0BC@HBLEBLNN@norwegian?9nynorsk?$AA@ 200701c8     LIBCMTD:getqloc.obj
 0002:000091dc       ??_C@_0BB@HMACDDCK@norwegian?9bokmal?$AA@ 200701dc     LIBCMTD:getqloc.obj
 0002:000091f0       ??_C@_09BAFFPPHE@norwegian?$AA@ 200701f0     LIBCMTD:getqloc.obj
 0002:000091fc       ??_C@_0O@EAJFJDFG@italian?9swiss?$AA@ 200701fc     LIBCMTD:getqloc.obj
 0002:0000920c       ??_C@_0O@CNOMPGD@irish?9english?$AA@ 2007020c     LIBCMTD:getqloc.obj
 0002:0000921c       ??_C@_0N@EDHBGCKG@german?9swiss?$AA@ 2007021c     LIBCMTD:getqloc.obj
 0002:0000922c       ??_C@_0BC@JACMHNBP@german?9luxembourg?$AA@ 2007022c     LIBCMTD:getqloc.obj
 0002:00009240       ??_C@_0BE@HBGMGFEG@german?9lichtenstein?$AA@ 20070240     LIBCMTD:getqloc.obj
 0002:00009254       ??_C@_0BA@HKKBIBKL@german?9austrian?$AA@ 20070254     LIBCMTD:getqloc.obj
 0002:00009264       ??_C@_0N@GCAEPEBK@french?9swiss?$AA@ 20070264     LIBCMTD:getqloc.obj
 0002:00009274       ??_C@_0BC@DJFJJCK@french?9luxembourg?$AA@ 20070274     LIBCMTD:getqloc.obj
 0002:00009288       ??_C@_0BA@NNCEDFIC@french?9canadian?$AA@ 20070288     LIBCMTD:getqloc.obj
 0002:00009298       ??_C@_0P@CMPOCLM@french?9belgian?$AA@ 20070298     LIBCMTD:getqloc.obj
 0002:000092a8       ??_C@_0M@GHHDJOK@english?9usa?$AA@ 200702a8     LIBCMTD:getqloc.obj
 0002:000092b4       ??_C@_0L@PLDJKEIL@english?9us?$AA@ 200702b4     LIBCMTD:getqloc.obj
 0002:000092c0       ??_C@_0L@HJCCDMNC@english?9uk?$AA@ 200702c0     LIBCMTD:getqloc.obj
 0002:000092cc       ??_C@_0BK@CKLIAGJB@english?9trinidad?5y?5tobago?$AA@ 200702cc     LIBCMTD:getqloc.obj
 0002:000092e8       ??_C@_0BF@JMJMGNNF@english?9south?5africa?$AA@ 200702e8     LIBCMTD:getqloc.obj
 0002:00009300       ??_C@_0L@DKIIFDFD@english?9nz?$AA@ 20070300     LIBCMTD:getqloc.obj
 0002:0000930c       ??_C@_0BA@ONHGJCLH@english?9jamaica?$AA@ 2007030c     LIBCMTD:getqloc.obj
 0002:0000931c       ??_C@_0M@HJBGHOPO@english?9ire?$AA@ 2007031c     LIBCMTD:getqloc.obj
 0002:00009328       ??_C@_0BC@LFEKMIFB@english?9caribbean?$AA@ 20070328     LIBCMTD:getqloc.obj
 0002:0000933c       ??_C@_0M@OLDPFKHI@english?9can?$AA@ 2007033c     LIBCMTD:getqloc.obj
 0002:00009348       ??_C@_0P@OMDEHBMP@english?9belize?$AA@ 20070348     LIBCMTD:getqloc.obj
 0002:00009358       ??_C@_0M@KFHFPFED@english?9aus?$AA@ 20070358     LIBCMTD:getqloc.obj
 0002:00009364       ??_C@_0BB@MNMBKDFE@english?9american?$AA@ 20070364     LIBCMTD:getqloc.obj
 0002:00009378       ??_C@_0O@KIDLNNBA@dutch?9belgian?$AA@ 20070378     LIBCMTD:getqloc.obj
 0002:00009388       ??_C@_0BE@JBKABBMH@chinese?9traditional?$AA@ 20070388     LIBCMTD:getqloc.obj
 0002:0000939c       ??_C@_0BC@MJJMPKCG@chinese?9singapore?$AA@ 2007039c     LIBCMTD:getqloc.obj
 0002:000093b0       ??_C@_0BD@FDKADDCP@chinese?9simplified?$AA@ 200703b0     LIBCMTD:getqloc.obj
 0002:000093c4       ??_C@_0BB@DBEFDDME@chinese?9hongkong?$AA@ 200703c4     LIBCMTD:getqloc.obj
 0002:000093d8       ??_C@_07DHNMFMCI@chinese?$AA@ 200703d8     LIBCMTD:getqloc.obj
 0002:000093e0       ??_C@_03FNDDCHI@chi?$AA@   200703e0     LIBCMTD:getqloc.obj
 0002:000093e4       ??_C@_03BMMIADDJ@chh?$AA@  200703e4     LIBCMTD:getqloc.obj
 0002:000093e8       ??_C@_08OAIPJDGI@canadian?$AA@ 200703e8     LIBCMTD:getqloc.obj
 0002:000093f4       ??_C@_07HBPMNPNJ@belgian?$AA@ 200703f4     LIBCMTD:getqloc.obj
 0002:000093fc       ??_C@_0L@OEKOPBEL@australian?$AA@ 200703fc     LIBCMTD:getqloc.obj
 0002:00009408       ??_C@_0BB@MEIMBEDG@american?9english?$AA@ 20070408     LIBCMTD:getqloc.obj
 0002:0000941c       ??_C@_0BB@DFMDPDGB@american?5english?$AA@ 2007041c     LIBCMTD:getqloc.obj
 0002:00009430       ??_C@_08IJLOKOLL@american?$AA@ 20070430     LIBCMTD:getqloc.obj
 0002:0000943c       ??_C@_0BC@NFIEMBLL@Norwegian?9Nynorsk?$AA@ 2007043c     LIBCMTD:getqloc.obj
 0002:00009450       ??_C@_03NFKLAGEF@OCP?$AA@  20070450     LIBCMTD:getqloc.obj
 0002:00009454       ??_C@_03DFHEHBHG@ACP?$AA@  20070454     LIBCMTD:getqloc.obj
 0002:00009464       ??_C@_09KJLOAKHC@mbctype?4c?$AA@ 20070464     LIBCMTD:mbctype.obj
 0002:0000947c       ??_C@_08NJPDFEGP@mbtowc?4c?$AA@ 2007047c     LIBCMTD:mbtowc.obj
 0002:00009488       ??_C@_0DD@FIIGOHOA@ptloci?9?$DOmb_cur_max?5?$DN?$DN?51?5?$HM?$HM?5ptloc@ 20070488     LIBCMTD:mbtowc.obj
 0002:000094bc       ??_C@_09OOOBBFNM@_filbuf?4c?$AA@ 200704bc     LIBCMTD:_filbuf.obj
 0002:000094c8       ??_C@_08CJEJHOKM@ungetc?4c?$AA@ 200704c8     LIBCMTD:ungetc.obj
 0002:000094e4       ??_C@_0CP@PEILCOHB@f?3?2vs70builds?23077?2vc?2crtbld?2crt@ 200704e4     LIBCMTD:snprintf.obj
 0002:00009514       ??_C@_0DA@KHEJFFIK@f?3?2vs70builds?23077?2vc?2crtbld?2crt@ 20070514     LIBCMTD:vsnprint.obj
 0002:00009544       ??_C@_0L@KBNGFDKM@convrtcp?4c?$AA@ 20070544     LIBCMTD:convrtcp.obj
 0002:0000957c       ??_C@_09PKAEMGHJ@_getbuf?4c?$AA@ 2007057c     LIBCMTD:_getbuf.obj
 0002:00009594       ??_C@_08GNMOIKDK@onexit?4c?$AA@ 20070594     LIBCMTD:onexit.obj
 0002:000095ac       ??_C@_09IFKHNCOH@_sftbuf?4c?$AA@ 200705ac     LIBCMTD:_sftbuf.obj
 0002:000095b8       ??_C@_0BH@HIGALIFJ@flag?5?$DN?$DN?50?5?$HM?$HM?5flag?5?$DN?$DN?51?$AA@ 200705b8     LIBCMTD:_sftbuf.obj
 0002:000095d0       ??_C@_0L@CKFHAPLH@_freebuf?4c?$AA@ 200705d0     LIBCMTD:_freebuf.obj
 0002:000095f0       ??_C@_0KA@JEHFIFGP@A?5buffer?5overrun?5has?5been?5detect@ 200705f0     LIBCMTD:secfail.obj
 0002:00009690       ??_C@_0BJ@MDEKIEOJ@Buffer?5overrun?5detected?$CB?$AA@ 20070690     LIBCMTD:secfail.obj
 0002:000096b0       ??_C@_0LB@BPLHHLFD@A?5security?5error?5of?5unknown?5caus@ 200706b0     LIBCMTD:secfail.obj
 0002:00009764       ??_C@_0CD@GMKACBEK@Unknown?5security?5failure?5detecte@ 20070764     LIBCMTD:secfail.obj
 0002:000097e4       ??_C@_09FNBBCGGI@sprintf?4c?$AA@ 200707e4     LIBCMTD:sprintf.obj
 0002:000097f0       ??_C@_0CG@PKBDLMEO@InitializeCriticalSectionAndSpin@ 200707f0     LIBCMTD:initcrit.obj
 0002:00009824       ___dnames                  20070824     LIBCMTD:timeset.obj
 0002:0000983c       ___mnames                  2007083c     LIBCMTD:timeset.obj
 0002:00009884       ??_C@_07LOOFNDIO@tzset?4c?$AA@ 20070884     LIBCMTD:tzset.obj
 0002:0000988c       ??_C@_02CLFPBFFP@TZ?$AA@   2007088c     LIBCMTD:tzset.obj
 0002:000098ac       ??_C@_0L@DILIPMN@inithelp?4c?$AA@ 200708ac     LIBCMTD:inithelp.obj
 0002:000098b8       ??_C@_06IMKFLFPG@1?$CDQNAN?$AA@ 200708b8     LIBCMTD:x10fout.obj
 0002:000098c0       ??_C@_05DNEBIAHO@1?$CDINF?$AA@ 200708c0     LIBCMTD:x10fout.obj
 0002:000098c8       ??_C@_05PHHOCPM@1?$CDIND?$AA@ 200708c8     LIBCMTD:x10fout.obj
 0002:000098d0       ??_C@_06PGGFOGJG@1?$CDSNAN?$AA@ 200708d0     LIBCMTD:x10fout.obj
 0002:000098e4       ??_C@_09MGNHMPHC@osfinfo?4c?$AA@ 200708e4     LIBCMTD:osfinfo.obj
 0002:00009934       ??_C@_08BDNGOBJJ@fclose?4c?$AA@ 20070934     LIBCMTD:fclose.obj
 0002:0000995c       ??_C@_07NIBBAFJP@w_loc?4c?$AA@ 2007095c     LIBCMTD:w_loc.obj
 0002:00009974       ??_C@_07GCMFDNDD@a_loc?4c?$AA@ 20070974     LIBCMTD:a_loc.obj
 0002:0000999c       ??_C@_0L@CELCHBFJ@wtombenv?4c?$AA@ 2007099c     LIBCMTD:wtombenv.obj
 0002:000099a8       ??_C@_07KLPPCEPH@a_cmp?4c?$AA@ 200709a8     LIBCMTD:a_cmp.obj
 0002:000099b0       ??_C@_0DN@NFIMOOFE@cchCount1?$DN?$DN0?5?$CG?$CG?5cchCount2?$DN?$DN1?5?$HM?$HM?5@ 200709b0     LIBCMTD:a_cmp.obj
 0002:00009a08       ??_C@_08BMJILFKN@setenv?4c?$AA@ 20070a08     LIBCMTD:setenv.obj
 0002:00009a14       ??_C@_05MAJJAKPI@FALSE?$AA@ 20070a14     LIBCMTD:setenv.obj
 0002:00009a74       ___rtc_iaa                 20070a74     LIBCMTD:initsect.obj
 0002:00009a78       ___rtc_izz                 20070a78     LIBCMTD:initsect.obj
 0002:00009a7c       ___rtc_taa                 20070a7c     LIBCMTD:initsect.obj
 0002:00009a80       ___rtc_tzz                 20070a80     LIBCMTD:initsect.obj
 0002:00009a84       __IMPORT_DESCRIPTOR_KERNEL32 20070a84     kernel32:KERNEL32.dll
 0002:00009a98       __NULL_IMPORT_DESCRIPTOR   20070a98     kernel32:KERNEL32.dll
 0003:00000000       ___xc_a                    20072000     LIBCMTD:crt0init.obj
 0003:00000008       ___xc_z                    20072008     LIBCMTD:crt0init.obj
 0003:0000000c       ___xi_a                    2007200c     LIBCMTD:crt0init.obj
 0003:00000020       ___xi_z                    20072020     LIBCMTD:crt0init.obj
 0003:00000024       ___xp_a                    20072024     LIBCMTD:crt0init.obj
 0003:0000002c       ___xp_z                    2007202c     LIBCMTD:crt0init.obj
 0003:00000030       ___xt_a                    20072030     LIBCMTD:crt0init.obj
 0003:00000034       ___xt_z                    20072034     LIBCMTD:crt0init.obj
 0003:00000070       _voiceCommands             20072070     ai_vcmd.obj
 0003:000000e8       _bg_itemlist               200720e8     bg_misc.obj
 0003:0000086c       _bg_numItems               2007286c     bg_misc.obj
 0003:00000870       _eventnames                20072870     bg_misc.obj
 0003:000009a0       _pm_stopspeed              200729a0     bg_pmove.obj
 0003:000009a4       _pm_duckScale              200729a4     bg_pmove.obj
 0003:000009a8       _pm_swimScale              200729a8     bg_pmove.obj
 0003:000009ac       _pm_wadeScale              200729ac     bg_pmove.obj
 0003:000009b0       _pm_accelerate             200729b0     bg_pmove.obj
 0003:000009b4       _pm_airaccelerate          200729b4     bg_pmove.obj
 0003:000009b8       _pm_wateraccelerate        200729b8     bg_pmove.obj
 0003:000009bc       _pm_flyaccelerate          200729bc     bg_pmove.obj
 0003:000009c0       _pm_friction               200729c0     bg_pmove.obj
 0003:000009c4       _pm_waterfriction          200729c4     bg_pmove.obj
 0003:000009c8       _pm_flightfriction         200729c8     bg_pmove.obj
 0003:000009cc       _pm_spectatorfriction      200729cc     bg_pmove.obj
 0003:00000a58       _modNames                  20072a58     g_combat.obj
 0003:00000fc8       _fields                    20072fc8     g_spawn.obj
 0003:00001118       _spawns                    20073118     g_spawn.obj
 0003:00001308       _axisDefault               20073308     q_math.obj
 0003:0000132c       _colorBlack                2007332c     q_math.obj
 0003:0000133c       _colorRed                  2007333c     q_math.obj
 0003:0000134c       _colorGreen                2007334c     q_math.obj
 0003:0000135c       _colorBlue                 2007335c     q_math.obj
 0003:0000136c       _colorYellow               2007336c     q_math.obj
 0003:0000137c       _colorMagenta              2007337c     q_math.obj
 0003:0000138c       _colorCyan                 2007338c     q_math.obj
 0003:0000139c       _colorWhite                2007339c     q_math.obj
 0003:000013ac       _colorLtGrey               200733ac     q_math.obj
 0003:000013bc       _colorMdGrey               200733bc     q_math.obj
 0003:000013cc       _colorDkGrey               200733cc     q_math.obj
 0003:000013e0       _g_color_table             200733e0     q_math.obj
 0003:00001460       _bytedirs                  20073460     q_math.obj
 0003:00001bf8       ?__LINE__Var@?1??ProjectPointOnPlane@@9@9 20073bf8     q_math.obj
 0003:00001c00       __fltused                  20073c00     LIBCMTD:fpinit.obj
 0003:00001c04       __ldused                   20073c04     LIBCMTD:fpinit.obj
 0003:00001c08       __FPinit                   20073c08     LIBCMTD:fpinit.obj
 0003:00001c0c       __FPmtinit                 20073c0c     LIBCMTD:fpinit.obj
 0003:00001c10       __FPmtterm                 20073c10     LIBCMTD:fpinit.obj
 0003:00001c84       __aexit_rtn                20073c84     LIBCMTD:dllcrt0.obj
 0003:00001c90       ___initiallocinfo          20073c90     LIBCMTD:setlocal.obj
 0003:00001ce4       ___ptlocinfo               20073ce4     LIBCMTD:setlocal.obj
 0003:00001e20       ___lc_category             20073e20     LIBCMTD:setlocal.obj
 0003:00001e68       ___tlsindex                20073e68     LIBCMTD:tidtable.obj
 0003:00001e70       __cfltcvt_tab              20073e70     LIBCMTD:cmiscdat.obj
 0003:00001e88       __crtAssertBusy            20073e88     LIBCMTD:dbgrpt.obj
 0003:00001e8c       __CrtDbgMode               20073e8c     LIBCMTD:dbgrpt.obj
 0003:00001e98       __CrtDbgFile               20073e98     LIBCMTD:dbgrpt.obj
 0003:00001eb0       __indefinite               20073eb0     LIBCMTD:87disp.obj
 0003:00001eba       __piby2                    20073eba     LIBCMTD:87disp.obj
 0003:00001fc8       __d_inf                    20073fc8     LIBCMTD:util.obj
 0003:00001fd0       __d_ind                    20073fd0     LIBCMTD:util.obj
 0003:00001fd8       __d_max                    20073fd8     LIBCMTD:util.obj
 0003:00001fe0       __d_min                    20073fe0     LIBCMTD:util.obj
 0003:00001fe8       __d_mzero                  20073fe8     LIBCMTD:util.obj
 0003:00002008       ___nullstring              20074008     LIBCMTD:output.obj
 0003:0000200c       ___wnullstring             2007400c     LIBCMTD:output.obj
 0003:00002010       __pmatherr                 20074010     LIBCMTD:libm_error.obj
 0003:00002020       __OP_ATAN2jmptab           20074020     LIBCMTD:87triga.obj
 0003:00002070       __iob                      20074070     LIBCMTD:_file.obj
 0003:000022f0       ___security_cookie         200742f0     LIBCMTD:seccook.obj
 0003:000022f4       __crtDbgFlag               200742f4     LIBCMTD:dbgheap.obj
 0003:000022fc       __crtBreakAlloc            200742fc     LIBCMTD:dbgheap.obj
 0003:00002318       ___badioinfo               20074318     LIBCMTD:ioinit.obj
 0003:0000233c       __amblksiz                 2007433c     LIBCMTD:heapinit.obj
 0003:00002340       __XcptActTab               20074340     LIBCMTD:winxfltr.obj
 0003:000023b8       __First_FPE_Indx           200743b8     LIBCMTD:winxfltr.obj
 0003:000023bc       __Num_FPE                  200743bc     LIBCMTD:winxfltr.obj
 0003:000023c0       __XcptActTabSize           200743c0     LIBCMTD:winxfltr.obj
 0003:000023c4       __XcptActTabCount          200743c4     LIBCMTD:winxfltr.obj
 0003:000023c8       __NLG_Destination          200743c8     LIBCMTD:exsup.obj
 0003:00002470       __pctype                   20074470     LIBCMTD:ctype.obj
 0003:00002474       __pwctype                  20074474     LIBCMTD:ctype.obj
 0003:00002478       ___lc_time_curr            20074478     LIBCMTD:strftime.obj
 0003:00002480       ___lc_time_c               20074480     LIBCMTD:strftime.obj
 0003:00002538       ___lconv_static_decimal    20074538     LIBCMTD:lconv.obj
 0003:0000253c       ___lconv_c                 2007453c     LIBCMTD:lconv.obj
 0003:0000256c       ___lconv                   2007456c     LIBCMTD:lconv.obj
 0003:00002690       ___mb_cur_max              20074690     LIBCMTD:nlsdata1.obj
 0003:00002694       ___decimal_point           20074694     LIBCMTD:nlsdata1.obj
 0003:00002698       ___decimal_point_length    20074698     LIBCMTD:nlsdata1.obj
 0003:0000269c       ___lc_clike                2007469c     LIBCMTD:nlsdata2.obj
 0003:00002938       __matherr_flag             20074938     LIBCMTD:matherr.obj
 0003:00002940       __pfnAllocHook             20074940     LIBCMTD:dbghook.obj
 0003:00002948       __timezone                 20074948     LIBCMTD:timeset.obj
 0003:0000294c       __daylight                 2007494c     LIBCMTD:timeset.obj
 0003:00002950       __dstbias                  20074950     LIBCMTD:timeset.obj
 0003:000029d8       __tzname                   200749d8     LIBCMTD:timeset.obj
 0003:00002a00       __lpdays                   20074a00     LIBCMTD:days.obj
 0003:00002a34       __days                     20074a34     LIBCMTD:days.obj
 0003:00002a70       __pow10pos                 20074a70     LIBCMTD:constpow.obj
 0003:00002bd0       __pow10neg                 20074bd0     LIBCMTD:constpow.obj
 0003:00002e68       _c_pmove                   20074e68     bg_pmove.obj
 0003:00048478       _remapCount                200ba478     g_utils.obj
 0003:000484ec       _vec3_origin               200ba4ec     q_math.obj
 0003:0005e708       ___fastflag                200d0708     LIBCMTD:fpinit.obj
 0003:0005e70c       __adjust_fdiv              200d070c     LIBCMTD:fpinit.obj
 0003:0005e714       __aenvptr                  200d0714     LIBCMTD:dllcrt0.obj
 0003:0005e718       __wenvptr                  200d0718     LIBCMTD:dllcrt0.obj
 0003:0005e71c       ___error_mode              200d071c     LIBCMTD:dllcrt0.obj
 0003:0005e720       ___app_type                200d0720     LIBCMTD:dllcrt0.obj
 0003:0005e730       _gpFlsAlloc                200d0730     LIBCMTD:tidtable.obj
 0003:0005e734       _gpFlsGetValue             200d0734     LIBCMTD:tidtable.obj
 0003:0005e738       _gpFlsSetValue             200d0738     LIBCMTD:tidtable.obj
 0003:0005e73c       _gpFlsFree                 200d073c     LIBCMTD:tidtable.obj
 0003:0005e748       __umaskval                 200d0748     LIBCMTD:crt0dat.obj
 0003:0005e74c       __osplatform               200d074c     LIBCMTD:crt0dat.obj
 0003:0005e750       __osver                    200d0750     LIBCMTD:crt0dat.obj
 0003:0005e754       __winver                   200d0754     LIBCMTD:crt0dat.obj
 0003:0005e758       __winmajor                 200d0758     LIBCMTD:crt0dat.obj
 0003:0005e75c       __winminor                 200d075c     LIBCMTD:crt0dat.obj
 0003:0005e760       ___argc                    200d0760     LIBCMTD:crt0dat.obj
 0003:0005e764       ___argv                    200d0764     LIBCMTD:crt0dat.obj
 0003:0005e768       ___wargv                   200d0768     LIBCMTD:crt0dat.obj
 0003:0005e76c       __environ                  200d076c     LIBCMTD:crt0dat.obj
 0003:0005e770       ___initenv                 200d0770     LIBCMTD:crt0dat.obj
 0003:0005e774       __wenviron                 200d0774     LIBCMTD:crt0dat.obj
 0003:0005e778       ___winitenv                200d0778     LIBCMTD:crt0dat.obj
 0003:0005e77c       __pgmptr                   200d077c     LIBCMTD:crt0dat.obj
 0003:0005e780       __wpgmptr                  200d0780     LIBCMTD:crt0dat.obj
 0003:0005e784       __exitflag                 200d0784     LIBCMTD:crt0dat.obj
 0003:0005e788       __C_Termination_Done       200d0788     LIBCMTD:crt0dat.obj
 0003:0005e78c       __C_Exit_Done              200d078c     LIBCMTD:crt0dat.obj
 0003:0005e7bc       __cflush                   200d07bc     LIBCMTD:_file.obj
 0003:0005e8ec       __adbgmsg                  200d08ec     LIBCMTD:crt0msg.obj
 0003:0005e8f4       ___lconv_static_null       200d08f4     LIBCMTD:lconv.obj
 0003:0005e8f8       ___lc_time_intl            200d08f8     LIBCMTD:inittime.obj
 0003:0005e8fc       ___lconv_intl              200d08fc     LIBCMTD:initmon.obj
 0003:0005ea50       ___lc_handle               200d0a50     LIBCMTD:nlsdata2.obj
 0003:0005ea68       ___lc_codepage             200d0a68     LIBCMTD:nlsdata2.obj
 0003:0005ea6c       ___lc_collate_cp           200d0a6c     LIBCMTD:nlsdata2.obj
 0003:0005ea70       ___lc_id                   200d0a70     LIBCMTD:nlsdata3.obj
 0003:0005eabc       __stdbuf                   200d0abc     LIBCMTD:_sftbuf.obj
 0003:0005eac8       __newmode                  200d0ac8     LIBCMTD:_newmode.obj
 0003:0005eacc       ?_pnhHeap@@3P6AHI@ZA       200d0acc     LIBCMTD:handler.obj
 0003:0005ec00       _remappedShaders           200d0c00     <common>
 0003:00062e00       _neutralObelisk            200d4e00     <common>
 0003:00062e20       _teamgame                  200d4e20     <common>
 0003:00062e60       _pushed                    200d4e60     <common>
 0003:0006ae60       _pushed_p                  200dce60     <common>
 0003:0006ae80       _g_password                200dce80     <common>
 0003:0006afa0       _g_smoothClients           200dcfa0     <common>
 0003:0006b0c0       _g_friendlyFire            200dd0c0     <common>
 0003:0006b1e0       _g_podiumDist              200dd1e0     <common>
 0003:0006b300       _g_gravity                 200dd300     <common>
 0003:0006b420       _g_filterBan               200dd420     <common>
 0003:0006b540       _g_entities                200dd540     <common>
 0003:00135540       _g_restarted               201a7540     <common>
 0003:00135660       _g_quadfactor              201a7660     <common>
 0003:00135780       _g_debugMove               201a7780     <common>
 0003:001358a0       _g_weaponTeamRespawn       201a78a0     <common>
 0003:001359c0       _g_fraglimit               201a79c0     <common>
 0003:00135ae0       _g_dmflags                 201a7ae0     <common>
 0003:00135c00       _g_maxclients              201a7c00     <common>
 0003:00135d20       _pmove_msec                201a7d20     <common>
 0003:00135e40       _g_synchronousClients      201a7e40     <common>
 0003:00135f60       _g_knockback               201a7f60     <common>
 0003:00136080       _g_warmup                  201a8080     <common>
 0003:001361a0       _g_weaponRespawn           201a81a0     <common>
 0003:001362c0       _g_allowVote               201a82c0     <common>
 0003:001363e0       _g_debugAlloc              201a83e0     <common>
 0003:00136500       _g_dedicated               201a8500     <common>
 0003:00136620       _g_rankings                201a8620     <common>
 0003:00136740       _g_timelimit               201a8740     <common>
 0003:00136860       _g_needpass                201a8860     <common>
 0003:00136980       _g_blood                   201a8980     <common>
 0003:00136aa0       _g_listEntity              201a8aa0     <common>
 0003:00136bc0       _g_inactivity              201a8bc0     <common>
 0003:00136ce0       _g_cheats                  201a8ce0     <common>
 0003:00136e00       _g_maxGameClients          201a8e00     <common>
 0003:00136f20       _g_speed                   201a8f20     <common>
 0003:00137040       _g_log                     201a9040     <common>
 0003:00137160       _g_teamForceBalance        201a9160     <common>
 0003:00137280       _g_banIPs                  201a9280     <common>
 0003:001373a0       _g_gametype                201a93a0     <common>
 0003:001374c0       _g_capturelimit            201a94c0     <common>
 0003:001375e0       _pmove_fixed               201a95e0     <common>
 0003:00137700       _g_doWarmup                201a9700     <common>
 0003:00137820       _g_logSync                 201a9820     <common>
 0003:00137940       _g_teamAutoJoin            201a9940     <common>
 0003:00137a60       _g_podiumDrop              201a9a60     <common>
 0003:00137b80       _g_motd                    201a9b80     <common>
 0003:00137ca0       _g_debugDamage             201a9ca0     <common>
 0003:00137dc0       _g_clients                 201a9dc0     <common>
 0003:00143fc0       _g_forcerespawn            201b5fc0     <common>
 0003:001440e0       _level                     201b60e0     <common>
 0003:001464e0       _itemRegistered            201b84e0     <common>
 0003:001468e0       _bot_minplayers            201b88e0     <common>
 0003:001469f0       _g_numArenas               201b89f0     <common>
 0003:001469f4       _podium1                   201b89f4     <common>
 0003:001469f8       _podium3                   201b89f8     <common>
 0003:001469fc       _podium2                   201b89fc     <common>
 0003:00146a00       _pml                       201b8a00     <common>
 0003:00146a8c       _pm                        201b8a8c     <common>
 0003:00146aa0       _ctftaskpreferences        201b8aa0     <common>
 0003:001474a0       _bot_interbreedcycle       201b94a0     <common>
 0003:001475c0       _bot_saveroutingcache      201b95c0     <common>
 0003:001476e0       _bot_interbreedbots        201b96e0     <common>
 0003:00147800       _bot_memorydump            201b9800     <common>
 0003:00147910       _bot_interbreed            201b9910     <common>
 0003:00147914       _floattime                 201b9914     <common>
 0003:00147920       _botstates                 201b9920     <common>
 0003:00147a20       _bot_interbreedchar        201b9a20     <common>
 0003:00147b40       _bot_developer             201b9b40     <common>
 0003:00147c60       _bot_report                201b9c60     <common>
 0003:00147d80       _bot_interbreedwrite       201b9d80     <common>
 0003:00147ea0       _bot_testsolid             201b9ea0     <common>
 0003:00147fb0       _regularupdate_time        201b9fb0     <common>
 0003:00147fb4       _numbots                   201b9fb4     <common>
 0003:00147fc0       _bot_testclusters          201b9fc0     <common>
 0003:001480d0       _bot_interbreedmatchcount  201ba0d0     <common>
 0003:001480e0       _bot_pause                 201ba0e0     <common>
 0003:00148200       _bot_thinktime             201ba200     <common>
 0003:00148320       _blue_altroutegoals        201ba320     <common>
 0003:00148620       _bot_nochat                201ba620     <common>
 0003:00148740       _bot_challenge             201ba740     <common>
 0003:00148860       _bot_rocketjump            201ba860     <common>
 0003:00148980       _ctf_redflag               201ba980     <common>
 0003:001489b8       _botai_freewaypoints       201ba9b8     <common>
 0003:001489c0       _bot_testrchat             201ba9c0     <common>
 0003:00148ae0       _bot_grapple               201baae0     <common>
 0003:00148bf0       _altroutegoals_setup       201babf0     <common>
 0003:00148c00       _lastteleport_origin       201bac00     <common>
 0003:00148c0c       _lastteleport_time         201bac0c     <common>
 0003:00148c10       _blue_numaltroutegoals     201bac10     <common>
 0003:00148c20       _bot_predictobstacles      201bac20     <common>
 0003:00148d30       _maxclients                201bad30     <common>
 0003:00148d40       _g_spSkill                 201bad40     <common>
 0003:00148e60       _red_altroutegoals         201bae60     <common>
 0003:00149160       _bot_fastchat              201bb160     <common>
 0003:00149280       _ctf_blueflag              201bb280     <common>
 0003:001492b8       _max_bspmodelindex         201bb2b8     <common>
 0003:001492bc       _red_numaltroutegoals      201bb2bc     <common>
 0003:001492c0       _gametype                  201bb2c0     <common>
 0003:001492e0       _botai_waypoints           201bb2e0     <common>
 0003:0014c4e0       _numnodeswitches           201be4e0     <common>
 0003:0014c500       _nodeswitch                201be500     <common>
 0003:0014e1c0       _notleader                 201c01c0     <common>
 0003:0014e2c0       ___sbh_initialized         201c02c0     <common>
 0003:0014e2c4       ___sbh_pHeaderDefer        201c02c4     <common>
 0003:0014e2c8       ___sbh_cntHeaderList       201c02c8     <common>
 0003:0014e2cc       ___sbh_pHeaderList         201c02cc     <common>
 0003:0014e2d0       ___sbh_threshold           201c02d0     <common>
 0003:0014e2d4       ___sbh_pHeaderScan         201c02d4     <common>
 0003:0014e2d8       ___sbh_sizeHeaderList      201c02d8     <common>
 0003:0014e2dc       ___sbh_indGroupDefer       201c02dc     <common>
 0003:0014e2e0       ___mblcid                  201c02e0     <common>
 0003:0014e2e4       ___ptmbcinfo               201c02e4     <common>
 0003:0014e2e8       ___ismbcodepage            201c02e8     <common>
 0003:0014e300       __mbctype                  201c0300     <common>
 0003:0014e404       ___mbcodepage              201c0404     <common>
 0003:0014e410       ___mbulinfo                201c0410     <common>
 0003:0014e420       __mbcasemap                201c0420     <common>
 0003:0014e520       ___ctype1                  201c0520     <common>
 0003:0014e524       ___ctype1_refcount         201c0524     <common>
 0003:0014e528       ___lconv_mon_refcount      201c0528     <common>
 0003:0014e52c       ___lconv_intl_refcount     201c052c     <common>
 0003:0014e530       ___lconv_num_refcount      201c0530     <common>
 0003:0014e534       __crtheap                  201c0534     <common>
 0003:0014e538       ___active_heap             201c0538     <common>
 0003:0014e53c       __nhandle                  201c053c     <common>
 0003:0014e540       ___pioinfo                 201c0540     <common>
 0003:0014e640       __pfnDumpClient            201c0640     <common>
 0003:0014e644       ___piob                    201c0644     <common>
 0003:0014e660       __bufin                    201c0660     <common>
 0003:0014f660       __nstream                  201c1660     <common>
 0003:0014f664       ___env_initialized         201c1664     <common>
 0003:0014f668       ___onexitend               201c1668     <common>
 0003:0014f66c       ___onexitbegin             201c166c     <common>
 0003:0014f670       ___mbctype_initialized     201c1670     <common>
 0003:0014f674       ___use_sse2_mathfcns       201c1674     <common>
 0003:0014f678       ___sse2_available          201c1678     <common>
 0003:0014f67c       __pfnReportHook            201c167c     <common>
 0003:0014f680       __pReportHookList          201c1680     <common>
 0003:0014f684       ___setlc_active            201c1684     <common>
 0003:0014f688       ___unguarded_readlc_active 201c1688     <common>
 0003:0014f68c       __acmdln                   201c168c     <common>
 0003:0014f690       __pRawDllMain              201c1690     <common>

 entry point at        0001:00048c10

 Static symbols

 0001:00005dc0       _VectorLength              20006dc0 f   ai_cmd.obj
 0001:00009150       _VectorLengthSquared       2000a150 f   ai_dmnet.obj
 0001:0000a0f0       _VectorLength              2000b0f0 f   ai_dmnet.obj
 0001:0000a930       _VectorCompare             2000b930 f   ai_dmnet.obj
 0001:0000dec0       _VectorLength              2000eec0 f   ai_dmq3.obj
 0001:00010410       _CrossProduct              20011410 f   ai_dmq3.obj
 0001:00010ba0       _VectorLengthSquared       20011ba0 f   ai_dmq3.obj
 0001:000130a0       _VectorCompare             200140a0 f   ai_dmq3.obj
 0001:0001f7f0       _PM_WaterJumpMove          200207f0 f   bg_pmove.obj
 0001:0001f870       _PM_WaterMove              20020870 f   bg_pmove.obj
 0001:0001fab0       _VectorLength              20020ab0 f   bg_pmove.obj
 0001:0001fb00       _PM_Friction               20020b00 f   bg_pmove.obj
 0001:0001fcc0       _PM_Accelerate             20020cc0 f   bg_pmove.obj
 0001:0001fd90       _PM_CmdScale               20020d90 f   bg_pmove.obj
 0001:0001fe80       _PM_CheckWaterJump         20020e80 f   bg_pmove.obj
 0001:00020020       _PM_FlyMove                20021020 f   bg_pmove.obj
 0001:00020130       _PM_AirMove                20021130 f   bg_pmove.obj
 0001:000202b0       _PM_SetMovementDir         200212b0 f   bg_pmove.obj
 0001:00020480       _PM_GrappleMove            20021480 f   bg_pmove.obj
 0001:000205e0       _PM_WalkMove               200215e0 f   bg_pmove.obj
 0001:000209b0       _PM_CheckJump              200219b0 f   bg_pmove.obj
 0001:00020ac0       _PM_ForceLegsAnim          20021ac0 f   bg_pmove.obj
 0001:00020af0       _PM_StartLegsAnim          20021af0 f   bg_pmove.obj
 0001:00020b50       _PM_DeadMove               20021b50 f   bg_pmove.obj
 0001:00020c30       _PM_NoclipMove             20021c30 f   bg_pmove.obj
 0001:00020ed0       _PM_GroundTrace            20021ed0 f   bg_pmove.obj
 0001:000211e0       _PM_CrashLand              200221e0 f   bg_pmove.obj
 0001:000213e0       _PM_FootstepForSurface     200223e0 f   bg_pmove.obj
 0001:00021420       _PM_CorrectAllSolid        20022420 f   bg_pmove.obj
 0001:00021610       _PM_GroundTraceMissed      20022610 f   bg_pmove.obj
 0001:00021760       _PM_SetWaterLevel          20022760 f   bg_pmove.obj
 0001:000218d0       _PM_CheckDuck              200228d0 f   bg_pmove.obj
 0001:00021ba0       _PM_Footsteps              20022ba0 f   bg_pmove.obj
 0001:00021e10       _PM_ContinueLegsAnim       20022e10 f   bg_pmove.obj
 0001:00021e60       _PM_WaterEvents            20022e60 f   bg_pmove.obj
 0001:00021f00       _PM_TorsoAnimation         20022f00 f   bg_pmove.obj
 0001:00021f50       _PM_ContinueTorsoAnim      20022f50 f   bg_pmove.obj
 0001:00021fa0       _PM_StartTorsoAnim         20022fa0 f   bg_pmove.obj
 0001:00021ff0       _PM_Weapon                 20022ff0 f   bg_pmove.obj
 0001:00022430       _PM_BeginWeaponChange      20023430 f   bg_pmove.obj
 0001:000224c0       _PM_FinishWeaponChange     200234c0 f   bg_pmove.obj
 0001:00022560       _PM_Animate                20023560 f   bg_pmove.obj
 0001:000225b0       _PM_DropTimers             200235b0 f   bg_pmove.obj
 0001:00022fd0       _CrossProduct              20023fd0 f   bg_slidemove.obj
 0001:000254d0       _SpawnModelOnVictoryPad    200264d0 f   g_arenas.obj
 0001:00025880       _CelebrateStart            20026880 f   g_arenas.obj
 0001:000258f0       _CelebrateStop             200268f0 f   g_arenas.obj
 0001:00025940       _SpawnPodium               20026940 f   g_arenas.obj
 0001:00025ae0       _PodiumPlacementThink      20026ae0 f   g_arenas.obj
 0001:00026a00       _PlayerIntroSound          20027a00 f   g_bot.obj
 0001:00026d20       _G_AddBot                  20027d20 f   g_bot.obj
 0001:000271e0       _AddBotToSpawnQueue        200281e0 f   g_bot.obj
 0001:00027680       _G_LoadArenas              20028680 f   g_bot.obj
 0001:00027820       _G_LoadArenasFromFile      20028820 f   g_bot.obj
 0001:00027910       _G_SpawnBots               20028910 f   g_bot.obj
 0001:00027a80       _G_LoadBots                20028a80 f   g_bot.obj
 0001:00027be0       _G_LoadBotsFromFile        20028be0 f   g_bot.obj
 0001:00027f30       _VectorLength              20028f30 f   g_client.obj
 0001:00029220       _ClientCleanName           2002a220 f   g_client.obj
 0001:0002ba60       _G_SayTo                   2002ca60 f   g_cmds.obj
 0001:0002bc10       _G_VoiceTo                 2002cc10 f   g_cmds.obj
 0001:0002d4c0       _Cmd_Say_f                 2002e4c0 f   g_cmds.obj
 0001:0002d520       _Cmd_Tell_f                2002e520 f   g_cmds.obj
 0001:0002d630       _Cmd_Voice_f               2002e630 f   g_cmds.obj
 0001:0002d690       _Cmd_VoiceTell_f           2002e690 f   g_cmds.obj
 0001:0002d7b0       _Cmd_VoiceTaunt_f          2002e7b0 f   g_cmds.obj
 0001:0002e0d0       _VectorLength              2002f0d0 f   g_combat.obj
 0001:000341d0       _CrossProduct              200351d0 f   g_misc.obj
 0001:00034320       _InitShooter_Finish        20035320 f   g_misc.obj
 0001:000345a0       _VectorLength              200355a0 f   g_missile.obj
 0001:00035e70       _VectorInverse             20036e70 f   g_mover.obj
 0001:00037240       _VectorLength              20038240 f   g_mover.obj
 0001:000373f0       _Touch_DoorTriggerSpectator 200383f0 f   g_mover.obj
 0001:00039b00       _AddIP                     2003ab00 f   g_svcmds.obj
 0001:00039ba0       _StringToFilter            2003aba0 f   g_svcmds.obj
 0001:00039d30       _UpdateIPBans              2003ad30 f   g_svcmds.obj
 0001:0003d5a0       _target_location_linkup    2003e5a0 f   g_target.obj
 0001:0003e5b0       _VectorLength              2003f5b0 f   g_team.obj
 0001:0003f7a0       _SortClients               200407a0 f   g_team.obj
 0001:0003fb50       _VectorCompare             20040b50 f   g_trigger.obj
 0001:00040d80       _VectorCompare             20041d80 f   g_utils.obj
 0001:00041750       _CrossProduct              20042750 f   g_utils.obj
 0001:000420e0       _CrossProduct              200430e0 f   g_weapon.obj
 0001:000433a0       _CrossProduct              200443a0 f   q_math.obj
 0001:000441f0       _VectorLength              200451f0 f   q_math.obj
 0001:000453d0       _SkipWhitespace            200463d0 f   q_shared.obj
 0001:00047a20       _$$$00001                  20048a20 f   LIBCMTD:strchr.obj
 0001:000482e0       _shortsort                 200492e0 f   LIBCMTD:qsort.obj
 0001:00048350       _swap                      20049350 f   LIBCMTD:qsort.obj
 0001:00049160       ___updatetlocinfo_lk       2004a160 f   LIBCMTD:setlocal.obj
 0001:00049550       __setlocale_lk             2004a550 f   LIBCMTD:setlocal.obj
 0001:00049900       __setlocale_set_cat        2004a900 f   LIBCMTD:setlocal.obj
 0001:00049cd0       __setlocale_get_all        2004acd0 f   LIBCMTD:setlocal.obj
 0001:0004aaa0       __cftoe2                   2004baa0 f   LIBCMTD:cvt.obj
 0001:0004ac90       __cftof2                   2004bc90 f   LIBCMTD:cvt.obj
 0001:0004af30       __shift                    2004bf30 f   LIBCMTD:cvt.obj
 0001:0004c8d0       __hextodec                 2004d8d0 f   LIBCMTD:input.obj
 0001:0004c900       __inc                      2004d900 f   LIBCMTD:input.obj
 0001:0004c960       __un_inc                   2004d960 f   LIBCMTD:input.obj
 0001:0004c980       __whiteout                 2004d980 f   LIBCMTD:input.obj
 0001:0004d190       _CrtMessageWindow          2004e190 f   LIBCMTD:dbgrpt.obj
 0001:0004d583       _$$$00003                  2004e583 f   LIBCMTD:87disp.obj
 0001:0004ddc0       _strncnt                   2004edc0 f   LIBCMTD:a_map.obj
 0001:0004e9a0       __get_fname                2004f9a0 f   LIBCMTD:fpexcept.obj
 0001:0004fdd0       _write_char                20050dd0 f   LIBCMTD:output.obj
 0001:0004fe70       _write_multi_char          20050e70 f   LIBCMTD:output.obj
 0001:0004feb0       _write_string              20050eb0 f   LIBCMTD:output.obj
 0001:0004ff20       _get_int_arg               20050f20 f   LIBCMTD:output.obj
 0001:0004ff40       _get_int64_arg             20050f40 f   LIBCMTD:output.obj
 0001:0004ff60       _get_short_arg             20050f60 f   LIBCMTD:output.obj
 0001:00050ab0       _has_osfxsr_set            20051ab0 f   LIBCMTD:cpu_disp.obj
 0001:00050c80       _$$$00001                  20051c80 f   LIBCMTD:87triga.obj
 0001:000510b0       _doexit                    200520b0 f   LIBCMTD:crt0dat.obj
 0001:00051250       __initterm                 20052250 f   LIBCMTD:crt0dat.obj
 0001:00051280       __initterm_e               20052280 f   LIBCMTD:crt0dat.obj
 0001:00051530       _ctrlevent_capture@4       20052530 f   LIBCMTD:winsig.obj
 0001:00051860       _siglookup                 20052860 f   LIBCMTD:winsig.obj
 0001:00051aa0       _xtoa                      20052aa0 f   LIBCMTD:xtoa.obj
 0001:00051c20       _x64toa@20                 20052c20 f   LIBCMTD:xtoa.obj
 0001:00052020       _flsall                    20053020 f   LIBCMTD:fflush.obj
 0001:00052690       _report_failure            20053690 f   LIBCMTD:secchk.obj
 0001:00052cb0       _realloc_help              20053cb0 f   LIBCMTD:dbgheap.obj
 0001:000539f0       _CheckBytes                200549f0 f   LIBCMTD:dbgheap.obj
 0001:00054740       __printMemBlockData        20055740 f   LIBCMTD:dbgheap.obj
 0001:00055560       _parse_cmdline             20056560 f   LIBCMTD:stdargv.obj
 0001:00055f40       _xcptlookup                20056f40 f   LIBCMTD:winxfltr.obj
 0001:00055fac       $$$00001                   20056fac f   LIBCMTD:exsup.obj
 0001:00055fcc       __unwind_handler           20056fcc f   LIBCMTD:exsup.obj
 0001:00055fcc       $$$00003                   20056fcc f   LIBCMTD:exsup.obj
 0001:00055fee       $$$00005                   20056fee f   LIBCMTD:exsup.obj
 0001:00056056       $$$00007                   20057056 f   LIBCMTD:exsup.obj
 0001:0005609a       $$$00011                   2005709a f   LIBCMTD:exsup.obj
 0001:000561a5       $$$00003                   200571a5 f   LIBCMTD:exsup3.obj
 0001:00056f60       __expandtime               20057f60 f   LIBCMTD:strftime.obj
 0001:00057540       __store_str                20058540 f   LIBCMTD:strftime.obj
 0001:00057590       __store_num                20058590 f   LIBCMTD:strftime.obj
 0001:00057640       __store_number             20058640 f   LIBCMTD:strftime.obj
 0001:000576f0       __store_winword            200586f0 f   LIBCMTD:strftime.obj
 0001:00058050       __get_lc_time              20059050 f   LIBCMTD:inittime.obj
 0001:00058b90       _fix_grouping              20059b90 f   LIBCMTD:initnum.obj
 0001:00059030       _fix_grouping              2005a030 f   LIBCMTD:initmon.obj
 0001:00059c30       _TranslateName             2005ac30 f   LIBCMTD:getqloc.obj
 0001:00059cc0       _GetLcidFromLangCountry    2005acc0 f   LIBCMTD:getqloc.obj
 0001:00059d80       _LangCountryEnumProc@4     2005ad80 f   LIBCMTD:getqloc.obj
 0001:0005a100       _GetLcidFromLanguage       2005b100 f   LIBCMTD:getqloc.obj
 0001:0005a170       _LanguageEnumProc@4        2005b170 f   LIBCMTD:getqloc.obj
 0001:0005a2c0       _GetLcidFromCountry        2005b2c0 f   LIBCMTD:getqloc.obj
 0001:0005a310       _CountryEnumProc@4         2005b310 f   LIBCMTD:getqloc.obj
 0001:0005a3e0       _GetLcidFromDefault        2005b3e0 f   LIBCMTD:getqloc.obj
 0001:0005a410       _ProcessCodePage           2005b410 f   LIBCMTD:getqloc.obj
 0001:0005a4c0       _TestDefaultCountry        2005b4c0 f   LIBCMTD:getqloc.obj
 0001:0005a510       _TestDefaultLanguage       2005b510 f   LIBCMTD:getqloc.obj
 0001:0005a5b0       _crtGetLocaleInfoA@16      2005b5b0 f   LIBCMTD:getqloc.obj
 0001:0005a740       _LcidFromHexString         2005b740 f   LIBCMTD:getqloc.obj
 0001:0005a7c0       _GetPrimaryLen             2005b7c0 f   LIBCMTD:getqloc.obj
 0001:0005aad0       _getSystemCP               2005bad0 f   LIBCMTD:mbctype.obj
 0001:0005ab30       __setmbcp_lk               2005bb30 f   LIBCMTD:mbctype.obj
 0001:0005ae20       _CPtoLCID                  2005be20 f   LIBCMTD:mbctype.obj
 0001:0005aea0       _setSBCS                   2005bea0 f   LIBCMTD:mbctype.obj
 0001:0005af20       _setSBUpLow                2005bf20 f   LIBCMTD:mbctype.obj
 0001:0005b390       __abstract_cw              2005c390 f   LIBCMTD:ieee87.obj
 0001:0005b4e0       __hw_cw                    2005c4e0 f   LIBCMTD:ieee87.obj
 0001:0005b640       __abstract_sw              2005c640 f   LIBCMTD:ieee87.obj
 0001:0005e320       __onexit_lk                2005f320 f   LIBCMTD:onexit.obj
 0001:000611b0       ___crtInitCritSecNoSpinCount@8 200621b0 f   LIBCMTD:initcrit.obj
 0001:000616c0       __tzset_lk                 200626c0 f   LIBCMTD:tzset.obj
 0001:00061b50       __isindst_lk               20062b50 f   LIBCMTD:tzset.obj
 0001:00061e20       _cvtdate                   20062e20 f   LIBCMTD:tzset.obj
 0001:00064f30       _strncnt                   20065f30 f   LIBCMTD:a_cmp.obj
 0001:00065300       _findenv                   20066300 f   LIBCMTD:setenv.obj
 0001:00065380       _copy_environ              20066380 f   LIBCMTD:setenv.obj
